 ConEmuTh.x64

 Timestamp is 5b32b111 (Wed Jun 27 00:33:05 2018)

 Preferred load address is 0000000180000000

 Start         Length     Name                   Class
 0001:00000000 00025470H .text$mn                CODE
 0001:00025470 00000020H .text$mn$00             CODE
 0001:00025490 000004b0H .text$x                 CODE
 0002:00000000 00000660H .idata$5                DATA
 0002:00000660 00000010H .00cfg                  DATA
 0002:00000670 00000008H .CRT$XCA                DATA
 0002:00000678 00000008H .CRT$XCZ                DATA
 0002:00000680 00000008H .CRT$XIA                DATA
 0002:00000688 00000018H .CRT$XIC                DATA
 0002:000006a0 00000008H .CRT$XIZ                DATA
 0002:000006a8 00000008H .CRT$XPA                DATA
 0002:000006b0 00000010H .CRT$XPX                DATA
 0002:000006c0 00000008H .CRT$XPXA               DATA
 0002:000006c8 00000008H .CRT$XPZ                DATA
 0002:000006d0 00000008H .CRT$XTA                DATA
 0002:000006d8 00000008H .CRT$XTZ                DATA
 0002:000006e0 00000000H .gfids$x                DATA
 0002:000006e0 00000000H .gfids$y                DATA
 0002:000006e0 000095e0H .rdata                  DATA
 0002:00009cc0 0000035cH .rdata$r                DATA
 0002:0000a01c 0000032cH .rdata$zzzdbg           DATA
 0002:0000a348 00000008H .rtc$IAA                DATA
 0002:0000a350 00000008H .rtc$IZZ                DATA
 0002:0000a358 00000008H .rtc$TAA                DATA
 0002:0000a360 00000008H .rtc$TZZ                DATA
 0002:0000a368 00001ac0H .xdata                  DATA
 0002:0000be28 00000088H .xdata$x                DATA
 0002:0000beb0 0000016cH .edata                  DATA
 0002:0000c01c 0000008cH .idata$2                DATA
 0002:0000c0a8 00000018H .idata$3                DATA
 0002:0000c0c0 00000660H .idata$4                DATA
 0002:0000c720 00000e08H .idata$6                DATA
 0003:00000000 000009e0H .data                   DATA
 0003:000009e0 00000180H .data$r                 DATA
 0003:00000b60 0002b108H .bss                    DATA
 0004:00000000 00001efcH .pdata                  DATA
 0005:00000000 00000130H .rsrc$01                DATA
 0005:00000130 00001560H .rsrc$02                DATA

  Address         Publics by Value              Rva+Base               Lib:Object

 0000:00000000       __dynamic_value_reloc_table 0000000000000000     <absolute>
 0000:00000000       __guard_iat_count          0000000000000000     <absolute>
 0000:00000000       __hybrid_code_map          0000000000000000     <absolute>
 0000:00000000       __hybrid_code_map_count    0000000000000000     <absolute>
 0000:00000000       __guard_iat_table          0000000000000000     <absolute>
 0000:00000000       __hybrid_auxiliary_iat     0000000000000000     <absolute>
 0000:00000000       __guard_longjmp_table      0000000000000000     <absolute>
 0000:00000000       __guard_longjmp_count      0000000000000000     <absolute>
 0000:00000000       __guard_fids_count         0000000000000000     <absolute>
 0000:00000000       __enclave_config           0000000000000000     <absolute>
 0000:00000000       ___safe_se_handler_table   0000000000000000     <absolute>
 0000:00000000       ___safe_se_handler_count   0000000000000000     <absolute>
 0000:00000000       __guard_fids_table         0000000000000000     <absolute>
 0000:00000100       __guard_flags              0000000000000100     <absolute>
 0000:00000000       __ImageBase                0000000180000000     <linker-defined>
 0001:00000000       ExitFARW                   0000000180001000 f   ConEmuTh.obj
 0001:00000000       ?ExitFARW3@@YAXPEAX@Z      0000000180001000 f   ConEmuTh.obj
 0001:00000038       ProcessSynchroEventW       0000000180001038 f   ConEmuTh.obj
 0001:00000040       ??$swprintf_c@$0CAA@@@YAHAEAY0CAA@_WPEB_WZZ 0000000180001040 f i ConEmuTh.obj
 0001:0000006c       ??1?$MFileMapping@UPanelViewSetMapping@@@@QEAA@XZ 000000018000106c f i ConEmuTh.obj
 0001:000000c4       ??_G?$MFileMapping@Utag_DetectedDialog@@@@QEAAPEAXI@Z 00000001800010c4 f i ConEmuTh.obj
 0001:000002a4       ?CheckConEmu@@YAHH@Z       00000001800012a4 f   ConEmuTh.obj
 0001:000003ac       ?CheckPanelSettings@@YAHH@Z 00000001800013ac f   ConEmuTh.obj
 0001:000003e4       ?CheckVarsInitialized@@YAXXZ 00000001800013e4 f   ConEmuTh.obj
 0001:00000534       ?CheckWindows@@YA_NXZ      0000000180001534 f   ConEmuTh.obj
 0001:000005d4       ?EntryPoint@@YAXH_J_N@Z    00000001800015d4 f   ConEmuTh.obj
 0001:0000078c       ?ExecuteInMainThread@@YAXPEAUConEmuThSynchroArg@@@Z 000000018000178c f   ConEmuTh.obj
 0001:00000810       ?ExitPlugin@@YAXXZ         0000000180001810 f   ConEmuTh.obj
 0001:00000948       ?FreeItem@CePluginPanelItem@@QEAAXXZ 0000000180001948 f   ConEmuTh.obj
 0001:00000968       ?FreeUserData@CePluginPanelItem@@QEAAXXZ 0000000180001968 f   ConEmuTh.obj
 0001:000009bc       ?GetActivePanel@@YAPEAUCeFullPanelInfo@@XZ 00000001800019bc f   ConEmuTh.obj
 0001:00000a00       ?GetFarRect@@YAHPEAU_SMALL_RECT@@@Z 0000000180001a00 f   ConEmuTh.obj
 0001:00000a70       ?GetFocusedThumbnails@@YAPEAUCeFullPanelInfo@@XZ 0000000180001a70 f   ConEmuTh.obj
 0001:00000acc       ?GetMainThreadId@@YAKXZ    0000000180001acc f   ConEmuTh.obj
 0001:00000b80       ?GetMsgW@@YAPEB_WH@Z       0000000180001b80 f   ConEmuTh.obj
 0001:00000bbc       ?GetPluginInfoWcmn@@YAXPEAX@Z 0000000180001bbc f   ConEmuTh.obj
 0001:00000be0       ?InitName@?$MFileMapping@Utag_DetectedDialog@@@@QEAAPEB_WPEB_WKK@Z 0000000180001be0 f i ConEmuTh.obj
 0001:00000be0       ?InitName@?$MFileMapping@UPanelViewSetMapping@@@@QEAAPEB_WPEB_WKK@Z 0000000180001be0 f i ConEmuTh.obj
 0001:00000c7c       ?InternalOpenCreate@?$MFileMapping@UPanelViewSetMapping@@@@IEAAPEAUPanelViewSetMapping@@HHH@Z 0000000180001c7c f i ConEmuTh.obj
 0001:00000e30       ?InternalOpenCreate@?$MFileMapping@Utag_DetectedDialog@@@@IEAAPEAUtag_DetectedDialog@@HHH@Z 0000000180001e30 f i ConEmuTh.obj
 0001:00000fe4       ?IsThumbnailsActive@@YAPEAUCeFullPanelInfo@@H@Z 0000000180001fe4 f   ConEmuTh.obj
 0001:000011ec       ?LoadFarVersion@@YAHXZ     00000001800021ec f   ConEmuTh.obj
 0001:00001578       ?LoadPanelItemInfo@@YAXPEAUCeFullPanelInfo@@_J@Z 0000000180002578 f   ConEmuTh.obj
 0001:000015b0       ?LoadThSet@@YAHK@Z         00000001800025b0 f   ConEmuTh.obj
 0001:000017e8       ?OnPostPeekConsole@@YAHPEAXPEAU_INPUT_RECORD@@KPEAKPEAH@Z 00000001800027e8 f   ConEmuTh.obj
 0001:00001828       ?OnPostReadConsole@@YAHPEAXPEAU_INPUT_RECORD@@KPEAKPEAH@Z 0000000180002828 f   ConEmuTh.obj
 0001:0000186c       ?OnPrePeekConsole@@YAHPEAXPEAU_INPUT_RECORD@@KPEAKPEAH@Z 000000018000286c f   ConEmuTh.obj
 0001:00001930       ?OnPreReadConsole@@YAHPEAXPEAU_INPUT_RECORD@@KPEAKPEAH@Z 0000000180002930 f   ConEmuTh.obj
 0001:0000194c       ?OnPreWriteConsoleOutput@@YAHPEAXPEBU_CHAR_INFO@@U_COORD@@2PEAU_SMALL_RECT@@@Z 000000018000294c f   ConEmuTh.obj
 0001:00001acc       ?OnReadyForPanelsReload@@YAXXZ 0000000180002acc f   ConEmuTh.obj
 0001:00001c38       ?OpenPluginWcmn@@YAPEAXH_J_N@Z 0000000180002c38 f   ConEmuTh.obj
 0001:00001ca4       ?OpenW@@YAPEAXPEBUOpenInfo@@@Z 0000000180002ca4 f   ConEmuTh.obj
 0001:00001cd4       ?PostMacro@@YAXPEA_W@Z     0000000180002cd4 f   ConEmuTh.obj
 0001:00001e6c       ?ProcessConsoleInput@@YAHHPEAU_INPUT_RECORD@@KPEAK@Z 0000000180002e6c f   ConEmuTh.obj
 0001:000021b0       ?ProcessSynchroEventCommon@@YAHHPEAX@Z 00000001800031b0 f   ConEmuTh.obj
 0001:00002360       ?ReloadPanelsInfo@@YAXXZ   0000000180003360 f   ConEmuTh.obj
 0001:00002508       ?ReloadResourcesW@@YAXXZ   0000000180003508 f   ConEmuTh.obj
 0001:000025a4       ?ResetUngetBuffer@@YAXXZ   00000001800035a4 f   ConEmuTh.obj
 0001:000025b4       ?SavePanelViewState@@YAXHK@Z 00000001800035b4 f   ConEmuTh.obj
 0001:000025fc       ?SettingsLoad@@YAHPEB_WPEAK@Z 00000001800035fc f   ConEmuTh.obj
 0001:00002634       ?SettingsLoadOther@@YAXPEB_W@Z 0000000180003634 f   ConEmuTh.obj
 0001:00002790       ?SettingsLoadReg@@YAHPEB_W0PEAK@Z 0000000180003790 f   ConEmuTh.obj
 0001:00002830       ?SettingsSave@@YAXPEB_WPEAK@Z 0000000180003830 f   ConEmuTh.obj
 0001:00002868       ?SettingsSaveReg@@YAXPEB_W0PEAK@Z 0000000180003868 f   ConEmuTh.obj
 0001:000028f0       ?ShowLastError@@YAHXZ      00000001800038f0 f   ConEmuTh.obj
 0001:00002988       ?ShowMessage@@YAHHH@Z      0000000180003988 f   ConEmuTh.obj
 0001:000029c0       ?ShowPluginMenu@@YAHXZ     00000001800039c0 f   ConEmuTh.obj
 0001:000029f8       ?StartPlugin@@YAXH@Z       00000001800039f8 f   ConEmuTh.obj
 0001:00002b6c       ?StringCchCatW@@YAJPEA_W_KPEB_W@Z 0000000180003b6c f i ConEmuTh.obj
 0001:00002c3c       ?StringCchCopyW@@YAJPEA_W_KPEB_W@Z 0000000180003c3c f i ConEmuTh.obj
 0001:00002cb4       ?StringCchVPrintfW@@YAJPEA_W_KPEB_WPEAD@Z 0000000180003cb4 f i ConEmuTh.obj
 0001:00002d58       ?UpdateEnvVar@@YAXH@Z      0000000180003d58 f   ConEmuTh.obj
 0001:00002d88       ?isPreloadByDefault@@YA_NXZ 0000000180003d88 f   ConEmuTh.obj
 0001:00002db0       DllMain                    0000000180003db0 f   ConEmuTh.obj
 0001:00002e7c       GetMinFarVersionW          0000000180003e7c f   ConEmuTh.obj
 0001:00002e84       SetStartupInfoW            0000000180003e84 f   ConEmuTh.obj
 0001:00002ee4       __local_stdio_printf_options 0000000180003ee4 f i ConEmuTh.obj
 0001:00002eec       ?CheckFarPanelsW1900@@YA_NXZ 0000000180003eec f   ConEmuTh1900.obj
 0001:00002f64       ?CheckPanelSettingsW1900@@YAHH@Z 0000000180003f64 f   ConEmuTh1900.obj
 0001:00003024       ?Color2BgIndex@Far3Color@@SAXKHAEAGPEBK@Z 0000000180004024 f i ConEmuTh1900.obj
 0001:00003138       ?Color2FgIndex@Far3Color@@SAXKAEAGPEBK@Z 0000000180004138 f i ConEmuTh1900.obj
 0001:00003224       ?ExecuteInMainThreadW1900@@YAXPEAUConEmuThSynchroArg@@@Z 0000000180004224 f   ConEmuTh1900.obj
 0001:00003250       ?ExitFARW1900@@YAXXZ       0000000180004250 f   ConEmuTh1900.obj
 0001:0000328c       ?FarColor_3_2@@YAEAEBUFarColor@@_N@Z 000000018000428c f i ConEmuTh1900.obj
 0001:0000334c       ?GetFarRectW1900@@YAXPEAU_SMALL_RECT@@@Z 000000018000434c f   ConEmuTh1900.obj
 0001:000033e0       ?GetMsgW1900@@YAPEB_WH@Z   00000001800043e0 f   ConEmuTh1900.obj
 0001:0000340c       ?GetPluginInfoW1900@@YAXPEAX@Z 000000018000440c f   ConEmuTh1900.obj
 0001:000035c8       ?LoadPanelInfoW1900@@YAHH@Z 00000001800045c8 f   ConEmuTh1900.obj
 0001:00003a80       ?LoadPanelItemInfoW1900@@YAXPEAUCeFullPanelInfo@@_J@Z 0000000180004a80 f   ConEmuTh1900.obj
 0001:00003cb0       ?OpenW1900@@YAPEAXPEBX@Z   0000000180004cb0 f   ConEmuTh1900.obj
 0001:00003d10       ?PostMacroW1900@@YAXPEA_W@Z 0000000180004d10 f   ConEmuTh1900.obj
 0001:00003db0       ?ReloadPanelsInfoW1900@@YAXXZ 0000000180004db0 f   ConEmuTh1900.obj
 0001:00003dd4       ?SetCurrentPanelItemW1900@@YAXH_J0@Z 0000000180004dd4 f   ConEmuTh1900.obj
 0001:00003f08       ?SetStartupInfoW1900@@YAXPEAX@Z 0000000180004f08 f   ConEmuTh1900.obj
 0001:00004054       _guard_check_icall_nop     0000000180005054 f   LIBCMT:guard_support.obj
 0001:00004054       ?FreeItem@?$CQueueProcessor@PEAUIMAGE_CACHE_INFO@@@@MEAAXAEBQEAUIMAGE_CACHE_INFO@@@Z 0000000180005054 f   ImgCache.obj
 0001:00004054       ?OnThreadStopped@?$CQueueProcessor@PEAUIMAGE_CACHE_INFO@@@@MEAAXXZ 0000000180005054 f   ImgCache.obj
 0001:00004054       ?SettingsLoadOtherW2800@@YAXXZ 0000000180005054 f   ConEmuTh2800.obj
 0001:00004054       ?OnItemReady@?$CQueueProcessor@PEAUIMAGE_CACHE_INFO@@@@MEAAXAEAPEAUIMAGE_CACHE_INFO@@_J@Z 0000000180005054 f   ImgCache.obj
 0001:00004054       ?LoadPanelItemInfoA@@YAXPEAUCeFullPanelInfo@@_J@Z 0000000180005054 f   ConEmuThA.obj
 0001:00004054       ?SettingsLoadOtherW1900@@YAXXZ 0000000180005054 f   ConEmuTh1900.obj
 0001:00004054       ?ApplyChanges@?$CQueueProcessor@PEAUIMAGE_CACHE_INFO@@@@MEAAXAEAPEAUIMAGE_CACHE_INFO@@AEBQEAU2@@Z 0000000180005054 f   ImgCache.obj
 0001:00004054       ?OnItemFailed@?$CQueueProcessor@PEAUIMAGE_CACHE_INFO@@@@MEAAXAEAPEAUIMAGE_CACHE_INFO@@_J@Z 0000000180005054 f   ImgCache.obj
 0001:00004058       ?SettingsLoadW1900@@YAHPEB_WPEAK@Z 0000000180005058 f   ConEmuTh1900.obj
 0001:0000413c       ?SettingsSaveW1900@@YAXPEB_WPEAK@Z 000000018000513c f   ConEmuTh1900.obj
 0001:00004228       ?ShowMessageW1900@@YAHHH@Z 0000000180005228 f   ConEmuTh1900.obj
 0001:00004270       ?ShowMessageW1900@@YAHPEB_WH@Z 0000000180005270 f   ConEmuTh1900.obj
 0001:000042f4       ?ShowPluginMenuW1900@@YAHXZ 00000001800052f4 f   ConEmuTh1900.obj
 0001:00004508       ??$swprintf_c@$0MI@@@YAHAEAY0MI@_WPEB_WZZ 0000000180005508 f i ConEmuTh2800.obj
 0001:00004534       ?CheckFarPanelsW2800@@YA_NXZ 0000000180005534 f   ConEmuTh2800.obj
 0001:000045c4       ?CheckPanelSettingsW2800@@YAHH@Z 00000001800055c4 f   ConEmuTh2800.obj
 0001:00004688       ?ExecuteInMainThreadW2800@@YAXPEAUConEmuThSynchroArg@@@Z 0000000180005688 f   ConEmuTh2800.obj
 0001:000046b4       ?ExitFARW2800@@YAXXZ       00000001800056b4 f   ConEmuTh2800.obj
 0001:000046f0       ?FreePanelItemUserData2800@@YAXPEAX_KP6A_JXZ@Z 00000001800056f0 f   ConEmuTh2800.obj
 0001:00004724       ?GetFarRectW2800@@YAXPEAU_SMALL_RECT@@@Z 0000000180005724 f   ConEmuTh2800.obj
 0001:000047c0       ?GetMsgW2800@@YAPEB_WH@Z   00000001800057c0 f   ConEmuTh2800.obj
 0001:000047ec       ?GetPluginInfoW2800@@YAXPEAX@Z 00000001800057ec f   ConEmuTh2800.obj
 0001:000049a8       ?LoadPanelInfoW2800@@YAHH@Z 00000001800059a8 f   ConEmuTh2800.obj
 0001:00004e60       ?LoadPanelItemInfoW2800@@YAXPEAUCeFullPanelInfo@@_J@Z 0000000180005e60 f   ConEmuTh2800.obj
 0001:000050cc       ?OpenW2800@@YAPEAXPEBX@Z   00000001800060cc f   ConEmuTh2800.obj
 0001:0000518c       ?PostMacroW2800@@YAXPEA_W@Z 000000018000618c f   ConEmuTh2800.obj
 0001:00005230       ?ProcessSynchroEventW3@@YA_JPEAX@Z 0000000180006230 f   ConEmuTh2800.obj
 0001:00005248       ?ReloadPanelsInfoW2800@@YAXXZ 0000000180006248 f   ConEmuTh2800.obj
 0001:0000526c       ?SetCurrentPanelItemW2800@@YAXH_J0@Z 000000018000626c f   ConEmuTh2800.obj
 0001:000053c4       ?SetCurrentPanelItemW2800Int@@YAXH_J0@Z 00000001800063c4 f   ConEmuTh2800.obj
 0001:000054fc       ?SetStartupInfoW2800@@YAXPEAX@Z 00000001800064fc f   ConEmuTh2800.obj
 0001:00005648       ?SettingsLoadW2800@@YAHPEB_WPEAK@Z 0000000180006648 f   ConEmuTh2800.obj
 0001:0000573c       ?SettingsSaveW2800@@YAXPEB_WPEAK@Z 000000018000673c f   ConEmuTh2800.obj
 0001:00005830       ?ShowMessageW2800@@YAHHH@Z 0000000180006830 f   ConEmuTh2800.obj
 0001:0000587c       ?ShowMessageW2800@@YAHPEB_WH@Z 000000018000687c f   ConEmuTh2800.obj
 0001:00005904       ?ShowPluginMenuW2800@@YAHXZ 0000000180006904 f   ConEmuTh2800.obj
 0001:00005b28       GetGlobalInfoW             0000000180006b28 f   ConEmuTh2800.obj
 0001:00005bc0       ?CheckFarPanelsW995@@YA_NXZ 0000000180006bc0 f   ConEmuTh995.obj
 0001:00005c38       ?CheckPanelSettingsW995@@YAHH@Z 0000000180006c38 f   ConEmuTh995.obj
 0001:00005cd0       ?ExecuteInMainThreadW995@@YAXPEAUConEmuThSynchroArg@@@Z 0000000180006cd0 f   ConEmuTh995.obj
 0001:00005cf8       ?ExitFARW995@@YAXXZ        0000000180006cf8 f   ConEmuTh995.obj
 0001:00005d4c       ?GetFarRectW995@@YAXPEAU_SMALL_RECT@@@Z 0000000180006d4c f   ConEmuTh995.obj
 0001:00005d8c       ?GetMsgW995@@YAPEB_WH@Z    0000000180006d8c f   ConEmuTh995.obj
 0001:00005db4       ?GetPluginInfoW995@@YAXPEAX@Z 0000000180006db4 f   ConEmuTh995.obj
 0001:00005e88       ?LoadPanelInfo995@@YAHH@Z  0000000180006e88 f   ConEmuTh995.obj
 0001:000061d4       ?LoadPanelItemInfoW995@@YAXPEAUCeFullPanelInfo@@_J@Z 00000001800071d4 f   ConEmuTh995.obj
 0001:0000635c       ?PostMacroW995@@YAXPEA_W@Z 000000018000735c f   ConEmuTh995.obj
 0001:000063dc       ?ReloadPanelsInfoW995@@YAXXZ 00000001800073dc f   ConEmuTh995.obj
 0001:00006400       ?SetCurrentPanelItemW995@@YAXH_J0@Z 0000000180007400 f   ConEmuTh995.obj
 0001:00006528       ?SetStartupInfoW995@@YAXPEAX@Z 0000000180007528 f   ConEmuTh995.obj
 0001:000066c8       ?SettingsLoadOtherW995@@YAXXZ 00000001800076c8 f   ConEmuTh995.obj
 0001:000066d4       ?SettingsLoadW995@@YAHPEB_WPEAK@Z 00000001800076d4 f   ConEmuTh995.obj
 0001:000066e8       ?SettingsSaveW995@@YAXPEB_WPEAK@Z 00000001800076e8 f   ConEmuTh995.obj
 0001:000066fc       ?ShowMessageW995@@YAHHH@Z  00000001800076fc f   ConEmuTh995.obj
 0001:00006740       ?ShowMessageW995@@YAHPEB_WH@Z 0000000180007740 f   ConEmuTh995.obj
 0001:00006780       ?ShowPluginMenuW995@@YAHXZ 0000000180007780 f   ConEmuTh995.obj
 0001:0000692c       OpenPluginW                000000018000792c f   ConEmuTh995.obj
 0001:0000694c       ?CheckFarPanelsA@@YA_NXZ   000000018000794c f   ConEmuThA.obj
 0001:000069d8       ?CheckPanelSettingsA@@YAHH@Z 00000001800079d8 f   ConEmuThA.obj
 0001:00006a84       ?GetMsgA@@YAPEB_WHPEA_W@Z  0000000180007a84 f   ConEmuThA.obj
 0001:00006b80       ?LoadPanelInfoA@@YAHH@Z    0000000180007b80 f   ConEmuThA.obj
 0001:00006f60       ?PostMacroA@@YAXPEAD@Z     0000000180007f60 f   ConEmuThA.obj
 0001:00006fdc       ?ReloadPanelsInfoA@@YAXXZ  0000000180007fdc f   ConEmuThA.obj
 0001:00007000       ?ReloadResourcesA@@YAXXZ   0000000180008000 f   ConEmuThA.obj
 0001:000070dc       ?SetCurrentPanelItemA@@YAXH_J0@Z 00000001800080dc f   ConEmuThA.obj
 0001:00007210       ?SettingsLoadA@@YAHPEB_WPEAK@Z 0000000180008210 f   ConEmuThA.obj
 0001:00007224       ?SettingsLoadOtherA@@YAXXZ 0000000180008224 f   ConEmuThA.obj
 0001:00007230       ?SettingsSaveA@@YAXPEB_WPEAK@Z 0000000180008230 f   ConEmuThA.obj
 0001:00007244       ?ShowMessageA@@YAHHH@Z     0000000180008244 f   ConEmuThA.obj
 0001:00007294       ?ShowMessageA@@YAHPEBDH@Z  0000000180008294 f   ConEmuThA.obj
 0001:000072d8       ?ShowPluginMenuA@@YAHXZ    00000001800082d8 f   ConEmuThA.obj
 0001:000074d0       ExitFAR                    00000001800084d0 f   ConEmuThA.obj
 0001:0000752c       GetMinFarVersion           000000018000852c f   ConEmuThA.obj
 0001:0000755c       GetPluginInfo              000000018000855c f   ConEmuThA.obj
 0001:000075dc       OpenPlugin                 00000001800085dc f   ConEmuThA.obj
 0001:00007618       SetStartupInfo             0000000180008618 f   ConEmuThA.obj
 0001:000077d8       ??$swprintf_c@$0IA@@@YAHAEAY0IA@_WPEB_WZZ 00000001800087d8 f i Display.obj
 0001:00007804       ?BisItem2CeItem@CeFullPanelInfo@@QEAAH_JH_KKKHH@Z 0000000180008804 f   Display.obj
 0001:000078a4       ?CalcTopPanelItem@CeFullPanelInfo@@QEAA_J_J0@Z 00000001800088a4 f   Display.obj
 0001:00007984       ?Close@CeFullPanelInfo@@QEAAXXZ 0000000180008984 f   Display.obj
 0001:000079c8       ?CreateView@CeFullPanelInfo@@QEAAPEAUHWND__@@XZ 00000001800089c8 f   Display.obj
 0001:00007d74       ?DisplayReloadPanel@CeFullPanelInfo@@QEAAXXZ 0000000180008d74 f   Display.obj
 0001:00007db0       ?DisplayThread@CeFullPanelInfo@@SAKPEAX@Z 0000000180008db0 f   Display.obj
 0001:00007ed0       ?DisplayWndProc@CeFullPanelInfo@@SA_JPEAUHWND__@@I_K_J@Z 0000000180008ed0 f   Display.obj
 0001:0000843c       ?DrawItemText@CeFullPanelInfo@@QEAAHPEAUHDC__@@PEAUtagRECT@@1PEAUCePluginPanelItem@@PEB_WPEAUHBRUSH__@@H@Z 000000018000943c f   Display.obj
 0001:00008aa8       ?FarItem2CeItem@CeFullPanelInfo@@QEAAH_JPEB_W1KU_FILETIME@@_KHPEAX3P6A_JXZ3K@Z 0000000180009aa8 f   Display.obj
 0001:00008e0c       ?FinalRelease@CeFullPanelInfo@@QEAAXXZ 0000000180009e0c f   Display.obj
 0001:00008f28       ?GetConCoordFromIndex@CeFullPanelInfo@@QEAAH_JAEAU_COORD@@@Z 0000000180009f28 f   Display.obj
 0001:00008fd0       ?GetIndexFromWndCoord@CeFullPanelInfo@@QEAAHHHAEA_J@Z 0000000180009fd0 f   Display.obj
 0001:00009068       ?GetItemColors@CeFullPanelInfo@@QEAAPEAUHBRUSH__@@_JPEAUCePluginPanelItem@@PEAUCePluginPanelItemColor@@HAEAK3@Z 000000018000a068 f   Display.obj
 0001:000090d0       ?Invalidate@CeFullPanelInfo@@QEAAXXZ 000000018000a0d0 f   Display.obj
 0001:00009124       ?InvalidateAll@CeFullPanelInfo@@SAXXZ 000000018000a124 f   Display.obj
 0001:00009174       ?LoadItemColors@CeFullPanelInfo@@QEAAX_JPEAUCePluginPanelItem@@PEAUCePluginPanelItemColor@@HH@Z 000000018000a174 f   Display.obj
 0001:000093d4       ?OnSettingsChanged@CeFullPanelInfo@@QEAAHH@Z 000000018000a3d4 f   Display.obj
 0001:00009508       ?Paint@CeFullPanelInfo@@QEAAXPEAUHWND__@@AEAUtagPAINTSTRUCT@@AEAUtagRECT@@@Z 000000018000a508 f   Display.obj
 0001:00009e0c       ?PaintItem@CeFullPanelInfo@@QEAAHPEAUHDC__@@_JHHPEAUCePluginPanelItem@@PEAUCePluginPanelItemColor@@HHPEAUHBRUSH__@@4K@Z 000000018000ae0c f   Display.obj
 0001:0000a344       ?ReallocItems@CeFullPanelInfo@@QEAAH_J@Z 000000018000b344 f   Display.obj
 0001:0000a4c8       ?RegisterPanelView@CeFullPanelInfo@@QEAAHXZ 000000018000b4c8 f   Display.obj
 0001:0000a7a8       ?RequestSetPos@CeFullPanelInfo@@QEAAX_J0H@Z 000000018000b7a8 f   Display.obj
 0001:0000a88c       ?UnregisterPanelView@CeFullPanelInfo@@QEAAH_N@Z 000000018000b88c f   Display.obj
 0001:0000a9c8       ??$SafeDelete@UMSectionSimple@@@@YAXAEAPEAUMSectionSimple@@@Z 000000018000b9c8 f i ImgCache.obj
 0001:0000aa10       ??0?$CQueueProcessor@PEAUIMAGE_CACHE_INFO@@@@QEAA@XZ 000000018000ba10 f i ImgCache.obj
 0001:0000aa94       ??0CImgCache@@QEAA@PEAUHINSTANCE__@@@Z 000000018000ba94 f   ImgCache.obj
 0001:0000abd0       ??1?$CQueueProcessor@PEAUIMAGE_CACHE_INFO@@@@UEAA@XZ 000000018000bbd0 f i ImgCache.obj
 0001:0000ac98       ??1CImgCache@@QEAA@XZ      000000018000bc98 f   ImgCache.obj
 0001:0000ad60       ??_E?$CQueueProcessor@PEAUIMAGE_CACHE_INFO@@@@UEAAPEAXI@Z 000000018000bd60 f i ImgCache.obj
 0001:0000ad60       ??_G?$CQueueProcessor@PEAUIMAGE_CACHE_INFO@@@@UEAAPEAXI@Z 000000018000bd60 f i ImgCache.obj
 0001:0000ad60       ??_ECImgLoader@@UEAAPEAXI@Z 000000018000bd60 f i ImgCache.obj
 0001:0000ad60       ??_GCImgLoader@@UEAAPEAXI@Z 000000018000bd60 f i ImgCache.obj
 0001:0000ad94       ?CheckDrawDibCreated@CImgCache@@IEAAHXZ 000000018000bd94 f   ImgCache.obj
 0001:0000af00       ?CheckHighPriority@?$CQueueProcessor@PEAUIMAGE_CACHE_INFO@@@@MEAA_NAEBQEAUIMAGE_CACHE_INFO@@@Z 000000018000bf00 f i ImgCache.obj
 0001:0000af00       ?Filter@?$MToolHelp@UtagPROCESSENTRY32W@@$1?Process32FirstW@@YAHPEAXPEAU1@@Z$1?Process32NextW@@YAH01@Z@@MEAA_NPEAUtagPROCESSENTRY32W@@@Z 000000018000bf00 f i common-kernel64:MProcess.obj
 0001:0000af00       ?CheckHighPriority@CImgLoader@@UEAA_NAEAPEBUIMAGE_CACHE_INFO@@@Z 000000018000bf00 f i ImgCache.obj
 0001:0000af00       __acrt_uninitialize_command_line 000000018000bf00 f i libucrt:argv_data.obj
 0001:0000af04       ?CheckLoadDibCreated@CImgCache@@IEAAHXZ 000000018000bf04 f   ImgCache.obj
 0001:0000b070       ?CheckThread@?$CQueueProcessor@PEAUIMAGE_CACHE_INFO@@@@IEAAJXZ 000000018000c070 f i ImgCache.obj
 0001:0000b12c       ?ClearQueue@?$CQueueProcessor@PEAUIMAGE_CACHE_INFO@@@@AEAAXXZ 000000018000c12c f i ImgCache.obj
 0001:0000b1b4       ?CopyBits@CImgCache@@IEAAXU_COORD@@PEAEK01@Z 000000018000c1b4 f   ImgCache.obj
 0001:0000b23c       ?CopyItem@?$CQueueProcessor@PEAUIMAGE_CACHE_INFO@@@@MEAAXPEBQEAUIMAGE_CACHE_INFO@@PEAPEAU2@@Z 000000018000c23c f i ImgCache.obj
 0001:0000b25c       ?FindInCache@CImgCache@@IEAAHPEAUCePluginPanelItem@@PEAHI@Z 000000018000c25c f   ImgCache.obj
 0001:0000b488       ?FindOrCreate@?$CQueueProcessor@PEAUIMAGE_CACHE_INFO@@@@AEAAPEAUProcessingItem@1@AEBQEAUIMAGE_CACHE_INFO@@_J_NW4ProcessingPriority@@@Z 000000018000c488 f i ImgCache.obj
 0001:0000b6e8       ?FreeModules@CImgCache@@IEAAXXZ 000000018000c6e8 f   ImgCache.obj
 0001:0000b754       ?Init@CImgCache@@QEAAXK@Z  000000018000c754 f   ImgCache.obj
 0001:0000b7b4       ?InitializeQueue@?$CQueueProcessor@PEAUIMAGE_CACHE_INFO@@@@AEAAXH@Z 000000018000c7b4 f i ImgCache.obj
 0001:0000b864       ?IsEqual@?$CQueueProcessor@PEAUIMAGE_CACHE_INFO@@@@MEAA_NAEBQEAUIMAGE_CACHE_INFO@@_J01@Z 000000018000c864 f i ImgCache.obj
 0001:0000b880       ?IsEqual@CImgLoader@@UEAA_NAEAPEBUIMAGE_CACHE_INFO@@_JAEAPEAU2@1@Z 000000018000c880 f i ImgCache.obj
 0001:0000b898       ?IsStopRequested@?$CQueueProcessor@PEAUIMAGE_CACHE_INFO@@@@UEAA_NAEBQEAUIMAGE_CACHE_INFO@@@Z 000000018000c898 f i ImgCache.obj
 0001:0000b8a8       ?IsTerminationRequested@CImgLoader@@UEAA_NXZ 000000018000c8a8 f i ImgCache.obj
 0001:0000b8a8       ?IsTerminationRequested@?$CQueueProcessor@PEAUIMAGE_CACHE_INFO@@@@MEAA_NXZ 000000018000c8a8 f i ImgCache.obj
 0001:0000b8ac       ?LoadModules@CImgCache@@IEAAXXZ 000000018000c8ac f   ImgCache.obj
 0001:0000bb14       ?LoadShellIcon@CImgCache@@QEAAHPEAUIMAGE_CACHE_INFO@@H@Z 000000018000cb14 f   ImgCache.obj
 0001:0000be48       ?LoadThumbnail@CImgCache@@QEAAHPEAUIMAGE_CACHE_INFO@@@Z 000000018000ce48 f   ImgCache.obj
 0001:0000c37c       ?OnThreadStarted@?$CQueueProcessor@PEAUIMAGE_CACHE_INFO@@@@MEAAJXZ 000000018000d37c f i ImgCache.obj
 0001:0000c380       ?OnThreadStarted@CImgLoader@@UEAAJXZ 000000018000d380 f i ImgCache.obj
 0001:0000c394       ?OnThreadStopped@CImgLoader@@UEAAXXZ 000000018000d394 f i ImgCache.obj
 0001:0000c39c       ?PaintItem@CImgCache@@QEAAHPEAUHDC__@@HHHPEAUCePluginPanelItem@@PEAPEB_WPEAH@Z 000000018000d39c f   ImgCache.obj
 0001:0000c8a0       ?ProcessItem@?$CQueueProcessor@PEAUIMAGE_CACHE_INFO@@@@IEAAJPEAUProcessingItem@1@@Z 000000018000d8a0 f i ImgCache.obj
 0001:0000c8cc       ?ProcessItem@?$CQueueProcessor@PEAUIMAGE_CACHE_INFO@@@@MEAAJAEAPEAUIMAGE_CACHE_INFO@@_J@Z 000000018000d8cc f i ImgCache.obj
 0001:0000c8d4       ?ProcessItem@CImgLoader@@UEAAJAEAPEAUIMAGE_CACHE_INFO@@_J@Z 000000018000d8d4 f i ImgCache.obj
 0001:0000c92c       ?ProcessingStep@?$CQueueProcessor@PEAUIMAGE_CACHE_INFO@@@@IEAA_NXZ 000000018000d92c f i ImgCache.obj
 0001:0000cb38       ?ProcessingThread@?$CQueueProcessor@PEAUIMAGE_CACHE_INFO@@@@KAKPEAX@Z 000000018000db38 f i ImgCache.obj
 0001:0000cb68       ?RequestItem@CImgCache@@QEAAHPEAUCePluginPanelItem@@I@Z 000000018000db68 f   ImgCache.obj
 0001:0000cc60       ?Reset@CImgCache@@QEAAXXZ  000000018000dc60 f   ImgCache.obj
 0001:0000ce30       ?SetCacheLocation@CImgCache@@QEAAXPEB_W@Z 000000018000de30 f   ImgCache.obj
 0001:0000ceaf       GetFileVersionInfoSizeW    000000018000deaf f   version:VERSION.dll
 0001:0000ceb5       GetFileVersionInfoW        000000018000deb5 f   version:VERSION.dll
 0001:0000cebb       VerQueryValueW             000000018000debb f   version:VERSION.dll
 0001:0000cec1       CreateToolhelp32Snapshot   000000018000dec1 f   kernel32:KERNEL32.dll
 0001:0000cec7       Thread32First              000000018000dec7 f   kernel32:KERNEL32.dll
 0001:0000cecd       Thread32Next               000000018000decd f   kernel32:KERNEL32.dll
 0001:0000ced4       ??2@YAPEAX_K@Z             000000018000ded4 f   common-kernel64:Memory.obj
 0001:0000cf08       ??3@YAXPEAX@Z              000000018000df08 f   common-kernel64:Memory.obj
 0001:0000cf08       ??_V@YAXPEAX@Z             000000018000df08 f   common-kernel64:Memory.obj
 0001:0000cf08       ?xf_free@@YAXPEAX@Z        000000018000df08 f   common-kernel64:Memory.obj
 0001:0000cf30       ??_U@YAPEAX_K@Z            000000018000df30 f   common-kernel64:Memory.obj
 0001:0000cf30       ?xf_malloc@@YAPEAX_K@Z     000000018000df30 f   common-kernel64:Memory.obj
 0001:0000cf44       ?HeapDeinitialize@@YAXXZ   000000018000df44 f   common-kernel64:Memory.obj
 0001:0000cf68       ?HeapInitialize@@YA_NXZ    000000018000df68 f   common-kernel64:Memory.obj
 0001:0000cf9c       ?xf_calloc@@YAPEAX_K0@Z    000000018000df9c f   common-kernel64:Memory.obj
 0001:0000cfb8       ?xf_realloc@@YAPEAXPEAX_K@Z 000000018000dfb8 f   common-kernel64:Memory.obj
 0001:0000cfec       ?StringCchVPrintfA@@YAJPEAD_KPEBD0@Z 000000018000dfec f i common-kernel64:MStrSafe.obj
 0001:0000d094       ?msprintf@@YAPEB_WPEA_W_KPEB_WZZ 000000018000e094 f   common-kernel64:MStrSafe.obj
 0001:0000d4b0       ?sprintf_c@@YAHPEAD_JPEBDZZ 000000018000e4b0 f   common-kernel64:MStrSafe.obj
 0001:0000d4f0       ?swprintf_c@@YAHPEA_W_JPEB_WZZ 000000018000e4f0 f   common-kernel64:MStrSafe.obj
 0001:0000d530       ?CommonShutdown@@YAXXZ     000000018000e530 f   common-kernel64:Common.obj
 0001:0000d540       ??_GMNullDesc@@QEAAPEAXI@Z 000000018000e540 f i common-kernel64:MSecurity.obj
 0001:0000d5b8       ?LoadAdvApi@MNullDesc@@IEAAHXZ 000000018000e5b8 f i common-kernel64:MSecurity.obj
 0001:0000d76c       ?LocalSecurity@@YAPEAU_SECURITY_ATTRIBUTES@@XZ 000000018000e76c f   common-kernel64:MSecurity.obj
 0001:0000d7c8       ?LocalSecurity@MNullDesc@@QEAAPEAU_SECURITY_ATTRIBUTES@@XZ 000000018000e7c8 f i common-kernel64:MSecurity.obj
 0001:0000d944       ?ShutdownSecurity@@YAXXZ   000000018000e944 f   common-kernel64:MSecurity.obj
 0001:0000d96c       ?ExecuteCmd@@YAPEAUCESERVER_REQ@@PEB_WPEAU1@KPEAUHWND__@@HKH@Z 000000018000e96c f   common-kernel64:ConEmuCheck.obj
 0001:0000db54       ?ExecuteFreeResult@@YAXAEAPEAUCESERVER_REQ@@@Z 000000018000eb54 f   common-kernel64:ConEmuCheck.obj
 0001:0000db74       ?ExecuteGuiCmd@@YAPEAUCESERVER_REQ@@PEAUHWND__@@PEAU1@0H@Z 000000018000eb74 f   common-kernel64:ConEmuCheck.obj
 0001:0000dc34       ?ExecuteNewCmd@@YAPEAUCESERVER_REQ@@K_K@Z 000000018000ec34 f   common-kernel64:ConEmuCheck.obj
 0001:0000dc98       ?ExecuteOpenPipe@@YAPEAXPEB_WAEAY0CAI@_W0KKHPEAXH@Z 000000018000ec98 f   common-kernel64:ConEmuCheck.obj
 0001:0000de48       ?ExecutePrepareCmd@@YAXPEAUCESERVER_REQ@@K_K@Z 000000018000ee48 f   common-kernel64:ConEmuCheck.obj
 0001:0000de84       ?ExecutePrepareCmd@@YAXPEAUCESERVER_REQ_HDR@@K_K@Z 000000018000ee84 f   common-kernel64:ConEmuCheck.obj
 0001:0000def4       ?ModuleName@@YAPEB_WPEB_W@Z 000000018000eef4 f   common-kernel64:ConEmuCheck.obj
 0001:0000dfb8       ??1?$MToolHelp@UtagPROCESSENTRY32W@@$1?Process32FirstW@@YAHPEAXPEAU1@@Z$1?Process32NextW@@YAH01@Z@@UEAA@XZ 000000018000efb8 f i common-kernel64:MProcess.obj
 0001:0000e050       ??_E?$MToolHelp@UtagPROCESSENTRY32W@@$1?Process32FirstW@@YAHPEAXPEAU1@@Z$1?Process32NextW@@YAH01@Z@@UEAAPEAXI@Z 000000018000f050 f i common-kernel64:MProcess.obj
 0001:0000e050       ??_GMToolHelpProcess@@UEAAPEAXI@Z 000000018000f050 f i common-kernel64:MProcess.obj
 0001:0000e050       ??_G?$MToolHelp@UtagPROCESSENTRY32W@@$1?Process32FirstW@@YAHPEAXPEAU1@@Z$1?Process32NextW@@YAH01@Z@@UEAAPEAXI@Z 000000018000f050 f i common-kernel64:MProcess.obj
 0001:0000e050       ??_EMToolHelpProcess@@UEAAPEAXI@Z 000000018000f050 f i common-kernel64:MProcess.obj
 0001:0000e084       ?Find@?$MToolHelp@UtagPROCESSENTRY32W@@$1?Process32FirstW@@YAHPEAXPEAU1@@Z$1?Process32NextW@@YAH01@Z@@QEAA_NP6A_NPEAUtagPROCESSENTRY32W@@_J@Z10@Z 000000018000f084 f i common-kernel64:MProcess.obj
 0001:0000e164       ?Open@?$MToolHelp@UtagPROCESSENTRY32W@@$1?Process32FirstW@@YAHPEAXPEAU1@@Z$1?Process32NextW@@YAH01@Z@@QEAA_NXZ 000000018000f164 f i common-kernel64:MProcess.obj
 0001:0000e1e8       ?addsize@?$MArray@UtagPROCESSENTRY32W@@@@QEAA_N_J@Z 000000018000f1e8 f i common-kernel64:MProcess.obj
 0001:0000e284       ?getNext@?$MToolHelp@UtagPROCESSENTRY32W@@$1?Process32FirstW@@YAHPEAXPEAU1@@Z$1?Process32NextW@@YAH01@Z@@IEAA_NXZ 000000018000f284 f i common-kernel64:MProcess.obj
 0001:0000e324       ?isTerminalMode@@YA_NXZ    000000018000f324 f   common-kernel64:MProcess.obj
 0001:0000e494       ?push_back@?$MArray@UtagPROCESSENTRY32W@@@@QEAA_JAEBUtagPROCESSENTRY32W@@@Z 000000018000f494 f i common-kernel64:MProcess.obj
 0001:0000e50c       ?Init@HkFunc@@QEAA_NPEB_WPEAUHINSTANCE__@@@Z 000000018000f50c f   common-kernel64:HkFunc.obj
 0001:0000e59c       ??0MSection@@QEAA@XZ       000000018000f59c f   common-kernel64:MSection.obj
 0001:0000e624       ??0MSectionLock@@QEAA@XZ   000000018000f624 f   common-kernel64:MSection.obj
 0001:0000e634       ??1MSection@@QEAA@XZ       000000018000f634 f   common-kernel64:MSection.obj
 0001:0000e6a8       ??1MSectionLock@@QEAA@XZ   000000018000f6a8 f   common-kernel64:MSection.obj
 0001:0000e6cc       ?AddRef@MSection@@IEAAXK@Z 000000018000f6cc f   common-kernel64:MSection.obj
 0001:0000e760       ?Lock@MSection@@IEAAHHK@Z  000000018000f760 f   common-kernel64:MSection.obj
 0001:0000e85c       ?Lock@MSectionLock@@QEAAHPEAVMSection@@HK@Z 000000018000f85c f   common-kernel64:MSection.obj
 0001:0000e8b0       ?MyEnterCriticalSection@MSection@@IEAA_NK@Z 000000018000f8b0 f   common-kernel64:MSection.obj
 0001:0000e9e0       ?ReleaseRef@MSection@@IEAAHK@Z 000000018000f9e0 f   common-kernel64:MSection.obj
 0001:0000ea80       ?Unlock@MSection@@IEAAXH@Z 000000018000fa80 f   common-kernel64:MSection.obj
 0001:0000ead8       ?Unlock@MSectionLock@@QEAAXXZ 000000018000fad8 f   common-kernel64:MSection.obj
 0001:0000eb04       ?WaitUnlocked@MSection@@IEAAXKK@Z 000000018000fb04 f   common-kernel64:MSection.obj
 0001:0000eb98       ??$sprintf_c@$0CI@@@YAHAEAY0CI@DPEBDZZ 000000018000fb98 f i common-kernel64:WThreads.obj
 0001:0000ebc4       ?SetThreadName@@YAXKPEAD@Z 000000018000fbc4 f   common-kernel64:WThreads.obj
 0001:0000ebfc       ?apiCreateThread@@YAPEAXP6AKPEAX@Z0PEAKPEBDH@Z 000000018000fbfc f   common-kernel64:WThreads.obj
 0001:0000ed50       ?apiTerminateThreadEx@@YAHPEAXKPEBDH@Z 000000018000fd50 f   common-kernel64:WThreads.obj
 0001:0000ee58       ?apiThreadHelper@@YAKPEAX@Z 000000018000fe58 f   common-kernel64:WThreads.obj
 0001:0000f064       ?ExpandEnvStr@@YAPEA_WPEB_W@Z 0000000180010064 f   common-kernel64:WObjects.obj
 0001:0000f10c       ?FileExists@@YA_NPEB_WPEAK@Z 000000018001010c f   common-kernel64:WObjects.obj
 0001:0000f298       ?GetEnvVar@@YAPEA_WPEB_W@Z 0000000180010298 f   common-kernel64:WObjects.obj
 0001:0000f33c       ?IsWindows64@@YA_NXZ       000000018001033c f   common-kernel64:WObjects.obj
 0001:0000f360       ?StringCchCopyNW@@YAJPEA_W_KPEB_W1@Z 0000000180010360 f i common-kernel64:WObjects.obj
 0001:0000f3e8       ?_VerifyVersionInfo@@YA_NPEAU_OSVERSIONINFOEXW@@K_K@Z 00000001800103e8 f   common-kernel64:WObjects.obj
 0001:0000f498       ?PointToExt@@YAPEB_WPEB_W@Z 0000000180010498 f   common-kernel64:CmdLine.obj
 0001:0000f4bc       ?PointToName@@YAPEB_WPEB_W@Z 00000001800104bc f   common-kernel64:CmdLine.obj
 0001:0000f518       ?Unquote@@YAPEB_WPEA_W_N@Z 0000000180010518 f   common-kernel64:CmdLine.obj
 0001:0000f580       ?lstrdup@@YAPEA_WPEB_W_K@Z 0000000180010580 f   common-kernel64:MStrDup.obj
 0001:0000f5f4       ?lstrmerge@@YAPEA_WPEB_W00000000@Z 00000001800105f4 f   common-kernel64:MStrDup.obj
 0001:0000f738       ??0MSectionLockSimple@@QEAA@XZ 0000000180010738 f   common-kernel64:MSectionSimple.obj
 0001:0000f744       ??0MSectionSimple@@QEAA@_N@Z 0000000180010744 f   common-kernel64:MSectionSimple.obj
 0001:0000f77c       ??1MSectionLockSimple@@QEAA@XZ 000000018001077c f   common-kernel64:MSectionSimple.obj
 0001:0000f790       ?Close@MSectionSimple@@QEAAXXZ 0000000180010790 f   common-kernel64:MSectionSimple.obj
 0001:0000f790       ??1MSectionSimple@@QEAA@XZ 0000000180010790 f   common-kernel64:MSectionSimple.obj
 0001:0000f7b0       ?Enter@MSectionSimple@@QEAAXXZ 00000001800107b0 f   common-kernel64:MSectionSimple.obj
 0001:0000f7b8       ?Init@MSectionSimple@@QEAAXXZ 00000001800107b8 f   common-kernel64:MSectionSimple.obj
 0001:0000f7d8       ?Leave@MSectionSimple@@QEAAXXZ 00000001800107d8 f   common-kernel64:MSectionSimple.obj
 0001:0000f7e0       ?Lock@MSectionLockSimple@@QEAAHPEAUMSectionSimple@@K@Z 00000001800107e0 f   common-kernel64:MSectionSimple.obj
 0001:0000f87c       ?RecreateAndLock@MSectionSimple@@QEAA_NXZ 000000018001087c f   common-kernel64:MSectionSimple.obj
 0001:0000f8ec       ?TryEnter@MSectionSimple@@QEAA_NXZ 00000001800108ec f   common-kernel64:MSectionSimple.obj
 0001:0000f914       ?Unlock@MSectionLockSimple@@QEAAXXZ 0000000180010914 f   common-kernel64:MSectionSimple.obj
 0001:0000f93c       ??0CEStr@@QEAA@PEB_W00000000@Z 000000018001093c f   common-kernel64:CEStr.obj
 0001:0000fa2c       ??1CEStr@@QEAA@XZ          0000000180010a2c f   common-kernel64:CEStr.obj
 0001:0000fa78       ??BCEStr@@QEBAPEB_WXZ      0000000180010a78 f   common-kernel64:CEStr.obj
 0001:0000fa7c       ?AttachInt@CEStr@@AEAAPEB_WAEAPEA_W@Z 0000000180010a7c f   common-kernel64:CEStr.obj
 0001:0000fb08       ?Empty@CEStr@@QEAAXXZ      0000000180010b08 f   common-kernel64:CEStr.obj
 0001:0000fb28       ?GetBuffer@CEStr@@QEAAPEA_W_J@Z 0000000180010b28 f   common-kernel64:CEStr.obj
 0001:0000fbe0       ?GetLen@CEStr@@QEBA_JXZ    0000000180010be0 f   common-kernel64:CEStr.obj
 0001:0000fc04       ?GetMaxCount@CEStr@@QEAA_JXZ 0000000180010c04 f   common-kernel64:CEStr.obj
 0001:0000fc30       ?SavePathVar@CEStr@@QEAAXPEB_W@Z 0000000180010c30 f   common-kernel64:CEStr.obj
 0001:0000fc68       ?Set@CEStr@@QEAAPEB_WPEB_W_J@Z 0000000180010c68 f   common-kernel64:CEStr.obj
 0001:0000fd54       ??0MModule@@QEAA@PEAUHINSTANCE__@@@Z 0000000180010d54 f   common-kernel64:MModule.obj
 0001:0000fd60       ??1MModule@@QEAA@XZ        0000000180010d60 f   common-kernel64:MModule.obj
 0001:0000fd68       ?Free@MModule@@QEAAXXZ     0000000180010d68 f   common-kernel64:MModule.obj
 0001:0000fd98       ??0CRgnDetect@@QEAA@XZ     0000000180010d98 f   common-user64:RgnDetect.obj
 0001:0000fe58       ??1CRgnDetect@@QEAA@XZ     0000000180010e58 f   common-user64:RgnDetect.obj
 0001:0000fec0       ?DetectDialog@CRgnDetect@@IEAA_NPEA_WPEAUtag_CharAttr@@HHHHPEAH2@Z 0000000180010ec0 f   common-user64:RgnDetect.obj
 0001:00010258       ?ExpandDialogFrame@CRgnDetect@@IEAA_NPEA_WPEAUtag_CharAttr@@HHAEAH2HH22@Z 0000000180011258 f   common-user64:RgnDetect.obj
 0001:000105a0       ?FindByBackground@CRgnDetect@@IEAA_NPEA_WPEAUtag_CharAttr@@HHAEAH222AEA_N@Z 00000001800115a0 f   common-user64:RgnDetect.obj
 0001:000106c8       ?FindDialog_Any@CRgnDetect@@IEAA_NPEA_WPEAUtag_CharAttr@@HHAEAH222AEA_N@Z 00000001800116c8 f   common-user64:RgnDetect.obj
 0001:00010964       ?FindDialog_Inner@CRgnDetect@@IEAA_NPEA_WPEAUtag_CharAttr@@HHAEAH2@Z 0000000180011964 f   common-user64:RgnDetect.obj
 0001:00010ad4       ?FindDialog_Left@CRgnDetect@@IEAA_NPEA_WPEAUtag_CharAttr@@HHAEAH222AEA_N@Z 0000000180011ad4 f   common-user64:RgnDetect.obj
 0001:00010cd0       ?FindDialog_Right@CRgnDetect@@IEAA_NPEA_WPEAUtag_CharAttr@@HHAEAH222AEA_N@Z 0000000180011cd0 f   common-user64:RgnDetect.obj
 0001:00010e38       ?FindDialog_TopLeft@CRgnDetect@@IEAA_NPEA_WPEAUtag_CharAttr@@HHAEAH222AEA_N@Z 0000000180011e38 f   common-user64:RgnDetect.obj
 0001:00010f44       ?FindDialog_TopRight@CRgnDetect@@IEAA_NPEA_WPEAUtag_CharAttr@@HHAEAH222AEA_N@Z 0000000180011f44 f   common-user64:RgnDetect.obj
 0001:0001105c       ?FindFrameBottom_ByLeft@CRgnDetect@@IEAA_NPEA_WPEAUtag_CharAttr@@HHAEAH22@Z 000000018001205c f   common-user64:RgnDetect.obj
 0001:000110f0       ?FindFrameBottom_ByRight@CRgnDetect@@IEAA_NPEA_WPEAUtag_CharAttr@@HHAEAH22@Z 00000001800120f0 f   common-user64:RgnDetect.obj
 0001:000111a4       ?FindFrameLeft_ByBottom@CRgnDetect@@IEAA_NPEA_WPEAUtag_CharAttr@@HHAEAH22@Z 00000001800121a4 f   common-user64:RgnDetect.obj
 0001:00011268       ?FindFrameLeft_ByTop@CRgnDetect@@IEAA_NPEA_WPEAUtag_CharAttr@@HHAEAH22@Z 0000000180012268 f   common-user64:RgnDetect.obj
 0001:000113f4       ?FindFrameRight_ByBottom@CRgnDetect@@IEAA_NPEA_WPEAUtag_CharAttr@@HHAEAH22@Z 00000001800123f4 f   common-user64:RgnDetect.obj
 0001:000114c4       ?FindFrameRight_ByTop@CRgnDetect@@IEAA_NPEA_WPEAUtag_CharAttr@@HHAEAH22@Z 00000001800124c4 f   common-user64:RgnDetect.obj
 0001:00011624       ?FindFrameTop_ByLeft@CRgnDetect@@IEAA_NPEA_WPEAUtag_CharAttr@@HHAEAH22@Z 0000000180012624 f   common-user64:RgnDetect.obj
 0001:000116a8       ?FindFrameTop_ByRight@CRgnDetect@@IEAA_NPEA_WPEAUtag_CharAttr@@HHAEAH22@Z 00000001800126a8 f   common-user64:RgnDetect.obj
 0001:00011750       ?FindFrame_TopLeft@CRgnDetect@@IEAA_NPEA_WPEAUtag_CharAttr@@HHAEAH222@Z 0000000180012750 f   common-user64:RgnDetect.obj
 0001:00011858       ?GetCharAttr@CRgnDetect@@QEAAHHHAEA_WAEAUtag_CharAttr@@@Z 0000000180012858 f   common-user64:RgnDetect.obj
 0001:000118d8       ?GetDetectedDialogsPtr@CRgnDetect@@QEBAPEBUtag_DetectedDialog@@XZ 00000001800128d8 f   common-user64:RgnDetect.obj
 0001:000118e0       ?GetFlags@CRgnDetect@@QEBAKXZ 00000001800128e0 f   common-user64:RgnDetect.obj
 0001:000118e8       ?InitializeSBI@CRgnDetect@@QEAAHPEBK@Z 00000001800128e8 f   common-user64:RgnDetect.obj
 0001:00011cc8       ?MarkDialog@CRgnDetect@@IEAAHPEA_WPEAUtag_CharAttr@@HHHHHHI_NK@Z 0000000180012cc8 f   common-user64:RgnDetect.obj
 0001:0001259c       ?OnWindowSizeChanged@CRgnDetect@@QEAAXXZ 000000018001359c f   common-user64:RgnDetect.obj
 0001:000125a4       ?OnWriteConsoleOutput@CRgnDetect@@QEAAXPEBU_CHAR_INFO@@U_COORD@@1PEAU_SMALL_RECT@@PEBK@Z 00000001800135a4 f   common-user64:RgnDetect.obj
 0001:00012814       ?PrepareTransparent@CRgnDetect@@QEAAXPEBUCEFAR_INFO_MAPPING@@PEBK@Z 0000000180013814 f   common-user64:RgnDetect.obj
 0001:000128e8       ?PrepareTransparent@CRgnDetect@@QEAAXPEBUCEFAR_INFO_MAPPING@@PEBKPEBU_CONSOLE_SCREEN_BUFFER_INFO@@PEA_WPEAUtag_CharAttr@@HH@Z 00000001800138e8 f   common-user64:RgnDetect.obj
 0001:00013114       ?SetFarRect@CRgnDetect@@QEAAXPEAU_SMALL_RECT@@@Z 0000000180014114 f   common-user64:RgnDetect.obj
 0001:00013184       ?TextHeight@CRgnDetect@@QEAAHXZ 0000000180014184 f   common-user64:RgnDetect.obj
 0001:000131b0       ?TextWidth@CRgnDetect@@QEAAHXZ 00000001800141b0 f   common-user64:RgnDetect.obj
 0001:000131dc       ?SearchAppPaths@@YA_NPEB_WAEAUCEStr@@_NPEAU1@@Z 00000001800141dc f   common-user64:WFiles.obj
 0001:000135dc       ?apiShowWindow@@YA_NPEAUHWND__@@H@Z 00000001800145dc f   common-user64:WUser.obj
 0001:000135f0       ??3@YAXPEAX_K@Z            00000001800145f0 f   LIBCMT:delete_scalar_size.obj
 0001:000135f8       __GSHandlerCheck           00000001800145f8 f   LIBCMT:_gshandler_.obj
 0001:00013618       __GSHandlerCheckCommon     0000000180014618 f   LIBCMT:_gshandler_.obj
 0001:00013674       __GSHandlerCheck_EH        0000000180014674 f   LIBCMT:gshandlereh.obj
 0001:00013710       __security_check_cookie    0000000180014710 f   LIBCMT:_amdsecgs_.obj
 0001:00013734       ??_Etype_info@@UEAAPEAXI@Z 0000000180014734 f i LIBCMT:std_type_info_static.obj
 0001:00013734       ??_Gtype_info@@UEAAPEAXI@Z 0000000180014734 f i LIBCMT:std_type_info_static.obj
 0001:00013a80       _DllMainCRTStartup         0000000180014a80 f   LIBCMT:dll_dllmain.obj
 0001:00013ac0       __raise_securityfailure    0000000180014ac0 f   LIBCMT:gs_report.obj
 0001:00013af4       __report_gsfailure         0000000180014af4 f   LIBCMT:gs_report.obj
 0001:00013bc8       __report_rangecheckfailure 0000000180014bc8 f   LIBCMT:gs_report.obj
 0001:00013bdc       __report_securityfailure   0000000180014bdc f   LIBCMT:gs_report.obj
 0001:00013d5c       __security_init_cookie     0000000180014d5c f   LIBCMT:gs_support.obj
 0001:00013e0c       ?__scrt_initialize_type_info@@YAXXZ 0000000180014e0c f   LIBCMT:tncleanup.obj
 0001:00013e1c       ?__scrt_uninitialize_type_info@@YAXXZ 0000000180014e1c f   LIBCMT:tncleanup.obj
 0001:00013e28       __local_stdio_scanf_options 0000000180014e28 f i LIBCMT:default_local_stdio_options.obj
 0001:00013e30       __scrt_initialize_default_local_stdio_options 0000000180014e30 f   LIBCMT:default_local_stdio_options.obj
 0001:00013e4c       __scrt_acquire_startup_lock 0000000180014e4c f   LIBCMT:utility.obj
 0001:00013e88       __scrt_dllmain_after_initialize_c 0000000180014e88 f   LIBCMT:utility.obj
 0001:00013ebc       __scrt_dllmain_before_initialize_c 0000000180014ebc f   LIBCMT:utility.obj
 0001:00013ed4       __scrt_dllmain_crt_thread_attach 0000000180014ed4 f   LIBCMT:utility.obj
 0001:00013efc       __scrt_dllmain_crt_thread_detach 0000000180014efc f   LIBCMT:utility.obj
 0001:00013f14       __scrt_dllmain_exception_filter 0000000180014f14 f   LIBCMT:utility.obj
 0001:00013f74       __scrt_dllmain_uninitialize_c 0000000180014f74 f   LIBCMT:utility.obj
 0001:00013fa4       __scrt_dllmain_uninitialize_critical 0000000180014fa4 f   LIBCMT:utility.obj
 0001:00013fb8       __scrt_initialize_crt      0000000180014fb8 f   LIBCMT:utility.obj
 0001:00014004       __scrt_initialize_onexit_tables 0000000180015004 f   LIBCMT:utility.obj
 0001:000140e0       __scrt_is_nonwritable_in_current_image 00000001800150e0 f   LIBCMT:utility.obj
 0001:0001417c       __scrt_release_startup_lock 000000018001517c f   LIBCMT:utility.obj
 0001:000141a0       __scrt_uninitialize_crt    00000001800151a0 f   LIBCMT:utility.obj
 0001:000141cc       __scrt_get_dyn_tls_init_callback 00000001800151cc f   LIBCMT:dyn_tls_init.obj
 0001:000141d4       __crt_debugger_hook        00000001800151d4 f   LIBCMT:utility_desktop.obj
 0001:000141dc       __scrt_fastfail            00000001800151dc f   LIBCMT:utility_desktop.obj
 0001:00014328       _RTC_Initialize            0000000180015328 f   LIBCMT:_initsect_.obj
 0001:00014364       _RTC_Terminate             0000000180015364 f   LIBCMT:_initsect_.obj
 0001:000143a0       __isa_available_init       00000001800153a0 f   LIBCMT:_cpu_disp_.obj
 0001:0001455c       _get_startup_argv_mode     000000018001555c f   LIBCMT:argv_mode.obj
 0001:00014564       __scrt_is_ucrt_dll_in_use  0000000180015564 f   LIBCMT:ucrt_detection.obj
 0001:00014570       wcsrchr                    0000000180015570 f   libvcruntime:wcsrchr.obj
 0001:00014624       ?_ExecutionInCatch@@YAHPEAU_xDISPATCHER_CONTEXT@@PEBU_s_FuncInfo@@@Z 0000000180015624 f   libvcruntime:risctrnsctrl.obj
 0001:00014698       ?_GetEstablisherFrame@@YAPEA_KPEA_KPEAU_xDISPATCHER_CONTEXT@@PEBU_s_FuncInfo@@0@Z 0000000180015698 f   libvcruntime:risctrnsctrl.obj
 0001:00014764       ?_GetRangeOfTrysToCheck@@YAPEBU_s_TryBlockMapEntry@@PEA_KPEBU_s_FuncInfo@@HHPEAI2PEAU_xDISPATCHER_CONTEXT@@@Z 0000000180015764 f   libvcruntime:risctrnsctrl.obj
 0001:00014890       ?__FrameUnwindToEmptyState@@YAXPEA_KPEAU_xDISPATCHER_CONTEXT@@PEBU_s_FuncInfo@@@Z 0000000180015890 f   libvcruntime:risctrnsctrl.obj
 0001:00014924       _CallSETranslator          0000000180015924 f   libvcruntime:risctrnsctrl.obj
 0001:00014978       _CreateFrameInfo           0000000180015978 f   libvcruntime:risctrnsctrl.obj
 0001:000149b4       _FindAndUnlinkFrame        00000001800159b4 f   libvcruntime:risctrnsctrl.obj
 0001:00014a08       _GetImageBase              0000000180015a08 f   libvcruntime:risctrnsctrl.obj
 0001:00014a1c       _GetThrowImageBase         0000000180015a1c f   libvcruntime:risctrnsctrl.obj
 0001:00014a30       _SetImageBase              0000000180015a30 f   libvcruntime:risctrnsctrl.obj
 0001:00014a48       _SetThrowImageBase         0000000180015a48 f   libvcruntime:risctrnsctrl.obj
 0001:00014a60       _UnwindNestedFrames        0000000180015a60 f   libvcruntime:risctrnsctrl.obj
 0001:00014b84       __CxxFrameHandler3         0000000180015b84 f   libvcruntime:risctrnsctrl.obj
 0001:00014c20       memcmp                     0000000180015c20 f   libvcruntime:memcmp.obj
 0001:00014d00       memcpy                     0000000180015d00 f   libvcruntime:memcpy.obj
 0001:00014d00       memmove                    0000000180015d00 f   libvcruntime:memcpy.obj
 0001:00015160       memset                     0000000180016160 f   libvcruntime:memset.obj
 0001:00015310       wcschr                     0000000180016310 f   libvcruntime:wcschr.obj
 0001:000153a4       __C_specific_handler       00000001800163a4 f   libvcruntime:_riscchandler_.obj
 0001:000155b0       strchr                     00000001800165b0 f   libvcruntime:strchr.obj
 0001:0001563c       strrchr                    000000018001663c f   libvcruntime:strrchr.obj
 0001:000157a0       memchr                     00000001800167a0 f   libvcruntime:memchr.obj
 0001:00015810       __std_type_info_compare    0000000180016810 f   libvcruntime:std_type_info.obj
 0001:00015838       __std_type_info_destroy_list 0000000180016838 f   libvcruntime:std_type_info.obj
 0001:00015864       __vcrt_initialize          0000000180016864 f   libvcruntime:initialization.obj
 0001:00015898       __vcrt_thread_attach       0000000180016898 f   libvcruntime:initialization.obj
 0001:000158ac       __vcrt_thread_detach       00000001800168ac f   libvcruntime:initialization.obj
 0001:000158c0       __vcrt_uninitialize        00000001800168c0 f   libvcruntime:initialization.obj
 0001:000158e0       __vcrt_uninitialize_critical 00000001800168e0 f   libvcruntime:initialization.obj
 0001:000158f0       __vcrt_freefls             00000001800168f0 f   libvcruntime:per_thread_data.obj
 0001:00015910       __vcrt_freeptd             0000000180016910 f   libvcruntime:per_thread_data.obj
 0001:00015960       __vcrt_getptd              0000000180016960 f   libvcruntime:per_thread_data.obj
 0001:0001597c       __vcrt_getptd_noexit       000000018001697c f   libvcruntime:per_thread_data.obj
 0001:00015a34       __vcrt_initialize_ptd      0000000180016a34 f   libvcruntime:per_thread_data.obj
 0001:00015a84       __vcrt_uninitialize_ptd    0000000180016a84 f   libvcruntime:per_thread_data.obj
 0001:00015aa8       ?__GetCurrentState@@YAHPEA_KPEAU_xDISPATCHER_CONTEXT@@PEBU_s_FuncInfo@@@Z 0000000180016aa8 f   libvcruntime:riscehstate.obj
 0001:00015ad0       ?__GetUnwindTryBlock@@YAHPEA_KPEAU_xDISPATCHER_CONTEXT@@PEBU_s_FuncInfo@@@Z 0000000180016ad0 f   libvcruntime:riscehstate.obj
 0001:00015afc       ?__SetState@@YAXPEA_KPEAU_xDISPATCHER_CONTEXT@@PEBU_s_FuncInfo@@H@Z 0000000180016afc f   libvcruntime:riscehstate.obj
 0001:00015b08       ?__SetUnwindTryBlock@@YAXPEA_KPEAU_xDISPATCHER_CONTEXT@@PEBU_s_FuncInfo@@H@Z 0000000180016b08 f   libvcruntime:riscehstate.obj
 0001:00015b44       ?__StateFromControlPc@@YAHPEBU_s_FuncInfo@@PEAU_xDISPATCHER_CONTEXT@@@Z 0000000180016b44 f   libvcruntime:riscehstate.obj
 0001:00015b4c       ?__StateFromIp@@YAHPEBU_s_FuncInfo@@PEAU_xDISPATCHER_CONTEXT@@_K@Z 0000000180016b4c f   libvcruntime:riscehstate.obj
 0001:00015bb4       ??0bad_exception@std@@QEAA@AEBV01@@Z 0000000180016bb4 f i libvcruntime:frame.obj
 0001:00015bf4       ??0bad_exception@std@@QEAA@XZ 0000000180016bf4 f i libvcruntime:frame.obj
 0001:00015c14       ??0exception@std@@QEAA@AEBV01@@Z 0000000180016c14 f i libvcruntime:frame.obj
 0001:00015c4c       ??1bad_exception@std@@UEAA@XZ 0000000180016c4c f i libvcruntime:frame.obj
 0001:00015c60       ??_Gbad_exception@std@@UEAAPEAXI@Z 0000000180016c60 f i libvcruntime:frame.obj
 0001:00015c60       ??_Eexception@std@@UEAAPEAXI@Z 0000000180016c60 f i libvcruntime:frame.obj
 0001:00015c60       ??_Gexception@std@@UEAAPEAXI@Z 0000000180016c60 f i libvcruntime:frame.obj
 0001:00015c60       ??_Ebad_exception@std@@UEAAPEAXI@Z 0000000180016c60 f i libvcruntime:frame.obj
 0001:000165cc       ?_CallMemberFunction1@@YAXQEAX00@Z 00000001800175cc f i libvcruntime:frame.obj
 0001:000165d8       ?_CallMemberFunction2@@YAXQEAX00H@Z 00000001800175d8 f i libvcruntime:frame.obj
 0001:000165e8       ?what@exception@std@@UEBAPEBDXZ 00000001800175e8 f i libvcruntime:frame.obj
 0001:000165fc       __BuildCatchObject         00000001800175fc f   libvcruntime:frame.obj
 0001:000166bc       __BuildCatchObjectHelper   00000001800176bc f   libvcruntime:frame.obj
 0001:000168bc       __CxxCallCatchBlock        00000001800178bc f   libvcruntime:frame.obj
 0001:00016aa8       __FrameUnwindToState       0000000180017aa8 f   libvcruntime:frame.obj
 0001:00016c3c       __InternalCxxFrameHandler  0000000180017c3c f   libvcruntime:frame.obj
 0001:00016e80       __TypeMatch                0000000180017e80 f   libvcruntime:frame.obj
 0001:00016fe0       _local_unwind              0000000180017fe0 f   libvcruntime:_jmpuwind_.obj
 0001:00017010       _NLG_Notify                0000000180018010 f   libvcruntime:_jmpuwind_.obj
 0001:00017030       __NLG_Dispatch2            0000000180018030 f   libvcruntime:_jmpuwind_.obj
 0001:00017040       __NLG_Return2              0000000180018040 f   libvcruntime:_jmpuwind_.obj
 0001:00017044       __except_validate_context_record 0000000180018044 f   libvcruntime:jbcxrval.obj
 0001:0001707c       __vcrt_initialize_locks    000000018001807c f   libvcruntime:locks.obj
 0001:000170c4       __vcrt_uninitialize_locks  00000001800180c4 f   libvcruntime:locks.obj
 0001:000172d4       __vcrt_FlsAlloc            00000001800182d4 f   libvcruntime:winapi_downlevel.obj
 0001:0001731c       __vcrt_FlsFree             000000018001831c f   libvcruntime:winapi_downlevel.obj
 0001:00017364       __vcrt_FlsGetValue         0000000180018364 f   libvcruntime:winapi_downlevel.obj
 0001:000173ac       __vcrt_FlsSetValue         00000001800183ac f   libvcruntime:winapi_downlevel.obj
 0001:00017400       __vcrt_InitializeCriticalSectionEx 0000000180018400 f   libvcruntime:winapi_downlevel.obj
 0001:00017464       __vcrt_initialize_winapi_thunks 0000000180018464 f   libvcruntime:winapi_downlevel.obj
 0001:00017494       __vcrt_uninitialize_winapi_thunks 0000000180018494 f   libvcruntime:winapi_downlevel.obj
 0001:000174d4       __vcrt_initialize_pure_virtual_call_handler 00000001800184d4 f   libvcruntime:purevirt_data.obj
 0001:00017500       _CallSettingFrame          0000000180018500 f   libvcruntime:handlers.obj
 0001:00017540       __DestructExceptionObject  0000000180018540 f   libvcruntime:ehhelpers.obj
 0001:000175b4       ?_CallMemberFunction0@@YAXQEAX0@Z 00000001800185b4 f i libvcruntime:ehhelpers.obj
 0001:000175b8       _IsExceptionObjectToBeDestroyed 00000001800185b8 f   libvcruntime:ehhelpers.obj
 0001:000175e8       __AdjustPointer            00000001800185e8 f   libvcruntime:ehhelpers.obj
 0001:0001760c       __FrameUnwindFilter        000000018001860c f   libvcruntime:ehhelpers.obj
 0001:00017658       __std_exception_copy       0000000180018658 f   libvcruntime:std_exception.obj
 0001:000176e8       __std_exception_destroy    00000001800186e8 f   libvcruntime:std_exception.obj
 0001:00017710       _CxxThrowException         0000000180018710 f   libvcruntime:throw.obj
 0001:000177d0       ??$ensure_buffer_is_big_enough@D@formatting_buffer@__crt_stdio_output@@QEAA_N_K@Z 00000001800187d0 f i libucrt:output.obj
 0001:0001787c       ??$is_wide_character_specifier@D@__crt_stdio_output@@YA_N_KDW4length_modifier@0@@Z 000000018001887c f i libucrt:output.obj
 0001:000178ac       ??$is_wide_character_specifier@_W@__crt_stdio_output@@YA_N_K_WW4length_modifier@0@@Z 00000001800188ac f i libucrt:output.obj
 0001:000178f0       ??$type_case_integer_parse_into_buffer@I@?$output_processor@DV?$string_output_adapter@D@__crt_stdio_output@@V?$standard_base@DV?$string_output_adapter@D@__crt_stdio_output@@@2@@__crt_stdio_output@@AEAAXII_N@Z 00000001800188f0 f i libucrt:output.obj
 0001:000178f0       ??$type_case_integer_parse_into_buffer@I@?$output_processor@_WV?$string_output_adapter@_W@__crt_stdio_output@@V?$standard_base@_WV?$string_output_adapter@_W@__crt_stdio_output@@@2@@__crt_stdio_output@@AEAAXII_N@Z 00000001800188f0 f i libucrt:output.obj
 0001:0001798c       ??$type_case_integer_parse_into_buffer@_K@?$output_processor@_WV?$string_output_adapter@_W@__crt_stdio_output@@V?$standard_base@_WV?$string_output_adapter@_W@__crt_stdio_output@@@2@@__crt_stdio_output@@AEAAX_KI_N@Z 000000018001898c f i libucrt:output.obj
 0001:0001798c       ??$type_case_integer_parse_into_buffer@_K@?$output_processor@DV?$string_output_adapter@D@__crt_stdio_output@@V?$standard_base@DV?$string_output_adapter@D@__crt_stdio_output@@@2@@__crt_stdio_output@@AEAAX_KI_N@Z 000000018001898c f i libucrt:output.obj
 0001:00017a28       ??$write_multiple_characters@V?$string_output_adapter@D@__crt_stdio_output@@D@__crt_stdio_output@@YAXAEBV?$string_output_adapter@D@0@DHQEAH@Z 0000000180018a28 f i libucrt:output.obj
 0001:00017a84       ??$write_multiple_characters@V?$string_output_adapter@_W@__crt_stdio_output@@D@__crt_stdio_output@@YAXAEBV?$string_output_adapter@_W@0@DHQEAH@Z 0000000180018a84 f i libucrt:output.obj
 0001:00017af4       ??0?$output_processor@DV?$string_output_adapter@D@__crt_stdio_output@@V?$standard_base@DV?$string_output_adapter@D@__crt_stdio_output@@@2@@__crt_stdio_output@@QEAA@AEBV?$string_output_adapter@D@1@_KQEBDQEAU__crt_locale_pointers@@QEAD@Z 0000000180018af4 f i libucrt:output.obj
 0001:00017b70       ??0?$output_processor@_WV?$string_output_adapter@_W@__crt_stdio_output@@V?$standard_base@_WV?$string_output_adapter@_W@__crt_stdio_output@@@2@@__crt_stdio_output@@QEAA@AEBV?$string_output_adapter@_W@1@_KQEB_WQEAU__crt_locale_pointers@@QEAD@Z 0000000180018b70 f i libucrt:output.obj
 0001:00017bf0       ??0_LocaleUpdate@@QEAA@QEAU__crt_locale_pointers@@@Z 0000000180018bf0 f i libucrt:output.obj
 0001:00017c80       ?force_decimal_point@__crt_stdio_output@@YAXPEADQEAU__crt_locale_pointers@@@Z 0000000180018c80 f i libucrt:output.obj
 0001:00017cf0       ?parse_int_from_format_string@?$output_processor@DV?$string_output_adapter@D@__crt_stdio_output@@V?$standard_base@DV?$string_output_adapter@D@__crt_stdio_output@@@2@@__crt_stdio_output@@AEAA_NQEAH@Z 0000000180018cf0 f i libucrt:output.obj
 0001:00017d74       ?parse_int_from_format_string@?$output_processor@_WV?$string_output_adapter@_W@__crt_stdio_output@@V?$standard_base@_WV?$string_output_adapter@_W@__crt_stdio_output@@@2@@__crt_stdio_output@@AEAA_NQEAH@Z 0000000180018d74 f i libucrt:output.obj
 0001:00017df4       ?process@?$output_processor@DV?$string_output_adapter@D@__crt_stdio_output@@V?$standard_base@DV?$string_output_adapter@D@__crt_stdio_output@@@2@@__crt_stdio_output@@QEAAHXZ 0000000180018df4 f i libucrt:output.obj
 0001:00017ff8       ?process@?$output_processor@_WV?$string_output_adapter@_W@__crt_stdio_output@@V?$standard_base@_WV?$string_output_adapter@_W@__crt_stdio_output@@@2@@__crt_stdio_output@@QEAAHXZ 0000000180018ff8 f i libucrt:output.obj
 0001:00018274       ?state_case_normal@?$output_processor@DV?$string_output_adapter@D@__crt_stdio_output@@V?$standard_base@DV?$string_output_adapter@D@__crt_stdio_output@@@2@@__crt_stdio_output@@AEAA_NXZ 0000000180019274 f i libucrt:output.obj
 0001:000182e8       ?state_case_normal_tchar@?$output_processor@DV?$string_output_adapter@D@__crt_stdio_output@@V?$standard_base@DV?$string_output_adapter@D@__crt_stdio_output@@@2@@__crt_stdio_output@@AEAA_ND@Z 00000001800192e8 f i libucrt:output.obj
 0001:00018380       ?state_case_size@?$output_processor@DV?$string_output_adapter@D@__crt_stdio_output@@V?$standard_base@DV?$string_output_adapter@D@__crt_stdio_output@@@2@@__crt_stdio_output@@AEAA_NXZ 0000000180019380 f i libucrt:output.obj
 0001:000184fc       ?state_case_size@?$output_processor@_WV?$string_output_adapter@_W@__crt_stdio_output@@V?$standard_base@_WV?$string_output_adapter@_W@__crt_stdio_output@@@2@@__crt_stdio_output@@AEAA_NXZ 00000001800194fc f i libucrt:output.obj
 0001:000186a0       ?state_case_type@?$output_processor@DV?$string_output_adapter@D@__crt_stdio_output@@V?$standard_base@DV?$string_output_adapter@D@__crt_stdio_output@@@2@@__crt_stdio_output@@AEAA_NXZ 00000001800196a0 f i libucrt:output.obj
 0001:0001891c       ?state_case_type@?$output_processor@_WV?$string_output_adapter@_W@__crt_stdio_output@@V?$standard_base@_WV?$string_output_adapter@_W@__crt_stdio_output@@@2@@__crt_stdio_output@@AEAA_NXZ 000000018001991c f i libucrt:output.obj
 0001:00018be8       ?type_case_Z@?$output_processor@DV?$string_output_adapter@D@__crt_stdio_output@@V?$standard_base@DV?$string_output_adapter@D@__crt_stdio_output@@@2@@__crt_stdio_output@@AEAA_NXZ 0000000180019be8 f i libucrt:output.obj
 0001:00018c68       ?type_case_Z@?$output_processor@_WV?$string_output_adapter@_W@__crt_stdio_output@@V?$standard_base@_WV?$string_output_adapter@_W@__crt_stdio_output@@@2@@__crt_stdio_output@@AEAA_NXZ 0000000180019c68 f i libucrt:output.obj
 0001:00018ce8       ?type_case_a@?$output_processor@DV?$string_output_adapter@D@__crt_stdio_output@@V?$standard_base@DV?$string_output_adapter@D@__crt_stdio_output@@@2@@__crt_stdio_output@@AEAA_NXZ 0000000180019ce8 f i libucrt:output.obj
 0001:00018f04       ?type_case_a@?$output_processor@_WV?$string_output_adapter@_W@__crt_stdio_output@@V?$standard_base@_WV?$string_output_adapter@_W@__crt_stdio_output@@@2@@__crt_stdio_output@@AEAA_NXZ 0000000180019f04 f i libucrt:output.obj
 0001:00019148       ?type_case_c_tchar@?$output_processor@DV?$string_output_adapter@D@__crt_stdio_output@@V?$standard_base@DV?$string_output_adapter@D@__crt_stdio_output@@@2@@__crt_stdio_output@@AEAA_ND@Z 000000018001a148 f i libucrt:output.obj
 0001:000191fc       ?type_case_c_tchar@?$output_processor@_WV?$string_output_adapter@_W@__crt_stdio_output@@V?$standard_base@_WV?$string_output_adapter@_W@__crt_stdio_output@@@2@@__crt_stdio_output@@AEAA_N_W@Z 000000018001a1fc f i libucrt:output.obj
 0001:000192a4       ?type_case_integer@?$output_processor@_WV?$string_output_adapter@_W@__crt_stdio_output@@V?$standard_base@_WV?$string_output_adapter@_W@__crt_stdio_output@@@2@@__crt_stdio_output@@AEAA_NI_N@Z 000000018001a2a4 f i libucrt:output.obj
 0001:000192a4       ?type_case_integer@?$output_processor@DV?$string_output_adapter@D@__crt_stdio_output@@V?$standard_base@DV?$string_output_adapter@D@__crt_stdio_output@@@2@@__crt_stdio_output@@AEAA_NI_N@Z 000000018001a2a4 f i libucrt:output.obj
 0001:00019444       ?type_case_n@?$output_processor@DV?$string_output_adapter@D@__crt_stdio_output@@V?$standard_base@DV?$string_output_adapter@D@__crt_stdio_output@@@2@@__crt_stdio_output@@AEAA_NXZ 000000018001a444 f i libucrt:output.obj
 0001:00019444       ?type_case_n@?$output_processor@_WV?$string_output_adapter@_W@__crt_stdio_output@@V?$standard_base@_WV?$string_output_adapter@_W@__crt_stdio_output@@@2@@__crt_stdio_output@@AEAA_NXZ 000000018001a444 f i libucrt:output.obj
 0001:00019520       ?type_case_s@?$output_processor@DV?$string_output_adapter@D@__crt_stdio_output@@V?$standard_base@DV?$string_output_adapter@D@__crt_stdio_output@@@2@@__crt_stdio_output@@AEAA_NXZ 000000018001a520 f i libucrt:output.obj
 0001:000195b0       ?type_case_s@?$output_processor@_WV?$string_output_adapter@_W@__crt_stdio_output@@V?$standard_base@_WV?$string_output_adapter@_W@__crt_stdio_output@@@2@@__crt_stdio_output@@AEAA_NXZ 000000018001a5b0 f i libucrt:output.obj
 0001:00019678       ?write_stored_string_tchar@?$output_processor@DV?$string_output_adapter@D@__crt_stdio_output@@V?$standard_base@DV?$string_output_adapter@D@__crt_stdio_output@@@2@@__crt_stdio_output@@AEAA_ND@Z 000000018001a678 f i libucrt:output.obj
 0001:00019750       ?write_stored_string_tchar@?$output_processor@_WV?$string_output_adapter@_W@__crt_stdio_output@@V?$standard_base@_WV?$string_output_adapter@_W@__crt_stdio_output@@@2@@__crt_stdio_output@@AEAA_N_W@Z 000000018001a750 f i libucrt:output.obj
 0001:00019840       ?write_string@?$string_output_adapter@D@__crt_stdio_output@@QEBAXQEBDHQEAH1@Z 000000018001a840 f i libucrt:output.obj
 0001:000198fc       ?write_string@?$string_output_adapter@_W@__crt_stdio_output@@QEBAXQEB_WHQEAH1@Z 000000018001a8fc f i libucrt:output.obj
 0001:000199bc       __stdio_common_vsprintf    000000018001a9bc f   libucrt:output.obj
 0001:00019bf0       __stdio_common_vswprintf   000000018001abf0 f   libucrt:output.obj
 0001:00019e28       wcsncmp                    000000018001ae28 f   libucrt:wcsncmp.obj
 0001:00019e54       ??$is_overflow_condition@K@__crt_strtox@@YA_NIK@Z 000000018001ae54 f i libucrt:strtox.obj
 0001:00019e80       ??$make_c_string_character_source@DPEAPEAD@__crt_strtox@@YA?AV?$c_string_character_source@D@0@QEBDQEAPEAD@Z 000000018001ae80 f i libucrt:strtox.obj
 0001:00019e80       ??$make_c_string_character_source@_WPEAPEA_W@__crt_strtox@@YA?AV?$c_string_character_source@_W@0@QEB_WQEAPEA_W@Z 000000018001ae80 f i libucrt:strtox.obj
 0001:00019e94       ??$parse_integer@KV?$c_string_character_source@D@__crt_strtox@@@__crt_strtox@@YAKQEAU__crt_locale_pointers@@V?$c_string_character_source@D@0@H_N@Z 000000018001ae94 f i libucrt:strtox.obj
 0001:0001a1a8       ??$parse_integer@KV?$c_string_character_source@_W@__crt_strtox@@@__crt_strtox@@YAKQEAU__crt_locale_pointers@@V?$c_string_character_source@_W@0@H_N@Z 000000018001b1a8 f i libucrt:strtox.obj
 0001:0001a87c       strtol                     000000018001b87c f   libucrt:strtox.obj
 0001:0001a8ac       wcstol                     000000018001b8ac f   libucrt:strtox.obj
 0001:0001a8dc       wcspbrk                    000000018001b8dc f   libucrt:wcspbrk.obj
 0001:0001a914       _initterm                  000000018001b914 f   libucrt:initterm.obj
 0001:0001a98c       _initterm_e                000000018001b98c f   libucrt:initterm.obj
 0001:0001a9d8       _seh_filter_dll            000000018001b9d8 f   libucrt:exception_filter.obj
 0001:0001a9ec       _seh_filter_exe            000000018001b9ec f   libucrt:exception_filter.obj
 0001:0001adac       __acrt_initialize_thread_local_exit_callback 000000018001bdac f   libucrt:exit.obj
 0001:0001adb4       _cexit                     000000018001bdb4 f   libucrt:exit.obj
 0001:0001adc4       _exit                      000000018001bdc4 f   libucrt:exit.obj
 0001:0001add0       _is_c_termination_complete 000000018001bdd0 f   libucrt:exit.obj
 0001:0001af94       __acrt_allocate_buffer_for_argv 000000018001bf94 f   libucrt:argv_parsing.obj
 0001:0001aff8       _configure_narrow_argv     000000018001bff8 f   libucrt:argv_parsing.obj
 0001:0001b354       __dcrt_uninitialize_environments_nolock 000000018001c354 f   libucrt:environment_initialization.obj
 0001:0001b38c       _initialize_narrow_environment 000000018001c38c f   libucrt:environment_initialization.obj
 0001:0001b394       ??$?RV<lambda_e24bbb7b643b32fcea6fa61b31d4c984>@@AEAV<lambda_275893d493268fdec8709772e3fcec0e>@@V<lambda_9d71df4d7cf3f480f8d633942495c3b0>@@@?$__crt_seh_guarded_call@H@@QEAAH$$QEAV<lambda_e24bbb7b643b32fcea6fa61b31d4c984>@@AEAV<lambda_275893d493268fdec8709772e3fcec0e>@@$$QEAV<lambda_9d71df4d7cf3f480f8d633942495c3b0>@@@Z 000000018001c394 f i libucrt:onexit.obj
 0001:0001b534       _execute_onexit_table      000000018001c534 f   libucrt:onexit.obj
 0001:0001b570       _initialize_onexit_table   000000018001c570 f   libucrt:onexit.obj
 0001:0001b6e4       __acrt_initialize          000000018001c6e4 f   libucrt:initialization.obj
 0001:0001b6f8       __acrt_thread_attach       000000018001c6f8 f   libucrt:initialization.obj
 0001:0001b70c       __acrt_thread_detach       000000018001c70c f   libucrt:initialization.obj
 0001:0001b71c       __acrt_uninitialize        000000018001c71c f   libucrt:initialization.obj
 0001:0001b730       __acrt_uninitialize_critical 000000018001c730 f   libucrt:initialization.obj
 0001:0001b740       terminate                  000000018001c740 f   libucrt:terminate.obj
 0001:0001b768       free                       000000018001c768 f   libucrt:free.obj
 0001:0001b770       malloc                     000000018001c770 f   libucrt:malloc.obj
 0001:0001b778       strcpy_s                   000000018001c778 f   libucrt:strcpy_s.obj
 0001:0001b7d8       abort                      000000018001c7d8 f   libucrt:abort.obj
 0001:0001b830       calloc                     000000018001c830 f   libucrt:calloc.obj
 0001:0001b850       strncmp                    000000018001c850 f   libucrt:strncmp.obj
 0001:0001b8d0       __acrt_call_reportfault    000000018001c8d0 f   libucrt:invalid_parameter.obj
 0001:0001ba2c       __acrt_initialize_invalid_parameter_handler 000000018001ca2c f   libucrt:invalid_parameter.obj
 0001:0001ba34       _invalid_parameter         000000018001ca34 f   libucrt:invalid_parameter.obj
 0001:0001badc       _invalid_parameter_noinfo  000000018001cadc f   libucrt:invalid_parameter.obj
 0001:0001bafc       _invoke_watson             000000018001cafc f   libucrt:invalid_parameter.obj
 0001:0001bb44       isdigit                    000000018001cb44 f i libucrt:_ctype.obj
 0001:0001bc08       _tolower_l                 000000018001cc08 f   libucrt:tolower_toupper.obj
 0001:0001bd48       tolower                    000000018001cd48 f   libucrt:tolower_toupper.obj
 0001:0001bd74       __acrt_errno_from_os_error 000000018001cd74 f   libucrt:errno.obj
 0001:0001bdbc       __acrt_errno_map_os_error  000000018001cdbc f   libucrt:errno.obj
 0001:0001be0c       __doserrno                 000000018001ce0c f   libucrt:errno.obj
 0001:0001be2c       _errno                     000000018001ce2c f   libucrt:errno.obj
 0001:0001be4c       _free_base                 000000018001ce4c f   libucrt:free_base.obj
 0001:0001be8c       _malloc_base               000000018001ce8c f   libucrt:malloc_base.obj
 0001:0001beec       _mbtowc_l                  000000018001ceec f   libucrt:mbtowc.obj
 0001:0001c034       mbtowc                     000000018001d034 f   libucrt:mbtowc.obj
 0001:0001c03c       _wctomb_s_l                000000018001d03c f   libucrt:wctomb.obj
 0001:0001c1c0       wctomb_s                   000000018001d1c0 f   libucrt:wctomb.obj
 0001:0001c1d4       strnlen                    000000018001d1d4 f   libucrt:strnlen.obj
 0001:0001c330       wcsnlen                    000000018001d330 f   libucrt:strnlen.obj
 0001:0001c520       ??$?RV<lambda_46352004c1216016012b18bd6f87e700>@@AEAV<lambda_3bd07e1a1191394380780325891bf33f>@@V<lambda_334532d3f185bcaa59b5be82d7d22bff>@@@?$__crt_seh_guarded_call@X@@QEAAX$$QEAV<lambda_46352004c1216016012b18bd6f87e700>@@AEAV<lambda_3bd07e1a1191394380780325891bf33f>@@$$QEAV<lambda_334532d3f185bcaa59b5be82d7d22bff>@@@Z 000000018001d520 f i libucrt:per_thread_data.obj
 0001:0001c580       ??$?RV<lambda_5e887d1dcbef67a5eb4283622ba103bf>@@AEAV<lambda_4466841279450cc726390878d4a41900>@@V<lambda_341c25c0346d94847f1f3c463c57e077>@@@?$__crt_seh_guarded_call@X@@QEAAX$$QEAV<lambda_5e887d1dcbef67a5eb4283622ba103bf>@@AEAV<lambda_4466841279450cc726390878d4a41900>@@$$QEAV<lambda_341c25c0346d94847f1f3c463c57e077>@@@Z 000000018001d580 f i libucrt:per_thread_data.obj
 0001:0001c5c8       ??$?RV<lambda_72d1df2b273a38828b1ce30cbf4cdab5>@@AEAV<lambda_876a65b173b8412d3a47c70a915b0cf4>@@V<lambda_41932305e351933ebe8f8be3ed8bb5dc>@@@?$__crt_seh_guarded_call@X@@QEAAX$$QEAV<lambda_72d1df2b273a38828b1ce30cbf4cdab5>@@AEAV<lambda_876a65b173b8412d3a47c70a915b0cf4>@@$$QEAV<lambda_41932305e351933ebe8f8be3ed8bb5dc>@@@Z 000000018001d5c8 f i libucrt:per_thread_data.obj
 0001:0001c608       ??$?RV<lambda_fb3a7dec4e47f37f22dae91bb15c9095>@@AEAV<lambda_698284760c8add0bfb0756c19673e34b>@@V<lambda_dfb8eca1e75fef3034a8fb18dd509707>@@@?$__crt_seh_guarded_call@X@@QEAAX$$QEAV<lambda_fb3a7dec4e47f37f22dae91bb15c9095>@@AEAV<lambda_698284760c8add0bfb0756c19673e34b>@@$$QEAV<lambda_dfb8eca1e75fef3034a8fb18dd509707>@@@Z 000000018001d608 f i libucrt:per_thread_data.obj
 0001:0001c898       __acrt_freeptd             000000018001d898 f   libucrt:per_thread_data.obj
 0001:0001c8dc       __acrt_getptd              000000018001d8dc f   libucrt:per_thread_data.obj
 0001:0001c970       __acrt_getptd_noexit       000000018001d970 f   libucrt:per_thread_data.obj
 0001:0001ca10       __acrt_initialize_ptd      000000018001da10 f   libucrt:per_thread_data.obj
 0001:0001ca4c       __acrt_uninitialize_ptd    000000018001da4c f   libucrt:per_thread_data.obj
 0001:0001ca70       __acrt_update_locale_info  000000018001da70 f   libucrt:locale_update.obj
 0001:0001caa4       __acrt_update_multibyte_info 000000018001daa4 f   libucrt:locale_update.obj
 0001:0001cad8       ?__acrt_fp_classify@@YA?AW4__acrt_fp_class@@AEBN@Z 000000018001dad8 f i libucrt:cvt.obj
 0001:0001d510       __acrt_fp_format           000000018001e510 f   libucrt:cvt.obj
 0001:0001d754       _fileno                    000000018001e754 f   libucrt:fileno.obj
 0001:0001d77c       __acrt_initialize_stdio    000000018001e77c f   libucrt:_file.obj
 0001:0001d89c       __acrt_uninitialize_stdio  000000018001e89c f   libucrt:_file.obj
 0001:0001d8f8       _lock_file                 000000018001e8f8 f   libucrt:_file.obj
 0001:0001d904       _unlock_file               000000018001e904 f   libucrt:_file.obj
 0001:0001d910       _get_printf_count_output   000000018001e910 f   libucrt:printf_count_output.obj
 0001:0001d928       __acrt_set_locale_changed  000000018001e928 f   libucrt:wsetlocale.obj
 0001:0001d934       __acrt_uninitialize_locale 000000018001e934 f   libucrt:wsetlocale.obj
 0001:0001db64       __acrt_initialize_lowio    000000018001eb64 f   libucrt:ioinit.obj
 0001:0001dba0       __acrt_uninitialize_lowio  000000018001eba0 f   libucrt:ioinit.obj
 0001:0001dbe0       __pctype_func              000000018001ebe0 f   libucrt:ctype.obj
 0001:0001dc10       iswctype                   000000018001ec10 f   libucrt:iswctype.obj
 0001:0001dc80       _isctype_l                 000000018001ec80 f   libucrt:isctype.obj
 0001:0001dd90       __acrt_initialize_locks    000000018001ed90 f   libucrt:locks.obj
 0001:0001ddd8       __acrt_lock                000000018001edd8 f   libucrt:locks.obj
 0001:0001ddf4       __acrt_uninitialize_locks  000000018001edf4 f   libucrt:locks.obj
 0001:0001de2c       __acrt_unlock              000000018001ee2c f   libucrt:locks.obj
 0001:0001dfe8       __acrt_FlsAlloc            000000018001efe8 f   libucrt:winapi_thunks.obj
 0001:0001e040       __acrt_FlsFree             000000018001f040 f   libucrt:winapi_thunks.obj
 0001:0001e098       __acrt_FlsGetValue         000000018001f098 f   libucrt:winapi_thunks.obj
 0001:0001e0f0       __acrt_FlsSetValue         000000018001f0f0 f   libucrt:winapi_thunks.obj
 0001:0001e158       __acrt_InitializeCriticalSectionEx 000000018001f158 f   libucrt:winapi_thunks.obj
 0001:0001e1d0       __acrt_LCMapStringEx       000000018001f1d0 f   libucrt:winapi_thunks.obj
 0001:0001e2c0       __acrt_LocaleNameToLCID    000000018001f2c0 f   libucrt:winapi_thunks.obj
 0001:0001e328       __acrt_initialize_winapi_thunks 000000018001f328 f   libucrt:winapi_thunks.obj
 0001:0001e360       __acrt_is_packaged_app     000000018001f360 f   libucrt:winapi_thunks.obj
 0001:0001e3e8       __acrt_uninitialize_winapi_thunks 000000018001f3e8 f   libucrt:winapi_thunks.obj
 0001:0001e42c       _calloc_base               000000018001f42c f   libucrt:calloc_base.obj
 0001:0001e980       ?expand_if_necessary@?$argument_list@D@?A0xca0879c4@@AEAAHXZ 000000018001f980 f i libucrt:argv_wildcards.obj
 0001:0001ea48       __acrt_expand_narrow_argv_wildcards 000000018001fa48 f   libucrt:argv_wildcards.obj
 0001:0001ea50       ??$?RV<lambda_99476a1ad63dd22509b5d3e65b0ffc95>@@AEAV<lambda_ad1ced32f4ac17aa236e5ef05d6b3b7c>@@V<lambda_f7424dd8d45958661754dc4f2697e9c3>@@@?$__crt_seh_guarded_call@X@@QEAAX$$QEAV<lambda_99476a1ad63dd22509b5d3e65b0ffc95>@@AEAV<lambda_ad1ced32f4ac17aa236e5ef05d6b3b7c>@@$$QEAV<lambda_f7424dd8d45958661754dc4f2697e9c3>@@@Z 000000018001fa50 f i libucrt:mbctype.obj
 0001:0001f14c       __acrt_initialize_multibyte 000000018002014c f   libucrt:mbctype.obj
 0001:0001f174       __acrt_update_thread_multibyte_data 0000000180020174 f   libucrt:mbctype.obj
 0001:0001f234       _setmbcp_nolock            0000000180020234 f   libucrt:mbctype.obj
 0001:0001f554       _ismbblead                 0000000180020554 f   libucrt:ismbbyte.obj
 0001:0001f568       __acrt_initialize_command_line 0000000180020568 f   libucrt:argv_data.obj
 0001:0001f590       __dcrt_get_narrow_environment_from_os 0000000180020590 f   libucrt:get_environment_from_os.obj
 0001:0001f694       _recalloc                  0000000180020694 f   libucrt:recalloc.obj
 0001:0001f69c       _recalloc_base             000000018002069c f   libucrt:recalloc.obj
 0001:0001f734       __acrt_initialize_heap     0000000180020734 f   libucrt:heap_handle.obj
 0001:0001f750       __acrt_uninitialize_heap   0000000180020750 f   libucrt:heap_handle.obj
 0001:0001f75c       __acrt_execute_initializers 000000018002075c f   libucrt:shared_initialization.obj
 0001:0001f7f0       __acrt_execute_uninitializers 00000001800207f0 f   libucrt:shared_initialization.obj
 0001:0001f840       __acrt_initialize_new_handler 0000000180020840 f   libucrt:new_handler.obj
 0001:0001f848       _callnewh                  0000000180020848 f   libucrt:new_handler.obj
 0001:0001f888       _query_new_handler         0000000180020888 f   libucrt:new_handler.obj
 0001:0001f8bc       ??$?RV<lambda_c36588078e9f5dfd39652860aa6b3aaf>@@AEAV<lambda_ec61778202f4f5fc7e7711acc23c3bca>@@V<lambda_dc9d2797ccde5d239b4a0efae8ebd7db>@@@?$__crt_seh_guarded_call@P6AXH@Z@@QEAAP6AXH@Z$$QEAV<lambda_c36588078e9f5dfd39652860aa6b3aaf>@@AEAV<lambda_ec61778202f4f5fc7e7711acc23c3bca>@@$$QEAV<lambda_dc9d2797ccde5d239b4a0efae8ebd7db>@@@Z 00000001800208bc f i libucrt:signal.obj
 0001:0001f904       __acrt_get_sigabrt_handler 0000000180020904 f   libucrt:signal.obj
 0001:0001f934       __acrt_initialize_signal_handlers 0000000180020934 f   libucrt:signal.obj
 0001:0001f954       raise                      0000000180020954 f   libucrt:signal.obj
 0001:0001fbf0       __acrt_has_user_matherr    0000000180020bf0 f   libucrt:matherr.obj
 0001:0001fc10       __acrt_initialize_user_matherr 0000000180020c10 f   libucrt:matherr.obj
 0001:0001fc18       __acrt_invoke_user_matherr 0000000180020c18 f   libucrt:matherr.obj
 0001:0001fc60       _isleadbyte_l              0000000180020c60 f i libucrt:_wctype.obj
 0001:0001fffc       __acrt_LCMapStringA        0000000180020ffc f   libucrt:lcmapstringa.obj
 0001:00020094       _query_new_mode            0000000180021094 f   libucrt:new_mode.obj
 0001:0002009c       __acrt_add_locale_ref      000000018002109c f   libucrt:locale_refcounting.obj
 0001:00020128       __acrt_free_locale         0000000180021128 f   libucrt:locale_refcounting.obj
 0001:000202a0       __acrt_locale_add_lc_time_reference 00000001800212a0 f   libucrt:locale_refcounting.obj
 0001:000202c8       __acrt_locale_free_lc_time_if_unreferenced 00000001800212c8 f   libucrt:locale_refcounting.obj
 0001:00020300       __acrt_locale_release_lc_time_reference 0000000180021300 f   libucrt:locale_refcounting.obj
 0001:00020328       __acrt_release_locale_ref  0000000180021328 f   libucrt:locale_refcounting.obj
 0001:000203d0       __acrt_update_thread_locale_data 00000001800213d0 f   libucrt:locale_refcounting.obj
 0001:00020440       _updatetlocinfoEx_nolock   0000000180021440 f   libucrt:locale_refcounting.obj
 0001:000204a8       __acrt_fp_strflt_to_string 00000001800214a8 f   libucrt:_fptostr.obj
 0001:00020570       ?divide@__crt_strtox@@YA_KAEAUbig_integer@1@AEBU21@@Z 0000000180021570 f i libucrt:cfout.obj
 0001:00020a40       __acrt_fltout              0000000180021a40 f   libucrt:cfout.obj
 0001:00021e34       _fcloseall                 0000000180022e34 f   libucrt:closeall.obj
 0001:00021ee8       __acrt_stdio_flush_nolock  0000000180022ee8 f   libucrt:fflush.obj
 0001:00021f60       _fflush_nolock             0000000180022f60 f   libucrt:fflush.obj
 0001:00021fac       _flushall                  0000000180022fac f   libucrt:fflush.obj
 0001:0002209c       __acrt_stdio_free_buffer_nolock 000000018002309c f   libucrt:_freebuf.obj
 0001:000220dc       _isatty                    00000001800230dc f   libucrt:isatty.obj
 0001:0002213c       __acrt_locale_free_monetary 000000018002313c f   libucrt:initmon.obj
 0001:00022248       __acrt_locale_free_numeric 0000000180023248 f   libucrt:initnum.obj
 0001:0002230c       __acrt_locale_free_time    000000018002330c f   libucrt:inittime.obj
 0001:00022414       __acrt_GetStringTypeA      0000000180023414 f   libucrt:getstringtypea.obj
 0001:000225c8       __acrt_lowio_create_handle_array 00000001800235c8 f   libucrt:osfinfo.obj
 0001:00022660       __acrt_lowio_destroy_handle_array 0000000180023660 f   libucrt:osfinfo.obj
 0001:000226b0       __acrt_lowio_ensure_fh_exists 00000001800236b0 f   libucrt:osfinfo.obj
 0001:00022768       __acrt_lowio_lock_fh       0000000180023768 f   libucrt:osfinfo.obj
 0001:0002278c       __acrt_lowio_unlock_fh     000000018002378c f   libucrt:osfinfo.obj
 0001:000227b0       _free_osfhnd               00000001800237b0 f   libucrt:osfinfo.obj
 0001:0002286c       _get_osfhandle             000000018002386c f   libucrt:osfinfo.obj
 0001:000229ac       __acrt_DownlevelLocaleNameToLCID 00000001800239ac f   libucrt:lcidtoname_downlevel.obj
 0001:00022ab0       qsort                      0000000180023ab0 f   libucrt:qsort.obj
 0001:00022de4       strncpy_s                  0000000180023de4 f   libucrt:strncpy_s.obj
 0001:00022eb8       strpbrk                    0000000180023eb8 f   libucrt:strpbrk.obj
 0001:00022f58       _mbsdec                    0000000180023f58 f   libucrt:mbsdec.obj
 0001:00022f60       _mbsdec_l                  0000000180023f60 f   libucrt:mbsdec.obj
 0001:00023010       _msize                     0000000180024010 f   libucrt:msize.obj
 0001:0002304c       _realloc_base              000000018002404c f   libucrt:realloc_base.obj
 0001:000230d0       __strncnt                  00000001800240d0 f   libucrt:strncnt.obj
 0001:000230e8       fegetenv                   00000001800240e8 f   libucrt:fegetenv.obj
 0001:00023108       fesetenv                   0000000180024108 f   libucrt:fesetenv.obj
 0001:00023154       feholdexcept               0000000180024154 f   libucrt:feholdexcept.obj
 0001:000231a4       ceil                       00000001800241a4 f   libucrt:ceil.obj
 0001:00023270       log10                      0000000180024270 f   libucrt:log10.obj
 0001:00023dbc       _write                     0000000180024dbc f   libucrt:write.obj
 0001:00023ea8       _write_nolock              0000000180024ea8 f   libucrt:write.obj
 0001:00024228       _lseeki64_nolock           0000000180025228 f   libucrt:lseek.obj
 0001:00024230       _fclose_nolock             0000000180025230 f   libucrt:fclose.obj
 0001:000242b4       fclose                     00000001800252b4 f   libucrt:fclose.obj
 0001:00024320       ??$?RV<lambda_b521505b218e5242e90febf6bfebc422>@@AEAV<lambda_6978c1fb23f02e42e1d9e99668cc68aa>@@V<lambda_314360699dd331753a4119843814e9a7>@@@?$__crt_seh_guarded_call@H@@QEAAH$$QEAV<lambda_b521505b218e5242e90febf6bfebc422>@@AEAV<lambda_6978c1fb23f02e42e1d9e99668cc68aa>@@$$QEAV<lambda_314360699dd331753a4119843814e9a7>@@@Z 0000000180025320 f i libucrt:commit.obj
 0001:000243ac       _commit                    00000001800253ac f   libucrt:commit.obj
 0001:00024440       _query_app_type            0000000180025440 f   libucrt:report_runtime_error.obj
 0001:00024448       _getfpcontrolword          0000000180025448 f   libucrt:_fenvutils.obj
 0001:00024460       _getfpstatusword           0000000180025460 f   libucrt:_fenvutils.obj
 0001:00024474       _setfpcontrolword          0000000180025474 f   libucrt:_fenvutils.obj
 0001:00024480       _setfpstatusword           0000000180025480 f   libucrt:_fenvutils.obj
 0001:000244d0       _clearfp                   00000001800254d0 f   libucrt:ieee.obj
 0001:00024524       _controlfp                 0000000180025524 f   libucrt:ieee.obj
 0001:00024530       _statusfp                  0000000180025530 f   libucrt:ieee.obj
 0001:00024934       _handle_error              0000000180025934 f   libucrt:libm_error.obj
 0001:00024a5c       _handle_nan                0000000180025a5c f   libucrt:libm_error.obj
 0001:00024a80       __acrt_initialize_fma3     0000000180025a80 f   libucrt:fma3_available.obj
 0001:00024af0       _log10_special             0000000180025af0 f   libucrt:log_special.obj
 0001:00024ba8       _putwch_nolock             0000000180025ba8 f   libucrt:putwch.obj
 0001:00024c04       ??$?RV<lambda_bfedae4ebbf01fab1bb6dcc6a9e276e0>@@AEAV<lambda_2fe9b910cf3cbf4a0ab98a02ba45b3ec>@@V<lambda_237c231691f317818eb88cc1d5d642d6>@@@?$__crt_seh_guarded_call@H@@QEAAH$$QEAV<lambda_bfedae4ebbf01fab1bb6dcc6a9e276e0>@@AEAV<lambda_2fe9b910cf3cbf4a0ab98a02ba45b3ec>@@$$QEAV<lambda_237c231691f317818eb88cc1d5d642d6>@@@Z 0000000180025c04 f i libucrt:close.obj
 0001:00024c78       _close                     0000000180025c78 f   libucrt:close.obj
 0001:00024d1c       _close_nolock              0000000180025d1c f   libucrt:close.obj
 0001:00024dd8       ?__acrt_stdio_free_stream@@YAXV__crt_stdio_stream@@@Z 0000000180025dd8 f   libucrt:stream.obj
 0001:00024e30       _get_fpsr                  0000000180025e30 f   libucrt:fpsr.obj
 0001:00024e40       _set_fpsr                  0000000180025e40 f   libucrt:fpsr.obj
 0001:00024e4a       _fclrf                     0000000180025e4a f   libucrt:fpsr.obj
 0001:00024e5e       _frnd                      0000000180025e5e f   libucrt:fpsr.obj
 0001:00024e80       _raise_exc                 0000000180025e80 f   libucrt:fpexcept.obj
 0001:00024ea8       _raise_exc_ex              0000000180025ea8 f   libucrt:fpexcept.obj
 0001:000251b0       _set_errno_from_matherr    00000001800261b0 f   libucrt:fpexcept.obj
 0001:000251e0       _clrfp                     00000001800261e0 f   libucrt:fpctrl.obj
 0001:00025200       _ctrlfp                    0000000180026200 f   libucrt:fpctrl.obj
 0001:0002527c       _set_statfp                000000018002627c f   libucrt:fpctrl.obj
 0001:0002529c       _statfp                    000000018002629c f   libucrt:fpctrl.obj
 0001:000252b0       __dcrt_lowio_initialize_console_output 00000001800262b0 f   libucrt:initcon.obj
 0001:000252ec       __dcrt_terminate_console_output 00000001800262ec f   libucrt:initcon.obj
 0001:0002530c       Process32FirstW            000000018002630c f   kernel32:KERNEL32.dll
 0001:00025312       Process32NextW             0000000180026312 f   kernel32:KERNEL32.dll
 0001:00025318       IsProcessorFeaturePresent  0000000180026318 f   kernel32:KERNEL32.dll
 0001:0002531e       RtlUnwindEx                000000018002631e f   kernel32:KERNEL32.dll
 0001:00025330       _FindPESection             0000000180026330 f   LIBCMT:pesect.obj
 0001:00025380       _IsNonwritableInCurrentImage 0000000180026380 f   LIBCMT:pesect.obj
 0001:000253d0       _ValidateImageBase         00000001800263d0 f   LIBCMT:pesect.obj
 0001:00025410       _alloca_probe              0000000180026410 f   LIBCMT:_chkstk_.obj
 0001:00025410       __chkstk                   0000000180026410 f   LIBCMT:_chkstk_.obj
 0001:00025480       _guard_dispatch_icall_nop  0000000180026480 f   LIBCMT:_guard_dispatch_.obj
 0002:00000000       __imp_RegSetValueExW       0000000180027000     advapi32:ADVAPI32.dll
 0002:00000008       __imp_RegQueryValueExW     0000000180027008     advapi32:ADVAPI32.dll
 0002:00000010       __imp_RegOpenKeyExW        0000000180027010     advapi32:ADVAPI32.dll
 0002:00000018       __imp_RegCreateKeyExW      0000000180027018     advapi32:ADVAPI32.dll
 0002:00000020       __imp_RegCloseKey          0000000180027020     advapi32:ADVAPI32.dll
 0002:00000028       \177ADVAPI32_NULL_THUNK_DATA 0000000180027028     advapi32:ADVAPI32.dll
 0002:00000030       __imp_GdiFlush             0000000180027030     gdi32:GDI32.dll
 0002:00000038       __imp_GetObjectW           0000000180027038     gdi32:GDI32.dll
 0002:00000040       __imp_CreateDIBSection     0000000180027040     gdi32:GDI32.dll
 0002:00000048       __imp_GdiAlphaBlend        0000000180027048     gdi32:GDI32.dll
 0002:00000050       __imp_SetStretchBltMode    0000000180027050     gdi32:GDI32.dll
 0002:00000058       __imp_StretchBlt           0000000180027058     gdi32:GDI32.dll
 0002:00000060       __imp_MoveToEx             0000000180027060     gdi32:GDI32.dll
 0002:00000068       __imp_SetTextColor         0000000180027068     gdi32:GDI32.dll
 0002:00000070       __imp_SetBkColor           0000000180027070     gdi32:GDI32.dll
 0002:00000078       __imp_SelectObject         0000000180027078     gdi32:GDI32.dll
 0002:00000080       __imp_Rectangle            0000000180027080     gdi32:GDI32.dll
 0002:00000088       __imp_LineTo               0000000180027088     gdi32:GDI32.dll
 0002:00000090       __imp_GetStockObject       0000000180027090     gdi32:GDI32.dll
 0002:00000098       __imp_DeleteObject         0000000180027098     gdi32:GDI32.dll
 0002:000000a0       __imp_DeleteDC             00000001800270a0     gdi32:GDI32.dll
 0002:000000a8       __imp_CreateSolidBrush     00000001800270a8     gdi32:GDI32.dll
 0002:000000b0       __imp_CreatePen            00000001800270b0     gdi32:GDI32.dll
 0002:000000b8       __imp_CreateFontW          00000001800270b8     gdi32:GDI32.dll
 0002:000000c0       __imp_CreateCompatibleDC   00000001800270c0     gdi32:GDI32.dll
 0002:000000c8       __imp_CreateCompatibleBitmap 00000001800270c8     gdi32:GDI32.dll
 0002:000000d0       __imp_BitBlt               00000001800270d0     gdi32:GDI32.dll
 0002:000000d8       \177GDI32_NULL_THUNK_DATA  00000001800270d8     gdi32:GDI32.dll
 0002:000000e0       __imp_GetExitCodeThread    00000001800270e0     kernel32:KERNEL32.dll
 0002:000000e8       __imp_SetEvent             00000001800270e8     kernel32:KERNEL32.dll
 0002:000000f0       __imp_WaitForMultipleObjects 00000001800270f0     kernel32:KERNEL32.dll
 0002:000000f8       __imp_Sleep                00000001800270f8     kernel32:KERNEL32.dll
 0002:00000100       __imp_FileTimeToSystemTime 0000000180027100     kernel32:KERNEL32.dll
 0002:00000108       __imp_CreateEventW         0000000180027108     kernel32:KERNEL32.dll
 0002:00000110       __imp_FreeLibrary          0000000180027110     kernel32:KERNEL32.dll
 0002:00000118       __imp_ResetEvent           0000000180027118     kernel32:KERNEL32.dll
 0002:00000120       __imp_FindClose            0000000180027120     kernel32:KERNEL32.dll
 0002:00000128       __imp_GetTickCount         0000000180027128     kernel32:KERNEL32.dll
 0002:00000130       __imp_LoadLibraryW         0000000180027130     kernel32:KERNEL32.dll
 0002:00000138       __imp_GetTempPathW         0000000180027138     kernel32:KERNEL32.dll
 0002:00000140       __imp_CreateFileW          0000000180027140     kernel32:KERNEL32.dll
 0002:00000148       __imp_FindFirstFileW       0000000180027148     kernel32:KERNEL32.dll
 0002:00000150       __imp_FindNextFileW        0000000180027150     kernel32:KERNEL32.dll
 0002:00000158       __imp_IsBadReadPtr         0000000180027158     kernel32:KERNEL32.dll
 0002:00000160       __imp_WriteConsoleW        0000000180027160     kernel32:KERNEL32.dll
 0002:00000168       __imp_FlushFileBuffers     0000000180027168     kernel32:KERNEL32.dll
 0002:00000170       __imp_SetFilePointerEx     0000000180027170     kernel32:KERNEL32.dll
 0002:00000178       __imp_GetConsoleMode       0000000180027178     kernel32:KERNEL32.dll
 0002:00000180       __imp_GetConsoleCP         0000000180027180     kernel32:KERNEL32.dll
 0002:00000188       __imp_HeapSize             0000000180027188     kernel32:KERNEL32.dll
 0002:00000190       __imp_SetStdHandle         0000000180027190     kernel32:KERNEL32.dll
 0002:00000198       __imp_GetProcessHeap       0000000180027198     kernel32:KERNEL32.dll
 0002:000001a0       __imp_LocalAlloc           00000001800271a0     kernel32:KERNEL32.dll
 0002:000001a8       __imp_FreeEnvironmentStringsW 00000001800271a8     kernel32:KERNEL32.dll
 0002:000001b0       __imp_GetEnvironmentStringsW 00000001800271b0     kernel32:KERNEL32.dll
 0002:000001b8       __imp_GetCommandLineW      00000001800271b8     kernel32:KERNEL32.dll
 0002:000001c0       __imp_GetCommandLineA      00000001800271c0     kernel32:KERNEL32.dll
 0002:000001c8       __imp_GetCPInfo            00000001800271c8     kernel32:KERNEL32.dll
 0002:000001d0       __imp_GetOEMCP             00000001800271d0     kernel32:KERNEL32.dll
 0002:000001d8       __imp_IsValidCodePage      00000001800271d8     kernel32:KERNEL32.dll
 0002:000001e0       __imp_FindNextFileA        00000001800271e0     kernel32:KERNEL32.dll
 0002:000001e8       __imp_FindFirstFileExA     00000001800271e8     kernel32:KERNEL32.dll
 0002:000001f0       __imp_LCMapStringW         00000001800271f0     kernel32:KERNEL32.dll
 0002:000001f8       __imp_GetStringTypeW       00000001800271f8     kernel32:KERNEL32.dll
 0002:00000200       __imp_GetFileType          0000000180027200     kernel32:KERNEL32.dll
 0002:00000208       __imp_GetACP               0000000180027208     kernel32:KERNEL32.dll
 0002:00000210       __imp_GetModuleFileNameA   0000000180027210     kernel32:KERNEL32.dll
 0002:00000218       __imp_GetModuleHandleExW   0000000180027218     kernel32:KERNEL32.dll
 0002:00000220       __imp_ExitProcess          0000000180027220     kernel32:KERNEL32.dll
 0002:00000228       __imp_RtlPcToFileHeader    0000000180027228     kernel32:KERNEL32.dll
 0002:00000230       __imp_LoadLibraryExW       0000000180027230     kernel32:KERNEL32.dll
 0002:00000238       __imp_TlsFree              0000000180027238     kernel32:KERNEL32.dll
 0002:00000240       __imp_MultiByteToWideChar  0000000180027240     kernel32:KERNEL32.dll
 0002:00000248       __imp_lstrlenA             0000000180027248     kernel32:KERNEL32.dll
 0002:00000250       __imp_lstrcpynA            0000000180027250     kernel32:KERNEL32.dll
 0002:00000258       __imp_lstrcmpW             0000000180027258     kernel32:KERNEL32.dll
 0002:00000260       __imp_Thread32Next         0000000180027260     kernel32:KERNEL32.dll
 0002:00000268       __imp_Thread32First        0000000180027268     kernel32:KERNEL32.dll
 0002:00000270       __imp_CreateToolhelp32Snapshot 0000000180027270     kernel32:KERNEL32.dll
 0002:00000278       __imp_WriteConsoleInputW   0000000180027278     kernel32:KERNEL32.dll
 0002:00000280       __imp_ReadConsoleInputW    0000000180027280     kernel32:KERNEL32.dll
 0002:00000288       __imp_WideCharToMultiByte  0000000180027288     kernel32:KERNEL32.dll
 0002:00000290       __imp_SetEnvironmentVariableW 0000000180027290     kernel32:KERNEL32.dll
 0002:00000298       __imp_GetModuleHandleW     0000000180027298     kernel32:KERNEL32.dll
 0002:000002a0       __imp_GetModuleFileNameW   00000001800272a0     kernel32:KERNEL32.dll
 0002:000002a8       __imp_OpenFileMappingW     00000001800272a8     kernel32:KERNEL32.dll
 0002:000002b0       __imp_CreateFileMappingW   00000001800272b0     kernel32:KERNEL32.dll
 0002:000002b8       __imp_lstrlenW             00000001800272b8     kernel32:KERNEL32.dll
 0002:000002c0       __imp_lstrcpyW             00000001800272c0     kernel32:KERNEL32.dll
 0002:000002c8       __imp_lstrcpynW            00000001800272c8     kernel32:KERNEL32.dll
 0002:000002d0       __imp_lstrcmpiW            00000001800272d0     kernel32:KERNEL32.dll
 0002:000002d8       __imp_UnmapViewOfFile      00000001800272d8     kernel32:KERNEL32.dll
 0002:000002e0       __imp_MapViewOfFile        00000001800272e0     kernel32:KERNEL32.dll
 0002:000002e8       __imp_GetStdHandle         00000001800272e8     kernel32:KERNEL32.dll
 0002:000002f0       __imp_WaitForSingleObject  00000001800272f0     kernel32:KERNEL32.dll
 0002:000002f8       __imp_GetLastError         00000001800272f8     kernel32:KERNEL32.dll
 0002:00000300       __imp_GetCurrentThreadId   0000000180027300     kernel32:KERNEL32.dll
 0002:00000308       __imp_GetCurrentProcessId  0000000180027308     kernel32:KERNEL32.dll
 0002:00000310       __imp_CloseHandle          0000000180027310     kernel32:KERNEL32.dll
 0002:00000318       __imp_TlsSetValue          0000000180027318     kernel32:KERNEL32.dll
 0002:00000320       __imp_VirtualProtect       0000000180027320     kernel32:KERNEL32.dll
 0002:00000328       __imp_LocalFree            0000000180027328     kernel32:KERNEL32.dll
 0002:00000330       __imp_TlsGetValue          0000000180027330     kernel32:KERNEL32.dll
 0002:00000338       __imp_GetProcAddress       0000000180027338     kernel32:KERNEL32.dll
 0002:00000340       __imp_HeapCreate           0000000180027340     kernel32:KERNEL32.dll
 0002:00000348       __imp_HeapDestroy          0000000180027348     kernel32:KERNEL32.dll
 0002:00000350       __imp_HeapAlloc            0000000180027350     kernel32:KERNEL32.dll
 0002:00000358       __imp_HeapReAlloc          0000000180027358     kernel32:KERNEL32.dll
 0002:00000360       __imp_HeapFree             0000000180027360     kernel32:KERNEL32.dll
 0002:00000368       __imp_DebugBreak           0000000180027368     kernel32:KERNEL32.dll
 0002:00000370       __imp_VerSetConditionMask  0000000180027370     kernel32:KERNEL32.dll
 0002:00000378       __imp_SetLastError         0000000180027378     kernel32:KERNEL32.dll
 0002:00000380       __imp_IsDebuggerPresent    0000000180027380     kernel32:KERNEL32.dll
 0002:00000388       __imp_WriteFile            0000000180027388     kernel32:KERNEL32.dll
 0002:00000390       __imp_ReadFile             0000000180027390     kernel32:KERNEL32.dll
 0002:00000398       __imp_SetNamedPipeHandleState 0000000180027398     kernel32:KERNEL32.dll
 0002:000003a0       __imp_TransactNamedPipe    00000001800273a0     kernel32:KERNEL32.dll
 0002:000003a8       __imp_WaitNamedPipeW       00000001800273a8     kernel32:KERNEL32.dll
 0002:000003b0       __imp_Process32FirstW      00000001800273b0     kernel32:KERNEL32.dll
 0002:000003b8       __imp_Process32NextW       00000001800273b8     kernel32:KERNEL32.dll
 0002:000003c0       __imp_OpenThread           00000001800273c0     kernel32:KERNEL32.dll
 0002:000003c8       __imp_RaiseException       00000001800273c8     kernel32:KERNEL32.dll
 0002:000003d0       __imp_CreateThread         00000001800273d0     kernel32:KERNEL32.dll
 0002:000003d8       __imp_TerminateThread      00000001800273d8     kernel32:KERNEL32.dll
 0002:000003e0       __imp_ResumeThread         00000001800273e0     kernel32:KERNEL32.dll
 0002:000003e8       __imp_GetFileInformationByHandle 00000001800273e8     kernel32:KERNEL32.dll
 0002:000003f0       __imp_GetEnvironmentVariableW 00000001800273f0     kernel32:KERNEL32.dll
 0002:000003f8       __imp_ExpandEnvironmentStringsW 00000001800273f8     kernel32:KERNEL32.dll
 0002:00000400       __imp_VerifyVersionInfoW   0000000180027400     kernel32:KERNEL32.dll
 0002:00000408       __imp_InitializeCriticalSection 0000000180027408     kernel32:KERNEL32.dll
 0002:00000410       __imp_EnterCriticalSection 0000000180027410     kernel32:KERNEL32.dll
 0002:00000418       __imp_LeaveCriticalSection 0000000180027418     kernel32:KERNEL32.dll
 0002:00000420       __imp_TryEnterCriticalSection 0000000180027420     kernel32:KERNEL32.dll
 0002:00000428       __imp_DeleteCriticalSection 0000000180027428     kernel32:KERNEL32.dll
 0002:00000430       __imp_ReadConsoleOutputW   0000000180027430     kernel32:KERNEL32.dll
 0002:00000438       __imp_GetConsoleScreenBufferInfo 0000000180027438     kernel32:KERNEL32.dll
 0002:00000440       __imp_GetCurrentProcess    0000000180027440     kernel32:KERNEL32.dll
 0002:00000448       __imp_RtlCaptureContext    0000000180027448     kernel32:KERNEL32.dll
 0002:00000450       __imp_RtlLookupFunctionEntry 0000000180027450     kernel32:KERNEL32.dll
 0002:00000458       __imp_RtlVirtualUnwind     0000000180027458     kernel32:KERNEL32.dll
 0002:00000460       __imp_UnhandledExceptionFilter 0000000180027460     kernel32:KERNEL32.dll
 0002:00000468       __imp_SetUnhandledExceptionFilter 0000000180027468     kernel32:KERNEL32.dll
 0002:00000470       __imp_TerminateProcess     0000000180027470     kernel32:KERNEL32.dll
 0002:00000478       __imp_IsProcessorFeaturePresent 0000000180027478     kernel32:KERNEL32.dll
 0002:00000480       __imp_QueryPerformanceCounter 0000000180027480     kernel32:KERNEL32.dll
 0002:00000488       __imp_GetSystemTimeAsFileTime 0000000180027488     kernel32:KERNEL32.dll
 0002:00000490       __imp_InitializeSListHead  0000000180027490     kernel32:KERNEL32.dll
 0002:00000498       __imp_GetStartupInfoW      0000000180027498     kernel32:KERNEL32.dll
 0002:000004a0       __imp_RtlUnwindEx          00000001800274a0     kernel32:KERNEL32.dll
 0002:000004a8       __imp_InterlockedFlushSList 00000001800274a8     kernel32:KERNEL32.dll
 0002:000004b0       __imp_EncodePointer        00000001800274b0     kernel32:KERNEL32.dll
 0002:000004b8       __imp_InitializeCriticalSectionAndSpinCount 00000001800274b8     kernel32:KERNEL32.dll
 0002:000004c0       __imp_TlsAlloc             00000001800274c0     kernel32:KERNEL32.dll
 0002:000004c8       \177KERNEL32_NULL_THUNK_DATA 00000001800274c8     kernel32:KERNEL32.dll
 0002:000004d0       __imp_SHGetFileInfoW       00000001800274d0     shell32:SHELL32.dll
 0002:000004d8       \177SHELL32_NULL_THUNK_DATA 00000001800274d8     shell32:SHELL32.dll
 0002:000004e0       __imp_GetIconInfo          00000001800274e0     user32:USER32.dll
 0002:000004e8       __imp_DrawIconEx           00000001800274e8     user32:USER32.dll
 0002:000004f0       __imp_DestroyIcon          00000001800274f0     user32:USER32.dll
 0002:000004f8       __imp_LoadIconW            00000001800274f8     user32:USER32.dll
 0002:00000500       __imp_ReleaseDC            0000000180027500     user32:USER32.dll
 0002:00000508       __imp_GetDC                0000000180027508     user32:USER32.dll
 0002:00000510       __imp_LoadCursorW          0000000180027510     user32:USER32.dll
 0002:00000518       __imp_SetWindowLongPtrW    0000000180027518     user32:USER32.dll
 0002:00000520       __imp_GetWindowLongPtrW    0000000180027520     user32:USER32.dll
 0002:00000528       __imp_SetWindowLongW       0000000180027528     user32:USER32.dll
 0002:00000530       __imp_FillRect             0000000180027530     user32:USER32.dll
 0002:00000538       __imp_InvalidateRect       0000000180027538     user32:USER32.dll
 0002:00000540       __imp_EndPaint             0000000180027540     user32:USER32.dll
 0002:00000548       __imp_BeginPaint           0000000180027548     user32:USER32.dll
 0002:00000550       __imp_DrawTextW            0000000180027550     user32:USER32.dll
 0002:00000558       __imp_ShowWindowAsync      0000000180027558     user32:USER32.dll
 0002:00000560       __imp_DestroyWindow        0000000180027560     user32:USER32.dll
 0002:00000568       __imp_IsWindow             0000000180027568     user32:USER32.dll
 0002:00000570       __imp_UnregisterClassW     0000000180027570     user32:USER32.dll
 0002:00000578       __imp_RegisterClassW       0000000180027578     user32:USER32.dll
 0002:00000580       __imp_DefWindowProcW       0000000180027580     user32:USER32.dll
 0002:00000588       __imp_PostThreadMessageW   0000000180027588     user32:USER32.dll
 0002:00000590       __imp_PostMessageW         0000000180027590     user32:USER32.dll
 0002:00000598       __imp_DispatchMessageW     0000000180027598     user32:USER32.dll
 0002:000005a0       __imp_GetMessageW          00000001800275a0     user32:USER32.dll
 0002:000005a8       __imp_RegisterWindowMessageW 00000001800275a8     user32:USER32.dll
 0002:000005b0       __imp_wsprintfW            00000001800275b0     user32:USER32.dll
 0002:000005b8       __imp_GetWindowThreadProcessId 00000001800275b8     user32:USER32.dll
 0002:000005c0       __imp_GetClassNameW        00000001800275c0     user32:USER32.dll
 0002:000005c8       __imp_IntersectRect        00000001800275c8     user32:USER32.dll
 0002:000005d0       __imp_ChildWindowFromPointEx 00000001800275d0     user32:USER32.dll
 0002:000005d8       __imp_WindowFromPoint      00000001800275d8     user32:USER32.dll
 0002:000005e0       __imp_MapWindowPoints      00000001800275e0     user32:USER32.dll
 0002:000005e8       __imp_MessageBoxW          00000001800275e8     user32:USER32.dll
 0002:000005f0       __imp_GetClientRect        00000001800275f0     user32:USER32.dll
 0002:000005f8       __imp_MapVirtualKeyW       00000001800275f8     user32:USER32.dll
 0002:00000600       __imp_GetKeyState          0000000180027600     user32:USER32.dll
 0002:00000608       __imp_IsWindowVisible      0000000180027608     user32:USER32.dll
 0002:00000610       __imp_CreateWindowExW      0000000180027610     user32:USER32.dll
 0002:00000618       __imp_ShowWindow           0000000180027618     user32:USER32.dll
 0002:00000620       \177USER32_NULL_THUNK_DATA 0000000180027620     user32:USER32.dll
 0002:00000628       __imp_GetFileVersionInfoW  0000000180027628     version:VERSION.dll
 0002:00000630       __imp_GetFileVersionInfoSizeW 0000000180027630     version:VERSION.dll
 0002:00000638       __imp_VerQueryValueW       0000000180027638     version:VERSION.dll
 0002:00000640       \177VERSION_NULL_THUNK_DATA 0000000180027640     version:VERSION.dll
 0002:00000648       __imp_CoInitialize         0000000180027648     ole32:ole32.dll
 0002:00000650       __imp_CoUninitialize       0000000180027650     ole32:ole32.dll
 0002:00000658       \177ole32_NULL_THUNK_DATA  0000000180027658     ole32:ole32.dll
 0002:00000660       __guard_check_icall_fptr   0000000180027660     LIBCMT:guard_support.obj
 0002:00000668       __guard_dispatch_icall_fptr 0000000180027668     LIBCMT:guard_support.obj
 0002:00000670       __xc_a                     0000000180027670     LIBCMT:initializers.obj
 0002:00000678       __xc_z                     0000000180027678     LIBCMT:initializers.obj
 0002:00000680       __xi_a                     0000000180027680     LIBCMT:initializers.obj
 0002:00000688       __acrt_stdio_initializer   0000000180027688     libucrt:stdio_initializer.obj
 0002:00000690       __acrt_multibyte_initializer 0000000180027690     libucrt:multibyte_initializer.obj
 0002:00000698       __acrt_tran_fma3_initializer 0000000180027698     libucrt:fma3_initializer.obj
 0002:000006a0       __xi_z                     00000001800276a0     LIBCMT:initializers.obj
 0002:000006a8       __xp_a                     00000001800276a8     LIBCMT:initializers.obj
 0002:000006b0       __acrt_locale_terminator   00000001800276b0     libucrt:locale_initializer.obj
 0002:000006b8       __dcrt_console_output_terminator 00000001800276b8     libucrt:console_output_initializer.obj
 0002:000006c0       __acrt_stdio_terminator    00000001800276c0     libucrt:stdio_initializer.obj
 0002:000006c8       __xp_z                     00000001800276c8     LIBCMT:initializers.obj
 0002:000006d0       __xt_a                     00000001800276d0     LIBCMT:initializers.obj
 0002:000006d8       __xt_z                     00000001800276d8     LIBCMT:initializers.obj
 0002:000006e0       ??_C@_08BCACMCCB@ExitFARW?$AA@ 00000001800276e0     ConEmuTh.obj
 0002:000006f0       ??_C@_0BF@NLPJFAHE@ProcessSynchroEventW?$AA@ 00000001800276f0     ConEmuTh.obj
 0002:00000780       ??_C@_11LOCGONAA@?$AA?$AA@ 0000000180027780     ConEmuTh.obj
 0002:00000784       ??_C@_13FPGAJAPJ@?$AA?2?$AA?$AA@ 0000000180027784     ConEmuTh.obj
 0002:00000790       ??_C@_1FG@DPPGENBC@?$AAL?$AAo?$AAa?$AAd?$AAA?$AAp?$AAp?$AAV?$AAe?$AAr?$AAs?$AAi?$AAo?$AAn?$AA?4?$AAV?$AAe?$AAr?$AAQ?$AAu?$AAe?$AAr?$AAy?$AAV?$AAa?$AAl?$AAu?$AAe?$AA?$CI?$AA?$CC?$AA?2?$AA?$CC@ 0000000180027790     ConEmuTh.obj
 0002:000007f0       ??_C@_1FK@HILEEFML@?$AAL?$AAo?$AAa?$AAd?$AAA?$AAp?$AAp?$AAV?$AAe?$AAr?$AAs?$AAi?$AAo?$AAn?$AA?4?$AAG?$AAe?$AAt?$AAF?$AAi?$AAl?$AAe?$AAV?$AAe?$AAr?$AAs?$AAi?$AAo?$AAn?$AAI?$AAn?$AAf@ 00000001800277f0     ConEmuTh.obj
 0002:00000850       ??_C@_1GC@BINFLBDC@?$AAL?$AAo?$AAa?$AAd?$AAA?$AAp?$AAp?$AAV?$AAe?$AAr?$AAs?$AAi?$AAo?$AAn?$AA?5?$AAf?$AAa?$AAi?$AAl?$AAe?$AAd?$AA?$CB?$AA?5?$AAC?$AAa?$AAn?$AA?8?$AAt?$AA?5?$AAa?$AAl?$AAl@ 0000000180027850     ConEmuTh.obj
 0002:000008c0       ??_C@_1GC@CPPHDKJK@?$AAL?$AAo?$AAa?$AAd?$AAA?$AAp?$AAp?$AAV?$AAe?$AAr?$AAs?$AAi?$AAo?$AAn?$AA?4?$AAG?$AAe?$AAt?$AAF?$AAi?$AAl?$AAe?$AAV?$AAe?$AAr?$AAs?$AAi?$AAo?$AAn?$AAI?$AAn?$AAf@ 00000001800278c0     ConEmuTh.obj
 0002:00000930       ??_C@_1EG@IINOBDEG@?$AAI?$AAn?$AAv?$AAa?$AAl?$AAi?$AAd?$AA?5?$AAa?$AAs?$AAM?$AAo?$AAd?$AAu?$AAl?$AAe?$AAP?$AAa?$AAt?$AAh?$AA?5?$AAw?$AAa?$AAs?$AA?5?$AAs?$AAp?$AAe?$AAc?$AAi?$AAf?$AAi@ 0000000180027930     ConEmuTh.obj
 0002:00000978       ??_C@_1CA@GGFPMHLH@?$AA?6?$AAE?$AAr?$AAr?$AAC?$AAo?$AAd?$AAe?$AA?$DN?$AA0?$AAx?$AA?$CF?$AA0?$AA8?$AAX?$AA?$AA@ 0000000180027978     ConEmuTh.obj
 0002:000009a0       ??_C@_1FG@LNADFPCE@?$AAL?$AAo?$AAa?$AAd?$AAF?$AAa?$AAr?$AAV?$AAe?$AAr?$AAs?$AAi?$AAo?$AAn?$AA?4?$AAG?$AAe?$AAt?$AAM?$AAo?$AAd?$AAu?$AAl?$AAe?$AAF?$AAi?$AAl?$AAe?$AAN?$AAa?$AAm?$AAe@ 00000001800279a0     ConEmuTh.obj
 0002:000009f8       ??_C@_1CC@MFEKNKAL@?$AAC?$AAo?$AAn?$AAE?$AAm?$AAu?$AAT?$AAh?$AA?4?$AAx?$AA6?$AA4?$AA?4?$AAd?$AAl?$AAl?$AA?$AA@ 00000001800279f8     ConEmuTh.obj
 0002:00000a20       ??_C@_1BO@ONHPLONP@?$AAC?$AAo?$AAn?$AAE?$AAm?$AAu?$AA?4?$AAx?$AA6?$AA4?$AA?4?$AAd?$AAl?$AAl?$AA?$AA@ 0000000180027a20     ConEmuTh.obj
 0002:00000a40       ??_C@_0BC@MKJHPCEO@RegisterPanelView?$AA@ 0000000180027a40     ConEmuTh.obj
 0002:00000a58       ??_C@_0M@FMNOKGGE@GetFarHWND2?$AA@ 0000000180027a58     ConEmuTh.obj
 0002:00000a68       ??_C@_1BM@HEIDIPPL@?$AAL?$AAe?$AAf?$AAt?$AAP?$AAa?$AAn?$AAe?$AAl?$AAV?$AAi?$AAe?$AAw?$AA?$AA@ 0000000180027a68     ConEmuTh.obj
 0002:00000a88       ??_C@_1BO@KCLMEFLE@?$AAR?$AAi?$AAg?$AAh?$AAt?$AAP?$AAa?$AAn?$AAe?$AAl?$AAV?$AAi?$AAe?$AAw?$AA?$AA@ 0000000180027a88     ConEmuTh.obj
 0002:00000aa8       ??_C@_0DH@EICPHJHO@t?3?2vcproject?2maximus5?2conemu?2src@ 0000000180027aa8     ConEmuTh.obj
 0002:00000ae0       ??_C@_1DM@JLCDNDHD@?$AAC?$AAo?$AAn?$AAE?$AAm?$AAu?$AAP?$AAa?$AAn?$AAe?$AAl?$AAV?$AAi?$AAe?$AAw?$AAD?$AAl?$AAg?$AAs?$AAM?$AAa?$AAp?$AAp?$AAi?$AAn?$AAg?$AA?4?$AA?$CF?$AAu?$AA?$AA@ 0000000180027ae0     ConEmuTh.obj
 0002:00000b20       ??_C@_1O@EMLLFJNI@?$AAA?$AAc?$AAt?$AAi?$AAv?$AAe?$AA?$AA@ 0000000180027b20     ConEmuTh.obj
 0002:00000b30       ??_C@_1BM@OLHABKH@?$AAF?$AAa?$AAr?$AAT?$AAh?$AAu?$AAm?$AAb?$AAn?$AAa?$AAi?$AAl?$AAs?$AA?$AA@ 0000000180027b30     ConEmuTh.obj
 0002:00000b50       ??_C@_1DG@DBEAEOKG@?$AAF?$AAa?$AAr?$AAP?$AAi?$AAc?$AAt?$AAu?$AAr?$AAe?$AAV?$AAi?$AAe?$AAw?$AAC?$AAo?$AAn?$AAt?$AAr?$AAo?$AAl?$AAC?$AAl?$AAa?$AAs?$AAs?$AA?$AA@ 0000000180027b50     ConEmuTh.obj
 0002:00000b88       ??_C@_1DC@FOGHAECG@?$AAF?$AAa?$AAr?$AAM?$AAu?$AAl?$AAt?$AAi?$AAV?$AAi?$AAe?$AAw?$AAC?$AAo?$AAn?$AAt?$AAr?$AAo?$AAl?$AAC?$AAl?$AAa?$AAs?$AAs?$AA?$AA@ 0000000180027b88     ConEmuTh.obj
 0002:00000bc0       ??_C@_1DA@BMIFHIMF@?$AAC?$AAo?$AAn?$AAE?$AAm?$AAu?$AAV?$AAi?$AAe?$AAw?$AAS?$AAe?$AAt?$AAM?$AAa?$AAp?$AAp?$AAi?$AAn?$AAg?$AA?4?$AA?$CF?$AAu?$AA?$AA@ 0000000180027bc0     ConEmuTh.obj
 0002:00000bf0       ??_C@_1BC@DJOGOIHN@?$AAC?$AAo?$AAn?$AAE?$AAm?$AAu?$AAT?$AAh?$AA?$AA@ 0000000180027bf0     ConEmuTh.obj
 0002:00000c08       ??_C@_1DM@OLPDHEPA@?$AAF?$AAa?$AAi?$AAl?$AAe?$AAd?$AA?5?$AAt?$AAo?$AA?5?$AAg?$AAe?$AAt?$AA?5?$AAC?$AAo?$AAn?$AAE?$AAm?$AAu?$AA?5?$AAp?$AAa?$AAl?$AAe?$AAt?$AAt?$AAe?$AA?$CB?$AA?$AA@ 0000000180027c08     ConEmuTh.obj
 0002:00000c48       ??_C@_1CG@HOMCPCN@?$AA?2?$AAP?$AAl?$AAu?$AAg?$AAi?$AAn?$AAs?$AA?2?$AAP?$AAa?$AAn?$AAe?$AAl?$AAT?$AAa?$AAb?$AAs?$AA?$AA@ 0000000180027c48     ConEmuTh.obj
 0002:00000c70       ??_C@_1BK@NFAPLMGI@?$AAS?$AAe?$AAp?$AAa?$AAr?$AAa?$AAt?$AAe?$AAT?$AAa?$AAb?$AAs?$AA?$AA@ 0000000180027c70     ConEmuTh.obj
 0002:00000c90       ??_C@_1BI@GILFJGEK@?$AAB?$AAu?$AAt?$AAt?$AAo?$AAn?$AAC?$AAo?$AAl?$AAo?$AAr?$AA?$AA@ 0000000180027c90     ConEmuTh.obj
 0002:00000cb0       ??_C@_1GK@OGACKIKJ@?$AAI?$AAn?$AAt?$AAe?$AAr?$AAn?$AAa?$AAl?$AA?5?$AAe?$AAr?$AAr?$AAo?$AAr?$AA?4?$AA?5?$AAM?$AAa?$AAp?$AAp?$AAi?$AAn?$AAg?$AA?5?$AAf?$AAi?$AAl?$AAe?$AA?5?$AAn?$AAa?$AAm@ 0000000180027cb0     ConEmuTh.obj
 0002:00000d20       ??_C@_1O@KBENBEFG@?$AAc?$AAr?$AAe?$AAa?$AAt?$AAe?$AA?$AA@ 0000000180027d20     ConEmuTh.obj
 0002:00000d30       ??_C@_19BDAJEHDN@?$AAo?$AAp?$AAe?$AAn?$AA?$AA@ 0000000180027d30     ConEmuTh.obj
 0002:00000d40       ??_C@_1GM@LGOLGABE@?$AAC?$AAa?$AAn?$AA?8?$AAt?$AA?5?$AA?$CF?$AAs?$AA?5?$AAc?$AAo?$AAn?$AAs?$AAo?$AAl?$AAe?$AA?5?$AAd?$AAa?$AAt?$AAa?$AA?5?$AAf?$AAi?$AAl?$AAe?$AA?5?$AAm?$AAa?$AAp?$AAp?$AAi@ 0000000180027d40     ConEmuTh.obj
 0002:00000db0       ??_C@_1BE@HADLJAO@?$AAR?$AAe?$AAa?$AAd?$AAW?$AAr?$AAi?$AAt?$AAe?$AA?$AA@ 0000000180027db0     ConEmuTh.obj
 0002:00000dc8       ??_C@_19EOHDNDII@?$AAR?$AAe?$AAa?$AAd?$AA?$AA@ 0000000180027dc8     ConEmuTh.obj
 0002:00000de0       ??_C@_1FO@BGAPBIGG@?$AAC?$AAa?$AAn?$AA?8?$AAt?$AA?5?$AAm?$AAa?$AAp?$AA?5?$AAc?$AAo?$AAn?$AAs?$AAo?$AAl?$AAe?$AA?5?$AAi?$AAn?$AAf?$AAo?$AA?5?$AA?$CI?$AA?$CF?$AAs?$AA?$CJ?$AA?4?$AA?5?$AAE?$AAr?$AAr@ 0000000180027de0     ConEmuTh.obj
 0002:00000e40       ??_C@_17JLFEDMMI@?$AA?$DP?$AA?$DP?$AA?$DP?$AA?$AA@ 0000000180027e40     ConEmuTh1900.obj
 0002:00000e48       ??_C@_1BI@EKLHEFDO@?$AAS?$AAh?$AAo?$AAw?$AAM?$AAe?$AAn?$AAu?$AAB?$AAa?$AAr?$AA?$AA@ 0000000180027e48     ConEmuTh1900.obj
 0002:00000e60       ??_C@_1O@PDEOIOBG@?$AAK?$AAe?$AAy?$AAB?$AAa?$AAr?$AA?$AA@ 0000000180027e60     ConEmuTh1900.obj
 0002:00000e70       ??_C@_1BK@MBFACEDG@?$AAC?$AAo?$AAl?$AAu?$AAm?$AAn?$AAT?$AAi?$AAt?$AAl?$AAe?$AAs?$AA?$AA@ 0000000180027e70     ConEmuTh1900.obj
 0002:00000e90       ??_C@_1BG@MHMKAABO@?$AAS?$AAt?$AAa?$AAt?$AAu?$AAs?$AAL?$AAi?$AAn?$AAe?$AA?$AA@ 0000000180027e90     ConEmuTh1900.obj
 0002:00000ea8       ??_C@_1BC@IALIJCAM@?$AAS?$AAo?$AAr?$AAt?$AAM?$AAo?$AAd?$AAe?$AA?$AA@ 0000000180027ea8     ConEmuTh1900.obj
 0002:00000ec0       ??_C@_1CG@DMGPLFKD@?$AAC?$AAo?$AAn?$AAE?$AAm?$AAu?$AA?5?$AAP?$AAa?$AAn?$AAe?$AAl?$AA?5?$AAV?$AAi?$AAe?$AAw?$AAs?$AA?$AA@ 0000000180027ec0     ConEmuTh2800.obj
 0002:00000ef0       ??_C@_1EM@OOFEGLCO@?$AAT?$AAh?$AAu?$AAm?$AAb?$AAn?$AAa?$AAi?$AAl?$AAs?$AA?5?$AAa?$AAn?$AAd?$AA?5?$AAT?$AAi?$AAl?$AAe?$AAs?$AA?5?$AAi?$AAn?$AA?5?$AAC?$AAo?$AAn?$AAE?$AAm?$AAu?$AA?5?$AAw@ 0000000180027ef0     ConEmuTh2800.obj
 0002:00000f40       ??_C@_1DE@DJEAMLPH@?$AAC?$AAo?$AAn?$AAE?$AAm?$AAu?$AA?4?$AAM?$AAa?$AAx?$AAi?$AAm?$AAu?$AAs?$AA5?$AA?$EA?$AAg?$AAm?$AAa?$AAi?$AAl?$AA?4?$AAc?$AAo?$AAm?$AA?$AA@ 0000000180027f40     ConEmuTh2800.obj
 0002:00000f78       ??_C@_1BG@LBJCGLOJ@?$AAS?$AAe?$AAt?$AAC?$AAu?$AAr?$AAI?$AAt?$AAe?$AAm?$AA?$AA@ 0000000180027f78     ConEmuTh2800.obj
 0002:00000f90       ??_C@_1EI@PNMHLKGC@?$AAi?$AAf?$AA?5?$AAA?$AAr?$AAe?$AAa?$AA?4?$AAS?$AAe?$AAa?$AAr?$AAc?$AAh?$AA?5?$AAt?$AAh?$AAe?$AAn?$AA?5?$AAK?$AAe?$AAy?$AAs?$AA?$CI?$AA?$CC?$AAE?$AAs?$AAc?$AA?$CC?$AA?$CJ?$AA?5@ 0000000180027f90     ConEmuTh2800.obj
 0002:00000fd8       ??_C@_1CA@GIGEMLLA@?$AAP?$AAl?$AAu?$AAg?$AAi?$AAn?$AA?4?$AAS?$AAy?$AAn?$AAc?$AAC?$AAa?$AAl?$AAl?$AA?$AA@ 0000000180027fd8     ConEmuTh2800.obj
 0002:00000ff8       ??_C@_1CM@IICFOBPI@?$AA$?$AAi?$AAf?$AA?5?$AA?$CI?$AAS?$AAe?$AAa?$AAr?$AAc?$AAh?$AA?$CJ?$AA?5?$AAE?$AAs?$AAc?$AA?5?$AA$?$AAe?$AAn?$AAd?$AA?$AA@ 0000000180027ff8     ConEmuTh2800.obj
 0002:00001028       ??_C@_1BG@PKDGNNAF@?$AAc?$AAa?$AAl?$AAl?$AAp?$AAl?$AAu?$AAg?$AAi?$AAn?$AA?$AA@ 0000000180028028     ConEmuTh2800.obj
 0002:00001040       ??_C@_1HI@BNDPAPFP@?$AA?$CF?$AAs?$AA?5?$AA?$CF?$AAs?$AA?$CI?$AA?$CC?$AAb?$AAd?$AA4?$AA5?$AA4?$AAd?$AA4?$AA8?$AA?9?$AA4?$AA4?$AA8?$AAe?$AA?9?$AA4?$AA6?$AAc?$AAc?$AA?9?$AA9?$AA0?$AA9?$AAd?$AA?9?$AAb@ 0000000180028040     ConEmuTh2800.obj
 0002:000010b8       ??_C@_1BE@LFJLOEAN@?$AAC?$AAo?$AAn?$AAE?$AAm?$AAu?$AAT?$AAh?$AA?2?$AA?$AA@ 00000001800280b8     ConEmuTh995.obj
 0002:00001140       ??_C@_0BG@FGMCOIHO@Thumbs?3?3DisplayThread?$AA@ 0000000180028140     Display.obj
 0002:00001158       ??_C@_19DKAIAFPE@?$AAL?$AAe?$AAf?$AAt?$AA?$AA@ 0000000180028158     Display.obj
 0002:00001168       ??_C@_1M@KDEMMBOH@?$AAR?$AAi?$AAg?$AAh?$AAt?$AA?$AA@ 0000000180028168     Display.obj
 0002:00001178       ??_C@_1CM@MJKKOLFD@?$AAC?$AAo?$AAn?$AAE?$AAm?$AAu?$AA?4?$AA?$CF?$AAs?$AAP?$AAa?$AAn?$AAe?$AAl?$AAV?$AAi?$AAe?$AAw?$AA?4?$AA?$CF?$AAi?$AA?$AA@ 0000000180028178     Display.obj
 0002:000011a8       ??_C@_1BO@IPKBELC@?$AAC?$AAo?$AAn?$AAE?$AAm?$AAu?$AAT?$AAh?$AA?3?$AA?3?$AAF?$AAa?$AAd?$AAe?$AA?$AA@ 00000001800281a8     Display.obj
 0002:000011c8       ??_C@_1CG@OILEFJJN@?$AAC?$AAo?$AAn?$AAE?$AAm?$AAu?$AAT?$AAh?$AA?3?$AA?3?$AAS?$AAe?$AAt?$AAt?$AAi?$AAn?$AAg?$AAs?$AA?$AA@ 00000001800281c8     Display.obj
 0002:000011f0       ??_C@_1CI@GNBJKMME@?$AAC?$AAo?$AAn?$AAE?$AAm?$AAu?$AAT?$AAh?$AA?3?$AA?3?$AAM?$AAa?$AAp?$AAC?$AAo?$AAo?$AAr?$AAd?$AAs?$AA?$AA@ 00000001800281f0     Display.obj
 0002:00001218       ??_C@_1CO@LEOKLKOD@?$AA?$CF?$AA0?$AA2?$AAi?$AA?4?$AA?$CF?$AA0?$AA2?$AAi?$AA?4?$AA?$CF?$AA0?$AA2?$AAi?$AA?5?$AA?$CF?$AAi?$AA?3?$AA?$CF?$AA0?$AA2?$AAi?$AA?$AA@ 0000000180028218     Display.obj
 0002:00001248       ??_C@_1O@NLGMKEDN@?$AAB?$AAK?$AAM?$AAG?$AAT?$AAP?$AA?$AA@ 0000000180028248     Display.obj
 0002:00001258       ??_C@_1BG@NLGHAGA@?$AA?$CF?$AAi?$AA?0?$AA?$CF?$AA0?$AA3?$AAi?$AA?5?$AA?$CF?$AAc?$AA?$AA@ 0000000180028258     Display.obj
 0002:00001270       ??_C@_1M@KOMOBEPM@?$AA?$CF?$AAi?$AA?5?$AA?$CF?$AAc?$AA?$AA@ 0000000180028270     Display.obj
 0002:00001280       ??_C@_1EK@NOCLDABL@?$AAi?$AAf?$AA?5?$AA?$CF?$AAc?$AAP?$AAa?$AAn?$AAe?$AAl?$AA?4?$AAL?$AAe?$AAf?$AAt?$AA?5?$AAt?$AAh?$AAe?$AAn?$AA?5?$AAK?$AAe?$AAy?$AAs?$AA?$CI?$AA?$CC?$AAT?$AAa?$AAb?$AA?$CC?$AA?$CJ@ 0000000180028280     Display.obj
 0002:000012d0       ??_C@_1DI@DLGGKEIH@?$AA$?$AAI?$AAf?$AA?5?$AA?$CI?$AA?$CF?$AAc?$AAP?$AAa?$AAn?$AAe?$AAl?$AA?4?$AAL?$AAe?$AAf?$AAt?$AA?$CJ?$AA?5?$AAT?$AAa?$AAb?$AA?5?$AA$?$AAE?$AAn?$AAd?$AA?$AA@ 00000001800282d0     Display.obj
 0002:00001400       ??_7?$CQueueProcessor@PEAUIMAGE_CACHE_INFO@@@@6B@ 0000000180028400     ImgCache.obj
 0002:00001470       ??_7CImgLoader@@6B@        0000000180028470     ImgCache.obj
 0002:000014e8       ??_C@_1M@KCMICNEG@?$AA?$CK?$AA?4?$AAt?$AA6?$AA4?$AA?$AA@ 00000001800284e8     ImgCache.obj
 0002:000014f8       ??_C@_08DHJJJJMJ@CET_Init?$AA@ 00000001800284f8     ImgCache.obj
 0002:00001508       ??_C@_08CBCDAPII@CET_Done?$AA@ 0000000180028508     ImgCache.obj
 0002:00001518       ??_C@_08DBEDCDF@CET_Load?$AA@ 0000000180028518     ImgCache.obj
 0002:00001528       ??_C@_08PFMFDMEL@CET_Free?$AA@ 0000000180028528     ImgCache.obj
 0002:00001538       ??_C@_0L@DOHHADLD@CET_Cancel?$AA@ 0000000180028538     ImgCache.obj
 0002:00001548       ??_C@_1BO@EOFABIPH@?$AAC?$AAo?$AAn?$AAE?$AAm?$AAu?$AAT?$AAh?$AA?4?$AAc?$AAa?$AAc?$AAh?$AAe?$AA?$AA@ 0000000180028548     ImgCache.obj
 0002:00001568       ??_C@_15DDHGOCBH@?$AA?4?$AA?4?$AA?$AA@ 0000000180028568     ImgCache.obj
 0002:00001570       ??_C@_19DDLLJDOO@?$AAF?$AAi?$AAl?$AAe?$AA?$AA@ 0000000180028570     ImgCache.obj
 0002:00001580       ??_C@_19HKLPDE@?$AA?4?$AAb?$AAm?$AAp?$AA?$AA@ 0000000180028580     ImgCache.obj
 0002:00001590       ??_C@_19KGHJPLAF@?$AA?4?$AAg?$AAi?$AAf?$AA?$AA@ 0000000180028590     ImgCache.obj
 0002:000015a0       ??_C@_19GPGAIFNL@?$AA?4?$AAi?$AAc?$AAo?$AA?$AA@ 00000001800285a0     ImgCache.obj
 0002:000015b0       ??_C@_19HFLOJEOK@?$AA?4?$AAp?$AAn?$AAg?$AA?$AA@ 00000001800285b0     ImgCache.obj
 0002:000015c0       ??_C@_19EBFDIIDI@?$AA?4?$AAw?$AAm?$AAf?$AA?$AA@ 00000001800285c0     ImgCache.obj
 0002:000015d0       ??_C@_1BE@DFPCIADA@?$AAP?$AAB?$AAF?$AAa?$AAr?$AA?4?$AAd?$AAl?$AAl?$AA?$AA@ 00000001800285d0     ImgCache.obj
 0002:000015e8       ??_C@_0N@DDFPJHDO@_GetFileData?$AA@ 00000001800285e8     ImgCache.obj
 0002:000015f8       ??_C@_0DL@MAJAEI@t?3?2vcproject?2maximus5?2conemu?2src@ 00000001800285f8     ImgCache.obj
 0002:00001638       ??_C@_0BJ@KDNBOADC@Thumbs?3?3ProcessingThread?$AA@ 0000000180028638     ImgCache.obj
 0002:00001660       __xmm@00000020000000200000000000000000 0000000180028660     ImgCache.obj
 0002:00001670       ??_C@_1BC@LMIJMNIA@?$AA0?$AA0?$AA0?$AA0?$AA0?$AA0?$AA0?$AA0?$AA?$AA@ 0000000180028670     common-kernel64:MStrSafe.obj
 0002:00001688       ??_C@_1BO@HJHEFHMO@?$AAK?$AAe?$AAr?$AAn?$AAe?$AAl?$AAB?$AAa?$AAs?$AAe?$AA?4?$AAd?$AAl?$AAl?$AA?$AA@ 0000000180028688     common-kernel64:MSecurity.obj
 0002:000016a8       ??_C@_1BK@BIGILECK@?$AAA?$AAd?$AAv?$AAa?$AAp?$AAi?$AA3?$AA2?$AA?4?$AAd?$AAl?$AAl?$AA?$AA@ 00000001800286a8     common-kernel64:MSecurity.obj
 0002:000016c8       ??_C@_0BE@IPKPLIM@AddAccessAllowedAce?$AA@ 00000001800286c8     common-kernel64:MSecurity.obj
 0002:000016e0       ??_C@_0BD@EIGAJLOG@AddAccessDeniedAce?$AA@ 00000001800286e0     common-kernel64:MSecurity.obj
 0002:000016f8       ??_C@_0BJ@ECIKFEOL@AllocateAndInitializeSid?$AA@ 00000001800286f8     common-kernel64:MSecurity.obj
 0002:00001718       ??_C@_0N@HBKDHKNL@GetLengthSid?$AA@ 0000000180028718     common-kernel64:MSecurity.obj
 0002:00001728       ??_C@_0O@GKCEJBAA@InitializeAcl?$AA@ 0000000180028728     common-kernel64:MSecurity.obj
 0002:00001738       ??_C@_0BN@FNLANPJJ@InitializeSecurityDescriptor?$AA@ 0000000180028738     common-kernel64:MSecurity.obj
 0002:00001758       ??_C@_0BK@DNNLOFO@SetSecurityDescriptorDacl?$AA@ 0000000180028758     common-kernel64:MSecurity.obj
 0002:00001778       ??_C@_1BA@LEPJIIOK@?$AAU?$AAn?$AAk?$AAn?$AAo?$AAw?$AAn?$AA?$AA@ 0000000180028778     common-kernel64:ConEmuCheck.obj
 0002:00001790       ??_C@_1EM@INHGIPLC@?$AA?$CF?$AAs?$AA?4?$AA?$CF?$AAu?$AA?3?$AA?5?$AAC?$AAr?$AAe?$AAa?$AAt?$AAe?$AAF?$AAi?$AAl?$AAe?$AA?$CI?$AA?$CF?$AAs?$AA?$CJ?$AA?5?$AAf?$AAa?$AAi?$AAl?$AAe?$AAd?$AA?0?$AA?5?$AAc?$AAo@ 0000000180028790     common-kernel64:ConEmuCheck.obj
 0002:000017dc       ??_C@_13JOFGPIOO@?$AA?4?$AA?$AA@ 00000001800287dc     common-kernel64:ConEmuCheck.obj
 0002:000017e0       ??_C@_1DC@MJLCOFMA@?$AA?2?$AA?2?$AA?$CF?$AAs?$AA?2?$AAp?$AAi?$AAp?$AAe?$AA?2?$AAC?$AAo?$AAn?$AAE?$AAm?$AAu?$AAG?$AAu?$AAi?$AA?4?$AA?$CF?$AA0?$AA8?$AAX?$AA?$AA@ 00000001800287e0     common-kernel64:ConEmuCheck.obj
 0002:00001820       ??_7?$MToolHelp@UtagPROCESSENTRY32W@@$1?Process32FirstW@@YAHPEAXPEAU1@@Z$1?Process32NextW@@YAH01@Z@@6B@ 0000000180028820     common-kernel64:MProcess.obj
 0002:00001838       ??_7MToolHelpProcess@@6B@  0000000180028838     common-kernel64:MProcess.obj
 0002:00001848       ??_C@_1BK@HHKNEJDC@?$AAt?$AAl?$AAn?$AAt?$AAs?$AAe?$AAs?$AAs?$AA?4?$AAe?$AAx?$AAe?$AA?$AA@ 0000000180028848     common-kernel64:MProcess.obj
 0002:00001868       ??_C@_1BI@MPDCNJBA@?$AAt?$AAl?$AAn?$AAt?$AAs?$AAv?$AAr?$AA?4?$AAe?$AAx?$AAe?$AA?$AA@ 0000000180028868     common-kernel64:MProcess.obj
 0002:00001880       ??_C@_1BO@MLCHEAGG@?$AAC?$AAo?$AAn?$AAE?$AAm?$AAu?$AAH?$AAk?$AA6?$AA4?$AA?4?$AAd?$AAl?$AAl?$AA?$AA@ 0000000180028880     common-kernel64:HkFunc.obj
 0002:000018a0       ??_C@_0BD@HGJIAJJM@RequestTrampolines?$AA@ 00000001800288a0     common-kernel64:HkFunc.obj
 0002:000018b4       ??_C@_05LCABBMOG@?$CFs?3?$CFi?$AA@ 00000001800288b4     common-kernel64:WThreads.obj
 0002:000018c0       ??_C@_19DOGDICKI@?$AA?4?$AAe?$AAx?$AAe?$AA?$AA@ 00000001800288c0     common-kernel64:WObjects.obj
 0002:000018d0       ??_C@_1BE@GJOFHIHD@?$AAn?$AAt?$AAd?$AAl?$AAl?$AA?4?$AAd?$AAl?$AAl?$AA?$AA@ 00000001800288d0     common-kernel64:WObjects.obj
 0002:000018e8       ??_C@_0BF@LOGLPPDD@RtlVerifyVersionInfo?$AA@ 00000001800288e8     common-kernel64:WObjects.obj
 0002:00001900       ??_C@_1EHK@JMHPNAMN@?$AAA?$AAC?$AAT?$AAI?$AAV?$AAA?$AAT?$AAE?$AA?$AA?$AAA?$AAL?$AAI?$AAA?$AAS?$AA?$AA?$AAA?$AAS?$AAS?$AAO?$AAC?$AA?$AA?$AAA?$AAT?$AAT?$AAR?$AAI?$AAB?$AA?$AA?$AAB?$AAE?$AAE?$AAP@ 0000000180028900     common-kernel64:CmdLine.obj
 0002:00001d7a       ??_C@_00CNPNBAHC@?$AA@     0000000180028d7a     common-kernel64:MStrDup.obj
 0002:00001d80       ??_C@_19IJOJOJIB@?$AAP?$AAA?$AAT?$AAH?$AA?$AA@ 0000000180028d80     common-kernel64:CEStr.obj
 0002:00001db8       ??_C@_1CA@DHOHMJCG@?$AAU?$AAn?$AAi?$AAc?$AAo?$AAd?$AAe?$AA?5?$AAC?$AAh?$AAa?$AAr?$AAM?$AAa?$AAp?$AA?$AA@ 0000000180028db8     common-user64:RgnDetect.obj
 0002:00001e00       ??_C@_1GK@PPEHOOAL@?$AAS?$AAO?$AAF?$AAT?$AAW?$AAA?$AAR?$AAE?$AA?2?$AAM?$AAi?$AAc?$AAr?$AAo?$AAs?$AAo?$AAf?$AAt?$AA?2?$AAW?$AAi?$AAn?$AAd?$AAo?$AAw?$AAs?$AA?2?$AAC?$AAu?$AAr?$AAr?$AAe@ 0000000180028e00     common-user64:WFiles.obj
 0002:00001e6c       ??_C@_13PJJBFPED@?$AA?$DL?$AA?$AA@ 0000000180028e6c     common-user64:WFiles.obj
 0002:00001e78       ??_7type_info@@6B@         0000000180028e78     LIBCMT:std_type_info_static.obj
 0002:00001e80       _pDefaultRawDllMain        0000000180028e80     LIBCMT:dll_dllmain.obj
 0002:00001e80       _pRawDllMain               0000000180028e80     LIBCMT:dll_dllmain.obj
 0002:00001f40       ??_7exception@std@@6B@     0000000180028f40     libvcruntime:frame.obj
 0002:00001f50       ??_C@_0BC@EOODALEL@Unknown?5exception?$AA@ 0000000180028f50     libvcruntime:frame.obj
 0002:00001f70       ??_7bad_exception@std@@6B@ 0000000180028f70     libvcruntime:frame.obj
 0002:00001f80       ??_C@_0O@DPKOEFFH@bad?5exception?$AA@ 0000000180028f80     libvcruntime:frame.obj
 0002:000022c0       ??_C@_08EHJDFFNH@__based?$CI?$AA@ 00000001800292c0     libvcruntime:undname.obj
 0002:000022d0       ??_C@_07KOLFKCDI@__cdecl?$AA@ 00000001800292d0     libvcruntime:undname.obj
 0002:000022d8       ??_C@_08GHMPAG@__pascal?$AA@ 00000001800292d8     libvcruntime:undname.obj
 0002:000022e8       ??_C@_09IFJBGAPI@__stdcall?$AA@ 00000001800292e8     libvcruntime:undname.obj
 0002:000022f8       ??_C@_0L@NPHFGOKO@__thiscall?$AA@ 00000001800292f8     libvcruntime:undname.obj
 0002:00002308       ??_C@_0L@JMKHOMEK@__fastcall?$AA@ 0000000180029308     libvcruntime:undname.obj
 0002:00002318       ??_C@_0N@BCKKPABJ@__vectorcall?$AA@ 0000000180029318     libvcruntime:undname.obj
 0002:00002328       ??_C@_09HIJEGCPM@__clrcall?$AA@ 0000000180029328     libvcruntime:undname.obj
 0002:00002334       ??_C@_06GHPCKEAG@__eabi?$AA@ 0000000180029334     libvcruntime:undname.obj
 0002:00002340       ??_C@_07EECFKIPL@__swift?$AA@ 0000000180029340     libvcruntime:undname.obj
 0002:00002348       ??_C@_07JOMMBBKO@__ptr64?$AA@ 0000000180029348     libvcruntime:undname.obj
 0002:00002350       ??_C@_0L@PILCLIHE@__restrict?$AA@ 0000000180029350     libvcruntime:undname.obj
 0002:00002360       ??_C@_0M@GFIIJFMG@__unaligned?$AA@ 0000000180029360     libvcruntime:undname.obj
 0002:00002370       ??_C@_09DHDLOLLB@restrict?$CI?$AA@ 0000000180029370     libvcruntime:undname.obj
 0002:0000237c       ??_C@_04NIHEBCM@?5new?$AA@ 000000018002937c     libvcruntime:undname.obj
 0002:00002388       ??_C@_07FPCDHGMM@?5delete?$AA@ 0000000180029388     libvcruntime:undname.obj
 0002:00002390       ??_C@_01NEMOKFLO@?$DN?$AA@ 0000000180029390     libvcruntime:undname.obj
 0002:00002394       ??_C@_02GPIOPFAK@?$DO?$DO?$AA@ 0000000180029394     libvcruntime:undname.obj
 0002:00002398       ??_C@_02FODMEDOG@?$DM?$DM?$AA@ 0000000180029398     libvcruntime:undname.obj
 0002:0000239c       ??_C@_01DCLJPIOD@?$CB?$AA@ 000000018002939c     libvcruntime:undname.obj
 0002:000023a0       ??_C@_02EGOFBIJA@?$DN?$DN?$AA@ 00000001800293a0     libvcruntime:undname.obj
 0002:000023a4       ??_C@_02FDNJECIE@?$CB?$DN?$AA@ 00000001800293a4     libvcruntime:undname.obj
 0002:000023a8       ??_C@_02GPECMEKF@?$FL?$FN?$AA@ 00000001800293a8     libvcruntime:undname.obj
 0002:000023b0       ??_C@_08LHJFAFGD@operator?$AA@ 00000001800293b0     libvcruntime:undname.obj
 0002:000023bc       ??_C@_02HBOOOICD@?9?$DO?$AA@ 00000001800293bc     libvcruntime:undname.obj
 0002:000023c0       ??_C@_01NBENCBCI@?$CK?$AA@ 00000001800293c0     libvcruntime:undname.obj
 0002:000023c4       ??_C@_02ECNGHCIF@?$CL?$CL?$AA@ 00000001800293c4     libvcruntime:undname.obj
 0002:000023c8       ??_C@_02BAABKJLB@?9?9?$AA@ 00000001800293c8     libvcruntime:undname.obj
 0002:000023cc       ??_C@_01JOAMLHOP@?9?$AA@   00000001800293cc     libvcruntime:undname.obj
 0002:000023d0       ??_C@_01MIFGBAGJ@?$CL?$AA@ 00000001800293d0     libvcruntime:undname.obj
 0002:000023d4       ??_C@_01HNPIGOCE@?$CG?$AA@ 00000001800293d4     libvcruntime:undname.obj
 0002:000023d8       ??_C@_03MNHNFDLC@?9?$DO?$CK?$AA@ 00000001800293d8     libvcruntime:undname.obj
 0002:000023dc       ??_C@_01KMDKNFGN@?1?$AA@   00000001800293dc     libvcruntime:undname.obj
 0002:000023e0       ??_C@_01FGNFDNOH@?$CF?$AA@ 00000001800293e0     libvcruntime:undname.obj
 0002:000023e4       ??_C@_01MNNFJEPP@?$DM?$AA@ 00000001800293e4     libvcruntime:undname.obj
 0002:000023e8       ??_C@_02EHCHHCKH@?$DM?$DN?$AA@ 00000001800293e8     libvcruntime:undname.obj
 0002:000023ec       ??_C@_01PPODPGHN@?$DO?$AA@ 00000001800293ec     libvcruntime:undname.obj
 0002:000023f0       ??_C@_02EEKDKGMJ@?$DO?$DN?$AA@ 00000001800293f0     libvcruntime:undname.obj
 0002:000023f4       ??_C@_01IHBHIGKO@?0?$AA@   00000001800293f4     libvcruntime:undname.obj
 0002:000023f8       ??_C@_02HCKGKOFO@?$CI?$CJ?$AA@ 00000001800293f8     libvcruntime:undname.obj
 0002:000023fc       ??_C@_01PJKLJHI@?$HO?$AA@  00000001800293fc     libvcruntime:undname.obj
 0002:00002400       ??_C@_01JKBOJNNK@?$FO?$AA@ 0000000180029400     libvcruntime:undname.obj
 0002:00002404       ??_C@_01DNKMNLPK@?$HM?$AA@ 0000000180029404     libvcruntime:undname.obj
 0002:00002408       ??_C@_02PPKAJPJL@?$CG?$CG?$AA@ 0000000180029408     libvcruntime:undname.obj
 0002:0000240c       ??_C@_02NONPIBCD@?$HM?$HM?$AA@ 000000018002940c     libvcruntime:undname.obj
 0002:00002410       ??_C@_02FPIMKNGF@?$CK?$DN?$AA@ 0000000180029410     libvcruntime:undname.obj
 0002:00002414       ??_C@_02FOEOMHFC@?$CL?$DN?$AA@ 0000000180029414     libvcruntime:undname.obj
 0002:00002418       ??_C@_02FKMDLLOA@?9?$DN?$AA@ 0000000180029418     libvcruntime:undname.obj
 0002:0000241c       ??_C@_02FJEHGPIO@?1?$DN?$AA@ 000000018002941c     libvcruntime:undname.obj
 0002:00002420       ??_C@_02FENAOKFI@?$CF?$DN?$AA@ 0000000180029420     libvcruntime:undname.obj
 0002:00002424       ??_C@_03IKFCCPFF@?$DO?$DO?$DN?$AA@ 0000000180029424     libvcruntime:undname.obj
 0002:00002428       ??_C@_03CDNPDDLA@?$DM?$DM?$DN?$AA@ 0000000180029428     libvcruntime:undname.obj
 0002:0000242c       ??_C@_02FGJGFEAB@?$CG?$DN?$AA@ 000000018002942c     libvcruntime:undname.obj
 0002:00002430       ??_C@_02DHLNPPGH@?$HM?$DN?$AA@ 0000000180029430     libvcruntime:undname.obj
 0002:00002434       ??_C@_02MHEGNOJ@?$FO?$DN?$AA@ 0000000180029434     libvcruntime:undname.obj
 0002:00002438       ??_C@_09IFPLHPGF@?$GAvftable?8?$AA@ 0000000180029438     libvcruntime:undname.obj
 0002:00002448       ??_C@_09BLBHBJP@?$GAvbtable?8?$AA@ 0000000180029448     libvcruntime:undname.obj
 0002:00002458       ??_C@_07FEEIOKP@?$GAvcall?8?$AA@ 0000000180029458     libvcruntime:undname.obj
 0002:00002460       ??_C@_08LLFFHHDJ@?$GAtypeof?8?$AA@ 0000000180029460     libvcruntime:undname.obj
 0002:00002470       ??_C@_0BF@KDPPACIK@?$GAlocal?5static?5guard?8?$AA@ 0000000180029470     libvcruntime:undname.obj
 0002:00002488       ??_C@_08OBABFOLI@?$GAstring?8?$AA@ 0000000180029488     libvcruntime:undname.obj
 0002:00002498       ??_C@_0BD@JDLKDPAB@?$GAvbase?5destructor?8?$AA@ 0000000180029498     libvcruntime:undname.obj
 0002:000024b0       ??_C@_0BN@DEGPLNFK@?$GAvector?5deleting?5destructor?8?$AA@ 00000001800294b0     libvcruntime:undname.obj
 0002:000024d0       ??_C@_0BO@OBMKPJIG@?$GAdefault?5constructor?5closure?8?$AA@ 00000001800294d0     libvcruntime:undname.obj
 0002:000024f0       ??_C@_0BN@IMDCHIKM@?$GAscalar?5deleting?5destructor?8?$AA@ 00000001800294f0     libvcruntime:undname.obj
 0002:00002510       ??_C@_0BO@PFGOCPJJ@?$GAvector?5constructor?5iterator?8?$AA@ 0000000180029510     libvcruntime:undname.obj
 0002:00002530       ??_C@_0BN@LFPFMEDL@?$GAvector?5destructor?5iterator?8?$AA@ 0000000180029530     libvcruntime:undname.obj
 0002:00002550       ??_C@_0CE@IKBNEHA@?$GAvector?5vbase?5constructor?5iterat@ 0000000180029550     libvcruntime:undname.obj
 0002:00002578       ??_C@_0BL@NILFHHPC@?$GAvirtual?5displacement?5map?8?$AA@ 0000000180029578     libvcruntime:undname.obj
 0002:00002598       ??_C@_0CB@JONCMFFK@?$GAeh?5vector?5constructor?5iterator?8@ 0000000180029598     libvcruntime:undname.obj
 0002:000025c0       ??_C@_0CA@GCEOPDGL@?$GAeh?5vector?5destructor?5iterator?8?$AA@ 00000001800295c0     libvcruntime:undname.obj
 0002:000025e0       ??_C@_0CH@OOJPLCPH@?$GAeh?5vector?5vbase?5constructor?5ite@ 00000001800295e0     libvcruntime:undname.obj
 0002:00002608       ??_C@_0BL@LLKPOHJI@?$GAcopy?5constructor?5closure?8?$AA@ 0000000180029608     libvcruntime:undname.obj
 0002:00002628       ??_C@_0BA@KBCDOMBN@?$GAudt?5returning?8?$AA@ 0000000180029628     libvcruntime:undname.obj
 0002:00002638       ??_C@_03KLGMFNMG@?$GAEH?$AA@ 0000000180029638     libvcruntime:undname.obj
 0002:0000263c       ??_C@_05KHLCHHI@?$GARTTI?$AA@ 000000018002963c     libvcruntime:undname.obj
 0002:00002648       ??_C@_0BA@KKLDJDLB@?$GAlocal?5vftable?8?$AA@ 0000000180029648     libvcruntime:undname.obj
 0002:00002658       ??_C@_0CE@IIHCMGGL@?$GAlocal?5vftable?5constructor?5closu@ 0000000180029658     libvcruntime:undname.obj
 0002:0000267c       ??_C@_06FHBGPFGH@?5new?$FL?$FN?$AA@ 000000018002967c     libvcruntime:undname.obj
 0002:00002688       ??_C@_09LBNFPBCA@?5delete?$FL?$FN?$AA@ 0000000180029688     libvcruntime:undname.obj
 0002:00002698       ??_C@_0P@HJKNJFNN@?$GAomni?5callsig?8?$AA@ 0000000180029698     libvcruntime:undname.obj
 0002:000026a8       ??_C@_0BL@CNOONJFP@?$GAplacement?5delete?5closure?8?$AA@ 00000001800296a8     libvcruntime:undname.obj
 0002:000026c8       ??_C@_0BN@CKNJLHMB@?$GAplacement?5delete?$FL?$FN?5closure?8?$AA@ 00000001800296c8     libvcruntime:undname.obj
 0002:000026e8       ??_C@_0CG@CFDHKGGD@?$GAmanaged?5vector?5constructor?5iter@ 00000001800296e8     libvcruntime:undname.obj
 0002:00002710       ??_C@_0CF@IMGKMJNO@?$GAmanaged?5vector?5destructor?5itera@ 0000000180029710     libvcruntime:undname.obj
 0002:00002738       ??_C@_0CG@HLDDJMAG@?$GAeh?5vector?5copy?5constructor?5iter@ 0000000180029738     libvcruntime:undname.obj
 0002:00002760       ??_C@_0CM@FCBBDIGB@?$GAeh?5vector?5vbase?5copy?5constructo@ 0000000180029760     libvcruntime:undname.obj
 0002:00002790       ??_C@_0BL@CLIPGLGB@?$GAdynamic?5initializer?5for?5?8?$AA@ 0000000180029790     libvcruntime:undname.obj
 0002:000027b0       ??_C@_0CB@PDBIFEP@?$GAdynamic?5atexit?5destructor?5for?5?8@ 00000001800297b0     libvcruntime:undname.obj
 0002:000027d8       ??_C@_0CD@CGAJBKEJ@?$GAvector?5copy?5constructor?5iterato@ 00000001800297d8     libvcruntime:undname.obj
 0002:00002800       ??_C@_0CJ@GJELGAMM@?$GAvector?5vbase?5copy?5constructor?5i@ 0000000180029800     libvcruntime:undname.obj
 0002:00002830       ??_C@_0CL@FGIJHLCE@?$GAmanaged?5vector?5copy?5constructor@ 0000000180029830     libvcruntime:undname.obj
 0002:00002860       ??_C@_0BM@PMGGMLDN@?$GAlocal?5static?5thread?5guard?8?$AA@ 0000000180029860     libvcruntime:undname.obj
 0002:00002880       ??_C@_0N@BDNMDMOL@operator?5?$CC?$CC?5?$AA@ 0000000180029880     libvcruntime:undname.obj
 0002:00002890       ??_C@_0BC@GGEBGALA@operator?5co_await?$AA@ 0000000180029890     libvcruntime:undname.obj
 0002:000028a8       ??_C@_0BC@DAFEJGAK@?5Type?5Descriptor?8?$AA@ 00000001800298a8     libvcruntime:undname.obj
 0002:000028c0       ??_C@_0BM@LDKODKLH@?5Base?5Class?5Descriptor?5at?5?$CI?$AA@ 00000001800298c0     libvcruntime:undname.obj
 0002:000028e0       ??_C@_0BD@LGICGFMM@?5Base?5Class?5Array?8?$AA@ 00000001800298e0     libvcruntime:undname.obj
 0002:000028f8       ??_C@_0BN@MECKDCOJ@?5Class?5Hierarchy?5Descriptor?8?$AA@ 00000001800298f8     libvcruntime:undname.obj
 0002:00002918       ??_C@_0BK@CFCOFLF@?5Complete?5Object?5Locator?8?$AA@ 0000000180029918     libvcruntime:undname.obj
 0002:00002950       ??_C@_1DM@KHCHBNEB@?$AAa?$AAp?$AAi?$AA?9?$AAm?$AAs?$AA?9?$AAw?$AAi?$AAn?$AA?9?$AAc?$AAo?$AAr?$AAe?$AA?9?$AAf?$AAi?$AAb?$AAe?$AAr?$AAs?$AA?9?$AAl?$AA1?$AA?9?$AA1?$AA?9?$AA1?$AA?$AA@ 0000000180029950     libvcruntime:winapi_downlevel.obj
 0002:00002990       ??_C@_1DK@LPPGFMPP@?$AAa?$AAp?$AAi?$AA?9?$AAm?$AAs?$AA?9?$AAw?$AAi?$AAn?$AA?9?$AAc?$AAo?$AAr?$AAe?$AA?9?$AAs?$AAy?$AAn?$AAc?$AAh?$AA?9?$AAl?$AA1?$AA?9?$AA2?$AA?9?$AA0?$AA?$AA@ 0000000180029990     libvcruntime:winapi_downlevel.obj
 0002:000029d0       ??_C@_1BC@GDMECMAK@?$AAk?$AAe?$AAr?$AAn?$AAe?$AAl?$AA3?$AA2?$AA?$AA@ 00000001800299d0     libvcruntime:winapi_downlevel.obj
 0002:000029e8       ??_C@_1BA@PFFKHIOG@?$AAa?$AAp?$AAi?$AA?9?$AAm?$AAs?$AA?9?$AA?$AA@ 00000001800299e8     libvcruntime:winapi_downlevel.obj
 0002:000029f8       ??_C@_1BA@IAIFMGEF@?$AAe?$AAx?$AAt?$AA?9?$AAm?$AAs?$AA?9?$AA?$AA@ 00000001800299f8     libvcruntime:winapi_downlevel.obj
 0002:00002a10       ??_C@_08KNHFBNJ@FlsAlloc?$AA@ 0000000180029a10     libvcruntime:winapi_downlevel.obj
 0002:00002a28       ??_C@_07PEJMOBNF@FlsFree?$AA@ 0000000180029a28     libvcruntime:winapi_downlevel.obj
 0002:00002a38       ??_C@_0M@GDNOONDI@FlsGetValue?$AA@ 0000000180029a38     libvcruntime:winapi_downlevel.obj
 0002:00002a50       ??_C@_0M@JCPCPOEF@FlsSetValue?$AA@ 0000000180029a50     libvcruntime:winapi_downlevel.obj
 0002:00002a68       ??_C@_0BM@HCFOFFN@InitializeCriticalSectionEx?$AA@ 0000000180029a68     libvcruntime:winapi_downlevel.obj
 0002:00002a88       _pDestructExceptionObject  0000000180029a88     libvcruntime:ehhelpers.obj
 0002:00002ad0       standard_lookup_table      0000000180029ad0     libucrt:output.obj
 0002:00002b2c       ??_C@_06OJHGLDPL@?$CInull?$CJ?$AA@ 0000000180029b2c     libucrt:output.obj
 0002:00002b38       ??_C@_1O@CEDCILHN@?$AA?$CI?$AAn?$AAu?$AAl?$AAl?$AA?$CJ?$AA?$AA@ 0000000180029b38     libucrt:output.obj
 0002:00002b50       __acrt_exception_action_table 0000000180029b50     libucrt:exception_filter.obj
 0002:00002c10       __acrt_signal_action_table_count 0000000180029c10     libucrt:exception_filter.obj
 0002:00002c18       __acrt_signal_action_first_fpe_index 0000000180029c18     libucrt:exception_filter.obj
 0002:00002c20       __acrt_signal_action_fpe_count 0000000180029c20     libucrt:exception_filter.obj
 0002:00002c28       ??_C@_1BI@BGOHAHKC@?$AAm?$AAs?$AAc?$AAo?$AAr?$AAe?$AAe?$AA?4?$AAd?$AAl?$AAl?$AA?$AA@ 0000000180029c28     libucrt:exit.obj
 0002:00002c40       ??_C@_0P@MIGLKIOC@CorExitProcess?$AA@ 0000000180029c40     libucrt:exit.obj
 0002:00002ea8       ??_C@_03OEIAHPBN@INF?$AA@  0000000180029ea8     libucrt:cvt.obj
 0002:00002eac       ??_C@_03OJHLLCGB@inf?$AA@  0000000180029eac     libucrt:cvt.obj
 0002:00002eb0       ??_C@_03LKNCIKJB@NAN?$AA@  0000000180029eb0     libucrt:cvt.obj
 0002:00002eb4       ??_C@_03LHCJEHON@nan?$AA@  0000000180029eb4     libucrt:cvt.obj
 0002:00002eb8       ??_C@_09OFJJIMPC@NAN?$CISNAN?$CJ?$AA@ 0000000180029eb8     libucrt:cvt.obj
 0002:00002ec8       ??_C@_09IPFBKMDL@nan?$CIsnan?$CJ?$AA@ 0000000180029ec8     libucrt:cvt.obj
 0002:00002ed8       ??_C@_08IKHNHAJ@NAN?$CIIND?$CJ?$AA@ 0000000180029ed8     libucrt:cvt.obj
 0002:00002ee8       ??_C@_08OFCDMILK@nan?$CIind?$CJ?$AA@ 0000000180029ee8     libucrt:cvt.obj
 0002:00002ef4       ??_C@_05KLBDPFGC@e?$CL000?$AA@ 0000000180029ef4     libucrt:cvt.obj
 0002:00002f00       __lc_time_c                0000000180029f00     libucrt:nlsdata.obj
 0002:000031c0       ??_C@_03KOEHGMDN@Sun?$AA@  000000018002a1c0     libucrt:nlsdata.obj
 0002:000031c4       ??_C@_03PDAGKDH@Mon?$AA@   000000018002a1c4     libucrt:nlsdata.obj
 0002:000031c8       ??_C@_03NAGEINEP@Tue?$AA@  000000018002a1c8     libucrt:nlsdata.obj
 0002:000031cc       ??_C@_03MHOMLAJA@Wed?$AA@  000000018002a1cc     libucrt:nlsdata.obj
 0002:000031d0       ??_C@_03IOFIKPDN@Thu?$AA@  000000018002a1d0     libucrt:nlsdata.obj
 0002:000031d4       ??_C@_03IDIOELNC@Fri?$AA@  000000018002a1d4     libucrt:nlsdata.obj
 0002:000031d8       ??_C@_03FEFJNEK@Sat?$AA@   000000018002a1d8     libucrt:nlsdata.obj
 0002:000031dc       ??_C@_06OOPIFAJ@Sunday?$AA@ 000000018002a1dc     libucrt:nlsdata.obj
 0002:000031e4       ??_C@_06JLEDEDGH@Monday?$AA@ 000000018002a1e4     libucrt:nlsdata.obj
 0002:000031f0       ??_C@_07BAAGCFCM@Tuesday?$AA@ 000000018002a1f0     libucrt:nlsdata.obj
 0002:000031f8       ??_C@_09DLIGFAKA@Wednesday?$AA@ 000000018002a1f8     libucrt:nlsdata.obj
 0002:00003208       ??_C@_08HACCIKIA@Thursday?$AA@ 000000018002a208     libucrt:nlsdata.obj
 0002:00003214       ??_C@_06JECMNKMI@Friday?$AA@ 000000018002a214     libucrt:nlsdata.obj
 0002:00003220       ??_C@_08INBOOONO@Saturday?$AA@ 000000018002a220     libucrt:nlsdata.obj
 0002:0000322c       ??_C@_03JIHJHPIE@Jan?$AA@  000000018002a22c     libucrt:nlsdata.obj
 0002:00003230       ??_C@_03HJBDCHOM@Feb?$AA@  000000018002a230     libucrt:nlsdata.obj
 0002:00003234       ??_C@_03ODNJBKGA@Mar?$AA@  000000018002a234     libucrt:nlsdata.obj
 0002:00003238       ??_C@_03LEOLGMJP@Apr?$AA@  000000018002a238     libucrt:nlsdata.obj
 0002:0000323c       ??_C@_03CNMDKL@May?$AA@    000000018002a23c     libucrt:nlsdata.obj
 0002:00003240       ??_C@_03IDFGHECI@Jun?$AA@  000000018002a240     libucrt:nlsdata.obj
 0002:00003244       ??_C@_03LBGABGKK@Jul?$AA@  000000018002a244     libucrt:nlsdata.obj
 0002:00003248       ??_C@_03IFJFEIGA@Aug?$AA@  000000018002a248     libucrt:nlsdata.obj
 0002:0000324c       ??_C@_03GGCAPAJC@Sep?$AA@  000000018002a24c     libucrt:nlsdata.obj
 0002:00003250       ??_C@_03BMAOKBAD@Oct?$AA@  000000018002a250     libucrt:nlsdata.obj
 0002:00003254       ??_C@_03JPJOFNIA@Nov?$AA@  000000018002a254     libucrt:nlsdata.obj
 0002:00003258       ??_C@_03MKABNOCG@Dec?$AA@  000000018002a258     libucrt:nlsdata.obj
 0002:00003260       ??_C@_07CGJPFGJA@January?$AA@ 000000018002a260     libucrt:nlsdata.obj
 0002:00003268       ??_C@_08GNJGEPFN@February?$AA@ 000000018002a268     libucrt:nlsdata.obj
 0002:00003274       ??_C@_05HPCKOFNC@March?$AA@ 000000018002a274     libucrt:nlsdata.obj
 0002:0000327c       ??_C@_05DMJDNLEJ@April?$AA@ 000000018002a27c     libucrt:nlsdata.obj
 0002:00003284       ??_C@_04CNLMGBGM@June?$AA@ 000000018002a284     libucrt:nlsdata.obj
 0002:0000328c       ??_C@_04MIEPOIFP@July?$AA@ 000000018002a28c     libucrt:nlsdata.obj
 0002:00003294       ??_C@_06LBBHFDDG@August?$AA@ 000000018002a294     libucrt:nlsdata.obj
 0002:000032a0       ??_C@_09BHHEALKD@September?$AA@ 000000018002a2a0     libucrt:nlsdata.obj
 0002:000032b0       ??_C@_07JJNFCEND@October?$AA@ 000000018002a2b0     libucrt:nlsdata.obj
 0002:000032b8       ??_C@_08HCHEGEOA@November?$AA@ 000000018002a2b8     libucrt:nlsdata.obj
 0002:000032c8       ??_C@_08EDHMEBNP@December?$AA@ 000000018002a2c8     libucrt:nlsdata.obj
 0002:000032d4       ??_C@_02DEDBPAFC@AM?$AA@   000000018002a2d4     libucrt:nlsdata.obj
 0002:000032d8       ??_C@_02CJNFDJBF@PM?$AA@   000000018002a2d8     libucrt:nlsdata.obj
 0002:000032e0       ??_C@_08BPBNCDIB@MM?1dd?1yy?$AA@ 000000018002a2e0     libucrt:nlsdata.obj
 0002:000032f0       ??_C@_0BE@CKGJFCPC@dddd?0?5MMMM?5dd?0?5yyyy?$AA@ 000000018002a2f0     libucrt:nlsdata.obj
 0002:00003308       ??_C@_08JCCMCCIL@HH?3mm?3ss?$AA@ 000000018002a308     libucrt:nlsdata.obj
 0002:00003318       ??_C@_17MBGCMIPB@?$AAS?$AAu?$AAn?$AA?$AA@ 000000018002a318     libucrt:nlsdata.obj
 0002:00003320       ??_C@_17KBOMKBF@?$AAM?$AAo?$AAn?$AA?$AA@ 000000018002a320     libucrt:nlsdata.obj
 0002:00003328       ??_C@_17BMKGEGOJ@?$AAT?$AAu?$AAe?$AA?$AA@ 000000018002a328     libucrt:nlsdata.obj
 0002:00003330       ??_C@_17CJEDCEPE@?$AAW?$AAe?$AAd?$AA?$AA@ 000000018002a330     libucrt:nlsdata.obj
 0002:00003338       ??_C@_17PDPHAADD@?$AAT?$AAh?$AAu?$AA?$AA@ 000000018002a338     libucrt:nlsdata.obj
 0002:00003340       ??_C@_17HFOLPPLP@?$AAF?$AAr?$AAi?$AA?$AA@ 000000018002a340     libucrt:nlsdata.obj
 0002:00003348       ??_C@_17GGIBDPIH@?$AAS?$AAa?$AAt?$AA?$AA@ 000000018002a348     libucrt:nlsdata.obj
 0002:00003350       ??_C@_1O@IHNHDHPB@?$AAS?$AAu?$AAn?$AAd?$AAa?$AAy?$AA?$AA@ 000000018002a350     libucrt:nlsdata.obj
 0002:00003360       ??_C@_1O@MMNBFLIA@?$AAM?$AAo?$AAn?$AAd?$AAa?$AAy?$AA?$AA@ 000000018002a360     libucrt:nlsdata.obj
 0002:00003370       ??_C@_1BA@ENFBFFEK@?$AAT?$AAu?$AAe?$AAs?$AAd?$AAa?$AAy?$AA?$AA@ 000000018002a370     libucrt:nlsdata.obj
 0002:00003380       ??_C@_1BE@EBOGMDOH@?$AAW?$AAe?$AAd?$AAn?$AAe?$AAs?$AAd?$AAa?$AAy?$AA?$AA@ 000000018002a380     libucrt:nlsdata.obj
 0002:00003398       ??_C@_1BC@HHMNLIHE@?$AAT?$AAh?$AAu?$AAr?$AAs?$AAd?$AAa?$AAy?$AA?$AA@ 000000018002a398     libucrt:nlsdata.obj
 0002:000033b0       ??_C@_1O@PDICJHAG@?$AAF?$AAr?$AAi?$AAd?$AAa?$AAy?$AA?$AA@ 000000018002a3b0     libucrt:nlsdata.obj
 0002:000033c0       ??_C@_1BC@ENMNNPAJ@?$AAS?$AAa?$AAt?$AAu?$AAr?$AAd?$AAa?$AAy?$AA?$AA@ 000000018002a3c0     libucrt:nlsdata.obj
 0002:000033d8       ??_C@_17DKNBKCHM@?$AAJ?$AAa?$AAn?$AA?$AA@ 000000018002a3d8     libucrt:nlsdata.obj
 0002:000033e0       ??_C@_17LMDJEKJN@?$AAF?$AAe?$AAb?$AA?$AA@ 000000018002a3e0     libucrt:nlsdata.obj
 0002:000033e8       ??_C@_17CKNLEDEC@?$AAM?$AAa?$AAr?$AA?$AA@ 000000018002a3e8     libucrt:nlsdata.obj
 0002:000033f0       ??_C@_17LFPOIHDD@?$AAA?$AAp?$AAr?$AA?$AA@ 000000018002a3f0     libucrt:nlsdata.obj
 0002:000033f8       ??_C@_17PNNKMEED@?$AAM?$AAa?$AAy?$AA?$AA@ 000000018002a3f8     libucrt:nlsdata.obj
 0002:00003400       ??_C@_17KCJGOCPB@?$AAJ?$AAu?$AAn?$AA?$AA@ 000000018002a400     libucrt:nlsdata.obj
 0002:00003408       ??_C@_17IJPCKHK@?$AAJ?$AAu?$AAl?$AA?$AA@ 000000018002a408     libucrt:nlsdata.obj
 0002:00003410       ??_C@_17ICPELBCN@?$AAA?$AAu?$AAg?$AA?$AA@ 000000018002a410     libucrt:nlsdata.obj
 0002:00003418       ??_C@_17HCHCOKMG@?$AAS?$AAe?$AAp?$AA?$AA@ 000000018002a418     libucrt:nlsdata.obj
 0002:00003420       ??_C@_17FNLKOI@?$AAO?$AAc?$AAt?$AA?$AA@ 000000018002a420     libucrt:nlsdata.obj
 0002:00003428       ??_C@_17BBDMLCIG@?$AAN?$AAo?$AAv?$AA?$AA@ 000000018002a428     libucrt:nlsdata.obj
 0002:00003430       ??_C@_17EGKACKIF@?$AAD?$AAe?$AAc?$AA?$AA@ 000000018002a430     libucrt:nlsdata.obj
 0002:00003438       ??_C@_1BA@EFMEIEBA@?$AAJ?$AAa?$AAn?$AAu?$AAa?$AAr?$AAy?$AA?$AA@ 000000018002a438     libucrt:nlsdata.obj
 0002:00003448       ??_C@_1BC@JGDDFFAM@?$AAF?$AAe?$AAb?$AAr?$AAu?$AAa?$AAr?$AAy?$AA?$AA@ 000000018002a448     libucrt:nlsdata.obj
 0002:00003460       ??_C@_1M@IKEENEDF@?$AAM?$AAa?$AAr?$AAc?$AAh?$AA?$AA@ 000000018002a460     libucrt:nlsdata.obj
 0002:00003470       ??_C@_1M@GJNLMHFD@?$AAA?$AAp?$AAr?$AAi?$AAl?$AA?$AA@ 000000018002a470     libucrt:nlsdata.obj
 0002:00003480       ??_C@_19EPFLPGAP@?$AAJ?$AAu?$AAn?$AAe?$AA?$AA@ 000000018002a480     libucrt:nlsdata.obj
 0002:00003490       ??_C@_19BIFMLPCD@?$AAJ?$AAu?$AAl?$AAy?$AA?$AA@ 000000018002a490     libucrt:nlsdata.obj
 0002:000034a0       ??_C@_1O@PAHLKOAC@?$AAA?$AAu?$AAg?$AAu?$AAs?$AAt?$AA?$AA@ 000000018002a4a0     libucrt:nlsdata.obj
 0002:000034b0       ??_C@_1BE@DKAAMBJL@?$AAS?$AAe?$AAp?$AAt?$AAe?$AAm?$AAb?$AAe?$AAr?$AA?$AA@ 000000018002a4b0     libucrt:nlsdata.obj
 0002:000034c8       ??_C@_1BA@EPANDLNG@?$AAO?$AAc?$AAt?$AAo?$AAb?$AAe?$AAr?$AA?$AA@ 000000018002a4c8     libucrt:nlsdata.obj
 0002:000034d8       ??_C@_1BC@BGLIFPF@?$AAN?$AAo?$AAv?$AAe?$AAm?$AAb?$AAe?$AAr?$AA?$AA@ 000000018002a4d8     libucrt:nlsdata.obj
 0002:000034f0       ??_C@_1BC@FEMKIFH@?$AAD?$AAe?$AAc?$AAe?$AAm?$AAb?$AAe?$AAr?$AA?$AA@ 000000018002a4f0     libucrt:nlsdata.obj
 0002:00003504       ??_C@_15ODEHAHHF@?$AAA?$AAM?$AA?$AA@ 000000018002a504     libucrt:nlsdata.obj
 0002:0000350c       ??_C@_15CLMNNGEL@?$AAP?$AAM?$AA?$AA@ 000000018002a50c     libucrt:nlsdata.obj
 0002:00003518       ??_C@_1BC@IEBCMHCM@?$AAM?$AAM?$AA?1?$AAd?$AAd?$AA?1?$AAy?$AAy?$AA?$AA@ 000000018002a518     libucrt:nlsdata.obj
 0002:00003530       ??_C@_1CI@KNAKOEBC@?$AAd?$AAd?$AAd?$AAd?$AA?0?$AA?5?$AAM?$AAM?$AAM?$AAM?$AA?5?$AAd?$AAd?$AA?0?$AA?5?$AAy?$AAy?$AAy?$AAy?$AA?$AA@ 000000018002a530     libucrt:nlsdata.obj
 0002:00003558       ??_C@_1BC@GDGBMEMK@?$AAH?$AAH?$AA?3?$AAm?$AAm?$AA?3?$AAs?$AAs?$AA?$AA@ 000000018002a558     libucrt:nlsdata.obj
 0002:00003570       ??_C@_1M@BMHNFIME@?$AAe?$AAn?$AA?9?$AAU?$AAS?$AA?$AA@ 000000018002a570     libucrt:nlsdata.obj
 0002:00003580       __newctype                 000000018002a580     libucrt:ctype.obj
 0002:00003880       __newclmap                 000000018002a880     libucrt:ctype.obj
 0002:00003a00       __newcumap                 000000018002aa00     libucrt:ctype.obj
 0002:00003b80       _wctype                    000000018002ab80     libucrt:ctype.obj
 0002:00003e30       ??_C@_1EG@CNNIPFIM@?$AAa?$AAp?$AAi?$AA?9?$AAm?$AAs?$AA?9?$AAw?$AAi?$AAn?$AA?9?$AAa?$AAp?$AAp?$AAm?$AAo?$AAd?$AAe?$AAl?$AA?9?$AAr?$AAu?$AAn?$AAt?$AAi?$AAm?$AAe?$AA?9?$AAl?$AA1?$AA?9?$AA1@ 000000018002ae30     libucrt:winapi_thunks.obj
 0002:00003e80       ??_C@_1EA@JGEFHKEI@?$AAa?$AAp?$AAi?$AA?9?$AAm?$AAs?$AA?9?$AAw?$AAi?$AAn?$AA?9?$AAc?$AAo?$AAr?$AAe?$AA?9?$AAd?$AAa?$AAt?$AAe?$AAt?$AAi?$AAm?$AAe?$AA?9?$AAl?$AA1?$AA?9?$AA1?$AA?9?$AA1?$AA?$AA@ 000000018002ae80     libucrt:winapi_thunks.obj
 0002:00003ec0       ??_C@_1DI@GCIAAENM@?$AAa?$AAp?$AAi?$AA?9?$AAm?$AAs?$AA?9?$AAw?$AAi?$AAn?$AA?9?$AAc?$AAo?$AAr?$AAe?$AA?9?$AAf?$AAi?$AAl?$AAe?$AA?9?$AAl?$AA2?$AA?9?$AA1?$AA?9?$AA1?$AA?$AA@ 000000018002aec0     libucrt:winapi_thunks.obj
 0002:00003f00       ??_C@_1EI@MPIAOHOC@?$AAa?$AAp?$AAi?$AA?9?$AAm?$AAs?$AA?9?$AAw?$AAi?$AAn?$AA?9?$AAc?$AAo?$AAr?$AAe?$AA?9?$AAl?$AAo?$AAc?$AAa?$AAl?$AAi?$AAz?$AAa?$AAt?$AAi?$AAo?$AAn?$AA?9?$AAl?$AA1?$AA?9@ 000000018002af00     libucrt:winapi_thunks.obj
 0002:00003f50       ??_C@_1FK@FPHCKFIE@?$AAa?$AAp?$AAi?$AA?9?$AAm?$AAs?$AA?9?$AAw?$AAi?$AAn?$AA?9?$AAc?$AAo?$AAr?$AAe?$AA?9?$AAl?$AAo?$AAc?$AAa?$AAl?$AAi?$AAz?$AAa?$AAt?$AAi?$AAo?$AAn?$AA?9?$AAo?$AAb?$AAs@ 000000018002af50     libucrt:winapi_thunks.obj
 0002:00003fb0       ??_C@_1EM@DILCGIIO@?$AAa?$AAp?$AAi?$AA?9?$AAm?$AAs?$AA?9?$AAw?$AAi?$AAn?$AA?9?$AAc?$AAo?$AAr?$AAe?$AA?9?$AAp?$AAr?$AAo?$AAc?$AAe?$AAs?$AAs?$AAt?$AAh?$AAr?$AAe?$AAa?$AAd?$AAs?$AA?9?$AAl@ 000000018002afb0     libucrt:winapi_thunks.obj
 0002:00004000       ??_C@_1DM@LNCGDDPN@?$AAa?$AAp?$AAi?$AA?9?$AAm?$AAs?$AA?9?$AAw?$AAi?$AAn?$AA?9?$AAc?$AAo?$AAr?$AAe?$AA?9?$AAs?$AAt?$AAr?$AAi?$AAn?$AAg?$AA?9?$AAl?$AA1?$AA?9?$AA1?$AA?9?$AA0?$AA?$AA@ 000000018002b000     libucrt:winapi_thunks.obj
 0002:00004040       ??_C@_1DO@FPAPJEMD@?$AAa?$AAp?$AAi?$AA?9?$AAm?$AAs?$AA?9?$AAw?$AAi?$AAn?$AA?9?$AAc?$AAo?$AAr?$AAe?$AA?9?$AAs?$AAy?$AAs?$AAi?$AAn?$AAf?$AAo?$AA?9?$AAl?$AA1?$AA?9?$AA2?$AA?9?$AA1?$AA?$AA@ 000000018002b040     libucrt:winapi_thunks.obj
 0002:00004080       ??_C@_1DK@NDHNAHIO@?$AAa?$AAp?$AAi?$AA?9?$AAm?$AAs?$AA?9?$AAw?$AAi?$AAn?$AA?9?$AAc?$AAo?$AAr?$AAe?$AA?9?$AAw?$AAi?$AAn?$AAr?$AAt?$AA?9?$AAl?$AA1?$AA?9?$AA1?$AA?9?$AA0?$AA?$AA@ 000000018002b080     libucrt:winapi_thunks.obj
 0002:000040c0       ??_C@_1DM@KGHDGBCM@?$AAa?$AAp?$AAi?$AA?9?$AAm?$AAs?$AA?9?$AAw?$AAi?$AAn?$AA?9?$AAc?$AAo?$AAr?$AAe?$AA?9?$AAx?$AAs?$AAt?$AAa?$AAt?$AAe?$AA?9?$AAl?$AA2?$AA?9?$AA1?$AA?9?$AA0?$AA?$AA@ 000000018002b0c0     libucrt:winapi_thunks.obj
 0002:00004100       ??_C@_1EO@IJIOEFOH@?$AAa?$AAp?$AAi?$AA?9?$AAm?$AAs?$AA?9?$AAw?$AAi?$AAn?$AA?9?$AAr?$AAt?$AAc?$AAo?$AAr?$AAe?$AA?9?$AAn?$AAt?$AAu?$AAs?$AAe?$AAr?$AA?9?$AAw?$AAi?$AAn?$AAd?$AAo?$AAw?$AA?9@ 000000018002b100     libucrt:winapi_thunks.obj
 0002:00004150       ??_C@_1FG@HHGEKANL@?$AAa?$AAp?$AAi?$AA?9?$AAm?$AAs?$AA?9?$AAw?$AAi?$AAn?$AA?9?$AAs?$AAe?$AAc?$AAu?$AAr?$AAi?$AAt?$AAy?$AA?9?$AAs?$AAy?$AAs?$AAt?$AAe?$AAm?$AAf?$AAu?$AAn?$AAc?$AAt?$AAi@ 000000018002b150     libucrt:winapi_thunks.obj
 0002:000041b0       ??_C@_1FG@NCKKOLKO@?$AAe?$AAx?$AAt?$AA?9?$AAm?$AAs?$AA?9?$AAw?$AAi?$AAn?$AA?9?$AAk?$AAe?$AAr?$AAn?$AAe?$AAl?$AA3?$AA2?$AA?9?$AAp?$AAa?$AAc?$AAk?$AAa?$AAg?$AAe?$AA?9?$AAc?$AAu?$AAr?$AAr@ 000000018002b1b0     libucrt:winapi_thunks.obj
 0002:00004210       ??_C@_1EG@DBIOJECG@?$AAe?$AAx?$AAt?$AA?9?$AAm?$AAs?$AA?9?$AAw?$AAi?$AAn?$AA?9?$AAn?$AAt?$AAu?$AAs?$AAe?$AAr?$AA?9?$AAd?$AAi?$AAa?$AAl?$AAo?$AAg?$AAb?$AAo?$AAx?$AA?9?$AAl?$AA1?$AA?9?$AA1@ 000000018002b210     libucrt:winapi_thunks.obj
 0002:00004260       ??_C@_1EO@FIHMJCLF@?$AAe?$AAx?$AAt?$AA?9?$AAm?$AAs?$AA?9?$AAw?$AAi?$AAn?$AA?9?$AAn?$AAt?$AAu?$AAs?$AAe?$AAr?$AA?9?$AAw?$AAi?$AAn?$AAd?$AAo?$AAw?$AAs?$AAt?$AAa?$AAt?$AAi?$AAo?$AAn?$AA?9@ 000000018002b260     libucrt:winapi_thunks.obj
 0002:000042b0       ??_C@_1BC@DNHGCMLG@?$AAa?$AAd?$AAv?$AAa?$AAp?$AAi?$AA3?$AA2?$AA?$AA@ 000000018002b2b0     libucrt:winapi_thunks.obj
 0002:000042c8       ??_C@_1O@BCCLBEOE@?$AAu?$AAs?$AAe?$AAr?$AA3?$AA2?$AA?$AA@ 000000018002b2c8     libucrt:winapi_thunks.obj
 0002:00004300       ??_C@_0BE@JOGNEJCI@GetCurrentPackageId?$AA@ 000000018002b300     libucrt:winapi_thunks.obj
 0002:00004328       ??_C@_0O@KKBNKAPF@LCMapStringEx?$AA@ 000000018002b328     libucrt:winapi_thunks.obj
 0002:00004340       ??_C@_0BB@HBDEELFH@LocaleNameToLCID?$AA@ 000000018002b340     libucrt:winapi_thunks.obj
 0002:00004378       ??_C@_1M@HPNHIDJI@?$AAj?$AAa?$AA?9?$AAJ?$AAP?$AA?$AA@ 000000018002b378     libucrt:mbctype.obj
 0002:00004388       ??_C@_1M@BIBDDEMK@?$AAz?$AAh?$AA?9?$AAC?$AAN?$AA?$AA@ 000000018002b388     libucrt:mbctype.obj
 0002:00004398       ??_C@_1M@JLOOOEGK@?$AAk?$AAo?$AA?9?$AAK?$AAR?$AA?$AA@ 000000018002b398     libucrt:mbctype.obj
 0002:000043a8       ??_C@_1M@CLNBBOPM@?$AAz?$AAh?$AA?9?$AAT?$AAW?$AA?$AA@ 000000018002b3a8     libucrt:mbctype.obj
 0002:000043c0       ?large_power_data@?1??multiply_by_power_of_ten@__crt_strtox@@YA_NAEAUbig_integer@2@I@Z@4QBIB 000000018002b3c0     libucrt:cfout.obj
 0002:00004cd0       ?large_power_indices@?1??multiply_by_power_of_ten@__crt_strtox@@YA_NAEAUbig_integer@2@I@Z@4QBUunpack_index@?1??12@YA_N0I@Z@B 000000018002bcd0     libucrt:cfout.obj
 0002:00004d68       ?small_powers_of_ten@?6??multiply_by_power_of_ten@__crt_strtox@@YA_NAEAUbig_integer@2@I@Z@4QBIB 000000018002bd68     libucrt:cfout.obj
 0002:00004d8c       ??_C@_01GBGANLPD@0?$AA@    000000018002bd8c     libucrt:cfout.obj
 0002:00004d90       ??_C@_05DNEBIAHO@1?$CDINF?$AA@ 000000018002bd90     libucrt:cfout.obj
 0002:00004d98       ??_C@_06IMKFLFPG@1?$CDQNAN?$AA@ 000000018002bd98     libucrt:cfout.obj
 0002:00004da0       ??_C@_06PGGFOGJG@1?$CDSNAN?$AA@ 000000018002bda0     libucrt:cfout.obj
 0002:00004da8       ??_C@_05PHHOCPM@1?$CDIND?$AA@ 000000018002bda8     libucrt:cfout.obj
 0002:00004db0       ??_C@_15PJPFLCCM@?$AAu?$AAk?$AA?$AA@ 000000018002bdb0     libucrt:get_qualified_locale.obj
 0002:00005c00       ??_C@_15EMKDOKLE@?$AAa?$AAr?$AA?$AA@ 000000018002cc00     libucrt:lcidtoname_downlevel.obj
 0002:00005c08       ??_C@_15KNPADPLH@?$AAb?$AAg?$AA?$AA@ 000000018002cc08     libucrt:lcidtoname_downlevel.obj
 0002:00005c10       ??_C@_15EDMHLDMO@?$AAc?$AAa?$AA?$AA@ 000000018002cc10     libucrt:lcidtoname_downlevel.obj
 0002:00005c18       ??_C@_1O@BPEAJADD@?$AAz?$AAh?$AA?9?$AAC?$AAH?$AAS?$AA?$AA@ 000000018002cc18     libucrt:lcidtoname_downlevel.obj
 0002:00005c28       ??_C@_15LJNHCMNK@?$AAc?$AAs?$AA?$AA@ 000000018002cc28     libucrt:lcidtoname_downlevel.obj
 0002:00005c30       ??_C@_15FOMCIDHG@?$AAd?$AAa?$AA?$AA@ 000000018002cc30     libucrt:lcidtoname_downlevel.obj
 0002:00005c38       ??_C@_15NBKABECB@?$AAd?$AAe?$AA?$AA@ 000000018002cc38     libucrt:lcidtoname_downlevel.obj
 0002:00005c40       ??_C@_15GHPEIIAO@?$AAe?$AAl?$AA?$AA@ 000000018002cc40     libucrt:lcidtoname_downlevel.obj
 0002:00005c48       ??_C@_15MNPNEAIF@?$AAe?$AAn?$AA?$AA@ 000000018002cc48     libucrt:lcidtoname_downlevel.obj
 0002:00005c50       ??_C@_15GPIOMPMH@?$AAe?$AAs?$AA?$AA@ 000000018002cc50     libucrt:lcidtoname_downlevel.obj
 0002:00005c58       ??_C@_15NGLOAKJC@?$AAf?$AAi?$AA?$AA@ 000000018002cc58     libucrt:lcidtoname_downlevel.obj
 0002:00005c60       ??_C@_15FBKGNKAM@?$AAf?$AAr?$AA?$AA@ 000000018002cc60     libucrt:lcidtoname_downlevel.obj
 0002:00005c68       ??_C@_15KGGCNEFK@?$AAh?$AAe?$AA?$AA@ 000000018002cc68     libucrt:lcidtoname_downlevel.obj
 0002:00005c70       ??_C@_15PGHLIDMF@?$AAh?$AAu?$AA?$AA@ 000000018002cc70     libucrt:lcidtoname_downlevel.obj
 0002:00005c78       ??_C@_15BIEMAPLM@?$AAi?$AAs?$AA?$AA@ 000000018002cc78     libucrt:lcidtoname_downlevel.obj
 0002:00005c80       ??_C@_15IFJLDHAF@?$AAi?$AAt?$AA?$AA@ 000000018002cc80     libucrt:lcidtoname_downlevel.obj
 0002:00005c88       ??_C@_15GEMIOCAG@?$AAj?$AAa?$AA?$AA@ 000000018002cc88     libucrt:lcidtoname_downlevel.obj
 0002:00005c90       ??_C@_15EPELEGJA@?$AAk?$AAo?$AA?$AA@ 000000018002cc90     libucrt:lcidtoname_downlevel.obj
 0002:00005c98       ??_C@_15NDDHIMN@?$AAn?$AAl?$AA?$AA@ 000000018002cc98     libucrt:lcidtoname_downlevel.obj
 0002:00005ca0       ??_C@_15BPIGNHCD@?$AAn?$AAo?$AA?$AA@ 000000018002cca0     libucrt:lcidtoname_downlevel.obj
 0002:00005ca8       ??_C@_15DEOPBLCG@?$AAp?$AAl?$AA?$AA@ 000000018002cca8     libucrt:lcidtoname_downlevel.obj
 0002:00005cb0       ??_C@_15KBECGEFG@?$AAp?$AAt?$AA?$AA@ 000000018002ccb0     libucrt:lcidtoname_downlevel.obj
 0002:00005cb8       ??_C@_15GLJCBFMD@?$AAr?$AAo?$AA?$AA@ 000000018002ccb8     libucrt:lcidtoname_downlevel.obj
 0002:00005cc0       ??_C@_15FEDGKCDI@?$AAr?$AAu?$AA?$AA@ 000000018002ccc0     libucrt:lcidtoname_downlevel.obj
 0002:00005cc8       ??_C@_15GLKMLLHM@?$AAh?$AAr?$AA?$AA@ 000000018002ccc8     libucrt:lcidtoname_downlevel.obj
 0002:00005cd0       ??_C@_15CPKMFBDB@?$AAs?$AAk?$AA?$AA@ 000000018002ccd0     libucrt:lcidtoname_downlevel.obj
 0002:00005cd8       ??_C@_15BAAIOGMK@?$AAs?$AAq?$AA?$AA@ 000000018002ccd8     libucrt:lcidtoname_downlevel.obj
 0002:00005ce0       ??_C@_15INNPNOHD@?$AAs?$AAv?$AA?$AA@ 000000018002cce0     libucrt:lcidtoname_downlevel.obj
 0002:00005ce8       ??_C@_15CABMMOGH@?$AAt?$AAh?$AA?$AA@ 000000018002cce8     libucrt:lcidtoname_downlevel.obj
 0002:00005cf0       ??_C@_15BPLIHJJM@?$AAt?$AAr?$AA?$AA@ 000000018002ccf0     libucrt:lcidtoname_downlevel.obj
 0002:00005cf8       ??_C@_15NEOEKKDJ@?$AAu?$AAr?$AA?$AA@ 000000018002ccf8     libucrt:lcidtoname_downlevel.obj
 0002:00005d00       ??_C@_15NFICGAJK@?$AAi?$AAd?$AA?$AA@ 000000018002cd00     libucrt:lcidtoname_downlevel.obj
 0002:00005d08       ??_C@_15HPJPHDM@?$AAb?$AAe?$AA?$AA@ 000000018002cd08     libucrt:lcidtoname_downlevel.obj
 0002:00005d10       ??_C@_15LCHLGJII@?$AAs?$AAl?$AA?$AA@ 000000018002cd10     libucrt:lcidtoname_downlevel.obj
 0002:00005d18       ??_C@_15PCFJPHHO@?$AAe?$AAt?$AA?$AA@ 000000018002cd18     libucrt:lcidtoname_downlevel.obj
 0002:00005d20       ??_C@_15HPFPGODN@?$AAl?$AAv?$AA?$AA@ 000000018002cd20     libucrt:lcidtoname_downlevel.obj
 0002:00005d28       ??_C@_15NFFGKGLG@?$AAl?$AAt?$AA?$AA@ 000000018002cd28     libucrt:lcidtoname_downlevel.obj
 0002:00005d30       ??_C@_15BDAKCCHN@?$AAf?$AAa?$AA?$AA@ 000000018002cd30     libucrt:lcidtoname_downlevel.obj
 0002:00005d38       ??_C@_15NFGIAIAJ@?$AAv?$AAi?$AA?$AA@ 000000018002cd38     libucrt:lcidtoname_downlevel.obj
 0002:00005d40       ??_C@_15LMKNDMHN@?$AAh?$AAy?$AA?$AA@ 000000018002cd40     libucrt:lcidtoname_downlevel.obj
 0002:00005d48       ??_C@_15IJBHMCFL@?$AAa?$AAz?$AA?$AA@ 000000018002cd48     libucrt:lcidtoname_downlevel.obj
 0002:00005d50       ??_C@_15EKOFJABL@?$AAe?$AAu?$AA?$AA@ 000000018002cd50     libucrt:lcidtoname_downlevel.obj
 0002:00005d58       ??_C@_15BGHADCNK@?$AAm?$AAk?$AA?$AA@ 000000018002cd58     libucrt:lcidtoname_downlevel.obj
 0002:00005d60       ??_C@_15JDNICKHM@?$AAa?$AAf?$AA?$AA@ 000000018002cd60     libucrt:lcidtoname_downlevel.obj
 0002:00005d68       ??_C@_15KPJEDBKD@?$AAk?$AAa?$AA?$AA@ 000000018002cd68     libucrt:lcidtoname_downlevel.obj
 0002:00005d70       ??_C@_15PDNFFFEO@?$AAf?$AAo?$AA?$AA@ 000000018002cd70     libucrt:lcidtoname_downlevel.obj
 0002:00005d78       ??_C@_15OMLEGLOC@?$AAh?$AAi?$AA?$AA@ 000000018002cd78     libucrt:lcidtoname_downlevel.obj
 0002:00005d80       ??_C@_15IDNNENKK@?$AAm?$AAs?$AA?$AA@ 000000018002cd80     libucrt:lcidtoname_downlevel.obj
 0002:00005d88       ??_C@_15MACJNBMH@?$AAk?$AAk?$AA?$AA@ 000000018002cd88     libucrt:lcidtoname_downlevel.obj
 0002:00005d90       ??_C@_15DKDJEOND@?$AAk?$AAy?$AA?$AA@ 000000018002cd90     libucrt:lcidtoname_downlevel.obj
 0002:00005d98       ??_C@_15DFGDLJBG@?$AAs?$AAw?$AA?$AA@ 000000018002cd98     libucrt:lcidtoname_downlevel.obj
 0002:00005da0       ??_C@_15BBFAICNG@?$AAu?$AAz?$AA?$AA@ 000000018002cda0     libucrt:lcidtoname_downlevel.obj
 0002:00005da8       ??_C@_15DKNDCGEA@?$AAt?$AAt?$AA?$AA@ 000000018002cda8     libucrt:lcidtoname_downlevel.obj
 0002:00005db0       ??_C@_15MGIFMDPL@?$AAp?$AAa?$AA?$AA@ 000000018002cdb0     libucrt:lcidtoname_downlevel.obj
 0002:00005db8       ??_C@_15HCNDBBA@?$AAg?$AAu?$AA?$AA@ 000000018002cdb8     libucrt:lcidtoname_downlevel.obj
 0002:00005dc0       ??_C@_15FNBEIBON@?$AAt?$AAa?$AA?$AA@ 000000018002cdc0     libucrt:lcidtoname_downlevel.obj
 0002:00005dc8       ??_C@_15NCHGBGLK@?$AAt?$AAe?$AA?$AA@ 000000018002cdc8     libucrt:lcidtoname_downlevel.obj
 0002:00005dd0       ??_C@_15PHPHCBPF@?$AAk?$AAn?$AA?$AA@ 000000018002cdd0     libucrt:lcidtoname_downlevel.obj
 0002:00005dd8       ??_C@_15DLGBCKMP@?$AAm?$AAr?$AA?$AA@ 000000018002cdd8     libucrt:lcidtoname_downlevel.obj
 0002:00005de0       ??_C@_15EABBLBFF@?$AAs?$AAa?$AA?$AA@ 000000018002cde0     libucrt:lcidtoname_downlevel.obj
 0002:00005de8       ??_C@_15CBKOMCOI@?$AAm?$AAn?$AA?$AA@ 000000018002cde8     libucrt:lcidtoname_downlevel.obj
 0002:00005df0       ??_C@_15CKDMCJAF@?$AAg?$AAl?$AA?$AA@ 000000018002cdf0     libucrt:lcidtoname_downlevel.obj
 0002:00005df8       ??_C@_17CNJFBPG@?$AAk?$AAo?$AAk?$AA?$AA@ 000000018002cdf8     libucrt:lcidtoname_downlevel.obj
 0002:00005e00       ??_C@_17FFBJICPL@?$AAs?$AAy?$AAr?$AA?$AA@ 000000018002ce00     libucrt:lcidtoname_downlevel.obj
 0002:00005e08       ??_C@_17KPNDCPAF@?$AAd?$AAi?$AAv?$AA?$AA@ 000000018002ce08     libucrt:lcidtoname_downlevel.obj
 0002:00005e10       ??_C@_1M@OKAHONE@?$AAa?$AAr?$AA?9?$AAS?$AAA?$AA?$AA@ 000000018002ce10     libucrt:lcidtoname_downlevel.obj
 0002:00005e20       ??_C@_1M@FFFIGIGK@?$AAb?$AAg?$AA?9?$AAB?$AAG?$AA?$AA@ 000000018002ce20     libucrt:lcidtoname_downlevel.obj
 0002:00005e30       ??_C@_1M@BJNKEDC@?$AAc?$AAa?$AA?9?$AAE?$AAS?$AA?$AA@ 000000018002ce30     libucrt:lcidtoname_downlevel.obj
 0002:00005e40       ??_C@_1M@IJJHFJHA@?$AAc?$AAs?$AA?9?$AAC?$AAZ?$AA?$AA@ 000000018002ce40     libucrt:lcidtoname_downlevel.obj
 0002:00005e50       ??_C@_1M@CLPEOBGI@?$AAd?$AAa?$AA?9?$AAD?$AAK?$AA?$AA@ 000000018002ce50     libucrt:lcidtoname_downlevel.obj
 0002:00005e60       ??_C@_1M@MCMADGCB@?$AAd?$AAe?$AA?9?$AAD?$AAE?$AA?$AA@ 000000018002ce60     libucrt:lcidtoname_downlevel.obj
 0002:00005e70       ??_C@_1M@OOCKEMAM@?$AAe?$AAl?$AA?9?$AAG?$AAR?$AA?$AA@ 000000018002ce70     libucrt:lcidtoname_downlevel.obj
 0002:00005e80       ??_C@_1M@DDNJFGID@?$AAf?$AAi?$AA?9?$AAF?$AAI?$AA?$AA@ 000000018002ce80     libucrt:lcidtoname_downlevel.obj
 0002:00005e90       ??_C@_1M@GLIPPMAC@?$AAf?$AAr?$AA?9?$AAF?$AAR?$AA?$AA@ 000000018002ce90     libucrt:lcidtoname_downlevel.obj
 0002:00005ea0       ??_C@_1M@GFMCHPE@?$AAh?$AAe?$AA?9?$AAI?$AAL?$AA?$AA@ 000000018002cea0     libucrt:lcidtoname_downlevel.obj
 0002:00005eb0       ??_C@_1M@MHLPGNKM@?$AAh?$AAu?$AA?9?$AAH?$AAU?$AA?$AA@ 000000018002ceb0     libucrt:lcidtoname_downlevel.obj
 0002:00005ec0       ??_C@_1M@LPDDNNPN@?$AAi?$AAs?$AA?9?$AAI?$AAS?$AA?$AA@ 000000018002cec0     libucrt:lcidtoname_downlevel.obj
 0002:00005ed0       ??_C@_1M@MADIPODN@?$AAi?$AAt?$AA?9?$AAI?$AAT?$AA?$AA@ 000000018002ced0     libucrt:lcidtoname_downlevel.obj
 0002:00005ee0       ??_C@_1M@IHBJJGG@?$AAn?$AAl?$AA?9?$AAN?$AAL?$AA?$AA@ 000000018002cee0     libucrt:lcidtoname_downlevel.obj
 0002:00005ef0       ??_C@_1M@EANAGDL@?$AAn?$AAb?$AA?9?$AAN?$AAO?$AA?$AA@ 000000018002cef0     libucrt:lcidtoname_downlevel.obj
 0002:00005f00       ??_C@_1M@NEIEMEGP@?$AAp?$AAl?$AA?9?$AAP?$AAL?$AA?$AA@ 000000018002cf00     libucrt:lcidtoname_downlevel.obj
 0002:00005f10       ??_C@_1M@BOCFIGEP@?$AAp?$AAt?$AA?9?$AAB?$AAR?$AA?$AA@ 000000018002cf10     libucrt:lcidtoname_downlevel.obj
 0002:00005f20       ??_C@_1M@IMPFOPBG@?$AAr?$AAo?$AA?9?$AAR?$AAO?$AA?$AA@ 000000018002cf20     libucrt:lcidtoname_downlevel.obj
 0002:00005f30       ??_C@_1M@IDNNEJMM@?$AAr?$AAu?$AA?9?$AAR?$AAU?$AA?$AA@ 000000018002cf30     libucrt:lcidtoname_downlevel.obj
 0002:00005f40       ??_C@_1M@LILEEOGM@?$AAh?$AAr?$AA?9?$AAH?$AAR?$AA?$AA@ 000000018002cf40     libucrt:lcidtoname_downlevel.obj
 0002:00005f50       ??_C@_1M@FKIFEHPB@?$AAs?$AAk?$AA?9?$AAS?$AAK?$AA?$AA@ 000000018002cf50     libucrt:lcidtoname_downlevel.obj
 0002:00005f60       ??_C@_1M@LJMAMNPJ@?$AAs?$AAq?$AA?9?$AAA?$AAL?$AA?$AA@ 000000018002cf60     libucrt:lcidtoname_downlevel.obj
 0002:00005f70       ??_C@_1M@GIAKDKJK@?$AAs?$AAv?$AA?9?$AAS?$AAE?$AA?$AA@ 000000018002cf70     libucrt:lcidtoname_downlevel.obj
 0002:00005f80       ??_C@_1M@MKJKIKCL@?$AAt?$AAh?$AA?9?$AAT?$AAH?$AA?$AA@ 000000018002cf80     libucrt:lcidtoname_downlevel.obj
 0002:00005f90       ??_C@_1M@MFLCCMPB@?$AAt?$AAr?$AA?9?$AAT?$AAR?$AA?$AA@ 000000018002cf90     libucrt:lcidtoname_downlevel.obj
 0002:00005fa0       ??_C@_1M@OIJHDKJN@?$AAu?$AAr?$AA?9?$AAP?$AAK?$AA?$AA@ 000000018002cfa0     libucrt:lcidtoname_downlevel.obj
 0002:00005fb0       ??_C@_1M@LHIPCIEK@?$AAi?$AAd?$AA?9?$AAI?$AAD?$AA?$AA@ 000000018002cfb0     libucrt:lcidtoname_downlevel.obj
 0002:00005fc0       ??_C@_1M@MFMOBGI@?$AAu?$AAk?$AA?9?$AAU?$AAA?$AA?$AA@ 000000018002cfc0     libucrt:lcidtoname_downlevel.obj
 0002:00005fd0       ??_C@_1M@OBGLJIPL@?$AAb?$AAe?$AA?9?$AAB?$AAY?$AA?$AA@ 000000018002cfd0     libucrt:lcidtoname_downlevel.obj
 0002:00005fe0       ??_C@_1M@BCFAJEAD@?$AAs?$AAl?$AA?9?$AAS?$AAI?$AA?$AA@ 000000018002cfe0     libucrt:lcidtoname_downlevel.obj
 0002:00005ff0       ??_C@_1M@FKFFEDDN@?$AAe?$AAt?$AA?9?$AAE?$AAE?$AA?$AA@ 000000018002cff0     libucrt:lcidtoname_downlevel.obj
 0002:00006000       ??_C@_1M@KGKKAACI@?$AAl?$AAv?$AA?9?$AAL?$AAV?$AA?$AA@ 000000018002d000     libucrt:lcidtoname_downlevel.obj
 0002:00006010       ??_C@_1M@IFGBIJO@?$AAl?$AAt?$AA?9?$AAL?$AAT?$AA?$AA@ 000000018002d010     libucrt:lcidtoname_downlevel.obj
 0002:00006020       ??_C@_1M@FGEAHEDM@?$AAf?$AAa?$AA?9?$AAI?$AAR?$AA?$AA@ 000000018002d020     libucrt:lcidtoname_downlevel.obj
 0002:00006030       ??_C@_1M@KBMAIBFN@?$AAv?$AAi?$AA?9?$AAV?$AAN?$AA?$AA@ 000000018002d030     libucrt:lcidtoname_downlevel.obj
 0002:00006040       ??_C@_1M@GPCBKDJK@?$AAh?$AAy?$AA?9?$AAA?$AAM?$AA?$AA@ 000000018002d040     libucrt:lcidtoname_downlevel.obj
 0002:00006050       ??_C@_1BG@BECMDDJB@?$AAa?$AAz?$AA?9?$AAA?$AAZ?$AA?9?$AAL?$AAa?$AAt?$AAn?$AA?$AA@ 000000018002d050     libucrt:lcidtoname_downlevel.obj
 0002:00006068       ??_C@_1M@MAOFCAEA@?$AAe?$AAu?$AA?9?$AAE?$AAS?$AA?$AA@ 000000018002d068     libucrt:lcidtoname_downlevel.obj
 0002:00006078       ??_C@_1M@IGHABKPI@?$AAm?$AAk?$AA?9?$AAM?$AAK?$AA?$AA@ 000000018002d078     libucrt:lcidtoname_downlevel.obj
 0002:00006088       ??_C@_1M@IAIGNEJG@?$AAt?$AAn?$AA?9?$AAZ?$AAA?$AA?$AA@ 000000018002d088     libucrt:lcidtoname_downlevel.obj
 0002:00006098       ??_C@_1M@IIJCOJFA@?$AAx?$AAh?$AA?9?$AAZ?$AAA?$AA?$AA@ 000000018002d098     libucrt:lcidtoname_downlevel.obj
 0002:000060a8       ??_C@_1M@LGPJHNJH@?$AAz?$AAu?$AA?9?$AAZ?$AAA?$AA?$AA@ 000000018002d0a8     libucrt:lcidtoname_downlevel.obj
 0002:000060b8       ??_C@_1M@HOKAOIO@?$AAa?$AAf?$AA?9?$AAZ?$AAA?$AA?$AA@ 000000018002d0b8     libucrt:lcidtoname_downlevel.obj
 0002:000060c8       ??_C@_1M@DPCLHLIE@?$AAk?$AAa?$AA?9?$AAG?$AAE?$AA?$AA@ 000000018002d0c8     libucrt:lcidtoname_downlevel.obj
 0002:000060d8       ??_C@_1M@BLKMHJBI@?$AAf?$AAo?$AA?9?$AAF?$AAO?$AA?$AA@ 000000018002d0d8     libucrt:lcidtoname_downlevel.obj
 0002:000060e8       ??_C@_1M@LGGJAPPB@?$AAh?$AAi?$AA?9?$AAI?$AAN?$AA?$AA@ 000000018002d0e8     libucrt:lcidtoname_downlevel.obj
 0002:000060f8       ??_C@_1M@FIKPIHFE@?$AAm?$AAt?$AA?9?$AAM?$AAT?$AA?$AA@ 000000018002d0f8     libucrt:lcidtoname_downlevel.obj
 0002:00006108       ??_C@_1M@HEGGPBFA@?$AAs?$AAe?$AA?9?$AAN?$AAO?$AA?$AA@ 000000018002d108     libucrt:lcidtoname_downlevel.obj
 0002:00006118       ??_C@_1M@EIBJEEPA@?$AAm?$AAs?$AA?9?$AAM?$AAY?$AA?$AA@ 000000018002d118     libucrt:lcidtoname_downlevel.obj
 0002:00006128       ??_C@_1M@FHLBGMPP@?$AAk?$AAk?$AA?9?$AAK?$AAZ?$AA?$AA@ 000000018002d128     libucrt:lcidtoname_downlevel.obj
 0002:00006138       ??_C@_1M@NGJJLCGI@?$AAk?$AAy?$AA?9?$AAK?$AAG?$AA?$AA@ 000000018002d138     libucrt:lcidtoname_downlevel.obj
 0002:00006148       ??_C@_1M@GIENNBFC@?$AAs?$AAw?$AA?9?$AAK?$AAE?$AA?$AA@ 000000018002d148     libucrt:lcidtoname_downlevel.obj
 0002:00006158       ??_C@_1BG@NDGMJIMJ@?$AAu?$AAz?$AA?9?$AAU?$AAZ?$AA?9?$AAL?$AAa?$AAt?$AAn?$AA?$AA@ 000000018002d158     libucrt:lcidtoname_downlevel.obj
 0002:00006170       ??_C@_1M@IDCCIHBC@?$AAt?$AAt?$AA?9?$AAR?$AAU?$AA?$AA@ 000000018002d170     libucrt:lcidtoname_downlevel.obj
 0002:00006180       ??_C@_1M@LOICPMOJ@?$AAb?$AAn?$AA?9?$AAI?$AAN?$AA?$AA@ 000000018002d180     libucrt:lcidtoname_downlevel.obj
 0002:00006190       ??_C@_1M@KPKKNEAH@?$AAp?$AAa?$AA?9?$AAI?$AAN?$AA?$AA@ 000000018002d190     libucrt:lcidtoname_downlevel.obj
 0002:000061a0       ??_C@_1M@PJGPPBOG@?$AAg?$AAu?$AA?9?$AAI?$AAN?$AA?$AA@ 000000018002d1a0     libucrt:lcidtoname_downlevel.obj
 0002:000061b0       ??_C@_1M@KMKMOPHI@?$AAt?$AAa?$AA?9?$AAI?$AAN?$AA?$AA@ 000000018002d1b0     libucrt:lcidtoname_downlevel.obj
 0002:000061c0       ??_C@_1M@KFEHEPAC@?$AAt?$AAe?$AA?9?$AAI?$AAN?$AA?$AA@ 000000018002d1c0     libucrt:lcidtoname_downlevel.obj
 0002:000061d0       ??_C@_1M@CDCLMGHI@?$AAk?$AAn?$AA?9?$AAI?$AAN?$AA?$AA@ 000000018002d1d0     libucrt:lcidtoname_downlevel.obj
 0002:000061e0       ??_C@_1M@MIODLDKF@?$AAm?$AAl?$AA?9?$AAI?$AAN?$AA?$AA@ 000000018002d1e0     libucrt:lcidtoname_downlevel.obj
 0002:000061f0       ??_C@_1M@PBIEACPO@?$AAm?$AAr?$AA?9?$AAI?$AAN?$AA?$AA@ 000000018002d1f0     libucrt:lcidtoname_downlevel.obj
 0002:00006200       ??_C@_1M@NIDEAGPH@?$AAs?$AAa?$AA?9?$AAI?$AAN?$AA?$AA@ 000000018002d200     libucrt:lcidtoname_downlevel.obj
 0002:00006210       ??_C@_1M@FHIHCBIO@?$AAm?$AAn?$AA?9?$AAM?$AAN?$AA?$AA@ 000000018002d210     libucrt:lcidtoname_downlevel.obj
 0002:00006220       ??_C@_1M@JAIJPENP@?$AAc?$AAy?$AA?9?$AAG?$AAB?$AA?$AA@ 000000018002d220     libucrt:lcidtoname_downlevel.obj
 0002:00006230       ??_C@_1M@PHGFBEPN@?$AAg?$AAl?$AA?9?$AAE?$AAS?$AA?$AA@ 000000018002d230     libucrt:lcidtoname_downlevel.obj
 0002:00006240       ??_C@_1O@KPIPDNCP@?$AAk?$AAo?$AAk?$AA?9?$AAI?$AAN?$AA?$AA@ 000000018002d240     libucrt:lcidtoname_downlevel.obj
 0002:00006250       ??_C@_1O@KNHJLDJA@?$AAs?$AAy?$AAr?$AA?9?$AAS?$AAY?$AA?$AA@ 000000018002d250     libucrt:lcidtoname_downlevel.obj
 0002:00006260       ??_C@_1O@MKEKBLAH@?$AAd?$AAi?$AAv?$AA?9?$AAM?$AAV?$AA?$AA@ 000000018002d260     libucrt:lcidtoname_downlevel.obj
 0002:00006270       ??_C@_1O@OHDCKDDF@?$AAq?$AAu?$AAz?$AA?9?$AAB?$AAO?$AA?$AA@ 000000018002d270     libucrt:lcidtoname_downlevel.obj
 0002:00006280       ??_C@_1M@LEPJNLFD@?$AAn?$AAs?$AA?9?$AAZ?$AAA?$AA?$AA@ 000000018002d280     libucrt:lcidtoname_downlevel.obj
 0002:00006290       ??_C@_1M@OMLEIIJB@?$AAm?$AAi?$AA?9?$AAN?$AAZ?$AA?$AA@ 000000018002d290     libucrt:lcidtoname_downlevel.obj
 0002:000062a0       ??_C@_1M@PMPEAILG@?$AAa?$AAr?$AA?9?$AAI?$AAQ?$AA?$AA@ 000000018002d2a0     libucrt:lcidtoname_downlevel.obj
 0002:000062b0       ??_C@_1M@CNKPNOEE@?$AAd?$AAe?$AA?9?$AAC?$AAH?$AA?$AA@ 000000018002d2b0     libucrt:lcidtoname_downlevel.obj
 0002:000062c0       ??_C@_1M@LKMGMLKO@?$AAe?$AAn?$AA?9?$AAG?$AAB?$AA?$AA@ 000000018002d2c0     libucrt:lcidtoname_downlevel.obj
 0002:000062d0       ??_C@_1M@PGKJFFGL@?$AAe?$AAs?$AA?9?$AAM?$AAX?$AA?$AA@ 000000018002d2d0     libucrt:lcidtoname_downlevel.obj
 0002:000062e0       ??_C@_1M@DNNANBDC@?$AAf?$AAr?$AA?9?$AAB?$AAE?$AA?$AA@ 000000018002d2e0     libucrt:lcidtoname_downlevel.obj
 0002:000062f0       ??_C@_1M@HLGMDFHM@?$AAi?$AAt?$AA?9?$AAC?$AAH?$AA?$AA@ 000000018002d2f0     libucrt:lcidtoname_downlevel.obj
 0002:00006300       ??_C@_1M@CLLBGJH@?$AAn?$AAl?$AA?9?$AAB?$AAE?$AA?$AA@ 000000018002d300     libucrt:lcidtoname_downlevel.obj
 0002:00006310       ??_C@_1M@BODBOGLF@?$AAn?$AAn?$AA?9?$AAN?$AAO?$AA?$AA@ 000000018002d310     libucrt:lcidtoname_downlevel.obj
 0002:00006320       ??_C@_1M@HFFAHKAD@?$AAp?$AAt?$AA?9?$AAP?$AAT?$AA?$AA@ 000000018002d320     libucrt:lcidtoname_downlevel.obj
 0002:00006330       ??_C@_1BG@LNOAKHIE@?$AAs?$AAr?$AA?9?$AAS?$AAP?$AA?9?$AAL?$AAa?$AAt?$AAn?$AA?$AA@ 000000018002d330     libucrt:lcidtoname_downlevel.obj
 0002:00006348       ??_C@_1M@HBMHBGAK@?$AAs?$AAv?$AA?9?$AAF?$AAI?$AA?$AA@ 000000018002d348     libucrt:lcidtoname_downlevel.obj
 0002:00006358       ??_C@_1BG@DGCJGJBE@?$AAa?$AAz?$AA?9?$AAA?$AAZ?$AA?9?$AAC?$AAy?$AAr?$AAl?$AA?$AA@ 000000018002d358     libucrt:lcidtoname_downlevel.obj
 0002:00006370       ??_C@_1M@KEJDAAHB@?$AAs?$AAe?$AA?9?$AAS?$AAE?$AA?$AA@ 000000018002d370     libucrt:lcidtoname_downlevel.obj
 0002:00006380       ??_C@_1M@HEIBJJAD@?$AAm?$AAs?$AA?9?$AAB?$AAN?$AA?$AA@ 000000018002d380     libucrt:lcidtoname_downlevel.obj
 0002:00006390       ??_C@_1BG@PBGJMCEM@?$AAu?$AAz?$AA?9?$AAU?$AAZ?$AA?9?$AAC?$AAy?$AAr?$AAl?$AA?$AA@ 000000018002d390     libucrt:lcidtoname_downlevel.obj
 0002:000063a8       ??_C@_1O@LAOBCMDF@?$AAq?$AAu?$AAz?$AA?9?$AAE?$AAC?$AA?$AA@ 000000018002d3a8     libucrt:lcidtoname_downlevel.obj
 0002:000063b8       ??_C@_1M@POEEMAIO@?$AAa?$AAr?$AA?9?$AAE?$AAG?$AA?$AA@ 000000018002d3b8     libucrt:lcidtoname_downlevel.obj
 0002:000063c8       ??_C@_1M@EFAKDEDL@?$AAz?$AAh?$AA?9?$AAH?$AAK?$AA?$AA@ 000000018002d3c8     libucrt:lcidtoname_downlevel.obj
 0002:000063d8       ??_C@_1M@HKKIJHGI@?$AAd?$AAe?$AA?9?$AAA?$AAT?$AA?$AA@ 000000018002d3d8     libucrt:lcidtoname_downlevel.obj
 0002:000063e8       ??_C@_1M@KBFBEHJF@?$AAe?$AAn?$AA?9?$AAA?$AAU?$AA?$AA@ 000000018002d3e8     libucrt:lcidtoname_downlevel.obj
 0002:000063f8       ??_C@_1M@MNPLFAAH@?$AAe?$AAs?$AA?9?$AAE?$AAS?$AA?$AA@ 000000018002d3f8     libucrt:lcidtoname_downlevel.obj
 0002:00006408       ??_C@_1M@HJOOJFMA@?$AAf?$AAr?$AA?9?$AAC?$AAA?$AA?$AA@ 000000018002d408     libucrt:lcidtoname_downlevel.obj
 0002:00006418       ??_C@_1BG@JPOFPNAB@?$AAs?$AAr?$AA?9?$AAS?$AAP?$AA?9?$AAC?$AAy?$AAr?$AAl?$AA?$AA@ 000000018002d418     libucrt:lcidtoname_downlevel.obj
 0002:00006430       ??_C@_1M@LNFOCMOB@?$AAs?$AAe?$AA?9?$AAF?$AAI?$AA?$AA@ 000000018002d430     libucrt:lcidtoname_downlevel.obj
 0002:00006440       ??_C@_1O@MGJBOAMB@?$AAq?$AAu?$AAz?$AA?9?$AAP?$AAE?$AA?$AA@ 000000018002d440     libucrt:lcidtoname_downlevel.obj
 0002:00006450       ??_C@_1M@GJINLBOK@?$AAa?$AAr?$AA?9?$AAL?$AAY?$AA?$AA@ 000000018002d450     libucrt:lcidtoname_downlevel.obj
 0002:00006460       ??_C@_1M@GGMNHJNL@?$AAz?$AAh?$AA?9?$AAS?$AAG?$AA?$AA@ 000000018002d460     libucrt:lcidtoname_downlevel.obj
 0002:00006470       ??_C@_1M@HOIKODND@?$AAd?$AAe?$AA?9?$AAL?$AAU?$AA?$AA@ 000000018002d470     libucrt:lcidtoname_downlevel.obj
 0002:00006480       ??_C@_1M@DDOCCGFG@?$AAe?$AAn?$AA?9?$AAC?$AAA?$AA?$AA@ 000000018002d480     libucrt:lcidtoname_downlevel.obj
 0002:00006490       ??_C@_1M@BNOEMJLF@?$AAe?$AAs?$AA?9?$AAG?$AAT?$AA?$AA@ 000000018002d490     libucrt:lcidtoname_downlevel.obj
 0002:000064a0       ??_C@_1M@EOGNKEK@?$AAf?$AAr?$AA?9?$AAC?$AAH?$AA?$AA@ 000000018002d4a0     libucrt:lcidtoname_downlevel.obj
 0002:000064b0       ??_C@_1M@FLIDJFHL@?$AAh?$AAr?$AA?9?$AAB?$AAA?$AA?$AA@ 000000018002d4b0     libucrt:lcidtoname_downlevel.obj
 0002:000064c0       ??_C@_1O@FMCELNAJ@?$AAs?$AAm?$AAj?$AA?9?$AAN?$AAO?$AA?$AA@ 000000018002d4c0     libucrt:lcidtoname_downlevel.obj
 0002:000064d0       ??_C@_1M@JHGLJMGJ@?$AAa?$AAr?$AA?9?$AAD?$AAZ?$AA?$AA@ 000000018002d4d0     libucrt:lcidtoname_downlevel.obj
 0002:000064e0       ??_C@_1M@JKKFDCNP@?$AAz?$AAh?$AA?9?$AAM?$AAO?$AA?$AA@ 000000018002d4e0     libucrt:lcidtoname_downlevel.obj
 0002:000064f0       ??_C@_1M@GEEFALPE@?$AAd?$AAe?$AA?9?$AAL?$AAI?$AA?$AA@ 000000018002d4f0     libucrt:lcidtoname_downlevel.obj
 0002:00006500       ??_C@_1M@IGEOFBG@?$AAe?$AAn?$AA?9?$AAN?$AAZ?$AA?$AA@ 000000018002d500     libucrt:lcidtoname_downlevel.obj
 0002:00006510       ??_C@_1M@KDBONEHP@?$AAe?$AAs?$AA?9?$AAC?$AAR?$AA?$AA@ 000000018002d510     libucrt:lcidtoname_downlevel.obj
 0002:00006520       ??_C@_1M@FHMDOHNN@?$AAf?$AAr?$AA?9?$AAL?$AAU?$AA?$AA@ 000000018002d520     libucrt:lcidtoname_downlevel.obj
 0002:00006530       ??_C@_1BG@NFKKMAFG@?$AAb?$AAs?$AA?9?$AAB?$AAA?$AA?9?$AAL?$AAa?$AAt?$AAn?$AA?$AA@ 000000018002d530     libucrt:lcidtoname_downlevel.obj
 0002:00006548       ??_C@_1O@IMNBEMCI@?$AAs?$AAm?$AAj?$AA?9?$AAS?$AAE?$AA?$AA@ 000000018002d548     libucrt:lcidtoname_downlevel.obj
 0002:00006558       ??_C@_1M@DHHMBNDP@?$AAa?$AAr?$AA?9?$AAM?$AAA?$AA?$AA@ 000000018002d558     libucrt:lcidtoname_downlevel.obj
 0002:00006568       ??_C@_1M@BNBLJCGH@?$AAe?$AAn?$AA?9?$AAI?$AAE?$AA?$AA@ 000000018002d568     libucrt:lcidtoname_downlevel.obj
 0002:00006578       ??_C@_1M@GEPAFMDL@?$AAe?$AAs?$AA?9?$AAP?$AAA?$AA?$AA@ 000000018002d578     libucrt:lcidtoname_downlevel.obj
 0002:00006588       ??_C@_1M@OJONDMDL@?$AAf?$AAr?$AA?9?$AAM?$AAC?$AA?$AA@ 000000018002d588     libucrt:lcidtoname_downlevel.obj
 0002:00006598       ??_C@_1BG@OBCNFJB@?$AAs?$AAr?$AA?9?$AAB?$AAA?$AA?9?$AAL?$AAa?$AAt?$AAn?$AA?$AA@ 000000018002d598     libucrt:lcidtoname_downlevel.obj
 0002:000065b0       ??_C@_1O@KEMEEGPO@?$AAs?$AAm?$AAa?$AA?9?$AAN?$AAO?$AA?$AA@ 000000018002d5b0     libucrt:lcidtoname_downlevel.obj
 0002:000065c0       ??_C@_1M@ELMGFODK@?$AAa?$AAr?$AA?9?$AAT?$AAN?$AA?$AA@ 000000018002d5c0     libucrt:lcidtoname_downlevel.obj
 0002:000065d0       ??_C@_1M@BHDLHFAF@?$AAe?$AAn?$AA?9?$AAZ?$AAA?$AA?$AA@ 000000018002d5d0     libucrt:lcidtoname_downlevel.obj
 0002:000065e0       ??_C@_1M@BMGIGLIF@?$AAe?$AAs?$AA?9?$AAD?$AAO?$AA?$AA@ 000000018002d5e0     libucrt:lcidtoname_downlevel.obj
 0002:000065f0       ??_C@_1BG@CMBHIPBE@?$AAs?$AAr?$AA?9?$AAB?$AAA?$AA?9?$AAC?$AAy?$AAr?$AAl?$AA?$AA@ 000000018002d5f0     libucrt:lcidtoname_downlevel.obj
 0002:00006608       ??_C@_1O@HEDBLHNP@?$AAs?$AAm?$AAa?$AA?9?$AAS?$AAE?$AA?$AA@ 000000018002d608     libucrt:lcidtoname_downlevel.obj
 0002:00006618       ??_C@_1M@DAGCADIM@?$AAa?$AAr?$AA?9?$AAO?$AAM?$AA?$AA@ 000000018002d618     libucrt:lcidtoname_downlevel.obj
 0002:00006628       ??_C@_1M@FODLMICG@?$AAe?$AAn?$AA?9?$AAJ?$AAM?$AA?$AA@ 000000018002d628     libucrt:lcidtoname_downlevel.obj
 0002:00006638       ??_C@_1M@DNMLCIHB@?$AAe?$AAs?$AA?9?$AAV?$AAE?$AA?$AA@ 000000018002d638     libucrt:lcidtoname_downlevel.obj
 0002:00006648       ??_C@_1O@EOKHMKJK@?$AAs?$AAm?$AAs?$AA?9?$AAF?$AAI?$AA?$AA@ 000000018002d648     libucrt:lcidtoname_downlevel.obj
 0002:00006658       ??_C@_1M@CAFJMKOF@?$AAa?$AAr?$AA?9?$AAY?$AAE?$AA?$AA@ 000000018002d658     libucrt:lcidtoname_downlevel.obj
 0002:00006668       ??_C@_1M@CBFHIJLI@?$AAe?$AAn?$AA?9?$AAC?$AAB?$AA?$AA@ 000000018002d668     libucrt:lcidtoname_downlevel.obj
 0002:00006678       ??_C@_1M@BGNFLDN@?$AAe?$AAs?$AA?9?$AAC?$AAO?$AA?$AA@ 000000018002d678     libucrt:lcidtoname_downlevel.obj
 0002:00006688       ??_C@_1O@JMPHMAMC@?$AAs?$AAm?$AAn?$AA?9?$AAF?$AAI?$AA?$AA@ 000000018002d688     libucrt:lcidtoname_downlevel.obj
 0002:00006698       ??_C@_1M@JLANABKE@?$AAa?$AAr?$AA?9?$AAS?$AAY?$AA?$AA@ 000000018002d698     libucrt:lcidtoname_downlevel.obj
 0002:000066a8       ??_C@_1M@HPKGCFGN@?$AAe?$AAn?$AA?9?$AAB?$AAZ?$AA?$AA@ 000000018002d6a8     libucrt:lcidtoname_downlevel.obj
 0002:000066b8       ??_C@_1M@OLJCMLGM@?$AAe?$AAs?$AA?9?$AAP?$AAE?$AA?$AA@ 000000018002d6b8     libucrt:lcidtoname_downlevel.obj
 0002:000066c8       ??_C@_1M@MKKGFKLE@?$AAa?$AAr?$AA?9?$AAJ?$AAO?$AA?$AA@ 000000018002d6c8     libucrt:lcidtoname_downlevel.obj
 0002:000066d8       ??_C@_1M@EKPGLDNI@?$AAe?$AAn?$AA?9?$AAT?$AAT?$AA?$AA@ 000000018002d6d8     libucrt:lcidtoname_downlevel.obj
 0002:000066e8       ??_C@_1M@OONGHFHE@?$AAe?$AAs?$AA?9?$AAA?$AAR?$AA?$AA@ 000000018002d6e8     libucrt:lcidtoname_downlevel.obj
 0002:000066f8       ??_C@_1M@OOJFGBHE@?$AAa?$AAr?$AA?9?$AAL?$AAB?$AA?$AA@ 000000018002d6f8     libucrt:lcidtoname_downlevel.obj
 0002:00006708       ??_C@_1M@GCEJHNEG@?$AAe?$AAn?$AA?9?$AAZ?$AAW?$AA?$AA@ 000000018002d708     libucrt:lcidtoname_downlevel.obj
 0002:00006718       ??_C@_1M@JNOCAHJI@?$AAe?$AAs?$AA?9?$AAE?$AAC?$AA?$AA@ 000000018002d718     libucrt:lcidtoname_downlevel.obj
 0002:00006728       ??_C@_1M@JEFHPGGB@?$AAa?$AAr?$AA?9?$AAK?$AAW?$AA?$AA@ 000000018002d728     libucrt:lcidtoname_downlevel.obj
 0002:00006738       ??_C@_1M@MLKIBJOJ@?$AAe?$AAn?$AA?9?$AAP?$AAH?$AA?$AA@ 000000018002d738     libucrt:lcidtoname_downlevel.obj
 0002:00006748       ??_C@_1M@BDNIPEND@?$AAe?$AAs?$AA?9?$AAC?$AAL?$AA?$AA@ 000000018002d748     libucrt:lcidtoname_downlevel.obj
 0002:00006758       ??_C@_1M@MPNMEKBD@?$AAa?$AAr?$AA?9?$AAA?$AAE?$AA?$AA@ 000000018002d758     libucrt:lcidtoname_downlevel.obj
 0002:00006768       ??_C@_1M@KBJALCPI@?$AAe?$AAs?$AA?9?$AAU?$AAY?$AA?$AA@ 000000018002d768     libucrt:lcidtoname_downlevel.obj
 0002:00006778       ??_C@_1M@LLCCOAGA@?$AAa?$AAr?$AA?9?$AAB?$AAH?$AA?$AA@ 000000018002d778     libucrt:lcidtoname_downlevel.obj
 0002:00006788       ??_C@_1M@PBFNCDEL@?$AAe?$AAs?$AA?9?$AAP?$AAY?$AA?$AA@ 000000018002d788     libucrt:lcidtoname_downlevel.obj
 0002:00006798       ??_C@_1M@EDGINPNP@?$AAa?$AAr?$AA?9?$AAQ?$AAA?$AA?$AA@ 000000018002d798     libucrt:lcidtoname_downlevel.obj
 0002:000067a8       ??_C@_1M@MKDBIIJI@?$AAe?$AAs?$AA?9?$AAB?$AAO?$AA?$AA@ 000000018002d7a8     libucrt:lcidtoname_downlevel.obj
 0002:000067b8       ??_C@_1M@CPKKEBLD@?$AAe?$AAs?$AA?9?$AAS?$AAV?$AA?$AA@ 000000018002d7b8     libucrt:lcidtoname_downlevel.obj
 0002:000067c8       ??_C@_1M@NDBGMMJL@?$AAe?$AAs?$AA?9?$AAH?$AAN?$AA?$AA@ 000000018002d7c8     libucrt:lcidtoname_downlevel.obj
 0002:000067d8       ??_C@_1M@JIJIBHDP@?$AAe?$AAs?$AA?9?$AAN?$AAI?$AA?$AA@ 000000018002d7d8     libucrt:lcidtoname_downlevel.obj
 0002:000067e8       ??_C@_1M@CGFMKEEK@?$AAe?$AAs?$AA?9?$AAP?$AAR?$AA?$AA@ 000000018002d7e8     libucrt:lcidtoname_downlevel.obj
 0002:000067f8       ??_C@_1O@ICJHKIIK@?$AAz?$AAh?$AA?9?$AAC?$AAH?$AAT?$AA?$AA@ 000000018002d7f8     libucrt:lcidtoname_downlevel.obj
 0002:00006808       ??_C@_15CLNEJCE@?$AAs?$AAr?$AA?$AA@ 000000018002d808     libucrt:lcidtoname_downlevel.obj
 0002:00007650       ??_C@_1M@KAHEKEIG@?$AAa?$AAf?$AA?9?$AAz?$AAa?$AA?$AA@ 000000018002e650     libucrt:lcidtoname_downlevel.obj
 0002:00007660       ??_C@_1M@GIECOABL@?$AAa?$AAr?$AA?9?$AAa?$AAe?$AA?$AA@ 000000018002e660     libucrt:lcidtoname_downlevel.obj
 0002:00007670       ??_C@_1M@BMLMEKGI@?$AAa?$AAr?$AA?9?$AAb?$AAh?$AA?$AA@ 000000018002e670     libucrt:lcidtoname_downlevel.obj
 0002:00007680       ??_C@_1M@DAPFDGGB@?$AAa?$AAr?$AA?9?$AAd?$AAz?$AA?$AA@ 000000018002e680     libucrt:lcidtoname_downlevel.obj
 0002:00007690       ??_C@_1M@FJNKGKIG@?$AAa?$AAr?$AA?9?$AAe?$AAg?$AA?$AA@ 000000018002e690     libucrt:lcidtoname_downlevel.obj
 0002:000076a0       ??_C@_1M@FLGKKCLO@?$AAa?$AAr?$AA?9?$AAi?$AAq?$AA?$AA@ 000000018002e6a0     libucrt:lcidtoname_downlevel.obj
 0002:000076b0       ??_C@_1M@GNDIPALM@?$AAa?$AAr?$AA?9?$AAj?$AAo?$AA?$AA@ 000000018002e6b0     libucrt:lcidtoname_downlevel.obj
 0002:000076c0       ??_C@_1M@DDMJFMGJ@?$AAa?$AAr?$AA?9?$AAk?$AAw?$AA?$AA@ 000000018002e6c0     libucrt:lcidtoname_downlevel.obj
 0002:000076d0       ??_C@_1M@EJALMLHM@?$AAa?$AAr?$AA?9?$AAl?$AAb?$AA?$AA@ 000000018002e6d0     libucrt:lcidtoname_downlevel.obj
 0002:000076e0       ??_C@_1M@MOBDBLOC@?$AAa?$AAr?$AA?9?$AAl?$AAy?$AA?$AA@ 000000018002e6e0     libucrt:lcidtoname_downlevel.obj
 0002:000076f0       ??_C@_1M@JAOCLHDH@?$AAa?$AAr?$AA?9?$AAm?$AAa?$AA?$AA@ 000000018002e6f0     libucrt:lcidtoname_downlevel.obj
 0002:00007700       ??_C@_1M@JHPMKJIE@?$AAa?$AAr?$AA?9?$AAo?$AAm?$AA?$AA@ 000000018002e700     libucrt:lcidtoname_downlevel.obj
 0002:00007710       ??_C@_1M@OEPGHFNH@?$AAa?$AAr?$AA?9?$AAq?$AAa?$AA?$AA@ 000000018002e710     libucrt:lcidtoname_downlevel.obj
 0002:00007720       ??_C@_1M@KJDONENM@?$AAa?$AAr?$AA?9?$AAs?$AAa?$AA?$AA@ 000000018002e720     libucrt:lcidtoname_downlevel.obj
 0002:00007730       ??_C@_1M@DMJDKLKM@?$AAa?$AAr?$AA?9?$AAs?$AAy?$AA?$AA@ 000000018002e730     libucrt:lcidtoname_downlevel.obj
 0002:00007740       ??_C@_1M@OMFIPEDC@?$AAa?$AAr?$AA?9?$AAt?$AAn?$AA?$AA@ 000000018002e740     libucrt:lcidtoname_downlevel.obj
 0002:00007750       ??_C@_1M@IHMHGAON@?$AAa?$AAr?$AA?9?$AAy?$AAe?$AA?$AA@ 000000018002e750     libucrt:lcidtoname_downlevel.obj
 0002:00007760       ??_C@_1BG@KDCPGJGB@?$AAa?$AAz?$AA?9?$AAa?$AAz?$AA?9?$AAc?$AAy?$AAr?$AAl?$AA?$AA@ 000000018002e760     libucrt:lcidtoname_downlevel.obj
 0002:00007778       ??_C@_1BG@IBCKDDOE@?$AAa?$AAz?$AA?9?$AAa?$AAz?$AA?9?$AAl?$AAa?$AAt?$AAn?$AA?$AA@ 000000018002e778     libucrt:lcidtoname_downlevel.obj
 0002:00007790       ??_C@_1M@EGPFDCPD@?$AAb?$AAe?$AA?9?$AAb?$AAy?$AA?$AA@ 000000018002e790     libucrt:lcidtoname_downlevel.obj
 0002:000077a0       ??_C@_1M@PCMGMCGC@?$AAb?$AAg?$AA?9?$AAb?$AAg?$AA?$AA@ 000000018002e7a0     libucrt:lcidtoname_downlevel.obj
 0002:000077b0       ??_C@_1M@BJBMFGOB@?$AAb?$AAn?$AA?9?$AAi?$AAn?$AA?$AA@ 000000018002e7b0     libucrt:lcidtoname_downlevel.obj
 0002:000077c0       ??_C@_1BG@EAKMMACD@?$AAb?$AAs?$AA?9?$AAb?$AAa?$AA?9?$AAl?$AAa?$AAt?$AAn?$AA?$AA@ 000000018002e7c0     libucrt:lcidtoname_downlevel.obj
 0002:000077d8       ??_C@_1M@KGADAODK@?$AAc?$AAa?$AA?9?$AAe?$AAs?$AA?$AA@ 000000018002e7d8     libucrt:lcidtoname_downlevel.obj
 0002:000077e8       ??_C@_1M@COAJPDHI@?$AAc?$AAs?$AA?9?$AAc?$AAz?$AA?$AA@ 000000018002e7e8     libucrt:lcidtoname_downlevel.obj
 0002:000077f8       ??_C@_1M@DHBHFONH@?$AAc?$AAy?$AA?9?$AAg?$AAb?$AA?$AA@ 000000018002e7f8     libucrt:lcidtoname_downlevel.obj
 0002:00007808       ??_C@_1M@IMGKELGA@?$AAd?$AAa?$AA?9?$AAd?$AAk?$AA?$AA@ 000000018002e808     libucrt:lcidtoname_downlevel.obj
 0002:00007818       ??_C@_1M@NNDGDNGA@?$AAd?$AAe?$AA?9?$AAa?$AAt?$AA?$AA@ 000000018002e818     libucrt:lcidtoname_downlevel.obj
 0002:00007828       ??_C@_1M@IKDBHEEM@?$AAd?$AAe?$AA?9?$AAc?$AAh?$AA?$AA@ 000000018002e828     libucrt:lcidtoname_downlevel.obj
 0002:00007838       ??_C@_1M@GFFOJMCJ@?$AAd?$AAe?$AA?9?$AAd?$AAe?$AA?$AA@ 000000018002e838     libucrt:lcidtoname_downlevel.obj
 0002:00007848       ??_C@_1M@MDNLKBPM@?$AAd?$AAe?$AA?9?$AAl?$AAi?$AA?$AA@ 000000018002e848     libucrt:lcidtoname_downlevel.obj
 0002:00007858       ??_C@_1M@NJBEEJNL@?$AAd?$AAe?$AA?9?$AAl?$AAu?$AA?$AA@ 000000018002e858     libucrt:lcidtoname_downlevel.obj
 0002:00007868       ??_C@_1O@GNNELBAP@?$AAd?$AAi?$AAv?$AA?9?$AAm?$AAv?$AA?$AA@ 000000018002e868     libucrt:lcidtoname_downlevel.obj
 0002:00007878       ??_C@_1M@EJLEOGAE@?$AAe?$AAl?$AA?9?$AAg?$AAr?$AA?$AA@ 000000018002e878     libucrt:lcidtoname_downlevel.obj
 0002:00007888       ??_C@_1M@GMPONJN@?$AAe?$AAn?$AA?9?$AAa?$AAu?$AA?$AA@ 000000018002e888     libucrt:lcidtoname_downlevel.obj
 0002:00007898       ??_C@_1M@NIDIIPGF@?$AAe?$AAn?$AA?9?$AAb?$AAz?$AA?$AA@ 000000018002e898     libucrt:lcidtoname_downlevel.obj
 0002:000078a8       ??_C@_1M@JEHMIMFO@?$AAe?$AAn?$AA?9?$AAc?$AAa?$AA?$AA@ 000000018002e8a8     libucrt:lcidtoname_downlevel.obj
 0002:000078b8       ??_C@_1M@IGMJCDLA@?$AAe?$AAn?$AA?9?$AAc?$AAb?$AA?$AA@ 000000018002e8b8     libucrt:lcidtoname_downlevel.obj
 0002:000078c8       ??_C@_1M@BNFIGBKG@?$AAe?$AAn?$AA?9?$AAg?$AAb?$AA?$AA@ 000000018002e8c8     libucrt:lcidtoname_downlevel.obj
 0002:000078d8       ??_C@_1M@LKIFDIGP@?$AAe?$AAn?$AA?9?$AAi?$AAe?$AA?$AA@ 000000018002e8d8     libucrt:lcidtoname_downlevel.obj
 0002:000078e8       ??_C@_1M@PJKFGCCO@?$AAe?$AAn?$AA?9?$AAj?$AAm?$AA?$AA@ 000000018002e8e8     libucrt:lcidtoname_downlevel.obj
 0002:000078f8       ??_C@_1M@KPPKEPBO@?$AAe?$AAn?$AA?9?$AAn?$AAz?$AA?$AA@ 000000018002e8f8     libucrt:lcidtoname_downlevel.obj
 0002:00007908       ??_C@_1M@GMDGLDOB@?$AAe?$AAn?$AA?9?$AAp?$AAh?$AA?$AA@ 000000018002e908     libucrt:lcidtoname_downlevel.obj
 0002:00007918       ??_C@_1M@ONGIBJNA@?$AAe?$AAn?$AA?9?$AAt?$AAt?$AA?$AA@ 000000018002e918     libucrt:lcidtoname_downlevel.obj
 0002:00007928       ??_C@_1M@LLODPCMM@?$AAe?$AAn?$AA?9?$AAu?$AAs?$AA?$AA@ 000000018002e928     libucrt:lcidtoname_downlevel.obj
 0002:00007938       ??_C@_1M@LAKFNPAN@?$AAe?$AAn?$AA?9?$AAz?$AAa?$AA?$AA@ 000000018002e938     libucrt:lcidtoname_downlevel.obj
 0002:00007948       ??_C@_1M@MFNHNHEO@?$AAe?$AAn?$AA?9?$AAz?$AAw?$AA?$AA@ 000000018002e948     libucrt:lcidtoname_downlevel.obj
 0002:00007958       ??_C@_1M@EJEINPHM@?$AAe?$AAs?$AA?9?$AAa?$AAr?$AA?$AA@ 000000018002e958     libucrt:lcidtoname_downlevel.obj
 0002:00007968       ??_C@_1M@GNKPCCJA@?$AAe?$AAs?$AA?9?$AAb?$AAo?$AA?$AA@ 000000018002e968     libucrt:lcidtoname_downlevel.obj
 0002:00007978       ??_C@_1M@LEEGFONL@?$AAe?$AAs?$AA?9?$AAc?$AAl?$AA?$AA@ 000000018002e978     libucrt:lcidtoname_downlevel.obj
 0002:00007988       ??_C@_1M@KGPDPBDF@?$AAe?$AAs?$AA?9?$AAc?$AAo?$AA?$AA@ 000000018002e988     libucrt:lcidtoname_downlevel.obj
 0002:00007998       ??_C@_1M@EIAHOHH@?$AAe?$AAs?$AA?9?$AAc?$AAr?$AA?$AA@ 000000018002e998     libucrt:lcidtoname_downlevel.obj
 0002:000079a8       ??_C@_1M@LLPGMBIN@?$AAe?$AAs?$AA?9?$AAd?$AAo?$AA?$AA@ 000000018002e9a8     libucrt:lcidtoname_downlevel.obj
 0002:000079b8       ??_C@_1M@DKHMKNJA@?$AAe?$AAs?$AA?9?$AAe?$AAc?$AA?$AA@ 000000018002e9b8     libucrt:lcidtoname_downlevel.obj
 0002:000079c8       ??_C@_1M@GKGFPKAP@?$AAe?$AAs?$AA?9?$AAe?$AAs?$AA?$AA@ 000000018002e9c8     libucrt:lcidtoname_downlevel.obj
 0002:000079d8       ??_C@_1M@LKHKGDLN@?$AAe?$AAs?$AA?9?$AAg?$AAt?$AA?$AA@ 000000018002e9d8     libucrt:lcidtoname_downlevel.obj
 0002:000079e8       ??_C@_1M@HEIIGGJD@?$AAe?$AAs?$AA?9?$AAh?$AAn?$AA?$AA@ 000000018002e9e8     libucrt:lcidtoname_downlevel.obj
 0002:000079f8       ??_C@_1M@FBDHPPGD@?$AAe?$AAs?$AA?9?$AAm?$AAx?$AA?$AA@ 000000018002e9f8     libucrt:lcidtoname_downlevel.obj
 0002:00007a08       ??_C@_1M@DPAGLNDH@?$AAe?$AAs?$AA?9?$AAn?$AAi?$AA?$AA@ 000000018002ea08     libucrt:lcidtoname_downlevel.obj
 0002:00007a18       ??_C@_1M@MDGOPGDD@?$AAe?$AAs?$AA?9?$AAp?$AAa?$AA?$AA@ 000000018002ea18     libucrt:lcidtoname_downlevel.obj
 0002:00007a28       ??_C@_1M@EMAMGBGE@?$AAe?$AAs?$AA?9?$AAp?$AAe?$AA?$AA@ 000000018002ea28     libucrt:lcidtoname_downlevel.obj
 0002:00007a38       ??_C@_1M@IBMCAOEC@?$AAe?$AAs?$AA?9?$AAp?$AAr?$AA?$AA@ 000000018002ea38     libucrt:lcidtoname_downlevel.obj
 0002:00007a48       ??_C@_1M@FGMDIJED@?$AAe?$AAs?$AA?9?$AAp?$AAy?$AA?$AA@ 000000018002ea48     libucrt:lcidtoname_downlevel.obj
 0002:00007a58       ??_C@_1M@IIDEOLLL@?$AAe?$AAs?$AA?9?$AAs?$AAv?$AA?$AA@ 000000018002ea58     libucrt:lcidtoname_downlevel.obj
 0002:00007a68       ??_C@_1M@GAOBIPA@?$AAe?$AAs?$AA?9?$AAu?$AAy?$AA?$AA@ 000000018002ea68     libucrt:lcidtoname_downlevel.obj
 0002:00007a78       ??_C@_1M@JKFFICHJ@?$AAe?$AAs?$AA?9?$AAv?$AAe?$AA?$AA@ 000000018002ea78     libucrt:lcidtoname_downlevel.obj
 0002:00007a88       ??_C@_1M@PNMLOJDF@?$AAe?$AAt?$AA?9?$AAe?$AAe?$AA?$AA@ 000000018002ea88     libucrt:lcidtoname_downlevel.obj
 0002:00007a98       ??_C@_1M@GHHLIKEI@?$AAe?$AAu?$AA?9?$AAe?$AAs?$AA?$AA@ 000000018002ea98     libucrt:lcidtoname_downlevel.obj
 0002:00007aa8       ??_C@_1M@PBNONODE@?$AAf?$AAa?$AA?9?$AAi?$AAr?$AA?$AA@ 000000018002eaa8     libucrt:lcidtoname_downlevel.obj
 0002:00007ab8       ??_C@_1M@JEEHPMIL@?$AAf?$AAi?$AA?9?$AAf?$AAi?$AA?$AA@ 000000018002eab8     libucrt:lcidtoname_downlevel.obj
 0002:00007ac8       ??_C@_1M@LMDCNDBA@?$AAf?$AAo?$AA?9?$AAf?$AAo?$AA?$AA@ 000000018002eac8     libucrt:lcidtoname_downlevel.obj
 0002:00007ad8       ??_C@_1M@JKEOHLDK@?$AAf?$AAr?$AA?9?$AAb?$AAe?$AA?$AA@ 000000018002ead8     libucrt:lcidtoname_downlevel.obj
 0002:00007ae8       ??_C@_1M@NOHADPMI@?$AAf?$AAr?$AA?9?$AAc?$AAa?$AA?$AA@ 000000018002eae8     libucrt:lcidtoname_downlevel.obj
 0002:00007af8       ??_C@_1M@KDHIHAEC@?$AAf?$AAr?$AA?9?$AAc?$AAh?$AA?$AA@ 000000018002eaf8     libucrt:lcidtoname_downlevel.obj
 0002:00007b08       ??_C@_1M@MMBBFGAK@?$AAf?$AAr?$AA?9?$AAf?$AAr?$AA?$AA@ 000000018002eb08     libucrt:lcidtoname_downlevel.obj
 0002:00007b18       ??_C@_1M@PAFNENNF@?$AAf?$AAr?$AA?9?$AAl?$AAu?$AA?$AA@ 000000018002eb18     libucrt:lcidtoname_downlevel.obj
 0002:00007b28       ??_C@_1M@EOHDJGDD@?$AAf?$AAr?$AA?9?$AAm?$AAc?$AA?$AA@ 000000018002eb28     libucrt:lcidtoname_downlevel.obj
 0002:00007b38       ??_C@_1M@FAPLLOPF@?$AAg?$AAl?$AA?9?$AAe?$AAs?$AA?$AA@ 000000018002eb38     libucrt:lcidtoname_downlevel.obj
 0002:00007b48       ??_C@_1M@FOPBFLOO@?$AAg?$AAu?$AA?9?$AAi?$AAn?$AA?$AA@ 000000018002eb48     libucrt:lcidtoname_downlevel.obj
 0002:00007b58       ??_C@_1M@KBMCINPM@?$AAh?$AAe?$AA?9?$AAi?$AAl?$AA?$AA@ 000000018002eb58     libucrt:lcidtoname_downlevel.obj
 0002:00007b68       ??_C@_1M@BBPHKFPJ@?$AAh?$AAi?$AA?9?$AAi?$AAn?$AA?$AA@ 000000018002eb68     libucrt:lcidtoname_downlevel.obj
 0002:00007b78       ??_C@_1M@PMBNDPHD@?$AAh?$AAr?$AA?9?$AAb?$AAa?$AA?$AA@ 000000018002eb78     libucrt:lcidtoname_downlevel.obj
 0002:00007b88       ??_C@_1M@BPCKOEGE@?$AAh?$AAr?$AA?9?$AAh?$AAr?$AA?$AA@ 000000018002eb88     libucrt:lcidtoname_downlevel.obj
 0002:00007b98       ??_C@_1M@GACBMHKE@?$AAh?$AAu?$AA?9?$AAh?$AAu?$AA?$AA@ 000000018002eb98     libucrt:lcidtoname_downlevel.obj
 0002:00007ba8       ??_C@_1M@MILPAJJC@?$AAh?$AAy?$AA?9?$AAa?$AAm?$AA?$AA@ 000000018002eba8     libucrt:lcidtoname_downlevel.obj
 0002:00007bb8       ??_C@_1M@BABBICEC@?$AAi?$AAd?$AA?9?$AAi?$AAd?$AA?$AA@ 000000018002ebb8     libucrt:lcidtoname_downlevel.obj
 0002:00007bc8       ??_C@_1M@BIKNHHPF@?$AAi?$AAs?$AA?9?$AAi?$AAs?$AA?$AA@ 000000018002ebc8     libucrt:lcidtoname_downlevel.obj
 0002:00007bd8       ??_C@_1M@NMPCJPHE@?$AAi?$AAt?$AA?9?$AAc?$AAh?$AA?$AA@ 000000018002ebd8     libucrt:lcidtoname_downlevel.obj
 0002:00007be8       ??_C@_1M@GHKGFEDF@?$AAi?$AAt?$AA?9?$AAi?$AAt?$AA?$AA@ 000000018002ebe8     libucrt:lcidtoname_downlevel.obj
 0002:00007bf8       ??_C@_1M@NIEJCJJA@?$AAj?$AAa?$AA?9?$AAj?$AAp?$AA?$AA@ 000000018002ebf8     libucrt:lcidtoname_downlevel.obj
 0002:00007c08       ??_C@_1M@JILFNBIM@?$AAk?$AAa?$AA?9?$AAg?$AAe?$AA?$AA@ 000000018002ec08     libucrt:lcidtoname_downlevel.obj
 0002:00007c18       ??_C@_1M@PACPMGPH@?$AAk?$AAk?$AA?9?$AAk?$AAz?$AA?$AA@ 000000018002ec18     libucrt:lcidtoname_downlevel.obj
 0002:00007c28       ??_C@_1M@IELFGMHA@?$AAk?$AAn?$AA?9?$AAi?$AAn?$AA?$AA@ 000000018002ec28     libucrt:lcidtoname_downlevel.obj
 0002:00007c38       ??_C@_1O@IBBJHCH@?$AAk?$AAo?$AAk?$AA?9?$AAi?$AAn?$AA?$AA@ 000000018002ec38     libucrt:lcidtoname_downlevel.obj
 0002:00007c48       ??_C@_1M@DMHAEOGC@?$AAk?$AAo?$AA?9?$AAk?$AAr?$AA?$AA@ 000000018002ec48     libucrt:lcidtoname_downlevel.obj
 0002:00007c58       ??_C@_1M@HBAHBIGA@?$AAk?$AAy?$AA?9?$AAk?$AAg?$AA?$AA@ 000000018002ec58     libucrt:lcidtoname_downlevel.obj
 0002:00007c68       ??_C@_1M@KPMILCJG@?$AAl?$AAt?$AA?9?$AAl?$AAt?$AA?$AA@ 000000018002ec68     libucrt:lcidtoname_downlevel.obj
 0002:00007c78       ??_C@_1M@BDEKKCA@?$AAl?$AAv?$AA?9?$AAl?$AAv?$AA?$AA@ 000000018002ec78     libucrt:lcidtoname_downlevel.obj
 0002:00007c88       ??_C@_1M@ELCKCCJJ@?$AAm?$AAi?$AA?9?$AAn?$AAz?$AA?$AA@ 000000018002ec88     libucrt:lcidtoname_downlevel.obj
 0002:00007c98       ??_C@_1M@CBOOLAPA@?$AAm?$AAk?$AA?9?$AAm?$AAk?$AA?$AA@ 000000018002ec98     libucrt:lcidtoname_downlevel.obj
 0002:00007ca8       ??_C@_1M@GPHNBJKN@?$AAm?$AAl?$AA?9?$AAi?$AAn?$AA?$AA@ 000000018002eca8     libucrt:lcidtoname_downlevel.obj
 0002:00007cb8       ??_C@_1M@PABJILIG@?$AAm?$AAn?$AA?9?$AAm?$AAn?$AA?$AA@ 000000018002ecb8     libucrt:lcidtoname_downlevel.obj
 0002:00007cc8       ??_C@_1M@FGBKKIPG@?$AAm?$AAr?$AA?9?$AAi?$AAn?$AA?$AA@ 000000018002ecc8     libucrt:lcidtoname_downlevel.obj
 0002:00007cd8       ??_C@_1M@NDBPDDAL@?$AAm?$AAs?$AA?9?$AAb?$AAn?$AA?$AA@ 000000018002ecd8     libucrt:lcidtoname_downlevel.obj
 0002:00007ce8       ??_C@_1M@OPIHOOPI@?$AAm?$AAs?$AA?9?$AAm?$AAy?$AA?$AA@ 000000018002ece8     libucrt:lcidtoname_downlevel.obj
 0002:00007cf8       ??_C@_1M@PPDBCNFM@?$AAm?$AAt?$AA?9?$AAm?$AAt?$AA?$AA@ 000000018002ecf8     libucrt:lcidtoname_downlevel.obj
 0002:00007d08       ??_C@_1M@KDJDKMDD@?$AAn?$AAb?$AA?9?$AAn?$AAo?$AA?$AA@ 000000018002ed08     libucrt:lcidtoname_downlevel.obj
 0002:00007d18       ??_C@_1M@KFCFLMJP@?$AAn?$AAl?$AA?9?$AAb?$AAe?$AA?$AA@ 000000018002ed18     libucrt:lcidtoname_downlevel.obj
 0002:00007d28       ??_C@_1M@KPOPDDGO@?$AAn?$AAl?$AA?9?$AAn?$AAl?$AA?$AA@ 000000018002ed28     libucrt:lcidtoname_downlevel.obj
 0002:00007d38       ??_C@_1M@LJKPEMLN@?$AAn?$AAn?$AA?9?$AAn?$AAo?$AA?$AA@ 000000018002ed38     libucrt:lcidtoname_downlevel.obj
 0002:00007d48       ??_C@_1M@BDGHHBFL@?$AAn?$AAs?$AA?9?$AAz?$AAa?$AA?$AA@ 000000018002ed48     libucrt:lcidtoname_downlevel.obj
 0002:00007d58       ??_C@_1M@IDEHOAP@?$AAp?$AAa?$AA?9?$AAi?$AAn?$AA?$AA@ 000000018002ed58     libucrt:lcidtoname_downlevel.obj
 0002:00007d68       ??_C@_1M@HDBKGOGH@?$AAp?$AAl?$AA?9?$AAp?$AAl?$AA?$AA@ 000000018002ed68     libucrt:lcidtoname_downlevel.obj
 0002:00007d78       ??_C@_1M@LJLLCMEH@?$AAp?$AAt?$AA?9?$AAb?$AAr?$AA?$AA@ 000000018002ed78     libucrt:lcidtoname_downlevel.obj
 0002:00007d88       ??_C@_1M@NCMONAAL@?$AAp?$AAt?$AA?9?$AAp?$AAt?$AA?$AA@ 000000018002ed88     libucrt:lcidtoname_downlevel.obj
 0002:00007d98       ??_C@_1O@EAKMAJDN@?$AAq?$AAu?$AAz?$AA?9?$AAb?$AAo?$AA?$AA@ 000000018002ed98     libucrt:lcidtoname_downlevel.obj
 0002:00007da8       ??_C@_1O@BHHPIGDN@?$AAq?$AAu?$AAz?$AA?9?$AAe?$AAc?$AA?$AA@ 000000018002eda8     libucrt:lcidtoname_downlevel.obj
 0002:00007db8       ??_C@_1O@GBAPEKMJ@?$AAq?$AAu?$AAz?$AA?9?$AAp?$AAe?$AA?$AA@ 000000018002edb8     libucrt:lcidtoname_downlevel.obj
 0002:00007dc8       ??_C@_1M@CLGLEFBO@?$AAr?$AAo?$AA?9?$AAr?$AAo?$AA?$AA@ 000000018002edc8     libucrt:lcidtoname_downlevel.obj
 0002:00007dd8       ??_C@_1M@CEEDODME@?$AAr?$AAu?$AA?9?$AAr?$AAu?$AA?$AA@ 000000018002edd8     libucrt:lcidtoname_downlevel.obj
 0002:00007de8       ??_C@_1M@HPKKKMPP@?$AAs?$AAa?$AA?9?$AAi?$AAn?$AA?$AA@ 000000018002ede8     libucrt:lcidtoname_downlevel.obj
 0002:00007df8       ??_C@_1M@BKMAIGOJ@?$AAs?$AAe?$AA?9?$AAf?$AAi?$AA?$AA@ 000000018002edf8     libucrt:lcidtoname_downlevel.obj
 0002:00007e08       ??_C@_1M@NDPIFLFI@?$AAs?$AAe?$AA?9?$AAn?$AAo?$AA?$AA@ 000000018002ee08     libucrt:lcidtoname_downlevel.obj
 0002:00007e18       ??_C@_1M@DANKKHJ@?$AAs?$AAe?$AA?9?$AAs?$AAe?$AA?$AA@ 000000018002ee18     libucrt:lcidtoname_downlevel.obj
 0002:00007e28       ??_C@_1M@PNBLONPJ@?$AAs?$AAk?$AA?9?$AAs?$AAk?$AA?$AA@ 000000018002ee28     libucrt:lcidtoname_downlevel.obj
 0002:00007e38       ??_C@_1M@LFMODOAL@?$AAs?$AAl?$AA?9?$AAs?$AAi?$AA?$AA@ 000000018002ee38     libucrt:lcidtoname_downlevel.obj
 0002:00007e48       ??_C@_1O@DFKOMPG@?$AAs?$AAm?$AAa?$AA?9?$AAn?$AAo?$AA?$AA@ 000000018002ee48     libucrt:lcidtoname_downlevel.obj
 0002:00007e58       ??_C@_1O@NDKPBNNH@?$AAs?$AAm?$AAa?$AA?9?$AAs?$AAe?$AA?$AA@ 000000018002ee58     libucrt:lcidtoname_downlevel.obj
 0002:00007e68       ??_C@_1O@PLLKBHAB@?$AAs?$AAm?$AAj?$AA?9?$AAn?$AAo?$AA?$AA@ 000000018002ee68     libucrt:lcidtoname_downlevel.obj
 0002:00007e78       ??_C@_1O@CLEPOGCA@?$AAs?$AAm?$AAj?$AA?9?$AAs?$AAe?$AA?$AA@ 000000018002ee78     libucrt:lcidtoname_downlevel.obj
 0002:00007e88       ??_C@_1O@DLGJGKMK@?$AAs?$AAm?$AAn?$AA?9?$AAf?$AAi?$AA?$AA@ 000000018002ee88     libucrt:lcidtoname_downlevel.obj
 0002:00007e98       ??_C@_1O@OJDJGAJC@?$AAs?$AAm?$AAs?$AA?9?$AAf?$AAi?$AA?$AA@ 000000018002ee98     libucrt:lcidtoname_downlevel.obj
 0002:00007ea8       ??_C@_1M@BOFOGHPB@?$AAs?$AAq?$AA?9?$AAa?$AAl?$AA?$AA@ 000000018002eea8     libucrt:lcidtoname_downlevel.obj
 0002:00007eb8       ??_C@_1BG@LJBBIPGB@?$AAs?$AAr?$AA?9?$AAb?$AAa?$AA?9?$AAc?$AAy?$AAr?$AAl?$AA?$AA@ 000000018002eeb8     libucrt:lcidtoname_downlevel.obj
 0002:00007ed0       ??_C@_1BG@JLBENFOE@?$AAs?$AAr?$AA?9?$AAb?$AAa?$AA?9?$AAl?$AAa?$AAt?$AAn?$AA?$AA@ 000000018002eed0     libucrt:lcidtoname_downlevel.obj
 0002:00007ee8       ??_C@_1BG@KODPNHE@?$AAs?$AAr?$AA?9?$AAs?$AAp?$AA?9?$AAc?$AAy?$AAr?$AAl?$AA?$AA@ 000000018002eee8     libucrt:lcidtoname_downlevel.obj
 0002:00007f00       ??_C@_1BG@CIOGKHPB@?$AAs?$AAr?$AA?9?$AAs?$AAp?$AA?9?$AAl?$AAa?$AAt?$AAn?$AA?$AA@ 000000018002ef00     libucrt:lcidtoname_downlevel.obj
 0002:00007f18       ??_C@_1M@NGFJLMAC@?$AAs?$AAv?$AA?9?$AAf?$AAi?$AA?$AA@ 000000018002ef18     libucrt:lcidtoname_downlevel.obj
 0002:00007f28       ??_C@_1M@MPJEJAJC@?$AAs?$AAv?$AA?9?$AAs?$AAe?$AA?$AA@ 000000018002ef28     libucrt:lcidtoname_downlevel.obj
 0002:00007f38       ??_C@_1M@MPNDHLFK@?$AAs?$AAw?$AA?9?$AAk?$AAe?$AA?$AA@ 000000018002ef38     libucrt:lcidtoname_downlevel.obj
 0002:00007f48       ??_C@_1O@KOHBJJI@?$AAs?$AAy?$AAr?$AA?9?$AAs?$AAy?$AA?$AA@ 000000018002ef48     libucrt:lcidtoname_downlevel.obj
 0002:00007f58       ??_C@_1M@LDCEFHA@?$AAt?$AAa?$AA?9?$AAi?$AAn?$AA?$AA@ 000000018002ef58     libucrt:lcidtoname_downlevel.obj
 0002:00007f68       ??_C@_1M@CNJOFAK@?$AAt?$AAe?$AA?9?$AAi?$AAn?$AA?$AA@ 000000018002ef68     libucrt:lcidtoname_downlevel.obj
 0002:00007f78       ??_C@_1M@GNAECACD@?$AAt?$AAh?$AA?9?$AAt?$AAh?$AA?$AA@ 000000018002ef78     libucrt:lcidtoname_downlevel.obj
 0002:00007f88       ??_C@_1M@CHBIHOJO@?$AAt?$AAn?$AA?9?$AAz?$AAa?$AA?$AA@ 000000018002ef88     libucrt:lcidtoname_downlevel.obj
 0002:00007f98       ??_C@_1M@GCCMIGPJ@?$AAt?$AAr?$AA?9?$AAt?$AAr?$AA?$AA@ 000000018002ef98     libucrt:lcidtoname_downlevel.obj
 0002:00007fa8       ??_C@_1M@CELMCNBK@?$AAt?$AAt?$AA?9?$AAr?$AAu?$AA?$AA@ 000000018002efa8     libucrt:lcidtoname_downlevel.obj
 0002:00007fb8       ??_C@_1M@KLMCELGA@?$AAu?$AAk?$AA?9?$AAu?$AAa?$AA?$AA@ 000000018002efb8     libucrt:lcidtoname_downlevel.obj
 0002:00007fc8       ??_C@_1M@EPAJJAJF@?$AAu?$AAr?$AA?9?$AAp?$AAk?$AA?$AA@ 000000018002efc8     libucrt:lcidtoname_downlevel.obj
 0002:00007fd8       ??_C@_1BG@GEGPMCDJ@?$AAu?$AAz?$AA?9?$AAu?$AAz?$AA?9?$AAc?$AAy?$AAr?$AAl?$AA?$AA@ 000000018002efd8     libucrt:lcidtoname_downlevel.obj
 0002:00007ff0       ??_C@_1BG@EGGKJILM@?$AAu?$AAz?$AA?9?$AAu?$AAz?$AA?9?$AAl?$AAa?$AAt?$AAn?$AA?$AA@ 000000018002eff0     libucrt:lcidtoname_downlevel.obj
 0002:00008008       ??_C@_1M@GFOCLFF@?$AAv?$AAi?$AA?9?$AAv?$AAn?$AA?$AA@ 000000018002f008     libucrt:lcidtoname_downlevel.obj
 0002:00008018       ??_C@_1M@CPAMEDFI@?$AAx?$AAh?$AA?9?$AAz?$AAa?$AA?$AA@ 000000018002f018     libucrt:lcidtoname_downlevel.obj
 0002:00008028       ??_C@_1O@EBKIFIGN@?$AAz?$AAh?$AA?9?$AAc?$AAh?$AAs?$AA?$AA@ 000000018002f028     libucrt:lcidtoname_downlevel.obj
 0002:00008038       ??_C@_1O@NMHPGANE@?$AAz?$AAh?$AA?9?$AAc?$AAh?$AAt?$AA?$AA@ 000000018002f038     libucrt:lcidtoname_downlevel.obj
 0002:00008048       ??_C@_1M@LPINJOMC@?$AAz?$AAh?$AA?9?$AAc?$AAn?$AA?$AA@ 000000018002f048     libucrt:lcidtoname_downlevel.obj
 0002:00008058       ??_C@_1M@OCJEJODD@?$AAz?$AAh?$AA?9?$AAh?$AAk?$AA?$AA@ 000000018002f058     libucrt:lcidtoname_downlevel.obj
 0002:00008068       ??_C@_1M@DNDLJINH@?$AAz?$AAh?$AA?9?$AAm?$AAo?$AA?$AA@ 000000018002f068     libucrt:lcidtoname_downlevel.obj
 0002:00008078       ??_C@_1M@MBFDNDND@?$AAz?$AAh?$AA?9?$AAs?$AAg?$AA?$AA@ 000000018002f078     libucrt:lcidtoname_downlevel.obj
 0002:00008088       ??_C@_1M@IMEPLEPE@?$AAz?$AAh?$AA?9?$AAt?$AAw?$AA?$AA@ 000000018002f088     libucrt:lcidtoname_downlevel.obj
 0002:00008098       ??_C@_1M@BBGHNHJP@?$AAz?$AAu?$AA?9?$AAz?$AAa?$AA?$AA@ 000000018002f098     libucrt:lcidtoname_downlevel.obj
 0002:000080a8       __real@3ff0000000000000    000000018002f0a8     libucrt:ceil.obj
 0002:00008300       __log10_256_lead           000000018002f300     libucrt:log10_256_lead_tail_table.obj
 0002:00008b10       __log10_256_tail           000000018002fb10     libucrt:log10_256_lead_tail_table.obj
 0002:00009320       __log_F_inv_qword          0000000180030320     libucrt:log_f_inv_qword_table.obj
 0002:00009b30       ??_C@_05HGHHAHAP@log10?$AA@ 0000000180030b30     libucrt:log_special.obj
 0002:00009b50       ??_C@_1BA@BALFACEM@?$AAC?$AAO?$AAN?$AAO?$AAU?$AAT?$AA$?$AA?$AA@ 0000000180030b50     libucrt:initcon.obj
 0002:00009bc0       _load_config_used          0000000180030bc0     LIBCMT:loadcfg.obj
 0002:00009cc0       ??_R4CImgLoader@@6B@       0000000180030cc0     ImgCache.obj
 0002:00009ce8       ??_R3CImgLoader@@8         0000000180030ce8     ImgCache.obj
 0002:00009d00       ??_R2CImgLoader@@8         0000000180030d00     ImgCache.obj
 0002:00009d18       ??_R1A@?0A@EA@CImgLoader@@8 0000000180030d18     ImgCache.obj
 0002:00009d40       ??_R1A@?0A@EA@?$CQueueProcessor@PEAUIMAGE_CACHE_INFO@@@@8 0000000180030d40     ImgCache.obj
 0002:00009d68       ??_R3?$CQueueProcessor@PEAUIMAGE_CACHE_INFO@@@@8 0000000180030d68     ImgCache.obj
 0002:00009d80       ??_R2?$CQueueProcessor@PEAUIMAGE_CACHE_INFO@@@@8 0000000180030d80     ImgCache.obj
 0002:00009d90       ??_R4?$CQueueProcessor@PEAUIMAGE_CACHE_INFO@@@@6B@ 0000000180030d90     ImgCache.obj
 0002:00009db8       ??_R4MToolHelpProcess@@6B@ 0000000180030db8     common-kernel64:MProcess.obj
 0002:00009de0       ??_R3MToolHelpProcess@@8   0000000180030de0     common-kernel64:MProcess.obj
 0002:00009df8       ??_R2MToolHelpProcess@@8   0000000180030df8     common-kernel64:MProcess.obj
 0002:00009e10       ??_R1A@?0A@EA@MToolHelpProcess@@8 0000000180030e10     common-kernel64:MProcess.obj
 0002:00009e38       ??_R1A@?0A@EA@?$MToolHelp@UtagPROCESSENTRY32W@@$1?Process32FirstW@@YAHPEAXPEAU1@@Z$1?Process32NextW@@YAH01@Z@@8 0000000180030e38     common-kernel64:MProcess.obj
 0002:00009e60       ??_R3?$MToolHelp@UtagPROCESSENTRY32W@@$1?Process32FirstW@@YAHPEAXPEAU1@@Z$1?Process32NextW@@YAH01@Z@@8 0000000180030e60     common-kernel64:MProcess.obj
 0002:00009e78       ??_R2?$MToolHelp@UtagPROCESSENTRY32W@@$1?Process32FirstW@@YAHPEAXPEAU1@@Z$1?Process32NextW@@YAH01@Z@@8 0000000180030e78     common-kernel64:MProcess.obj
 0002:00009e88       ??_R4?$MToolHelp@UtagPROCESSENTRY32W@@$1?Process32FirstW@@YAHPEAXPEAU1@@Z$1?Process32NextW@@YAH01@Z@@6B@ 0000000180030e88     common-kernel64:MProcess.obj
 0002:00009eb0       ??_R4type_info@@6B@        0000000180030eb0     LIBCMT:std_type_info_static.obj
 0002:00009ed8       ??_R3type_info@@8          0000000180030ed8     LIBCMT:std_type_info_static.obj
 0002:00009ef0       ??_R2type_info@@8          0000000180030ef0     LIBCMT:std_type_info_static.obj
 0002:00009f00       ??_R1A@?0A@EA@type_info@@8 0000000180030f00     LIBCMT:std_type_info_static.obj
 0002:00009f28       ??_R4exception@std@@6B@    0000000180030f28     libvcruntime:frame.obj
 0002:00009f50       ??_R3exception@std@@8      0000000180030f50     libvcruntime:frame.obj
 0002:00009f68       ??_R2exception@std@@8      0000000180030f68     libvcruntime:frame.obj
 0002:00009f78       ??_R1A@?0A@EA@exception@std@@8 0000000180030f78     libvcruntime:frame.obj
 0002:00009fa0       ??_R4bad_exception@std@@6B@ 0000000180030fa0     libvcruntime:frame.obj
 0002:00009fc8       ??_R3bad_exception@std@@8  0000000180030fc8     libvcruntime:frame.obj
 0002:00009fe0       ??_R2bad_exception@std@@8  0000000180030fe0     libvcruntime:frame.obj
 0002:00009ff8       ??_R1A@?0A@EA@bad_exception@std@@8 0000000180030ff8     libvcruntime:frame.obj
 0002:0000a348       __rtc_iaa                  0000000180031348     LIBCMT:_initsect_.obj
 0002:0000a350       __rtc_izz                  0000000180031350     LIBCMT:_initsect_.obj
 0002:0000a358       __rtc_taa                  0000000180031358     LIBCMT:_initsect_.obj
 0002:0000a360       __rtc_tzz                  0000000180031360     LIBCMT:_initsect_.obj
 0002:0000be28       _TI2?AVbad_exception@std@@ 0000000180032e28     libvcruntime:frame.obj
 0002:0000be48       _CTA2?AVbad_exception@std@@ 0000000180032e48     libvcruntime:frame.obj
 0002:0000be60       _CT??_R0?AVbad_exception@std@@@8??0bad_exception@std@@QEAA@AEBV01@@Z24 0000000180032e60     libvcruntime:frame.obj
 0002:0000be88       _CT??_R0?AVexception@std@@@8??0exception@std@@QEAA@AEBV01@@Z24 0000000180032e88     libvcruntime:frame.obj
 0002:0000c01c       __IMPORT_DESCRIPTOR_VERSION 000000018003301c     version:VERSION.dll
 0002:0000c030       __IMPORT_DESCRIPTOR_KERNEL32 0000000180033030     kernel32:KERNEL32.dll
 0002:0000c044       __IMPORT_DESCRIPTOR_USER32 0000000180033044     user32:USER32.dll
 0002:0000c058       __IMPORT_DESCRIPTOR_GDI32  0000000180033058     gdi32:GDI32.dll
 0002:0000c06c       __IMPORT_DESCRIPTOR_ADVAPI32 000000018003306c     advapi32:ADVAPI32.dll
 0002:0000c080       __IMPORT_DESCRIPTOR_SHELL32 0000000180033080     shell32:SHELL32.dll
 0002:0000c094       __IMPORT_DESCRIPTOR_ole32  0000000180033094     ole32:ole32.dll
 0002:0000c0a8       __NULL_IMPORT_DESCRIPTOR   00000001800330a8     version:VERSION.dll
 0003:00000000       ?gcrCurColors@@3PEAKEA     0000000180035000     ConEmuTh.obj
 0003:00000008       ?gbPreloadByDefault@@3HA   0000000180035008     ConEmuTh.obj
 0003:00000010       ?Far3Func@@3PAUExportFunc@@A 0000000180035010     ConEmuTh.obj
 0003:00000060       ?StdPalette@?1??GetStdPalette@Far3Color@@SAPEBKXZ@4PAKA 0000000180035060     ConEmuTh1900.obj
 0003:000000a0       ?guid_ConEmuTh@@3U_GUID@@A 00000001800350a0     ConEmuTh2800.obj
 0003:000000b0       ?guid_ConEmuThPluginMenu@@3U_GUID@@A 00000001800350b0     ConEmuTh2800.obj
 0003:000000c0       ?g_TerminatedThreadIdx@@3JA 00000001800350c0     common-kernel64:WThreads.obj
 0003:000000c8       ?gsInternalCommands@@3PEB_WEB 00000001800350c8     common-kernel64:CmdLine.obj
 0003:000000d0       __security_cookie          00000001800350d0     LIBCMT:gs_cookie.obj
 0003:000000d8       __security_cookie_complement 00000001800350d8     LIBCMT:gs_cookie.obj
 0003:000000e0       __scrt_native_dllmain_reason 00000001800350e0     LIBCMT:utility.obj
 0003:000000e8       __isa_available            00000001800350e8     LIBCMT:_cpu_disp_.obj
 0003:000000ec       __isa_enabled              00000001800350ec     LIBCMT:_cpu_disp_.obj
 0003:000000f0       __memcpy_nt_iters          00000001800350f0     LIBCMT:_cpu_disp_.obj
 0003:00000110       __abort_behavior           0000000180035110     libucrt:abort.obj
 0003:00000130       _iob                       0000000180035130     libucrt:_file.obj
 0003:00000240       __acrt_initial_locale_data 0000000180035240     libucrt:nlsdata.obj
 0003:00000398       __acrt_initial_locale_pointers 0000000180035398     libucrt:nlsdata.obj
 0003:000003a8       __acrt_wide_c_locale_string 00000001800353a8     libucrt:nlsdata.obj
 0003:000003b0       _pwctype                   00000001800353b0     libucrt:ctype.obj
 0003:000003c0       __acrt_initial_multibyte_data 00000001800353c0     libucrt:mbctype.obj
 0003:000005e8       __acrt_current_multibyte_data 00000001800355e8     libucrt:mbctype.obj
 0003:000006f0       _mbctype                   00000001800356f0     libucrt:mbctype.obj
 0003:00000800       _mbcasemap                 0000000180035800     libucrt:mbctype.obj
 0003:00000900       __globallocalestatus       0000000180035900     libucrt:glstatus.obj
 0003:00000910       __acrt_lconv_c             0000000180035910     libucrt:localeconv.obj
 0003:000009a8       __acrt_lconv_static_decimal 00000001800359a8     libucrt:localeconv.obj
 0003:000009ac       __acrt_lconv_static_W_decimal 00000001800359ac     libucrt:localeconv.obj
 0003:000009c8       __dcrt_lowio_console_output_handle 00000001800359c8     libucrt:initcon.obj
 0003:000009d0       _fltused                   00000001800359d0     LIBCMT:fltused.obj
 0003:000009e0       ??_R0?AVCImgLoader@@@8     00000001800359e0     ImgCache.obj
 0003:00000a08       ??_R0?AV?$CQueueProcessor@PEAUIMAGE_CACHE_INFO@@@@@8 0000000180035a08     ImgCache.obj
 0003:00000a48       ??_R0?AVMToolHelpProcess@@@8 0000000180035a48     common-kernel64:MProcess.obj
 0003:00000a70       ??_R0?AV?$MToolHelp@UtagPROCESSENTRY32W@@$1?Process32FirstW@@YAHPEAXPEAU1@@Z$1?Process32NextW@@YAH01@Z@@@8 0000000180035a70     common-kernel64:MProcess.obj
 0003:00000ae8       ??_R0?AVtype_info@@@8      0000000180035ae8     LIBCMT:std_type_info_static.obj
 0003:00000b08       ??_R0?AVbad_exception@std@@@8 0000000180035b08     libvcruntime:frame.obj
 0003:00000b30       ??_R0?AVexception@std@@@8  0000000180035b30     libvcruntime:frame.obj
 0003:00000b60       ?gThSet@@3UPanelViewSetMapping@@A 0000000180035b60     ConEmuTh.obj
 0003:00000d78       ?ghConEmuRoot@@3PEAUHWND__@@EA 0000000180035d78     ConEmuTh.obj
 0003:00000d80       ?gThPal@@3UCESERVER_PALETTE@@A 0000000180035d80     ConEmuTh.obj
 0003:00000e00       ?ghConEmuWnd@@3PEAUHWND__@@EA 0000000180035e00     ConEmuTh.obj
 0003:00000e08       ?ghPluginModule@@3PEAUHINSTANCE__@@EA 0000000180035e08     ConEmuTh.obj
 0003:00000e10       ?gnSelfPID@@3KA            0000000180035e10     ConEmuTh.obj
 0003:00000e14       ?gnMainThreadId@@3KA       0000000180035e14     ConEmuTh.obj
 0003:00000e18       ?gFarVersion@@3UFarVersion@@A 0000000180035e18     ConEmuTh.obj
 0003:00000e24       ?gnDisplayThreadId@@3KA    0000000180035e24     ConEmuTh.obj
 0003:00000e28       ?ghDisplayThread@@3PEAXEA  0000000180035e28     ConEmuTh.obj
 0003:00000e30       ?pviLeft@@3UCeFullPanelInfo@@A 0000000180035e30     ConEmuTh.obj
 0003:000010f0       ?pviRight@@3UCeFullPanelInfo@@A 00000001800360f0     ConEmuTh.obj
 0003:000013b0       ?gnWaitForKeySeqTick@@3KA  00000001800363b0     ConEmuTh.obj
 0003:000013b4       ?gFarPanelSettings@@3UCEFarPanelSettings@@A 00000001800363b4     ConEmuTh.obj
 0003:000013b8       ?gFarInterfaceSettings@@3UCEFarInterfaceSettings@@A 00000001800363b8     ConEmuTh.obj
 0003:000013bc       ?gbFadeColors@@3_NA        00000001800363bc     ConEmuTh.obj
 0003:000013bd       ?gbFarPanelsReady@@3_NA    00000001800363bd     ConEmuTh.obj
 0003:000013be       ?gbSynchoRedrawPanelRequested@@3_NA 00000001800363be     ConEmuTh.obj
 0003:000013bf       ?gbConsoleChangesSyncho@@3_NA 00000001800363bf     ConEmuTh.obj
 0003:000013c0       ?gsFolder@@3PA_WA          00000001800363c0     ConEmuTh.obj
 0003:00001440       ?gsSymLink@@3PA_WA         0000000180036440     ConEmuTh.obj
 0003:000014c0       ?gsJunction@@3PA_WA        00000001800364c0     ConEmuTh.obj
 0003:00001540       ?gsTitleThumbs@@3PA_WA     0000000180036540     ConEmuTh.obj
 0003:000015c0       ?gsTitleTiles@@3PA_WA      00000001800365c0     ConEmuTh.obj
 0003:00001640       ?gpRgnDetect@@3PEAVCRgnDetect@@EA 0000000180036640     ConEmuTh.obj
 0003:00001648       ?gnRgnDetectFlags@@3KA     0000000180036648     ConEmuTh.obj
 0003:0000164c       ?TerminalMode@@3HA         000000018003664c     ConEmuTh.obj
 0003:00001650       ?gFarInfo@@3UCEFAR_INFO_MAPPING@@A 0000000180036650     ConEmuTh.obj
 0003:00021988       ?gpLastSynchroArg@@3PEAUConEmuThSynchroArg@@EA 0000000180056988     ConEmuTh.obj
 0003:00021990       ?gfRegisterPanelView@@3P6AHPEAUPanelViewInit@@@ZEA 0000000180056990     ConEmuTh.obj
 0003:00021998       ?gfGetFarHWND2@@3P6APEAUHWND__@@H@ZEA 0000000180056998     ConEmuTh.obj
 0003:000219a0       ?gdwModes@@3PAKA           00000001800569a0     ConEmuTh.obj
 0003:000219a8       ?gnMainThreadIdInitial@@3KA 00000001800569a8     ConEmuTh.obj
 0003:000219ac       ?wScanCodeUp@@3GA          00000001800569ac     ConEmuTh.obj
 0003:000219b0       ?gsHardLink@@3PA_WA        00000001800569b0     ConEmuTh.obj
 0003:00021a30       ?wScanCodeDown@@3GA        0000000180056a30     ConEmuTh.obj
 0003:00021a34       ?gnConsoleChanges@@3KA     0000000180056a34     ConEmuTh.obj
 0003:00021a38       ?gpDbgDlg@@3PEAV?$MFileMapping@Utag_DetectedDialog@@@@EA 0000000180056a38     ConEmuTh.obj
 0003:00021a40       ?gbInfoW_OK@@3HA           0000000180056a40     ConEmuTh.obj
 0003:00021a48       ?gpImgCache@@3PEAVCImgCache@@EA 0000000180056a48     ConEmuTh.obj
 0003:00021a50       ?_OptionsStorage@?1??__local_stdio_printf_options@@9@4_KA 0000000180056a50     ConEmuTh.obj
 0003:00021a60       ?InfoW1900@@3PEAUPluginStartupInfo@@EA 0000000180056a60     ConEmuTh1900.obj
 0003:00021a68       ?FSFW1900@@3PEAUFarStandardFunctions@@EA 0000000180056a68     ConEmuTh1900.obj
 0003:00021a70       ?LastColor@?1??Color2FgIndex@Far3Color@@SAXKAEAGPEBK@Z@4KA 0000000180056a70     ConEmuTh1900.obj
 0003:00021a74       ?LastIndex@?1??Color2FgIndex@Far3Color@@SAXKAEAGPEBK@Z@4HA 0000000180056a74     ConEmuTh1900.obj
 0003:00021a78       ?LastColor@?1??Color2BgIndex@Far3Color@@SAXKHAEAGPEBK@Z@4KA 0000000180056a78     ConEmuTh1900.obj
 0003:00021a7c       ?LastIndex@?1??Color2BgIndex@Far3Color@@SAXKHAEAGPEBK@Z@4HA 0000000180056a7c     ConEmuTh1900.obj
 0003:00021c90       ?InfoW2800@@3PEAUPluginStartupInfo@@EA 0000000180056c90     ConEmuTh2800.obj
 0003:00021c98       ?FSFW2800@@3PEAUFarStandardFunctions@@EA 0000000180056c98     ConEmuTh2800.obj
 0003:00021eb0       ?InfoW995@@3PEAUPluginStartupInfo@@EA 0000000180056eb0     ConEmuTh995.obj
 0003:00021eb8       ?FSFW995@@3PEAUFarStandardFunctions@@EA 0000000180056eb8     ConEmuTh995.obj
 0003:000220d0       ?InfoA@@3PEAUPluginStartupInfo@@EA 00000001800570d0     ConEmuThA.obj
 0003:000220d8       ?FSFA@@3PEAUFarStandardFunctions@@EA 00000001800570d8     ConEmuThA.obj
 0003:000221f0       ?ghCreateEvent@@3PEAXEA    00000001800571f0     Display.obj
 0003:000221f8       ?gnConEmuFadeMsg@@3IA      00000001800571f8     Display.obj
 0003:000221fc       ?gnConEmuSettingsMsg@@3IA  00000001800571fc     Display.obj
 0003:00022200       ?gnMapCoordMsg@@3IA        0000000180057200     Display.obj
 0003:00022204       ?gbCancelAll@@3HA          0000000180057204     Display.obj
 0003:00022208       ?gnCreateViewError@@3HA    0000000180057208     Display.obj
 0003:0002220c       ?gnWin32Error@@3KA         000000018005720c     Display.obj
 0003:00022218       ?ghUpIcon@@3PEAUHICON__@@EA 0000000180057218     ImgCache.obj
 0003:00022220       ?ghHeap@@3PEAXEA           0000000180057220     common-kernel64:Memory.obj
 0003:00022228       ?g_LastDeletePtr@@3PEAXEA  0000000180057228     common-kernel64:Memory.obj
 0003:00022230       ?gbInCommonShutdown@@3HA   0000000180057230     common-kernel64:Common.obj
 0003:00022238       ?gNullDesc@@3PEAVMNullDesc@@EA 0000000180057238     common-kernel64:MSecurity.obj
 0003:00022240       ?gpLocalSecurity@@3PEAU_SECURITY_ATTRIBUTES@@EA 0000000180057240     common-kernel64:ConEmuCheck.obj
 0003:00022248       ?ghWorkingModule@@3UHANDLE2@@A 0000000180057248     common-kernel64:ConEmuCheck.obj
 0003:00022250       ?gfGetRealConsoleWindow@@3P6APEAUHWND__@@XZEA 0000000180057250     common-kernel64:ConEmuCheck.obj
 0003:000222a4       ?hkFunc@@3UHkFunc@@A       00000001800572a4     common-kernel64:HkFunc.obj
 0003:000222b0       ?g_ThreadsIdx@@3JA         00000001800572b0     common-kernel64:WThreads.obj
 0003:0002aac8       ?gfnSearchAppPaths@@3P6A_NPEB_WAEAUCEStr@@_NPEAU1@@ZEA 000000018005fac8     common-kernel64:WObjects.obj
 0003:0002b060       ?__type_info_root_node@@3U__type_info_node@@A 0000000180060060     LIBCMT:tncleanup.obj
 0003:0002b070       ?_OptionsStorage@?1??__local_stdio_scanf_options@@9@4_KA 0000000180060070     LIBCMT:default_local_stdio_options.obj
 0003:0002b078       __scrt_current_native_startup_state 0000000180060078     LIBCMT:utility.obj
 0003:0002b080       __scrt_native_startup_lock 0000000180060080     LIBCMT:utility.obj
 0003:0002b0bc       __scrt_debugger_hook_flag  00000001800600bc     LIBCMT:utility_desktop.obj
 0003:0002b0c0       __favor                    00000001800600c0     LIBCMT:_cpu_disp_.obj
 0003:0002b148       ?m_pGetParameter@UnDecorator@@0P6APEADJ@ZEA 0000000180060148     libvcruntime:undname.obj
 0003:0002b150       ?m_CHPENameOffset@UnDecorator@@0KA 0000000180060150     libvcruntime:undname.obj
 0003:0002b154       ?m_recursionLevel@UnDecorator@@0KA 0000000180060154     libvcruntime:undname.obj
 0003:0002b158       ?pArgList@UnDecorator@@0PEAVReplicator@@EA 0000000180060158     libvcruntime:undname.obj
 0003:0002b160       ?pZNameList@UnDecorator@@0PEAVReplicator@@EA 0000000180060160     libvcruntime:undname.obj
 0003:0002b168       ?pTemplateArgList@UnDecorator@@0PEAVReplicator@@EA 0000000180060168     libvcruntime:undname.obj
 0003:0002b170       ?gName@UnDecorator@@0PEBDEB 0000000180060170     libvcruntime:undname.obj
 0003:0002b178       ?name@UnDecorator@@0PEBDEB 0000000180060178     libvcruntime:undname.obj
 0003:0002b180       ?disableFlags@UnDecorator@@0KA 0000000180060180     libvcruntime:undname.obj
 0003:0002b184       ?fExplicitTemplateParams@UnDecorator@@0_NA 0000000180060184     libvcruntime:undname.obj
 0003:0002b185       ?fGetTemplateArgumentList@UnDecorator@@0_NA 0000000180060185     libvcruntime:undname.obj
 0003:0002b220       __pPurecall                0000000180060220     libvcruntime:purevirt_data.obj
 0003:0002b228       ?__WinRTOutOfMemoryExceptionCallback@@3P6APEAXXZEA 0000000180060228     libvcruntime:ehhelpers.obj
 0003:0002b358       _environ_table             0000000180060358     libucrt:environment_initialization.obj
 0003:0002b360       _wenviron_table            0000000180060360     libucrt:environment_initialization.obj
 0003:0002b368       __dcrt_initial_wide_environment 0000000180060368     libucrt:environment_initialization.obj
 0003:0002b370       __dcrt_initial_narrow_environment 0000000180060370     libucrt:environment_initialization.obj
 0003:0002b378       __acrt_atexit_table        0000000180060378     libucrt:onexit.obj
 0003:0002b390       __acrt_at_quick_exit_table 0000000180060390     libucrt:onexit.obj
 0003:0002b3b0       _nstream                   00000001800603b0     libucrt:_file.obj
 0003:0002b3b8       __piob                     00000001800603b8     libucrt:_file.obj
 0003:0002b3c8       __acrt_stdout_buffer       00000001800603c8     libucrt:_sftbuf.obj
 0003:0002b3d0       __acrt_stderr_buffer       00000001800603d0     libucrt:_sftbuf.obj
 0003:0002b3d8       __acrt_locale_changed_data 00000001800603d8     libucrt:wsetlocale.obj
 0003:0002b3e0       __acrt_current_locale_data 00000001800603e0     libucrt:nlsdata.obj
 0003:0002b3f0       __pioinfo                  00000001800603f0     libucrt:ioinit.obj
 0003:0002b7f0       _nhandle                   00000001800607f0     libucrt:ioinit.obj
 0003:0002bbb4       __mbcodepage               0000000180060bb4     libucrt:mbctype.obj
 0003:0002bbb8       __ismbcodepage             0000000180060bb8     libucrt:mbctype.obj
 0003:0002bbc0       __mbulinfo                 0000000180060bc0     libucrt:mbctype.obj
 0003:0002bbd0       __mblocalename             0000000180060bd0     libucrt:mbctype.obj
 0003:0002bbdc       __argc                     0000000180060bdc     libucrt:argv_data.obj
 0003:0002bbe0       __argv                     0000000180060be0     libucrt:argv_data.obj
 0003:0002bbe8       __wargv                    0000000180060be8     libucrt:argv_data.obj
 0003:0002bbf0       _acmdln                    0000000180060bf0     libucrt:argv_data.obj
 0003:0002bbf8       _wcmdln                    0000000180060bf8     libucrt:argv_data.obj
 0003:0002bc00       _pgmptr                    0000000180060c00     libucrt:argv_data.obj
 0003:0002bc08       __acrt_heap                0000000180060c08     libucrt:heap_handle.obj
 0003:0002bc44       __acrt_lconv_static_null   0000000180060c44     libucrt:localeconv.obj
 0003:0002bc48       __acrt_lconv_static_W_null 0000000180060c48     libucrt:localeconv.obj
 0003:0002bc50       __fma3_is_available        0000000180060c50     libucrt:fma3_available.obj
 0003:0002bc54       __use_fma3_lib             0000000180060c54     libucrt:fma3_available.obj
 0003:0002bc58       __scrt_ucrt_dll_is_in_use  0000000180060c58     <common>
 0003:0002bc60       __dyn_tls_init_callback    0000000180060c60     <common>

 entry point at        0001:00013a80

 Static symbols

 0000:fff9a000       .debug$S                   0000000180000000     kernel32:KERNEL32.dll
 0000:fff9a000       .debug$S                   0000000180000000     advapi32:ADVAPI32.dll
 0000:fff9a000       .debug$S                   0000000180000000     gdi32:GDI32.dll
 0000:fff9a000       .debug$S                   0000000180000000     ole32:ole32.dll
 0000:fff9a000       .debug$S                   0000000180000000     ole32:ole32.dll
 0000:fff9a000       .debug$S                   0000000180000000     shell32:SHELL32.dll
 0000:fff9a000       .debug$S                   0000000180000000     advapi32:ADVAPI32.dll
 0000:fff9a000       .debug$S                   0000000180000000     advapi32:ADVAPI32.dll
 0000:fff9a000       .debug$S                   0000000180000000     advapi32:ADVAPI32.dll
 0000:fff9a000       .debug$S                   0000000180000000     version:VERSION.dll
 0000:fff9a000       .debug$S                   0000000180000000     version:VERSION.dll
 0000:fff9a000       .debug$S                   0000000180000000     version:VERSION.dll
 0000:fff9a000       .debug$S                   0000000180000000     kernel32:KERNEL32.dll
 0000:fff9a000       .debug$S                   0000000180000000     kernel32:KERNEL32.dll
 0000:fff9a000       .debug$S                   0000000180000000     kernel32:KERNEL32.dll
 0000:fff9a000       .debug$S                   0000000180000000     kernel32:KERNEL32.dll
 0000:fff9a000       .debug$S                   0000000180000000     kernel32:KERNEL32.dll
 0000:fff9a000       .debug$S                   0000000180000000     kernel32:KERNEL32.dll
 0000:fff9a000       .debug$S                   0000000180000000     kernel32:KERNEL32.dll
 0000:fff9a000       .debug$S                   0000000180000000     kernel32:KERNEL32.dll
 0000:fff9a000       .debug$S                   0000000180000000     kernel32:KERNEL32.dll
 0000:fff9a000       .debug$S                   0000000180000000     ConEmuTh.x64.exp
 0000:fff9a000       .debug$S                   0000000180000000     kernel32:KERNEL32.dll
 0000:fff9a000       .debug$S                   0000000180000000     kernel32:KERNEL32.dll
 0000:fff9a000       .debug$S                   0000000180000000     kernel32:KERNEL32.dll
 0000:fff9a000       .debug$S                   0000000180000000     kernel32:KERNEL32.dll
 0000:fff9a000       .debug$S                   0000000180000000     kernel32:KERNEL32.dll
 0000:fff9a000       .debug$S                   0000000180000000     kernel32:KERNEL32.dll
 0000:fff9a000       .debug$S                   0000000180000000     kernel32:KERNEL32.dll
 0000:fff9a000       .debug$S                   0000000180000000     kernel32:KERNEL32.dll
 0000:fff9a000       .debug$S                   0000000180000000     advapi32:ADVAPI32.dll
 0000:fff9a000       .debug$S                   0000000180000000     advapi32:ADVAPI32.dll
 0000:fff9a000       .debug$S                   0000000180000000     advapi32:ADVAPI32.dll
 0000:fff9a000       .debug$S                   0000000180000000     advapi32:ADVAPI32.dll
 0000:fff9a000       .debug$S                   0000000180000000     advapi32:ADVAPI32.dll
 0000:fff9a000       .debug$S                   0000000180000000     advapi32:ADVAPI32.dll
 0000:fff9a000       .debug$S                   0000000180000000     advapi32:ADVAPI32.dll
 0000:fff9a000       .debug$S                   0000000180000000     user32:USER32.dll
 0000:fff9a000       .debug$S                   0000000180000000     user32:USER32.dll
 0000:fff9a000       .debug$S                   0000000180000000     user32:USER32.dll
 0000:fff9a000       .debug$S                   0000000180000000     user32:USER32.dll
 0000:fff9a000       .debug$S                   0000000180000000     user32:USER32.dll
 0000:fff9a000       .debug$S                   0000000180000000     user32:USER32.dll
 0000:fff9a000       .debug$S                   0000000180000000     kernel32:KERNEL32.dll
 0000:fff9a000       .debug$S                   0000000180000000     kernel32:KERNEL32.dll
 0000:fff9a000       .debug$S                   0000000180000000     kernel32:KERNEL32.dll
 0000:fff9a000       .debug$S                   0000000180000000     kernel32:KERNEL32.dll
 0000:fff9a000       .debug$S                   0000000180000000     kernel32:KERNEL32.dll
 0000:fff9a000       .debug$S                   0000000180000000     kernel32:KERNEL32.dll
 0000:fff9a000       .debug$S                   0000000180000000     kernel32:KERNEL32.dll
 0000:fff9a000       .debug$S                   0000000180000000     kernel32:KERNEL32.dll
 0000:fff9a000       .debug$S                   0000000180000000     kernel32:KERNEL32.dll
 0000:fff9a000       .debug$S                   0000000180000000     kernel32:KERNEL32.dll
 0000:fff9a000       .debug$S                   0000000180000000     kernel32:KERNEL32.dll
 0000:fff9a000       .debug$S                   0000000180000000     kernel32:KERNEL32.dll
 0000:fff9a000       .debug$S                   0000000180000000     kernel32:KERNEL32.dll
 0000:fff9a000       .debug$S                   0000000180000000     kernel32:KERNEL32.dll
 0000:fff9a000       .debug$S                   0000000180000000     kernel32:KERNEL32.dll
 0000:fff9a000       .debug$S                   0000000180000000     kernel32:KERNEL32.dll
 0000:fff9a000       .debug$S                   0000000180000000     kernel32:KERNEL32.dll
 0000:fff9a000       .debug$S                   0000000180000000     kernel32:KERNEL32.dll
 0000:fff9a000       .debug$S                   0000000180000000     kernel32:KERNEL32.dll
 0000:fff9a000       .debug$S                   0000000180000000     kernel32:KERNEL32.dll
 0000:fff9a000       .debug$S                   0000000180000000     kernel32:KERNEL32.dll
 0000:fff9a000       .debug$S                   0000000180000000     kernel32:KERNEL32.dll
 0000:fff9a000       .debug$S                   0000000180000000     kernel32:KERNEL32.dll
 0000:fff9a000       .debug$S                   0000000180000000     kernel32:KERNEL32.dll
 0000:fff9a000       .debug$S                   0000000180000000     kernel32:KERNEL32.dll
 0000:fff9a000       .debug$S                   0000000180000000     kernel32:KERNEL32.dll
 0000:fff9a000       .debug$S                   0000000180000000     kernel32:KERNEL32.dll
 0000:fff9a000       .debug$S                   0000000180000000     kernel32:KERNEL32.dll
 0000:fff9a000       .debug$S                   0000000180000000     kernel32:KERNEL32.dll
 0000:fff9a000       .debug$S                   0000000180000000     kernel32:KERNEL32.dll
 0000:fff9a000       .debug$S                   0000000180000000     kernel32:KERNEL32.dll
 0000:fff9a000       .debug$S                   0000000180000000     kernel32:KERNEL32.dll
 0000:fff9a000       .debug$S                   0000000180000000     kernel32:KERNEL32.dll
 0000:fff9a000       .debug$S                   0000000180000000     kernel32:KERNEL32.dll
 0000:fff9a000       .debug$S                   0000000180000000     kernel32:KERNEL32.dll
 0000:fff9a000       .debug$S                   0000000180000000     kernel32:KERNEL32.dll
 0000:fff9a000       .debug$S                   0000000180000000     kernel32:KERNEL32.dll
 0000:fff9a000       .debug$S                   0000000180000000     kernel32:KERNEL32.dll
 0000:fff9a000       .debug$S                   0000000180000000     kernel32:KERNEL32.dll
 0000:fff9a000       .debug$S                   0000000180000000     kernel32:KERNEL32.dll
 0000:fff9a000       .debug$S                   0000000180000000     kernel32:KERNEL32.dll
 0000:fff9a000       .debug$S                   0000000180000000     kernel32:KERNEL32.dll
 0000:fff9a000       .debug$S                   0000000180000000     kernel32:KERNEL32.dll
 0000:fff9a000       .debug$S                   0000000180000000     kernel32:KERNEL32.dll
 0000:fff9a000       .debug$S                   0000000180000000     kernel32:KERNEL32.dll
 0000:fff9a000       .debug$S                   0000000180000000     kernel32:KERNEL32.dll
 0000:fff9a000       .debug$S                   0000000180000000     kernel32:KERNEL32.dll
 0000:fff9a000       .debug$S                   0000000180000000     kernel32:KERNEL32.dll
 0000:fff9a000       .debug$S                   0000000180000000     kernel32:KERNEL32.dll
 0000:fff9a000       .debug$S                   0000000180000000     kernel32:KERNEL32.dll
 0000:fff9a000       .debug$S                   0000000180000000     kernel32:KERNEL32.dll
 0000:fff9a000       .debug$S                   0000000180000000     kernel32:KERNEL32.dll
 0000:fff9a000       .debug$S                   0000000180000000     kernel32:KERNEL32.dll
 0000:fff9a000       .debug$S                   0000000180000000     kernel32:KERNEL32.dll
 0000:fff9a000       .debug$S                   0000000180000000     kernel32:KERNEL32.dll
 0000:fff9a000       .debug$S                   0000000180000000     kernel32:KERNEL32.dll
 0000:fff9a000       .debug$S                   0000000180000000     kernel32:KERNEL32.dll
 0000:fff9a000       .debug$S                   0000000180000000     kernel32:KERNEL32.dll
 0000:fff9a000       .debug$S                   0000000180000000     kernel32:KERNEL32.dll
 0000:fff9a000       .debug$S                   0000000180000000     kernel32:KERNEL32.dll
 0000:fff9a000       .debug$S                   0000000180000000     kernel32:KERNEL32.dll
 0000:fff9a000       .debug$S                   0000000180000000     kernel32:KERNEL32.dll
 0000:fff9a000       .debug$S                   0000000180000000     kernel32:KERNEL32.dll
 0000:fff9a000       .debug$S                   0000000180000000     kernel32:KERNEL32.dll
 0000:fff9a000       .debug$S                   0000000180000000     kernel32:KERNEL32.dll
 0000:fff9a000       .debug$S                   0000000180000000     kernel32:KERNEL32.dll
 0000:fff9a000       .debug$S                   0000000180000000     kernel32:KERNEL32.dll
 0000:fff9a000       .debug$S                   0000000180000000     kernel32:KERNEL32.dll
 0000:fff9a000       .debug$S                   0000000180000000     kernel32:KERNEL32.dll
 0000:fff9a000       .debug$S                   0000000180000000     kernel32:KERNEL32.dll
 0000:fff9a000       .debug$S                   0000000180000000     kernel32:KERNEL32.dll
 0000:fff9a000       .debug$S                   0000000180000000     kernel32:KERNEL32.dll
 0000:fff9a000       .debug$S                   0000000180000000     kernel32:KERNEL32.dll
 0000:fff9a000       .debug$S                   0000000180000000     kernel32:KERNEL32.dll
 0000:fff9a000       .debug$S                   0000000180000000     kernel32:KERNEL32.dll
 0000:fff9a000       .debug$S                   0000000180000000     kernel32:KERNEL32.dll
 0000:fff9a000       .debug$S                   0000000180000000     kernel32:KERNEL32.dll
 0000:fff9a000       .debug$S                   0000000180000000     kernel32:KERNEL32.dll
 0000:fff9a000       .debug$S                   0000000180000000     kernel32:KERNEL32.dll
 0000:fff9a000       .debug$S                   0000000180000000     kernel32:KERNEL32.dll
 0000:fff9a000       .debug$S                   0000000180000000     kernel32:KERNEL32.dll
 0000:fff9a000       .debug$S                   0000000180000000     kernel32:KERNEL32.dll
 0000:fff9a000       .debug$S                   0000000180000000     kernel32:KERNEL32.dll
 0000:fff9a000       .debug$S                   0000000180000000     kernel32:KERNEL32.dll
 0000:fff9a000       .debug$S                   0000000180000000     kernel32:KERNEL32.dll
 0000:fff9a000       .debug$S                   0000000180000000     kernel32:KERNEL32.dll
 0000:fff9a000       .debug$S                   0000000180000000     kernel32:KERNEL32.dll
 0000:fff9a000       .debug$S                   0000000180000000     kernel32:KERNEL32.dll
 0000:fff9a000       .debug$S                   0000000180000000     kernel32:KERNEL32.dll
 0000:fff9a000       .debug$S                   0000000180000000     kernel32:KERNEL32.dll
 0000:fff9a000       .debug$S                   0000000180000000     kernel32:KERNEL32.dll
 0000:fff9a000       .debug$S                   0000000180000000     kernel32:KERNEL32.dll
 0000:fff9a000       .debug$S                   0000000180000000     gdi32:GDI32.dll
 0000:fff9a000       .debug$S                   0000000180000000     kernel32:KERNEL32.dll
 0000:fff9a000       .debug$S                   0000000180000000     kernel32:KERNEL32.dll
 0000:fff9a000       .debug$S                   0000000180000000     kernel32:KERNEL32.dll
 0000:fff9a000       .debug$S                   0000000180000000     kernel32:KERNEL32.dll
 0000:fff9a000       .debug$S                   0000000180000000     kernel32:KERNEL32.dll
 0000:fff9a000       .debug$S                   0000000180000000     kernel32:KERNEL32.dll
 0000:fff9a000       .debug$S                   0000000180000000     kernel32:KERNEL32.dll
 0000:fff9a000       .debug$S                   0000000180000000     kernel32:KERNEL32.dll
 0000:fff9a000       .debug$S                   0000000180000000     kernel32:KERNEL32.dll
 0000:fff9a000       .debug$S                   0000000180000000     kernel32:KERNEL32.dll
 0000:fff9a000       .debug$S                   0000000180000000     kernel32:KERNEL32.dll
 0000:fff9a000       .debug$S                   0000000180000000     kernel32:KERNEL32.dll
 0000:fff9a000       .debug$S                   0000000180000000     kernel32:KERNEL32.dll
 0000:fff9a000       .debug$S                   0000000180000000     kernel32:KERNEL32.dll
 0000:fff9a000       .debug$S                   0000000180000000     kernel32:KERNEL32.dll
 0000:fff9a000       .debug$S                   0000000180000000     kernel32:KERNEL32.dll
 0000:fff9a000       .debug$S                   0000000180000000     kernel32:KERNEL32.dll
 0000:fff9a000       .debug$S                   0000000180000000     kernel32:KERNEL32.dll
 0000:fff9a000       .debug$S                   0000000180000000     kernel32:KERNEL32.dll
 0000:fff9a000       .debug$S                   0000000180000000     kernel32:KERNEL32.dll
 0000:fff9a000       .debug$S                   0000000180000000     kernel32:KERNEL32.dll
 0000:fff9a000       .debug$S                   0000000180000000     kernel32:KERNEL32.dll
 0000:fff9a000       .debug$S                   0000000180000000     kernel32:KERNEL32.dll
 0000:fff9a000       .debug$S                   0000000180000000     kernel32:KERNEL32.dll
 0000:fff9a000       .debug$S                   0000000180000000     kernel32:KERNEL32.dll
 0000:fff9a000       .debug$S                   0000000180000000     kernel32:KERNEL32.dll
 0000:fff9a000       .debug$S                   0000000180000000     kernel32:KERNEL32.dll
 0000:fff9a000       .debug$S                   0000000180000000     kernel32:KERNEL32.dll
 0000:fff9a000       .debug$S                   0000000180000000     kernel32:KERNEL32.dll
 0000:fff9a000       .debug$S                   0000000180000000     kernel32:KERNEL32.dll
 0000:fff9a000       .debug$S                   0000000180000000     kernel32:KERNEL32.dll
 0000:fff9a000       .debug$S                   0000000180000000     kernel32:KERNEL32.dll
 0000:fff9a000       .debug$S                   0000000180000000     kernel32:KERNEL32.dll
 0000:fff9a000       .debug$S                   0000000180000000     kernel32:KERNEL32.dll
 0000:fff9a000       .debug$S                   0000000180000000     kernel32:KERNEL32.dll
 0000:fff9a000       .debug$S                   0000000180000000     kernel32:KERNEL32.dll
 0000:fff9a000       .debug$S                   0000000180000000     kernel32:KERNEL32.dll
 0000:fff9a000       .debug$S                   0000000180000000     kernel32:KERNEL32.dll
 0000:fff9a000       .debug$S                   0000000180000000     kernel32:KERNEL32.dll
 0000:fff9a000       .debug$S                   0000000180000000     kernel32:KERNEL32.dll
 0000:fff9a000       .debug$S                   0000000180000000     kernel32:KERNEL32.dll
 0000:fff9a000       .debug$S                   0000000180000000     kernel32:KERNEL32.dll
 0000:fff9a000       .debug$S                   0000000180000000     kernel32:KERNEL32.dll
 0000:fff9a000       .debug$S                   0000000180000000     kernel32:KERNEL32.dll
 0000:fff9a000       .debug$S                   0000000180000000     kernel32:KERNEL32.dll
 0000:fff9a000       .debug$S                   0000000180000000     user32:USER32.dll
 0000:fff9a000       .debug$S                   0000000180000000     user32:USER32.dll
 0000:fff9a000       .debug$S                   0000000180000000     user32:USER32.dll
 0000:fff9a000       .debug$S                   0000000180000000     user32:USER32.dll
 0000:fff9a000       .debug$S                   0000000180000000     user32:USER32.dll
 0000:fff9a000       .debug$S                   0000000180000000     user32:USER32.dll
 0000:fff9a000       .debug$S                   0000000180000000     user32:USER32.dll
 0000:fff9a000       .debug$S                   0000000180000000     user32:USER32.dll
 0000:fff9a000       .debug$S                   0000000180000000     user32:USER32.dll
 0000:fff9a000       .debug$S                   0000000180000000     user32:USER32.dll
 0000:fff9a000       .debug$S                   0000000180000000     user32:USER32.dll
 0000:fff9a000       .debug$S                   0000000180000000     user32:USER32.dll
 0000:fff9a000       .debug$S                   0000000180000000     user32:USER32.dll
 0000:fff9a000       .debug$S                   0000000180000000     user32:USER32.dll
 0000:fff9a000       .debug$S                   0000000180000000     user32:USER32.dll
 0000:fff9a000       .debug$S                   0000000180000000     user32:USER32.dll
 0000:fff9a000       .debug$S                   0000000180000000     user32:USER32.dll
 0000:fff9a000       .debug$S                   0000000180000000     user32:USER32.dll
 0000:fff9a000       .debug$S                   0000000180000000     user32:USER32.dll
 0000:fff9a000       .debug$S                   0000000180000000     user32:USER32.dll
 0000:fff9a000       .debug$S                   0000000180000000     user32:USER32.dll
 0000:fff9a000       .debug$S                   0000000180000000     user32:USER32.dll
 0000:fff9a000       .debug$S                   0000000180000000     user32:USER32.dll
 0000:fff9a000       .debug$S                   0000000180000000     user32:USER32.dll
 0000:fff9a000       .debug$S                   0000000180000000     user32:USER32.dll
 0000:fff9a000       .debug$S                   0000000180000000     user32:USER32.dll
 0000:fff9a000       .debug$S                   0000000180000000     user32:USER32.dll
 0000:fff9a000       .debug$S                   0000000180000000     user32:USER32.dll
 0000:fff9a000       .debug$S                   0000000180000000     user32:USER32.dll
 0000:fff9a000       .debug$S                   0000000180000000     user32:USER32.dll
 0000:fff9a000       .debug$S                   0000000180000000     user32:USER32.dll
 0000:fff9a000       .debug$S                   0000000180000000     user32:USER32.dll
 0000:fff9a000       .debug$S                   0000000180000000     user32:USER32.dll
 0000:fff9a000       .debug$S                   0000000180000000     user32:USER32.dll
 0000:fff9a000       .debug$S                   0000000180000000     user32:USER32.dll
 0000:fff9a000       .debug$S                   0000000180000000     user32:USER32.dll
 0000:fff9a000       .debug$S                   0000000180000000     user32:USER32.dll
 0000:fff9a000       .debug$S                   0000000180000000     user32:USER32.dll
 0000:fff9a000       .debug$S                   0000000180000000     user32:USER32.dll
 0000:fff9a000       .debug$S                   0000000180000000     gdi32:GDI32.dll
 0000:fff9a000       .debug$S                   0000000180000000     gdi32:GDI32.dll
 0000:fff9a000       .debug$S                   0000000180000000     gdi32:GDI32.dll
 0000:fff9a000       .debug$S                   0000000180000000     gdi32:GDI32.dll
 0000:fff9a000       .debug$S                   0000000180000000     gdi32:GDI32.dll
 0000:fff9a000       .debug$S                   0000000180000000     gdi32:GDI32.dll
 0000:fff9a000       .debug$S                   0000000180000000     gdi32:GDI32.dll
 0000:fff9a000       .debug$S                   0000000180000000     gdi32:GDI32.dll
 0000:fff9a000       .debug$S                   0000000180000000     gdi32:GDI32.dll
 0000:fff9a000       .debug$S                   0000000180000000     gdi32:GDI32.dll
 0000:fff9a000       .debug$S                   0000000180000000     gdi32:GDI32.dll
 0000:fff9a000       .debug$S                   0000000180000000     gdi32:GDI32.dll
 0000:fff9a000       .debug$S                   0000000180000000     gdi32:GDI32.dll
 0000:fff9a000       .debug$S                   0000000180000000     gdi32:GDI32.dll
 0000:fff9a000       .debug$S                   0000000180000000     gdi32:GDI32.dll
 0000:fff9a000       .debug$S                   0000000180000000     gdi32:GDI32.dll
 0000:fff9a000       .debug$S                   0000000180000000     gdi32:GDI32.dll
 0000:fff9a000       .debug$S                   0000000180000000     gdi32:GDI32.dll
 0000:fff9a000       .debug$S                   0000000180000000     gdi32:GDI32.dll
 0000:fff9a000       .debug$S                   0000000180000000     advapi32:ADVAPI32.dll
 0001:0000013c       ?ChangeExports@@YA_NPEBUExportFunc@@PEAUHINSTANCE__@@@Z 000000018000113c f   ConEmuTh.obj
 0001:00001260       ?LoadFarVersion@@YA_NAEAUFarVersion@@AEAY0CAA@_W@Z 0000000180002260 f   ConEmuTh.obj
 0001:00001370       ?LoadModuleVersion@@YA_NPEB_WAEAUtagVS_FIXEDFILEINFO@@PEA_W_K@Z 0000000180002370 f   ConEmuTh.obj
 0001:00003390       ?GetFarSetting@@YAHPEAX_KPEB_W@Z 0000000180004390 f   ConEmuTh1900.obj
 0001:0000347c       ?LoadFarSettingsW1900@@YAXPEAUCEFarInterfaceSettings@@PEAUCEFarPanelSettings@@@Z 000000018000447c f   ConEmuTh1900.obj
 0001:00004768       ?GetFarSetting@@YAHPEAX_KPEB_W@Z 0000000180005768 f   ConEmuTh2800.obj
 0001:0000485c       ?LoadFarSettingsW2800@@YAXPEAUCEFarInterfaceSettings@@PEAUCEFarPanelSettings@@@Z 000000018000585c f   ConEmuTh2800.obj
 0001:00005e2c       ?LoadFarSettingsW995@@YAXPEAUCEFarInterfaceSettings@@PEAUCEFarPanelSettings@@@Z 0000000180006e2c f   ConEmuTh995.obj
 0001:00006b20       ?LoadFarSettingsA@@YAXPEAUCEFarInterfaceSettings@@PEAUCEFarPanelSettings@@@Z 0000000180007b20 f   ConEmuThA.obj
 0001:0000af00       uninitialize_global_state_isolation 000000018000bf00 f i libucrt:initialization.obj
 0001:0000af00       initialize_global_state_isolation 000000018000bf00 f i libucrt:initialization.obj
 0001:0000af00       initialize_environment     000000018000bf00 f i libucrt:initialization.obj
 0001:0000af00       uninitialize_c             000000018000bf00 f i libucrt:initialization.obj
 0001:0000af00       report_memory_leaks        000000018000bf00 f i libucrt:initialization.obj
 0001:0000e27c       ?compare@cmp@?1??Find@MToolHelpProcess@@QEAA_NKPEAUtagPROCESSENTRY32W@@@Z@SA_N0_J@Z 000000018000f27c f   common-kernel64:MProcess.obj
 0001:00013700       $$000000                   0000000180014700     LIBCMT:_amdsecgs_.obj
 0001:00013760       ?dllmain_crt_dispatch@@YAHQEAUHINSTANCE__@@KQEAX@Z 0000000180014760 f   LIBCMT:dll_dllmain.obj
 0001:000137b0       ?dllmain_crt_process_attach@@YAHQEAUHINSTANCE__@@QEAX@Z 00000001800147b0 f   LIBCMT:dll_dllmain.obj
 0001:000138c8       ?dllmain_crt_process_detach@@YAH_N@Z 00000001800148c8 f   LIBCMT:dll_dllmain.obj
 0001:0001394c       ?dllmain_dispatch@@YAHQEAUHINSTANCE__@@KQEAX@Z 000000018001494c f   LIBCMT:dll_dllmain.obj
 0001:00013c78       capture_current_context    0000000180014c78 f   LIBCMT:gs_report.obj
 0001:00013ce8       capture_previous_context   0000000180014ce8 f   LIBCMT:gs_report.obj
 0001:00014c10       $$000000                   0000000180015c10     libvcruntime:memcmp.obj
 0001:00014cf0       $$000000                   0000000180015cf0     libvcruntime:memcpy.obj
 0001:00014d97       MoveSmall                  0000000180015d97     libvcruntime:memcpy.obj
 0001:00015150       $$000000                   0000000180016150     libvcruntime:memset.obj
 0001:0001524c       MsetTab                    000000018001624c     libvcruntime:memset.obj
 0001:00015790       $$000000                   0000000180016790     libvcruntime:memchr.obj
 0001:00015ca4       ?CatchIt@@YAXPEAUEHExceptionRecord@@PEA_KPEAU_CONTEXT@@PEAU_xDISPATCHER_CONTEXT@@PEBU_s_FuncInfo@@PEBU_s_HandlerType@@PEBU_s_CatchableType@@PEBU_s_TryBlockMapEntry@@H1EE@Z 0000000180016ca4 f   libvcruntime:frame.obj
 0001:00015d68       ?ExFilterRethrow@@YAHPEAU_EXCEPTION_POINTERS@@PEAUEHExceptionRecord@@PEAH@Z 0000000180016d68 f   libvcruntime:frame.obj
 0001:00015df0       ?FindHandler@@YAXPEAUEHExceptionRecord@@PEA_KPEAU_CONTEXT@@PEAU_xDISPATCHER_CONTEXT@@PEBU_s_FuncInfo@@EH1@Z 0000000180016df0 f   libvcruntime:frame.obj
 0001:000162a0       ?FindHandlerForForeignException@@YAXPEAUEHExceptionRecord@@PEA_KPEAU_CONTEXT@@PEAU_xDISPATCHER_CONTEXT@@PEBU_s_FuncInfo@@HH1@Z 00000001800172a0 f   libvcruntime:frame.obj
 0001:000164f8       ?IsInExceptionSpec@@YAEPEAUEHExceptionRecord@@PEBU_s_ESTypeList@@@Z 00000001800174f8 f   libvcruntime:frame.obj
 0001:00016fd0       $$000000                   0000000180017fd0     libvcruntime:_jmpuwind_.obj
 0001:000170fc       ?try_get_function@@YAPEAXW4function_id@?A0x89697e75@@QEBDQEBW4module_id@2@2@Z 00000001800180fc f   libvcruntime:winapi_downlevel.obj
 0001:000174f0       $$000000                   00000001800184f0     libvcruntime:handlers.obj
 0001:0001ab7c       ?atexit_exception_filter@@YAHK@Z 000000018001bb7c f   libucrt:exit.obj
 0001:0001ab88       ?common_exit@@YAXHW4_crt_exit_cleanup_mode@@W4_crt_exit_return_mode@@@Z 000000018001bb88 f   libucrt:exit.obj
 0001:0001acf4       ?exit_or_terminate_process@@YAXI@Z 000000018001bcf4 f   libucrt:exit.obj
 0001:0001ad40       ?try_cor_exit_process@@YAXI@Z 000000018001bd40 f   libucrt:exit.obj
 0001:0001add8       ??$parse_command_line@D@@YAXPEADPEAPEAD0PEA_K2@Z 000000018001bdd8 f   libucrt:argv_parsing.obj
 0001:0001b170       ??$common_initialize_environment_nolock@D@@YAHXZ 000000018001c170 f   libucrt:environment_initialization.obj
 0001:0001b1dc       ??$create_environment@D@@YAQEAPEADQEAD@Z 000000018001c1dc f   libucrt:environment_initialization.obj
 0001:0001b2d8       ??$free_environment@D@@YAXQEAPEAD@Z 000000018001c2d8 f   libucrt:environment_initialization.obj
 0001:0001b2d8       ??$free_environment@_W@@YAXQEAPEA_W@Z 000000018001c2d8 f   libucrt:environment_initialization.obj
 0001:0001b31c       ??$uninitialize_environment_internal@D@@YAXAEAPEAPEAD@Z 000000018001c31c f   libucrt:environment_initialization.obj
 0001:0001b338       ??$uninitialize_environment_internal@_W@@YAXAEAPEAPEA_W@Z 000000018001c338 f   libucrt:environment_initialization.obj
 0001:0001b5b0       initialize_global_variables 000000018001c5b0 f   libucrt:initialization.obj
 0001:0001b5c4       initialize_c               000000018001c5c4 f   libucrt:initialization.obj
 0001:0001b5e8       uninitialize_environment   000000018001c5e8 f   libucrt:initialization.obj
 0001:0001b5f8       initialize_pointers        000000018001c5f8 f   libucrt:initialization.obj
 0001:0001b64c       uninitialize_vcruntime     000000018001c64c f   libucrt:initialization.obj
 0001:0001b654       uninitialize_allocated_memory 000000018001c654 f   libucrt:initialization.obj
 0001:0001b840       $$000000                   000000018001c840     libucrt:strncmp.obj
 0001:0001bbb8       ?internal_isupper_l@@YA_NHQEAU__crt_locale_pointers@@@Z 000000018001cbb8 f   libucrt:tolower_toupper.obj
 0001:0001c648       ?construct_ptd_array@@YAXQEAU__acrt_ptd@@@Z 000000018001d648 f   libucrt:per_thread_data.obj
 0001:0001c718       ?destroy_fls@@YAXPEAX@Z    000000018001d718 f   libucrt:per_thread_data.obj
 0001:0001c738       ?destroy_ptd_array@@YAXQEAU__acrt_ptd@@@Z 000000018001d738 f   libucrt:per_thread_data.obj
 0001:0001c830       ?replace_current_thread_locale_nolock@@YAXQEAU__acrt_ptd@@QEAU__crt_locale_data@@@Z 000000018001d830 f   libucrt:per_thread_data.obj
 0001:0001cb40       ?fp_format_a@@YAHQEBNPEAD_KQEAD2H_NIQEAU__crt_locale_pointers@@@Z 000000018001db40 f   libucrt:cvt.obj
 0001:0001cea0       ?fp_format_e@@YAHQEBNQEAD_K12H_NIQEAU__crt_locale_pointers@@@Z 000000018001dea0 f   libucrt:cvt.obj
 0001:0001cf70       ?fp_format_e_internal@@YAHQEAD_KH_NIQEAU_strflt@@2QEAU__crt_locale_pointers@@@Z 000000018001df70 f   libucrt:cvt.obj
 0001:0001d14c       ?fp_format_f_internal@@YAHQEAD_KHQEAU_strflt@@_NQEAU__crt_locale_pointers@@@Z 000000018001e14c f   libucrt:cvt.obj
 0001:0001d294       ?fp_format_g@@YAHQEBNQEAD_K12H_NIQEAU__crt_locale_pointers@@@Z 000000018001e294 f   libucrt:cvt.obj
 0001:0001d3cc       ?fp_format_nan_or_infinity@@YAHW4__acrt_fp_class@@_NPEAD_K1@Z 000000018001e3cc f   libucrt:cvt.obj
 0001:0001d97c       ?initialize_inherited_file_handles_nolock@@YAXXZ 000000018001e97c f   libucrt:ioinit.obj
 0001:0001da68       ?initialize_stdio_handles_nolock@@YAXXZ 000000018001ea68 f   libucrt:ioinit.obj
 0001:0001de48       ?try_get_function@@YAPEAXW4function_id@?A0x63058377@@QEBDQEBW4module_id@2@2@Z 000000018001ee48 f   libucrt:winapi_thunks.obj
 0001:0001e4a4       ?<helper_func_cdecl>@<lambda_2feae5270eb4d0d5532525f423405775>@@CAHPEBX0@Z 000000018001f4a4 f   libucrt:argv_wildcards.obj
 0001:0001e4b8       ??$common_expand_argv_wildcards@D@@YAHQEAPEADQEAPEAPEAD@Z 000000018001f4b8 f   libucrt:argv_wildcards.obj
 0001:0001e6c4       ??$copy_and_add_argument_to_buffer@D@@YAHQEBD0_KAEAV?$argument_list@D@?A0xca0879c4@@@Z 000000018001f6c4 f   libucrt:argv_wildcards.obj
 0001:0001e7d4       ??$expand_argument_wildcards@D@@YAHQEAD0AEAV?$argument_list@D@?A0xca0879c4@@@Z 000000018001f7d4 f   libucrt:argv_wildcards.obj
 0001:0001ea88       ??R<lambda_ad1ced32f4ac17aa236e5ef05d6b3b7c>@@QEBAXXZ 000000018001fa88 f   libucrt:mbctype.obj
 0001:0001eca0       ?getSystemCP@@YAHH@Z       000000018001fca0 f   libucrt:mbctype.obj
 0001:0001ed20       ?setSBCS@@YAXPEAU__crt_multibyte_data@@@Z 000000018001fd20 f   libucrt:mbctype.obj
 0001:0001edb0       ?setSBUpLow@@YAXPEAU__crt_multibyte_data@@@Z 000000018001fdb0 f   libucrt:mbctype.obj
 0001:0001ef94       ?setmbcp_internal@@YAHH_N@Z 000000018001ff94 f   libucrt:mbctype.obj
 0001:0001f4dc       ?x_ismbbtype_l@@YAHPEAU__crt_locale_pointers@@IHH@Z 00000001800204dc f   libucrt:ismbbyte.obj
 0001:0001fca0       ?__acrt_LCMapStringA_stat@@YAHPEAU__crt_locale_pointers@@PEB_WKPEBDHPEADHHH@Z 0000000180020ca0 f   libucrt:lcmapstringa.obj
 0001:00021dac       memcpy_s                   0000000180022dac f   libucrt:cfout.obj
 0001:00021fb8       common_flush_all           0000000180022fb8 f   libucrt:fflush.obj
 0001:000222b4       ?free_crt_array_internal@@YAXQEAPEBX_K@Z 00000001800232b4 f   libucrt:inittime.obj
 0001:000228e4       ?GetTableIndexFromLocaleName@@YAHPEB_W@Z 00000001800238e4 f   libucrt:lcidtoname_downlevel.obj
 0001:000229e0       ?shortsort@@YAXPEAD0_KP6AHPEBX2@Z@Z 00000001800239e0 f   libucrt:qsort.obj
 0001:00022ff8       ?initialize_multibyte@@YAHXZ 0000000180023ff8 f   libucrt:multibyte_initializer.obj
 0001:00023270       $$000000                   0000000180024270     libucrt:log10.obj
 0001:0002381c       ?write_double_translated_ansi_nolock@@YA?AUwrite_result@?A0x9c548279@@HQEBDI@Z 000000018002481c f   libucrt:write.obj
 0001:00023a24       ?write_text_ansi_nolock@@YA?AUwrite_result@?A0x9c548279@@HQEBDI@Z 0000000180024a24 f   libucrt:write.obj
 0001:00023b2c       ?write_text_utf16le_nolock@@YA?AUwrite_result@?A0x9c548279@@HQEBDI@Z 0000000180024b2c f   libucrt:write.obj
 0001:00023c48       ?write_text_utf8_nolock@@YA?AUwrite_result@?A0x9c548279@@HQEBDI@Z 0000000180024c48 f   libucrt:write.obj
 0001:0002418c       ??$common_lseek_nolock@_J@@YA_JH_JH@Z 000000018002518c f   libucrt:lseek.obj
 0001:00024578       common_control87           0000000180025578 f   libucrt:ieee.obj
 0001:00024810       _call_matherr              0000000180025810 f   libucrt:libm_error.obj
 0001:00024878       _exception_enabled         0000000180025878 f   libucrt:libm_error.obj
 0001:00024b10       _log_special_common        0000000180025b10 f   libucrt:log_special.obj
 0001:00024e20       $$000000                   0000000180025e20     libucrt:fpsr.obj
 0001:00025400       $$000000                   0000000180026400     LIBCMT:_chkstk_.obj
 0001:00025470       $$000000                   0000000180026470     LIBCMT:_guard_dispatch_.obj
 0001:00025490       ?dtor$0@?0??CheckVarsInitialized@@YAXXZ@4HA 0000000180026490 f   ConEmuTh.obj
 0001:000254ad       ?dtor$1@?0??CheckVarsInitialized@@YAXXZ@4HA 00000001800264ad f   ConEmuTh.obj
 0001:000254ad       ?dtor$2@?0??CheckVarsInitialized@@YAXXZ@4HA 00000001800264ad f   ConEmuTh.obj
 0001:000254ca       ?dtor$0@?0??LoadThSet@@YAHK@Z@4HA 00000001800264ca f   ConEmuTh.obj
 0001:000254d6       ?dtor$0@?0??StartPlugin@@YAXH@Z@4HA 00000001800264d6 f   ConEmuTh.obj
 0001:000254f3       ?dtor$0@?0??Paint@CeFullPanelInfo@@QEAAXPEAUHWND__@@AEAUtagPAINTSTRUCT@@AEAUtagRECT@@@Z@4HA 00000001800264f3 f   Display.obj
 0001:000254ff       ?dtor$0@?0??ReallocItems@CeFullPanelInfo@@QEAAH_J@Z@4HA 00000001800264ff f   Display.obj
 0001:0002550b       ?dtor$0@?0???0?$CQueueProcessor@PEAUIMAGE_CACHE_INFO@@@@QEAA@XZ@4HA 000000018002650b f   ImgCache.obj
 0001:00025528       ?dtor$0@?0??FindOrCreate@?$CQueueProcessor@PEAUIMAGE_CACHE_INFO@@@@AEAAPEAUProcessingItem@1@AEBQEAUIMAGE_CACHE_INFO@@_J_NW4ProcessingPriority@@@Z@4HA 0000000180026528 f   ImgCache.obj
 0001:00025534       ?dtor$0@?0??ProcessingStep@?$CQueueProcessor@PEAUIMAGE_CACHE_INFO@@@@IEAA_NXZ@4HA 0000000180026534 f   ImgCache.obj
 0001:00025540       ?dtor$0@?0??RequestItem@CImgCache@@QEAAHPEAUCePluginPanelItem@@I@Z@4HA 0000000180026540 f   ImgCache.obj
 0001:0002555d       ?dtor$0@?0??SearchAppPaths@@YA_NPEB_WAEAUCEStr@@_NPEAU1@@Z@4HA 000000018002655d f   common-user64:WFiles.obj
 0001:00025569       ?fin$0@?0??dllmain_crt_process_attach@@YAHQEAUHINSTANCE__@@QEAX@Z@4HA 0000000180026569 f   LIBCMT:dll_dllmain.obj
 0001:00025580       ?fin$0@?0??dllmain_crt_process_detach@@YAH_N@Z@4HA 0000000180026580 f   LIBCMT:dll_dllmain.obj
 0001:0002559c       ?filt$0@?0??dllmain_dispatch@@YAHQEAUHINSTANCE__@@KQEAX@Z@4HA 000000018002659c f   LIBCMT:dll_dllmain.obj
 0001:000255d2       __scrt_is_nonwritable_in_current_image$filt$0 00000001800265d2 f   LIBCMT:utility.obj
 0001:000255ea       _CallSETranslator$filt$0   00000001800265ea f   libvcruntime:risctrnsctrl.obj
 0001:0002567b       __CxxCallCatchBlock$filt$0 000000018002667b f   libvcruntime:frame.obj
 0001:000256a0       __CxxCallCatchBlock$fin$1  00000001800266a0 f   libvcruntime:frame.obj
 0001:00025718       __FrameUnwindToState$filt$0 0000000180026718 f   libvcruntime:frame.obj
 0001:0002572e       __FrameUnwindToState$fin$1 000000018002672e f   libvcruntime:frame.obj
 0001:00025751       __DestructExceptionObject$filt$0 0000000180026751 f   libvcruntime:ehhelpers.obj
 0001:00025769       ?filt$0@?0??common_exit@@YAXHW4_crt_exit_cleanup_mode@@W4_crt_exit_return_mode@@@Z@4HA 0000000180026769 f   libucrt:exit.obj
 0001:00025784       ?fin$1@?0??common_exit@@YAXHW4_crt_exit_cleanup_mode@@W4_crt_exit_return_mode@@@Z@4HA 0000000180026784 f   libucrt:exit.obj
 0001:0002579d       ?fin$0@?0???$?RV<lambda_e24bbb7b643b32fcea6fa61b31d4c984>@@AEAV<lambda_275893d493268fdec8709772e3fcec0e>@@V<lambda_9d71df4d7cf3f480f8d633942495c3b0>@@@?$__crt_seh_guarded_call@H@@QEAAH$$QEAV<lambda_e24bbb7b643b32fcea6fa61b31d4c984>@@AEAV<lambda_275893d493268fdec8709772e3fcec0e>@@$$QEAV<lambda_9d71df4d7cf3f480f8d633942495c3b0>@@@Z@4HA 000000018002679d f   libucrt:onexit.obj
 0001:000257ba       ?fin$0@?0???$?RV<lambda_5e887d1dcbef67a5eb4283622ba103bf>@@AEAV<lambda_4466841279450cc726390878d4a41900>@@V<lambda_341c25c0346d94847f1f3c463c57e077>@@@?$__crt_seh_guarded_call@X@@QEAAX$$QEAV<lambda_5e887d1dcbef67a5eb4283622ba103bf>@@AEAV<lambda_4466841279450cc726390878d4a41900>@@$$QEAV<lambda_341c25c0346d94847f1f3c463c57e077>@@@Z@4HA 00000001800267ba f   libucrt:per_thread_data.obj
 0001:000257ba       ?fin$0@?0???$?RV<lambda_c36588078e9f5dfd39652860aa6b3aaf>@@AEAV<lambda_ec61778202f4f5fc7e7711acc23c3bca>@@V<lambda_dc9d2797ccde5d239b4a0efae8ebd7db>@@@?$__crt_seh_guarded_call@P6AXH@Z@@QEAAP6AXH@Z$$QEAV<lambda_c36588078e9f5dfd39652860aa6b3aaf>@@AEAV<lambda_ec61778202f4f5fc7e7711acc23c3bca>@@$$QEAV<lambda_dc9d2797ccde5d239b4a0efae8ebd7db>@@@Z@4HA 00000001800267ba f   libucrt:signal.obj
 0001:000257ba       ?fin$0@?0???$?RV<lambda_46352004c1216016012b18bd6f87e700>@@AEAV<lambda_3bd07e1a1191394380780325891bf33f>@@V<lambda_334532d3f185bcaa59b5be82d7d22bff>@@@?$__crt_seh_guarded_call@X@@QEAAX$$QEAV<lambda_46352004c1216016012b18bd6f87e700>@@AEAV<lambda_3bd07e1a1191394380780325891bf33f>@@$$QEAV<lambda_334532d3f185bcaa59b5be82d7d22bff>@@@Z@4HA 00000001800267ba f   libucrt:per_thread_data.obj
 0001:000257ba       ?fin$0@?0???$?RV<lambda_99476a1ad63dd22509b5d3e65b0ffc95>@@AEAV<lambda_ad1ced32f4ac17aa236e5ef05d6b3b7c>@@V<lambda_f7424dd8d45958661754dc4f2697e9c3>@@@?$__crt_seh_guarded_call@X@@QEAAX$$QEAV<lambda_99476a1ad63dd22509b5d3e65b0ffc95>@@AEAV<lambda_ad1ced32f4ac17aa236e5ef05d6b3b7c>@@$$QEAV<lambda_f7424dd8d45958661754dc4f2697e9c3>@@@Z@4HA 00000001800267ba f   libucrt:mbctype.obj
 0001:000257ba       ?fin$0@?0???$?RV<lambda_72d1df2b273a38828b1ce30cbf4cdab5>@@AEAV<lambda_876a65b173b8412d3a47c70a915b0cf4>@@V<lambda_41932305e351933ebe8f8be3ed8bb5dc>@@@?$__crt_seh_guarded_call@X@@QEAAX$$QEAV<lambda_72d1df2b273a38828b1ce30cbf4cdab5>@@AEAV<lambda_876a65b173b8412d3a47c70a915b0cf4>@@$$QEAV<lambda_41932305e351933ebe8f8be3ed8bb5dc>@@@Z@4HA 00000001800267ba f   libucrt:per_thread_data.obj
 0001:000257ba       ?fin$0@?0???$?RV<lambda_fb3a7dec4e47f37f22dae91bb15c9095>@@AEAV<lambda_698284760c8add0bfb0756c19673e34b>@@V<lambda_dfb8eca1e75fef3034a8fb18dd509707>@@@?$__crt_seh_guarded_call@X@@QEAAX$$QEAV<lambda_fb3a7dec4e47f37f22dae91bb15c9095>@@AEAV<lambda_698284760c8add0bfb0756c19673e34b>@@$$QEAV<lambda_dfb8eca1e75fef3034a8fb18dd509707>@@@Z@4HA 00000001800267ba f   libucrt:per_thread_data.obj
 0001:000257d4       __acrt_uninitialize_locale$fin$0 00000001800267d4 f   libucrt:wsetlocale.obj
 0001:000257d4       __acrt_update_thread_locale_data$fin$0 00000001800267d4 f   libucrt:locale_refcounting.obj
 0001:000257ed       __acrt_initialize_lowio$fin$0 00000001800267ed f   libucrt:ioinit.obj
 0001:000257ed       __acrt_lowio_ensure_fh_exists$fin$0 00000001800267ed f   libucrt:osfinfo.obj
 0001:00025806       __acrt_update_thread_multibyte_data$fin$0 0000000180026806 f   libucrt:mbctype.obj
 0001:0002581f       _query_new_handler$fin$0   000000018002681f f   libucrt:new_handler.obj
 0001:00025835       raise$fin$0                0000000180026835 f   libucrt:signal.obj
 0001:00025859       _fcloseall$fin$0           0000000180026859 f   libucrt:closeall.obj
 0001:00025872       common_flush_all$fin$0     0000000180026872 f   libucrt:fflush.obj
 0001:0002588c       common_flush_all$fin$1     000000018002688c f   libucrt:fflush.obj
 0001:000258a5       _write$fin$0               00000001800268a5 f   libucrt:write.obj
 0001:000258bc       fclose$fin$0               00000001800268bc f   libucrt:fclose.obj
 0001:000258d4       ?fin$0@?0???$?RV<lambda_b521505b218e5242e90febf6bfebc422>@@AEAV<lambda_6978c1fb23f02e42e1d9e99668cc68aa>@@V<lambda_314360699dd331753a4119843814e9a7>@@@?$__crt_seh_guarded_call@H@@QEAAH$$QEAV<lambda_b521505b218e5242e90febf6bfebc422>@@AEAV<lambda_6978c1fb23f02e42e1d9e99668cc68aa>@@$$QEAV<lambda_314360699dd331753a4119843814e9a7>@@@Z@4HA 00000001800268d4 f   libucrt:commit.obj
 0001:000258d4       ?fin$0@?0???$?RV<lambda_bfedae4ebbf01fab1bb6dcc6a9e276e0>@@AEAV<lambda_2fe9b910cf3cbf4a0ab98a02ba45b3ec>@@V<lambda_237c231691f317818eb88cc1d5d642d6>@@@?$__crt_seh_guarded_call@H@@QEAAH$$QEAV<lambda_bfedae4ebbf01fab1bb6dcc6a9e276e0>@@AEAV<lambda_2fe9b910cf3cbf4a0ab98a02ba45b3ec>@@$$QEAV<lambda_237c231691f317818eb88cc1d5d642d6>@@@Z@4HA 00000001800268d4 f   libucrt:close.obj
 0001:000258ee       _ctrlfp$filt$0             00000001800268ee f   libucrt:fpctrl.obj
 0001:000258ee       common_control87$filt$0    00000001800268ee f   libucrt:ieee.obj
 0001:00025920       _IsNonwritableInCurrentImage$filt$0 0000000180026920 f   LIBCMT:pesect.obj
 0002:00000708       $cppxdata$?LoadThSet@@YAHK@Z 0000000180027708     ConEmuTh.obj
 0002:00000730       $cppxdata$?StartPlugin@@YAXH@Z 0000000180027730     ConEmuTh.obj
 0002:00000758       $cppxdata$?CheckVarsInitialized@@YAXXZ 0000000180027758     ConEmuTh.obj
 0002:000010d0       ?gsDisplayClassName@@3QB_WB 00000001800280d0     Display.obj
 0002:000010f0       $cppxdata$?ReallocItems@CeFullPanelInfo@@QEAAH_J@Z 00000001800280f0     Display.obj
 0002:00001118       $cppxdata$?Paint@CeFullPanelInfo@@QEAAXPEAUHWND__@@AEAUtagPAINTSTRUCT@@AEAUtagRECT@@@Z 0000000180028118     Display.obj
 0002:00001308       $cppxdata$??1CImgCache@@QEAA@XZ 0000000180028308     ImgCache.obj
 0002:00001330       $cppxdata$?RequestItem@CImgCache@@QEAAHPEAUCePluginPanelItem@@I@Z 0000000180028330     ImgCache.obj
 0002:00001358       $cppxdata$?FindOrCreate@?$CQueueProcessor@PEAUIMAGE_CACHE_INFO@@@@AEAAPEAUProcessingItem@1@AEBQEAUIMAGE_CACHE_INFO@@_J_NW4ProcessingPriority@@@Z 0000000180028358     ImgCache.obj
 0002:00001380       $cppxdata$??0?$CQueueProcessor@PEAUIMAGE_CACHE_INFO@@@@QEAA@XZ 0000000180028380     ImgCache.obj
 0002:000013a8       $cppxdata$??1?$CQueueProcessor@PEAUIMAGE_CACHE_INFO@@@@UEAA@XZ 00000001800283a8     ImgCache.obj
 0002:000013d0       $cppxdata$?ProcessingStep@?$CQueueProcessor@PEAUIMAGE_CACHE_INFO@@@@IEAA_NXZ 00000001800283d0     ImgCache.obj
 0002:00001d90       $cppxdata$??1CRgnDetect@@QEAA@XZ 0000000180028d90     common-user64:RgnDetect.obj
 0002:00001dd8       $cppxdata$?SearchAppPaths@@YA_NPEB_WAEAUCEStr@@_NPEAU1@@Z 0000000180028dd8     common-user64:WFiles.obj
 0002:00001e88       GS_ExceptionPointers       0000000180028e88     LIBCMT:gs_report.obj
 0002:00001ea0       ?ExceptionTemplate@?1??_UnwindNestedFrames@@9@4U_EXCEPTION_RECORD@@B 0000000180028ea0     libvcruntime:risctrnsctrl.obj
 0002:00001f90       ?tokenTable@@3QBQEBDB      0000000180028f90     libvcruntime:undname.obj
 0002:00002008       ?rttiTable@@3QBQEBDB       0000000180029008     libvcruntime:undname.obj
 0002:00002030       ?nameTable@@3QBQEBDB       0000000180029030     libvcruntime:undname.obj
 0002:00002938       ?module_names@?A0x89697e75@@3QBQEB_WB 0000000180029938     libvcruntime:winapi_downlevel.obj
 0002:00002a08       ?candidate_modules@?1??try_get_FlsAlloc@@YAP6AKP6AXPEAX@Z@ZXZ@4QBW4module_id@?A0x89697e75@@B 0000000180029a08     libvcruntime:winapi_downlevel.obj
 0002:00002a20       ?candidate_modules@?1??try_get_FlsFree@@YAP6AHK@ZXZ@4QBW4module_id@?A0x89697e75@@B 0000000180029a20     libvcruntime:winapi_downlevel.obj
 0002:00002a30       ?candidate_modules@?1??try_get_FlsGetValue@@YAP6APEAXK@ZXZ@4QBW4module_id@?A0x89697e75@@B 0000000180029a30     libvcruntime:winapi_downlevel.obj
 0002:00002a48       ?candidate_modules@?1??try_get_FlsSetValue@@YAP6AHKPEAX@ZXZ@4QBW4module_id@?A0x89697e75@@B 0000000180029a48     libvcruntime:winapi_downlevel.obj
 0002:00002a60       ?candidate_modules@?1??try_get_InitializeCriticalSectionEx@@YAP6AHPEAU_RTL_CRITICAL_SECTION@@KK@ZXZ@4QBW4module_id@?A0x89697e75@@B 0000000180029a60     libvcruntime:winapi_downlevel.obj
 0002:00002a90       ?ExceptionTemplate@?1??_CxxThrowException@@9@4UEHExceptionRecord@@B 0000000180029a90     libvcruntime:throw.obj
 0002:00002c50       __acrt_initializers        0000000180029c50     libucrt:initialization.obj
 0002:00002d40       errtable                   0000000180029d40     libucrt:errno.obj
 0002:00003d90       module_names               000000018002ad90     libucrt:winapi_thunks.obj
 0002:000042d8       ?candidate_modules@?1??try_get_FlsAlloc@@YAP6AKP6AXPEAX@Z@ZXZ@4QBW4module_id@?A0x63058377@@B 000000018002b2d8     libucrt:winapi_thunks.obj
 0002:000042e0       ?candidate_modules@?1??try_get_FlsFree@@YAP6AHK@ZXZ@4QBW4module_id@?A0x63058377@@B 000000018002b2e0     libucrt:winapi_thunks.obj
 0002:000042e8       ?candidate_modules@?1??try_get_FlsGetValue@@YAP6APEAXK@ZXZ@4QBW4module_id@?A0x63058377@@B 000000018002b2e8     libucrt:winapi_thunks.obj
 0002:000042f0       ?candidate_modules@?1??try_get_FlsSetValue@@YAP6AHKPEAX@ZXZ@4QBW4module_id@?A0x63058377@@B 000000018002b2f0     libucrt:winapi_thunks.obj
 0002:000042f8       ?candidate_modules@?1??try_get_GetCurrentPackageId@@YAP6AJPEAIPEAE@ZXZ@4QBW4module_id@?A0x63058377@@B 000000018002b2f8     libucrt:winapi_thunks.obj
 0002:00004318       ?candidate_modules@?1??try_get_InitializeCriticalSectionEx@@YAP6AHPEAU_RTL_CRITICAL_SECTION@@KK@ZXZ@4QBW4module_id@?A0x63058377@@B 000000018002b318     libucrt:winapi_thunks.obj
 0002:00004320       ?candidate_modules@?1??try_get_LCMapStringEx@@YAP6AHPEB_WK0HPEA_WHPEAU_nlsversioninfo@@PEAX_J@ZXZ@4QBW4module_id@?A0x63058377@@B 000000018002b320     libucrt:winapi_thunks.obj
 0002:00004338       ?candidate_modules@?1??try_get_LocaleNameToLCID@@YAP6AKPEB_WK@ZXZ@4QBW4module_id@?A0x63058377@@B 000000018002b338     libucrt:winapi_thunks.obj
 0002:00004358       _mb_locale_names           000000018002b358     libucrt:mbctype.obj
 0002:00004dc0       LcidToLocaleNameTable      000000018002bdc0     libucrt:lcidtoname_downlevel.obj
 0002:00006810       LocaleNameToIndexTable     000000018002d810     libucrt:lcidtoname_downlevel.obj
 0002:000080b0       __real_ninf                000000018002f0b0     libucrt:log10.obj
 0002:000080c0       __real_inf                 000000018002f0c0     libucrt:log10.obj
 0002:000080d0       __real_neg_qnan            000000018002f0d0     libucrt:log10.obj
 0002:000080e0       __real_qnanbit             000000018002f0e0     libucrt:log10.obj
 0002:000080f0       __int_1023                 000000018002f0f0     libucrt:log10.obj
 0002:00008100       __mask_001                 000000018002f100     libucrt:log10.obj
 0002:00008110       __mask_mant                000000018002f110     libucrt:log10.obj
 0002:00008120       __mask_mant_top8           000000018002f120     libucrt:log10.obj
 0002:00008130       __mask_mant9               000000018002f130     libucrt:log10.obj
 0002:00008140       __real_log10_e             000000018002f140     libucrt:log10.obj
 0002:00008150       __real_log10_e_lead        000000018002f150     libucrt:log10.obj
 0002:00008160       __real_log10_e_tail        000000018002f160     libucrt:log10.obj
 0002:00008170       __real_log10_2_lead        000000018002f170     libucrt:log10.obj
 0002:00008180       __real_log10_2_tail        000000018002f180     libucrt:log10.obj
 0002:00008190       __real_two                 000000018002f190     libucrt:log10.obj
 0002:000081a0       __real_one                 000000018002f1a0     libucrt:log10.obj
 0002:000081b0       __real_half                000000018002f1b0     libucrt:log10.obj
 0002:000081c0       __mask_100                 000000018002f1c0     libucrt:log10.obj
 0002:000081d0       __real_1_over_512          000000018002f1d0     libucrt:log10.obj
 0002:000081e0       __real_1_over_2            000000018002f1e0     libucrt:log10.obj
 0002:000081f0       __real_1_over_3            000000018002f1f0     libucrt:log10.obj
 0002:00008200       __real_1_over_4            000000018002f200     libucrt:log10.obj
 0002:00008210       __real_1_over_5            000000018002f210     libucrt:log10.obj
 0002:00008220       __real_1_over_6            000000018002f220     libucrt:log10.obj
 0002:00008230       __real_neg_1023            000000018002f230     libucrt:log10.obj
 0002:00008240       __mask_2045                000000018002f240     libucrt:log10.obj
 0002:00008250       __real_threshold           000000018002f250     libucrt:log10.obj
 0002:00008260       __real_near_one_lt         000000018002f260     libucrt:log10.obj
 0002:00008270       __real_near_one_gt         000000018002f270     libucrt:log10.obj
 0002:00008280       __real_min_norm            000000018002f280     libucrt:log10.obj
 0002:00008290       __real_notsign             000000018002f290     libucrt:log10.obj
 0002:000082a0       __real_ca1                 000000018002f2a0     libucrt:log10.obj
 0002:000082b0       __real_ca2                 000000018002f2b0     libucrt:log10.obj
 0002:000082c0       __real_ca3                 000000018002f2c0     libucrt:log10.obj
 0002:000082d0       __real_ca4                 000000018002f2d0     libucrt:log10.obj
 0002:000082e0       __mask_lower               000000018002f2e0     libucrt:log10.obj
 0002:000082f0       __flag_x_zero              000000018002f2f0     libucrt:log10.obj
 0002:000082f4       __flag_x_neg               000000018002f2f4     libucrt:log10.obj
 0002:000082f8       __flag_x_nan               000000018002f2f8     libucrt:log10.obj
 0002:00009b40       __real@433fffffffffffff    0000000180030b40     libucrt:fpsr.obj
 0002:00009b48       __real@c33fffffffffffff    0000000180030b48     libucrt:fpsr.obj
 0002:0000a368       $unwind$?GetIndexFromWndCoord@CeFullPanelInfo@@QEAAHHHAEA_J@Z 0000000180031368     Display.obj
 0002:0000a368       $unwind$?StringCchCatW@@YAJPEA_W_KPEB_W@Z 0000000180031368     ConEmuTh.obj
 0002:0000a368       $unwind$?FindFrameLeft_ByBottom@CRgnDetect@@IEAA_NPEA_WPEAUtag_CharAttr@@HHAEAH22@Z 0000000180031368     common-user64:RgnDetect.obj
 0002:0000a368       $unwind$?CalcTopPanelItem@CeFullPanelInfo@@QEAA_J_J0@Z 0000000180031368     Display.obj
 0002:0000a368       $unwind$??$type_case_integer_parse_into_buffer@I@?$output_processor@_WV?$string_output_adapter@_W@__crt_stdio_output@@V?$standard_base@_WV?$string_output_adapter@_W@__crt_stdio_output@@@2@@__crt_stdio_output@@AEAAXII_N@Z 0000000180031368     libucrt:output.obj
 0002:0000a368       $unwind$?FindFrameTop_ByLeft@CRgnDetect@@IEAA_NPEA_WPEAUtag_CharAttr@@HHAEAH22@Z 0000000180031368     common-user64:RgnDetect.obj
 0002:0000a368       $unwind$?FindFrameTop_ByRight@CRgnDetect@@IEAA_NPEA_WPEAUtag_CharAttr@@HHAEAH22@Z 0000000180031368     common-user64:RgnDetect.obj
 0002:0000a368       $unwind$??$type_case_integer_parse_into_buffer@_K@?$output_processor@_WV?$string_output_adapter@_W@__crt_stdio_output@@V?$standard_base@_WV?$string_output_adapter@_W@__crt_stdio_output@@@2@@__crt_stdio_output@@AEAAX_KI_N@Z 0000000180031368     libucrt:output.obj
 0002:0000a368       $unwind$??$type_case_integer_parse_into_buffer@I@?$output_processor@DV?$string_output_adapter@D@__crt_stdio_output@@V?$standard_base@DV?$string_output_adapter@D@__crt_stdio_output@@@2@@__crt_stdio_output@@AEAAXII_N@Z 0000000180031368     libucrt:output.obj
 0002:0000a368       $unwind$??$type_case_integer_parse_into_buffer@_K@?$output_processor@DV?$string_output_adapter@D@__crt_stdio_output@@V?$standard_base@DV?$string_output_adapter@D@__crt_stdio_output@@@2@@__crt_stdio_output@@AEAAX_KI_N@Z 0000000180031368     libucrt:output.obj
 0002:0000a368       $unwind$?Color2FgIndex@Far3Color@@SAXKAEAGPEBK@Z 0000000180031368     ConEmuTh1900.obj
 0002:0000a368       $unwind$??$write_multiple_characters@V?$string_output_adapter@D@__crt_stdio_output@@D@__crt_stdio_output@@YAXAEBV?$string_output_adapter@D@0@DHQEAH@Z 0000000180031368     libucrt:output.obj
 0002:0000a368       $unwind$?StringCchCopyW@@YAJPEA_W_KPEB_W@Z 0000000180031368     ConEmuTh.obj
 0002:0000a368       $unwind$?StringCchCopyNW@@YAJPEA_W_KPEB_W1@Z 0000000180031368     common-kernel64:WObjects.obj
 0002:0000a370       $unwind$??$create_environment@D@@YAQEAPEADQEAD@Z 0000000180031370     libucrt:environment_initialization.obj
 0002:0000a370       $unwind$?StringCchVPrintfW@@YAJPEA_W_KPEB_WPEAD@Z 0000000180031370     ConEmuTh.obj
 0002:0000a388       $unwind$?dllmain_crt_dispatch@@YAHQEAUHINSTANCE__@@KQEAX@Z 0000000180031388     LIBCMT:dll_dllmain.obj
 0002:0000a388       $unwind$?ReloadPanelsInfoW995@@YAXXZ 0000000180031388     ConEmuTh995.obj
 0002:0000a388       $unwind$?state_case_size@?$output_processor@_WV?$string_output_adapter@_W@__crt_stdio_output@@V?$standard_base@_WV?$string_output_adapter@_W@__crt_stdio_output@@@2@@__crt_stdio_output@@AEAA_NXZ 0000000180031388     libucrt:output.obj
 0002:0000a388       $unwind$?CopyItem@?$CQueueProcessor@PEAUIMAGE_CACHE_INFO@@@@MEAAXPEBQEAUIMAGE_CACHE_INFO@@PEAPEAU2@@Z 0000000180031388     ImgCache.obj
 0002:0000a388       $unwind$_msize             0000000180031388     libucrt:msize.obj
 0002:0000a388       $unwind$__acrt_uninitialize_ptd 0000000180031388     libucrt:per_thread_data.obj
 0002:0000a388       $unwind$?ExecuteInMainThreadW2800@@YAXPEAUConEmuThSynchroArg@@@Z 0000000180031388     ConEmuTh2800.obj
 0002:0000a388       $unwind$?PointToExt@@YAPEB_WPEB_W@Z 0000000180031388     common-kernel64:CmdLine.obj
 0002:0000a388       $unwind$__report_rangecheckfailure 0000000180031388     LIBCMT:gs_report.obj
 0002:0000a388       $unwind$?OnThreadStarted@CImgLoader@@UEAAJXZ 0000000180031388     ImgCache.obj
 0002:0000a388       $unwind$?ExecuteInMainThreadW1900@@YAXPEAUConEmuThSynchroArg@@@Z 0000000180031388     ConEmuTh1900.obj
 0002:0000a388       $unwind$_invoke_watson     0000000180031388     libucrt:invalid_parameter.obj
 0002:0000a388       $unwind$__scrt_initialize_default_local_stdio_options 0000000180031388     LIBCMT:default_local_stdio_options.obj
 0002:0000a388       $unwind$??1MSectionLockSimple@@QEAA@XZ 0000000180031388     common-kernel64:MSectionSimple.obj
 0002:0000a388       $unwind$__scrt_acquire_startup_lock 0000000180031388     LIBCMT:utility.obj
 0002:0000a388       $unwind$?ExitFARW1900@@YAXXZ 0000000180031388     ConEmuTh1900.obj
 0002:0000a388       $unwind$__acrt_initialize_command_line 0000000180031388     libucrt:argv_data.obj
 0002:0000a388       $unwind$?ExecuteInMainThreadW995@@YAXPEAUConEmuThSynchroArg@@@Z 0000000180031388     ConEmuTh995.obj
 0002:0000a388       $unwind$__acrt_DownlevelLocaleNameToLCID 0000000180031388     libucrt:lcidtoname_downlevel.obj
 0002:0000a388       $unwind$abort              0000000180031388     libucrt:abort.obj
 0002:0000a388       $unwind$__FrameUnwindFilter 0000000180031388     libvcruntime:ehhelpers.obj
 0002:0000a388       $unwind$?ProcessSynchroEventW3@@YA_JPEAX@Z 0000000180031388     ConEmuTh2800.obj
 0002:0000a388       $unwind$?initialize_multibyte@@YAHXZ 0000000180031388     libucrt:multibyte_initializer.obj
 0002:0000a388       $unwind$?ReloadPanelsInfoW2800@@YAXXZ 0000000180031388     ConEmuTh2800.obj
 0002:0000a388       $unwind$__dcrt_terminate_console_output 0000000180031388     libucrt:initcon.obj
 0002:0000a388       $unwind$__acrt_initialize_heap 0000000180031388     libucrt:heap_handle.obj
 0002:0000a388       $unwind$uninitialize_environment 0000000180031388     libucrt:initialization.obj
 0002:0000a388       $unwind$__acrt_initialize_ptd 0000000180031388     libucrt:per_thread_data.obj
 0002:0000a388       $unwind$__GSHandlerCheck   0000000180031388     LIBCMT:_gshandler_.obj
 0002:0000a388       $unwind$__scrt_dllmain_before_initialize_c 0000000180031388     LIBCMT:utility.obj
 0002:0000a388       $unwind$_errno             0000000180031388     libucrt:errno.obj
 0002:0000a388       $unwind$initialize_c       0000000180031388     libucrt:initialization.obj
 0002:0000a388       $unwind$_statfp            0000000180031388     libucrt:fpctrl.obj
 0002:0000a388       $unwind$ExitFAR            0000000180031388     ConEmuThA.obj
 0002:0000a388       $unwind$?ExitFARW995@@YAXXZ 0000000180031388     ConEmuTh995.obj
 0002:0000a388       $unwind$__scrt_dllmain_after_initialize_c 0000000180031388     LIBCMT:utility.obj
 0002:0000a388       $unwind$?ReloadPanelsInfoW1900@@YAXXZ 0000000180031388     ConEmuTh1900.obj
 0002:0000a388       $unwind$__acrt_thread_detach 0000000180031388     libucrt:initialization.obj
 0002:0000a388       $unwind$GetMinFarVersion   0000000180031388     ConEmuThA.obj
 0002:0000a388       $unwind$_set_errno_from_matherr 0000000180031388     libucrt:fpexcept.obj
 0002:0000a388       $unwind$?state_case_normal_tchar@?$output_processor@DV?$string_output_adapter@D@__crt_stdio_output@@V?$standard_base@DV?$string_output_adapter@D@__crt_stdio_output@@@2@@__crt_stdio_output@@AEAA_ND@Z 0000000180031388     libucrt:output.obj
 0002:0000a388       $unwind$__scrt_dllmain_uninitialize_c 0000000180031388     LIBCMT:utility.obj
 0002:0000a388       $unwind$__acrt_thread_attach 0000000180031388     libucrt:initialization.obj
 0002:0000a388       $unwind$?state_case_size@?$output_processor@DV?$string_output_adapter@D@__crt_stdio_output@@V?$standard_base@DV?$string_output_adapter@D@__crt_stdio_output@@@2@@__crt_stdio_output@@AEAA_NXZ 0000000180031388     libucrt:output.obj
 0002:0000a388       $unwind$__scrt_dllmain_uninitialize_critical 0000000180031388     LIBCMT:utility.obj
 0002:0000a388       $unwind$__acrt_uninitialize_critical 0000000180031388     libucrt:initialization.obj
 0002:0000a388       $unwind$_isatty            0000000180031388     libucrt:isatty.obj
 0002:0000a388       $unwind$__scrt_dllmain_crt_thread_attach 0000000180031388     LIBCMT:utility.obj
 0002:0000a388       $unwind$?UpdateEnvVar@@YAXH@Z 0000000180031388     ConEmuTh.obj
 0002:0000a388       $unwind$__scrt_dllmain_crt_thread_detach 0000000180031388     LIBCMT:utility.obj
 0002:0000a388       $unwind$?ExecuteFreeResult@@YAXAEAPEAUCESERVER_REQ@@@Z 0000000180031388     common-kernel64:ConEmuCheck.obj
 0002:0000a388       $unwind$?__GetCurrentState@@YAHPEA_KPEAU_xDISPATCHER_CONTEXT@@PEBU_s_FuncInfo@@@Z 0000000180031388     libvcruntime:riscehstate.obj
 0002:0000a388       $unwind$__vcrt_freefls     0000000180031388     libvcruntime:per_thread_data.obj
 0002:0000a388       $unwind$_get_osfhandle     0000000180031388     libucrt:osfinfo.obj
 0002:0000a388       $unwind$?ExitFARW2800@@YAXXZ 0000000180031388     ConEmuTh2800.obj
 0002:0000a388       $unwind$__acrt_release_locale_ref 0000000180031388     libucrt:locale_refcounting.obj
 0002:0000a388       $unwind$__acrt_initialize_multibyte 0000000180031388     libucrt:mbctype.obj
 0002:0000a388       $unwind$__vcrt_getptd      0000000180031388     libvcruntime:per_thread_data.obj
 0002:0000a388       $unwind$?ShutdownSecurity@@YAXXZ 0000000180031388     common-kernel64:MSecurity.obj
 0002:0000a388       $unwind$__vcrt_uninitialize_ptd 0000000180031388     libvcruntime:per_thread_data.obj
 0002:0000a388       $unwind$?LocalSecurity@@YAPEAU_SECURITY_ATTRIBUTES@@XZ 0000000180031388     common-kernel64:MSecurity.obj
 0002:0000a388       $unwind$?ExitFARW3@@YAXPEAX@Z 0000000180031388     ConEmuTh.obj
 0002:0000a388       $unwind$_GetImageBase      0000000180031388     libvcruntime:risctrnsctrl.obj
 0002:0000a388       $unwind$__vcrt_initialize_ptd 0000000180031388     libvcruntime:per_thread_data.obj
 0002:0000a388       $unwind$?apiShowWindow@@YA_NPEAUHWND__@@H@Z 0000000180031388     common-user64:WUser.obj
 0002:0000a388       $unwind$?xf_free@@YAXPEAX@Z 0000000180031388     common-kernel64:Memory.obj
 0002:0000a388       $unwind$?HeapDeinitialize@@YAXXZ 0000000180031388     common-kernel64:Memory.obj
 0002:0000a388       $unwind$ExitFARW           0000000180031388     ConEmuTh.obj
 0002:0000a388       $unwind$__pctype_func      0000000180031388     libucrt:ctype.obj
 0002:0000a388       $unwind$DllMain            0000000180031388     ConEmuTh.obj
 0002:0000a388       $unwind$__vcrt_thread_detach 0000000180031388     libvcruntime:initialization.obj
 0002:0000a388       $unwind$_getfpstatusword   0000000180031388     libucrt:_fenvutils.obj
 0002:0000a388       $unwind$_getfpcontrolword  0000000180031388     libucrt:_fenvutils.obj
 0002:0000a388       $unwind$?OpenW@@YAPEAXPEBUOpenInfo@@@Z 0000000180031388     ConEmuTh.obj
 0002:0000a388       $unwind$__vcrt_thread_attach 0000000180031388     libvcruntime:initialization.obj
 0002:0000a388       $unwind$?HeapInitialize@@YA_NXZ 0000000180031388     common-kernel64:Memory.obj
 0002:0000a388       $unwind$__vcrt_uninitialize_critical 0000000180031388     libvcruntime:initialization.obj
 0002:0000a388       $unwind$__vcrt_uninitialize 0000000180031388     libvcruntime:initialization.obj
 0002:0000a388       $unwind$__vcrt_initialize  0000000180031388     libvcruntime:initialization.obj
 0002:0000a388       $unwind$??_V@YAXPEAX@Z     0000000180031388     common-kernel64:Memory.obj
 0002:0000a388       $unwind$__doserrno         0000000180031388     libucrt:errno.obj
 0002:0000a388       $unwind$?ReloadPanelsInfoA@@YAXXZ 0000000180031388     ConEmuThA.obj
 0002:0000a388       $unwind$??$uninitialize_environment_internal@D@@YAXAEAPEAPEAD@Z 0000000180031388     libucrt:environment_initialization.obj
 0002:0000a388       $unwind$??$uninitialize_environment_internal@_W@@YAXAEAPEAPEA_W@Z 0000000180031388     libucrt:environment_initialization.obj
 0002:0000a388       $unwind$??3@YAXPEAX@Z      0000000180031388     common-kernel64:Memory.obj
 0002:0000a388       $unwind$??2@YAPEAX_K@Z     0000000180031388     common-kernel64:Memory.obj
 0002:0000a388       $unwind$tolower            0000000180031388     libucrt:tolower_toupper.obj
 0002:0000a388       $unwind$?InvalidateAll@CeFullPanelInfo@@SAXXZ 0000000180031388     Display.obj
 0002:0000a388       $unwind$_GetThrowImageBase 0000000180031388     libvcruntime:risctrnsctrl.obj
 0002:0000a388       $unwind$_fileno            0000000180031388     libucrt:fileno.obj
 0002:0000a388       $unwind$__dcrt_uninitialize_environments_nolock 0000000180031388     libucrt:environment_initialization.obj
 0002:0000a390       $unwind$??1MSectionLock@@QEAA@XZ 0000000180031390     common-kernel64:MSection.obj
 0002:0000a390       $unwind$_SetThrowImageBase 0000000180031390     libvcruntime:risctrnsctrl.obj
 0002:0000a390       $unwind$__acrt_uninitialize_stdio 0000000180031390     libucrt:_file.obj
 0002:0000a390       $unwind$?OnPostReadConsole@@YAHPEAXPEAU_INPUT_RECORD@@KPEAKPEAH@Z 0000000180031390     ConEmuTh.obj
 0002:0000a390       $unwind$SetStartupInfoW    0000000180031390     ConEmuTh.obj
 0002:0000a390       $unwind$_CreateFrameInfo   0000000180031390     libvcruntime:risctrnsctrl.obj
 0002:0000a390       $unwind$__std_type_info_destroy_list 0000000180031390     libvcruntime:std_type_info.obj
 0002:0000a390       $unwind$_SetImageBase      0000000180031390     libvcruntime:risctrnsctrl.obj
 0002:0000a390       $unwind$_setfpstatusword   0000000180031390     libucrt:_fenvutils.obj
 0002:0000a390       $unwind$_clearfp           0000000180031390     libucrt:ieee.obj
 0002:0000a390       $unwind$__acrt_allocate_buffer_for_argv 0000000180031390     libucrt:argv_parsing.obj
 0002:0000a390       $unwind$__acrt_initialize_locks 0000000180031390     libucrt:locks.obj
 0002:0000a390       $unwind$__acrt_uninitialize_locks 0000000180031390     libucrt:locks.obj
 0002:0000a390       $unwind$__acrt_fp_strflt_to_string 0000000180031390     libucrt:_fptostr.obj
 0002:0000a390       $unwind$__vcrt_freeptd     0000000180031390     libvcruntime:per_thread_data.obj
 0002:0000a390       $unwind$?ShowMessageA@@YAHHH@Z 0000000180031390     ConEmuThA.obj
 0002:0000a390       $unwind$?ExitPlugin@@YAXXZ 0000000180031390     ConEmuTh.obj
 0002:0000a390       $unwind$?exit_or_terminate_process@@YAXI@Z 0000000180031390     libucrt:exit.obj
 0002:0000a390       $unwind$?ReloadResourcesW@@YAXXZ 0000000180031390     ConEmuTh.obj
 0002:0000a390       $unwind$?__GetUnwindTryBlock@@YAHPEA_KPEAU_xDISPATCHER_CONTEXT@@PEBU_s_FuncInfo@@@Z 0000000180031390     libvcruntime:riscehstate.obj
 0002:0000a390       $unwind$?Close@CeFullPanelInfo@@QEAAXXZ 0000000180031390     Display.obj
 0002:0000a390       $unwind$?__StateFromIp@@YAHPEBU_s_FuncInfo@@PEAU_xDISPATCHER_CONTEXT@@_K@Z 0000000180031390     libvcruntime:riscehstate.obj
 0002:0000a390       $unwind$?OnReadyForPanelsReload@@YAXXZ 0000000180031390     ConEmuTh.obj
 0002:0000a390       $unwind$__acrt_uninitialize_winapi_thunks 0000000180031390     libucrt:winapi_thunks.obj
 0002:0000a390       $unwind$__acrt_update_multibyte_info 0000000180031390     libucrt:locale_update.obj
 0002:0000a390       $unwind$??1?$MFileMapping@UPanelViewSetMapping@@@@QEAA@XZ 0000000180031390     ConEmuTh.obj
 0002:0000a390       $unwind$__acrt_update_locale_info 0000000180031390     libucrt:locale_update.obj
 0002:0000a390       $unwind$?ShowMessageW2800@@YAHHH@Z 0000000180031390     ConEmuTh2800.obj
 0002:0000a390       $unwind$__acrt_stdio_free_buffer_nolock 0000000180031390     libucrt:_freebuf.obj
 0002:0000a390       $unwind$??0exception@std@@QEAA@AEBV01@@Z 0000000180031390     libvcruntime:frame.obj
 0002:0000a390       $unwind$_clrfp             0000000180031390     libucrt:fpctrl.obj
 0002:0000a390       $unwind$_set_statfp        0000000180031390     libucrt:fpctrl.obj
 0002:0000a390       $unwind$??0bad_exception@std@@QEAA@AEBV01@@Z 0000000180031390     libvcruntime:frame.obj
 0002:0000a390       $unwind$?state_case_normal@?$output_processor@DV?$string_output_adapter@D@__crt_stdio_output@@V?$standard_base@DV?$string_output_adapter@D@__crt_stdio_output@@@2@@__crt_stdio_output@@AEAA_NXZ 0000000180031390     libucrt:output.obj
 0002:0000a390       $unwind$initialize_pointers 0000000180031390     libucrt:initialization.obj
 0002:0000a390       $unwind$__scrt_uninitialize_crt 0000000180031390     LIBCMT:utility.obj
 0002:0000a390       $unwind$uninitialize_allocated_memory 0000000180031390     libucrt:initialization.obj
 0002:0000a390       $unwind$__scrt_initialize_crt 0000000180031390     LIBCMT:utility.obj
 0002:0000a390       $unwind$_calloc_base       0000000180031390     libucrt:calloc_base.obj
 0002:0000a390       $unwind$strcpy_s           0000000180031390     libucrt:strcpy_s.obj
 0002:0000a390       $unwind$__scrt_release_startup_lock 0000000180031390     LIBCMT:utility.obj
 0002:0000a390       $unwind$?ExFilterRethrow@@YAHPEAU_EXCEPTION_POINTERS@@PEAUEHExceptionRecord@@PEAH@Z 0000000180031390     libvcruntime:frame.obj
 0002:0000a390       $unwind$?Lock@MSectionLock@@QEAAHPEAVMSection@@HK@Z 0000000180031390     common-kernel64:MSection.obj
 0002:0000a390       $unwind$?Unlock@MSectionLock@@QEAAXXZ 0000000180031390     common-kernel64:MSection.obj
 0002:0000a390       $unwind$_malloc_base       0000000180031390     libucrt:malloc_base.obj
 0002:0000a390       $unwind$?type_case_integer@?$output_processor@_WV?$string_output_adapter@_W@__crt_stdio_output@@V?$standard_base@_WV?$string_output_adapter@_W@__crt_stdio_output@@@2@@__crt_stdio_output@@AEAA_NI_N@Z 0000000180031390     libucrt:output.obj
 0002:0000a390       $unwind$__vcrt_initialize_locks 0000000180031390     libvcruntime:locks.obj
 0002:0000a390       $unwind$__vcrt_uninitialize_locks 0000000180031390     libvcruntime:locks.obj
 0002:0000a390       $unwind$??0?$output_processor@DV?$string_output_adapter@D@__crt_stdio_output@@V?$standard_base@DV?$string_output_adapter@D@__crt_stdio_output@@@2@@__crt_stdio_output@@QEAA@AEBV?$string_output_adapter@D@1@_KQEBDQEAU__crt_locale_pointers@@QEAD@Z 0000000180031390     libucrt:output.obj
 0002:0000a390       $unwind$_fflush_nolock     0000000180031390     libucrt:fflush.obj
 0002:0000a390       $unwind$?ShowMessageW995@@YAHHH@Z 0000000180031390     ConEmuTh995.obj
 0002:0000a390       $unwind$__raise_securityfailure 0000000180031390     LIBCMT:gs_report.obj
 0002:0000a390       $unwind$__acrt_freeptd     0000000180031390     libucrt:per_thread_data.obj
 0002:0000a390       $unwind$?ShowMessageW1900@@YAHHH@Z 0000000180031390     ConEmuTh1900.obj
 0002:0000a390       $unwind$__vcrt_FlsAlloc    0000000180031390     libvcruntime:winapi_downlevel.obj
 0002:0000a390       $unwind$__vcrt_FlsFree     0000000180031390     libvcruntime:winapi_downlevel.obj
 0002:0000a390       $unwind$__vcrt_FlsGetValue 0000000180031390     libvcruntime:winapi_downlevel.obj
 0002:0000a390       $unwind$?ProcessItem@CImgLoader@@UEAAJAEAPEAUIMAGE_CACHE_INFO@@_J@Z 0000000180031390     ImgCache.obj
 0002:0000a390       $unwind$?ProcessingThread@?$CQueueProcessor@PEAUIMAGE_CACHE_INFO@@@@KAKPEAX@Z 0000000180031390     ImgCache.obj
 0002:0000a390       $unwind$?OnPostPeekConsole@@YAHPEAXPEAU_INPUT_RECORD@@KPEAKPEAH@Z 0000000180031390     ConEmuTh.obj
 0002:0000a390       $unwind$??0?$output_processor@_WV?$string_output_adapter@_W@__crt_stdio_output@@V?$standard_base@_WV?$string_output_adapter@_W@__crt_stdio_output@@@2@@__crt_stdio_output@@QEAA@AEBV?$string_output_adapter@_W@1@_KQEB_WQEAU__crt_locale_pointers@@QEAD@Z 0000000180031390     libucrt:output.obj
 0002:0000a390       $unwind$?CheckWindows@@YA_NXZ 0000000180031390     ConEmuTh.obj
 0002:0000a390       $unwind$fegetenv           0000000180031390     libucrt:fegetenv.obj
 0002:0000a390       $unwind$??0MSectionSimple@@QEAA@_N@Z 0000000180031390     common-kernel64:MSectionSimple.obj
 0002:0000a390       $unwind$?type_case_integer@?$output_processor@DV?$string_output_adapter@D@__crt_stdio_output@@V?$standard_base@DV?$string_output_adapter@D@__crt_stdio_output@@@2@@__crt_stdio_output@@AEAA_NI_N@Z 0000000180031390     libucrt:output.obj
 0002:0000a390       $unwind$feholdexcept       0000000180031390     libucrt:feholdexcept.obj
 0002:0000a390       $unwind$??1MSectionSimple@@QEAA@XZ 0000000180031390     common-kernel64:MSectionSimple.obj
 0002:0000a390       $unwind$?Init@MSectionSimple@@QEAAXXZ 0000000180031390     common-kernel64:MSectionSimple.obj
 0002:0000a390       $unwind$?Close@MSectionSimple@@QEAAXXZ 0000000180031390     common-kernel64:MSectionSimple.obj
 0002:0000a390       $unwind$?TryEnter@MSectionSimple@@QEAA_NXZ 0000000180031390     common-kernel64:MSectionSimple.obj
 0002:0000a390       $unwind$?Unlock@MSectionLockSimple@@QEAAXXZ 0000000180031390     common-kernel64:MSectionSimple.obj
 0002:0000a390       $unwind$fesetenv           0000000180031390     libucrt:fesetenv.obj
 0002:0000a390       $unwind$_IsExceptionObjectToBeDestroyed 0000000180031390     libvcruntime:ehhelpers.obj
 0002:0000a390       $unwind$?GetMaxCount@CEStr@@QEAA_JXZ 0000000180031390     common-kernel64:CEStr.obj
 0002:0000a390       $unwind$??_Gtype_info@@UEAAPEAXI@Z 0000000180031390     LIBCMT:std_type_info_static.obj
 0002:0000a390       $unwind$?SavePathVar@CEStr@@QEAAXPEB_W@Z 0000000180031390     common-kernel64:CEStr.obj
 0002:0000a390       $unwind$__std_exception_destroy 0000000180031390     libvcruntime:std_exception.obj
 0002:0000a390       $unwind$?Free@MModule@@QEAAXXZ 0000000180031390     common-kernel64:MModule.obj
 0002:0000a398       $unwind$?LoadModuleVersion@@YA_NPEB_WAEAUtagVS_FIXEDFILEINFO@@PEA_W_K@Z 0000000180031398     ConEmuTh.obj
 0002:0000a3b8       $unwind$?LoadFarVersion@@YA_NAEAUFarVersion@@AEAY0CAA@_W@Z 00000001800313b8     ConEmuTh.obj
 0002:0000a3d4       $unwind$__acrt_locale_free_numeric 00000001800313d4     libucrt:initnum.obj
 0002:0000a3d4       $unwind$?FreeItem@CePluginPanelItem@@QEAAXXZ 00000001800313d4     ConEmuTh.obj
 0002:0000a3d4       $unwind$_free_base         00000001800313d4     libucrt:free_base.obj
 0002:0000a3d4       $unwind$?ExecuteInMainThread@@YAXPEAUConEmuThSynchroArg@@@Z 00000001800313d4     ConEmuTh.obj
 0002:0000a3d4       $unwind$?Invalidate@CeFullPanelInfo@@QEAAXXZ 00000001800313d4     Display.obj
 0002:0000a3d4       $unwind$?FreeUserData@CePluginPanelItem@@QEAAXXZ 00000001800313d4     ConEmuTh.obj
 0002:0000a3d4       $unwind$?destroy_fls@@YAXPEAX@Z 00000001800313d4     libucrt:per_thread_data.obj
 0002:0000a3d4       $unwind$__acrt_locale_free_lc_time_if_unreferenced 00000001800313d4     libucrt:locale_refcounting.obj
 0002:0000a3dc       $unwind$?LoadThSet@@YAHK@Z 00000001800313dc     ConEmuTh.obj
 0002:0000a400       $stateUnwindMap$?LoadThSet@@YAHK@Z 0000000180031400     ConEmuTh.obj
 0002:0000a408       $ip2state$?LoadThSet@@YAHK@Z 0000000180031408     ConEmuTh.obj
 0002:0000a418       $unwind$?Set@CEStr@@QEAAPEB_WPEB_W_J@Z 0000000180031418     common-kernel64:CEStr.obj
 0002:0000a418       $unwind$??0CImgCache@@QEAA@PEAUHINSTANCE__@@@Z 0000000180031418     ImgCache.obj
 0002:0000a418       $unwind$??$ensure_buffer_is_big_enough@D@formatting_buffer@__crt_stdio_output@@QEAA_N_K@Z 0000000180031418     libucrt:output.obj
 0002:0000a418       $unwind$__scrt_dllmain_exception_filter 0000000180031418     LIBCMT:utility.obj
 0002:0000a418       $unwind$__acrt_InitializeCriticalSectionEx 0000000180031418     libucrt:winapi_thunks.obj
 0002:0000a418       $unwind$?Init@HkFunc@@QEAA_NPEB_WPEAUHINSTANCE__@@@Z 0000000180031418     common-kernel64:HkFunc.obj
 0002:0000a418       $unwind$?_ExecutionInCatch@@YAHPEAU_xDISPATCHER_CONTEXT@@PEBU_s_FuncInfo@@@Z 0000000180031418     libvcruntime:risctrnsctrl.obj
 0002:0000a418       $unwind$?lstrdup@@YAPEA_WPEB_W_K@Z 0000000180031418     common-kernel64:MStrDup.obj
 0002:0000a418       $unwind$__acrt_execute_initializers 0000000180031418     libucrt:shared_initialization.obj
 0002:0000a418       $unwind$?Reset@CImgCache@@QEAAXXZ 0000000180031418     ImgCache.obj
 0002:0000a418       $unwind$?AddRef@MSection@@IEAAXK@Z 0000000180031418     common-kernel64:MSection.obj
 0002:0000a418       $unwind$?expand_if_necessary@?$argument_list@D@?A0xca0879c4@@AEAAHXZ 0000000180031418     libucrt:argv_wildcards.obj
 0002:0000a418       $unwind$__acrt_free_locale 0000000180031418     libucrt:locale_refcounting.obj
 0002:0000a418       $unwind$__acrt_lowio_create_handle_array 0000000180031418     libucrt:osfinfo.obj
 0002:0000a418       $unwind$_seh_filter_exe    0000000180031418     libucrt:exception_filter.obj
 0002:0000a418       $unwind$_recalloc_base     0000000180031418     libucrt:recalloc.obj
 0002:0000a418       $unwind$?ExecuteNewCmd@@YAPEAUCESERVER_REQ@@K_K@Z 0000000180031418     common-kernel64:ConEmuCheck.obj
 0002:0000a418       $unwind$?setSBCS@@YAXPEAU__crt_multibyte_data@@@Z 0000000180031418     libucrt:mbctype.obj
 0002:0000a418       $unwind$?GetEnvVar@@YAPEA_WPEB_W@Z 0000000180031418     common-kernel64:WObjects.obj
 0002:0000a418       $unwind$?ExpandEnvStr@@YAPEA_WPEB_W@Z 0000000180031418     common-kernel64:WObjects.obj
 0002:0000a418       $unwind$?ReleaseRef@MSection@@IEAAHK@Z 0000000180031418     common-kernel64:MSection.obj
 0002:0000a418       $unwind$?Lock@MSection@@IEAAHHK@Z 0000000180031418     common-kernel64:MSection.obj
 0002:0000a418       $unwind$?OpenPluginWcmn@@YAPEAXH_J_N@Z 0000000180031418     ConEmuTh.obj
 0002:0000a42c       $unwind$?SettingsLoadReg@@YAHPEB_W0PEAK@Z 000000018003142c     ConEmuTh.obj
 0002:0000a43c       $unwind$?SettingsLoadOther@@YAXPEB_W@Z 000000018003143c     ConEmuTh.obj
 0002:0000a450       $unwind$?SettingsSaveReg@@YAXPEB_W0PEAK@Z 0000000180031450     ConEmuTh.obj
 0002:0000a45c       $unwind$__report_securityfailure 000000018003145c     LIBCMT:gs_report.obj
 0002:0000a45c       $unwind$?SavePanelViewState@@YAXHK@Z 000000018003145c     ConEmuTh.obj
 0002:0000a464       $unwind$?CopyBits@CImgCache@@IEAAXU_COORD@@PEAEK01@Z 0000000180031464     ImgCache.obj
 0002:0000a464       $unwind$?EntryPoint@@YAXH_J_N@Z 0000000180031464     ConEmuTh.obj
 0002:0000a47c       $unwind$?LoadFarVersion@@YAHXZ 000000018003147c     ConEmuTh.obj
 0002:0000a47c       $unwind$?ShowLastError@@YAHXZ 000000018003147c     ConEmuTh.obj
 0002:0000a490       $unwind$?StartPlugin@@YAXH@Z 0000000180031490     ConEmuTh.obj
 0002:0000a4ac       $stateUnwindMap$?StartPlugin@@YAXH@Z 00000001800314ac     ConEmuTh.obj
 0002:0000a4b8       $ip2state$?StartPlugin@@YAXH@Z 00000001800314b8     ConEmuTh.obj
 0002:0000a4d0       $unwind$?fin$0@?0???$?RV<lambda_5e887d1dcbef67a5eb4283622ba103bf>@@AEAV<lambda_4466841279450cc726390878d4a41900>@@V<lambda_341c25c0346d94847f1f3c463c57e077>@@@?$__crt_seh_guarded_call@X@@QEAAX$$QEAV<lambda_5e887d1dcbef67a5eb4283622ba103bf>@@AEAV<lambda_4466841279450cc726390878d4a41900>@@$$QEAV<lambda_341c25c0346d94847f1f3c463c57e077>@@@Z@4HA 00000001800314d0     libucrt:per_thread_data.obj
 0002:0000a4d0       $unwind$?fin$0@?0???$?RV<lambda_bfedae4ebbf01fab1bb6dcc6a9e276e0>@@AEAV<lambda_2fe9b910cf3cbf4a0ab98a02ba45b3ec>@@V<lambda_237c231691f317818eb88cc1d5d642d6>@@@?$__crt_seh_guarded_call@H@@QEAAH$$QEAV<lambda_bfedae4ebbf01fab1bb6dcc6a9e276e0>@@AEAV<lambda_2fe9b910cf3cbf4a0ab98a02ba45b3ec>@@$$QEAV<lambda_237c231691f317818eb88cc1d5d642d6>@@@Z@4HA 00000001800314d0     libucrt:close.obj
 0002:0000a4d0       $unwind$common_flush_all$fin$1 00000001800314d0     libucrt:fflush.obj
 0002:0000a4d0       $unwind$?fin$0@?0???$?RV<lambda_fb3a7dec4e47f37f22dae91bb15c9095>@@AEAV<lambda_698284760c8add0bfb0756c19673e34b>@@V<lambda_dfb8eca1e75fef3034a8fb18dd509707>@@@?$__crt_seh_guarded_call@X@@QEAAX$$QEAV<lambda_fb3a7dec4e47f37f22dae91bb15c9095>@@AEAV<lambda_698284760c8add0bfb0756c19673e34b>@@$$QEAV<lambda_dfb8eca1e75fef3034a8fb18dd509707>@@@Z@4HA 00000001800314d0     libucrt:per_thread_data.obj
 0002:0000a4d0       $unwind$?fin$0@?0???$?RV<lambda_72d1df2b273a38828b1ce30cbf4cdab5>@@AEAV<lambda_876a65b173b8412d3a47c70a915b0cf4>@@V<lambda_41932305e351933ebe8f8be3ed8bb5dc>@@@?$__crt_seh_guarded_call@X@@QEAAX$$QEAV<lambda_72d1df2b273a38828b1ce30cbf4cdab5>@@AEAV<lambda_876a65b173b8412d3a47c70a915b0cf4>@@$$QEAV<lambda_41932305e351933ebe8f8be3ed8bb5dc>@@@Z@4HA 00000001800314d0     libucrt:per_thread_data.obj
 0002:0000a4d0       $unwind$common_flush_all$fin$0 00000001800314d0     libucrt:fflush.obj
 0002:0000a4d0       $unwind$raise$fin$0        00000001800314d0     libucrt:signal.obj
 0002:0000a4d0       $unwind$?dtor$0@?0???0?$CQueueProcessor@PEAUIMAGE_CACHE_INFO@@@@QEAA@XZ@4HA 00000001800314d0     ImgCache.obj
 0002:0000a4d0       $unwind$__CxxCallCatchBlock$filt$0 00000001800314d0     libvcruntime:frame.obj
 0002:0000a4d0       $unwind$_fcloseall$fin$0   00000001800314d0     libucrt:closeall.obj
 0002:0000a4d0       $unwind$?filt$0@?0??common_exit@@YAXHW4_crt_exit_cleanup_mode@@W4_crt_exit_return_mode@@@Z@4HA 00000001800314d0     libucrt:exit.obj
 0002:0000a4d0       $unwind$?fin$1@?0??common_exit@@YAXHW4_crt_exit_cleanup_mode@@W4_crt_exit_return_mode@@@Z@4HA 00000001800314d0     libucrt:exit.obj
 0002:0000a4d0       $unwind$__acrt_update_thread_multibyte_data$fin$0 00000001800314d0     libucrt:mbctype.obj
 0002:0000a4d0       $unwind$?dtor$2@?0??CheckVarsInitialized@@YAXXZ@4HA 00000001800314d0     ConEmuTh.obj
 0002:0000a4d0       $unwind$__DestructExceptionObject$filt$0 00000001800314d0     libvcruntime:ehhelpers.obj
 0002:0000a4d0       $unwind$common_control87$filt$0 00000001800314d0     libucrt:ieee.obj
 0002:0000a4d0       $unwind$_ctrlfp$filt$0     00000001800314d0     libucrt:fpctrl.obj
 0002:0000a4d0       $unwind$?dtor$1@?0??CheckVarsInitialized@@YAXXZ@4HA 00000001800314d0     ConEmuTh.obj
 0002:0000a4d0       $unwind$?dtor$0@?0??StartPlugin@@YAXH@Z@4HA 00000001800314d0     ConEmuTh.obj
 0002:0000a4d0       $unwind$?fin$0@?0???$?RV<lambda_99476a1ad63dd22509b5d3e65b0ffc95>@@AEAV<lambda_ad1ced32f4ac17aa236e5ef05d6b3b7c>@@V<lambda_f7424dd8d45958661754dc4f2697e9c3>@@@?$__crt_seh_guarded_call@X@@QEAAX$$QEAV<lambda_99476a1ad63dd22509b5d3e65b0ffc95>@@AEAV<lambda_ad1ced32f4ac17aa236e5ef05d6b3b7c>@@$$QEAV<lambda_f7424dd8d45958661754dc4f2697e9c3>@@@Z@4HA 00000001800314d0     libucrt:mbctype.obj
 0002:0000a4d0       $unwind$?fin$0@?0???$?RV<lambda_e24bbb7b643b32fcea6fa61b31d4c984>@@AEAV<lambda_275893d493268fdec8709772e3fcec0e>@@V<lambda_9d71df4d7cf3f480f8d633942495c3b0>@@@?$__crt_seh_guarded_call@H@@QEAAH$$QEAV<lambda_e24bbb7b643b32fcea6fa61b31d4c984>@@AEAV<lambda_275893d493268fdec8709772e3fcec0e>@@$$QEAV<lambda_9d71df4d7cf3f480f8d633942495c3b0>@@@Z@4HA 00000001800314d0     libucrt:onexit.obj
 0002:0000a4d0       $unwind$?fin$0@?0??dllmain_crt_process_detach@@YAH_N@Z@4HA 00000001800314d0     LIBCMT:dll_dllmain.obj
 0002:0000a4d0       $unwind$?dtor$0@?0??CheckVarsInitialized@@YAXXZ@4HA 00000001800314d0     ConEmuTh.obj
 0002:0000a4d0       $unwind$_write$fin$0       00000001800314d0     libucrt:write.obj
 0002:0000a4d0       $unwind$__acrt_initialize_lowio$fin$0 00000001800314d0     libucrt:ioinit.obj
 0002:0000a4d0       $unwind$?fin$0@?0???$?RV<lambda_b521505b218e5242e90febf6bfebc422>@@AEAV<lambda_6978c1fb23f02e42e1d9e99668cc68aa>@@V<lambda_314360699dd331753a4119843814e9a7>@@@?$__crt_seh_guarded_call@H@@QEAAH$$QEAV<lambda_b521505b218e5242e90febf6bfebc422>@@AEAV<lambda_6978c1fb23f02e42e1d9e99668cc68aa>@@$$QEAV<lambda_314360699dd331753a4119843814e9a7>@@@Z@4HA 00000001800314d0     libucrt:commit.obj
 0002:0000a4d0       $unwind$?fin$0@?0??dllmain_crt_process_attach@@YAHQEAUHINSTANCE__@@QEAX@Z@4HA 00000001800314d0     LIBCMT:dll_dllmain.obj
 0002:0000a4d0       $unwind$__acrt_update_thread_locale_data$fin$0 00000001800314d0     libucrt:locale_refcounting.obj
 0002:0000a4d0       $unwind$?fin$0@?0???$?RV<lambda_c36588078e9f5dfd39652860aa6b3aaf>@@AEAV<lambda_ec61778202f4f5fc7e7711acc23c3bca>@@V<lambda_dc9d2797ccde5d239b4a0efae8ebd7db>@@@?$__crt_seh_guarded_call@P6AXH@Z@@QEAAP6AXH@Z$$QEAV<lambda_c36588078e9f5dfd39652860aa6b3aaf>@@AEAV<lambda_ec61778202f4f5fc7e7711acc23c3bca>@@$$QEAV<lambda_dc9d2797ccde5d239b4a0efae8ebd7db>@@@Z@4HA 00000001800314d0     libucrt:signal.obj
 0002:0000a4d0       $unwind$__acrt_lowio_ensure_fh_exists$fin$0 00000001800314d0     libucrt:osfinfo.obj
 0002:0000a4d0       $unwind$__FrameUnwindToState$filt$0 00000001800314d0     libvcruntime:frame.obj
 0002:0000a4d0       $unwind$_IsNonwritableInCurrentImage$filt$0 00000001800314d0     LIBCMT:pesect.obj
 0002:0000a4d0       $unwind$?dtor$0@?0??RequestItem@CImgCache@@QEAAHPEAUCePluginPanelItem@@I@Z@4HA 00000001800314d0     ImgCache.obj
 0002:0000a4d0       $unwind$__acrt_uninitialize_locale$fin$0 00000001800314d0     libucrt:wsetlocale.obj
 0002:0000a4d0       $unwind$__FrameUnwindToState$fin$1 00000001800314d0     libvcruntime:frame.obj
 0002:0000a4d0       $unwind$fclose$fin$0       00000001800314d0     libucrt:fclose.obj
 0002:0000a4d0       $unwind$?fin$0@?0???$?RV<lambda_46352004c1216016012b18bd6f87e700>@@AEAV<lambda_3bd07e1a1191394380780325891bf33f>@@V<lambda_334532d3f185bcaa59b5be82d7d22bff>@@@?$__crt_seh_guarded_call@X@@QEAAX$$QEAV<lambda_46352004c1216016012b18bd6f87e700>@@AEAV<lambda_3bd07e1a1191394380780325891bf33f>@@$$QEAV<lambda_334532d3f185bcaa59b5be82d7d22bff>@@@Z@4HA 00000001800314d0     libucrt:per_thread_data.obj
 0002:0000a4d0       $unwind$_query_new_handler$fin$0 00000001800314d0     libucrt:new_handler.obj
 0002:0000a4d8       $unwind$?PostMacro@@YAXPEA_W@Z 00000001800314d8     ConEmuTh.obj
 0002:0000a4f8       $unwind$?GetMainThreadId@@YAKXZ 00000001800314f8     ConEmuTh.obj
 0002:0000a4f8       $unwind$?ReloadPanelsInfo@@YAXXZ 00000001800314f8     ConEmuTh.obj
 0002:0000a510       $unwind$?IsThumbnailsActive@@YAPEAUCeFullPanelInfo@@H@Z 0000000180031510     ConEmuTh.obj
 0002:0000a530       $unwind$_FindAndUnlinkFrame 0000000180031530     libvcruntime:risctrnsctrl.obj
 0002:0000a530       $unwind$??0_LocaleUpdate@@QEAA@QEAU__crt_locale_pointers@@@Z 0000000180031530     libucrt:output.obj
 0002:0000a530       $unwind$_updatetlocinfoEx_nolock 0000000180031530     libucrt:locale_refcounting.obj
 0002:0000a530       $unwind$??_G?$MFileMapping@Utag_DetectedDialog@@@@QEAAPEAXI@Z 0000000180031530     ConEmuTh.obj
 0002:0000a530       $unwind$??_GCImgLoader@@UEAAPEAXI@Z 0000000180031530     ImgCache.obj
 0002:0000a530       $unwind$?LoadFarSettingsA@@YAXPEAUCEFarInterfaceSettings@@PEAUCEFarPanelSettings@@@Z 0000000180031530     ConEmuThA.obj
 0002:0000a530       $unwind$__acrt_uninitialize_lowio 0000000180031530     libucrt:ioinit.obj
 0002:0000a530       $unwind$_realloc_base      0000000180031530     libucrt:realloc_base.obj
 0002:0000a530       $unwind$__vcrt_FlsSetValue 0000000180031530     libvcruntime:winapi_downlevel.obj
 0002:0000a530       $unwind$??_GMNullDesc@@QEAAPEAXI@Z 0000000180031530     common-kernel64:MSecurity.obj
 0002:0000a530       $unwind$?GetItemColors@CeFullPanelInfo@@QEAAPEAUHBRUSH__@@_JPEAUCePluginPanelItem@@PEAUCePluginPanelItemColor@@HAEAK3@Z 0000000180031530     Display.obj
 0002:0000a530       $unwind$??_G?$CQueueProcessor@PEAUIMAGE_CACHE_INFO@@@@UEAAPEAXI@Z 0000000180031530     ImgCache.obj
 0002:0000a530       $unwind$?GetFarRectW995@@YAXPEAU_SMALL_RECT@@@Z 0000000180031530     ConEmuTh995.obj
 0002:0000a530       $unwind$_RTC_Terminate     0000000180031530     LIBCMT:_initsect_.obj
 0002:0000a530       $unwind$_callnewh          0000000180031530     libucrt:new_handler.obj
 0002:0000a530       $unwind$_RTC_Initialize    0000000180031530     LIBCMT:_initsect_.obj
 0002:0000a530       $unwind$__acrt_FlsAlloc    0000000180031530     libucrt:winapi_thunks.obj
 0002:0000a530       $unwind$?force_decimal_point@__crt_stdio_output@@YAXPEADQEAU__crt_locale_pointers@@@Z 0000000180031530     libucrt:output.obj
 0002:0000a530       $unwind$_fclose_nolock     0000000180031530     libucrt:fclose.obj
 0002:0000a530       $unwind$__acrt_FlsFree     0000000180031530     libucrt:winapi_thunks.obj
 0002:0000a530       $unwind$_close_nolock      0000000180031530     libucrt:close.obj
 0002:0000a530       $unwind$__acrt_FlsGetValue 0000000180031530     libucrt:winapi_thunks.obj
 0002:0000a530       $unwind$?__SetUnwindTryBlock@@YAXPEA_KPEAU_xDISPATCHER_CONTEXT@@PEBU_s_FuncInfo@@H@Z 0000000180031530     libvcruntime:riscehstate.obj
 0002:0000a530       $unwind$?try_cor_exit_process@@YAXI@Z 0000000180031530     libucrt:exit.obj
 0002:0000a530       $unwind$?GetPluginInfoW2800@@YAXPEAX@Z 0000000180031530     ConEmuTh2800.obj
 0002:0000a530       $unwind$__acrt_errno_map_os_error 0000000180031530     libucrt:errno.obj
 0002:0000a530       $unwind$?getNext@?$MToolHelp@UtagPROCESSENTRY32W@@$1?Process32FirstW@@YAHPEAXPEAU1@@Z$1?Process32NextW@@YAH01@Z@@IEAA_NXZ 0000000180031530     common-kernel64:MProcess.obj
 0002:0000a530       $unwind$OpenPlugin         0000000180031530     ConEmuThA.obj
 0002:0000a530       $unwind$??1?$MToolHelp@UtagPROCESSENTRY32W@@$1?Process32FirstW@@YAHPEAXPEAU1@@Z$1?Process32NextW@@YAH01@Z@@UEAA@XZ 0000000180031530     common-kernel64:MProcess.obj
 0002:0000a530       $unwind$strncpy_s          0000000180031530     libucrt:strncpy_s.obj
 0002:0000a530       $unwind$?Open@?$MToolHelp@UtagPROCESSENTRY32W@@$1?Process32FirstW@@YAHPEAXPEAU1@@Z$1?Process32NextW@@YAH01@Z@@QEAA_NXZ 0000000180031530     common-kernel64:MProcess.obj
 0002:0000a530       $unwind$?OpenW2800@@YAPEAXPEBX@Z 0000000180031530     ConEmuTh2800.obj
 0002:0000a530       $unwind$??_G?$MToolHelp@UtagPROCESSENTRY32W@@$1?Process32FirstW@@YAHPEAXPEAU1@@Z$1?Process32NextW@@YAH01@Z@@UEAAPEAXI@Z 0000000180031530     common-kernel64:MProcess.obj
 0002:0000a530       $unwind$??_GMToolHelpProcess@@UEAAPEAXI@Z 0000000180031530     common-kernel64:MProcess.obj
 0002:0000a530       $unwind$?GetPluginInfoW1900@@YAXPEAX@Z 0000000180031530     ConEmuTh1900.obj
 0002:0000a530       $unwind$??0MSection@@QEAA@XZ 0000000180031530     common-kernel64:MSection.obj
 0002:0000a530       $unwind$??$SafeDelete@UMSectionSimple@@@@YAXAEAPEAUMSectionSimple@@@Z 0000000180031530     ImgCache.obj
 0002:0000a530       $unwind$??1MSection@@QEAA@XZ 0000000180031530     common-kernel64:MSection.obj
 0002:0000a530       $unwind$?type_case_c_tchar@?$output_processor@DV?$string_output_adapter@D@__crt_stdio_output@@V?$standard_base@DV?$string_output_adapter@D@__crt_stdio_output@@@2@@__crt_stdio_output@@AEAA_ND@Z 0000000180031530     libucrt:output.obj
 0002:0000a530       $unwind$?Unlock@MSection@@IEAAXH@Z 0000000180031530     common-kernel64:MSection.obj
 0002:0000a530       $unwind$?OnPrePeekConsole@@YAHPEAXPEAU_INPUT_RECORD@@KPEAKPEAH@Z 0000000180031530     ConEmuTh.obj
 0002:0000a530       $unwind$GetPluginInfo      0000000180031530     ConEmuThA.obj
 0002:0000a530       $unwind$?DisplayReloadPanel@CeFullPanelInfo@@QEAAXXZ 0000000180031530     Display.obj
 0002:0000a530       $unwind$?replace_current_thread_locale_nolock@@YAXQEAU__acrt_ptd@@QEAU__crt_locale_data@@@Z 0000000180031530     libucrt:per_thread_data.obj
 0002:0000a530       $unwind$?PointToName@@YAPEB_WPEB_W@Z 0000000180031530     common-kernel64:CmdLine.obj
 0002:0000a530       $unwind$??_Gexception@std@@UEAAPEAXI@Z 0000000180031530     libvcruntime:frame.obj
 0002:0000a530       $unwind$__acrt_getptd      0000000180031530     libucrt:per_thread_data.obj
 0002:0000a530       $unwind$?GetFarRectW1900@@YAXPEAU_SMALL_RECT@@@Z 0000000180031530     ConEmuTh1900.obj
 0002:0000a530       $unwind$?GetFarRect@@YAHPEAU_SMALL_RECT@@@Z 0000000180031530     ConEmuTh.obj
 0002:0000a530       $unwind$?GetFarRectW2800@@YAXPEAU_SMALL_RECT@@@Z 0000000180031530     ConEmuTh2800.obj
 0002:0000a530       $unwind$?SetCacheLocation@CImgCache@@QEAAXPEB_W@Z 0000000180031530     ImgCache.obj
 0002:0000a530       $unwind$??_Gbad_exception@std@@UEAAPEAXI@Z 0000000180031530     libvcruntime:frame.obj
 0002:0000a530       $unwind$__acrt_invoke_user_matherr 0000000180031530     libucrt:matherr.obj
 0002:0000a530       $unwind$?internal_isupper_l@@YA_NHQEAU__crt_locale_pointers@@@Z 0000000180031530     libucrt:tolower_toupper.obj
 0002:0000a530       $unwind$?GetPluginInfoW995@@YAXPEAX@Z 0000000180031530     ConEmuTh995.obj
 0002:0000a530       $unwind$??1CEStr@@QEAA@XZ  0000000180031530     common-kernel64:CEStr.obj
 0002:0000a530       $unwind$??0CRgnDetect@@QEAA@XZ 0000000180031530     common-user64:RgnDetect.obj
 0002:0000a530       $unwind$?LoadFarSettingsW995@@YAXPEAUCEFarInterfaceSettings@@PEAUCEFarPanelSettings@@@Z 0000000180031530     ConEmuTh995.obj
 0002:0000a530       $unwind$??$common_initialize_environment_nolock@D@@YAHXZ 0000000180031530     libucrt:environment_initialization.obj
 0002:0000a530       $unwind$?CheckConEmu@@YAHH@Z 0000000180031530     ConEmuTh.obj
 0002:0000a53c       $unwind$?OnPreWriteConsoleOutput@@YAHPEAXPEBU_CHAR_INFO@@U_COORD@@2PEAU_SMALL_RECT@@@Z 000000018003153c     ConEmuTh.obj
 0002:0000a558       $unwind$?CheckVarsInitialized@@YAXXZ 0000000180031558     ConEmuTh.obj
 0002:0000a568       $stateUnwindMap$?CheckVarsInitialized@@YAXXZ 0000000180031568     ConEmuTh.obj
 0002:0000a580       $ip2state$?CheckVarsInitialized@@YAXXZ 0000000180031580     ConEmuTh.obj
 0002:0000a5b8       $unwind$?ProcessConsoleInput@@YAHHPEAU_INPUT_RECORD@@KPEAK@Z 00000001800315b8     ConEmuTh.obj
 0002:0000a5dc       $unwind$?ChangeExports@@YA_NPEBUExportFunc@@PEAUHINSTANCE__@@@Z 00000001800315dc     ConEmuTh.obj
 0002:0000a5f8       $unwind$?InitName@?$MFileMapping@UPanelViewSetMapping@@@@QEAAPEB_WPEB_WKK@Z 00000001800315f8     ConEmuTh.obj
 0002:0000a5f8       $unwind$?InitName@?$MFileMapping@Utag_DetectedDialog@@@@QEAAPEB_WPEB_WKK@Z 00000001800315f8     ConEmuTh.obj
 0002:0000a60c       $unwind$?InternalOpenCreate@?$MFileMapping@Utag_DetectedDialog@@@@IEAAPEAUtag_DetectedDialog@@HHH@Z 000000018003160c     ConEmuTh.obj
 0002:0000a60c       $unwind$??$copy_and_add_argument_to_buffer@D@@YAHQEBD0_KAEAV?$argument_list@D@?A0xca0879c4@@@Z 000000018003160c     libucrt:argv_wildcards.obj
 0002:0000a60c       $unwind$?InternalOpenCreate@?$MFileMapping@UPanelViewSetMapping@@@@IEAAPEAUPanelViewSetMapping@@HHH@Z 000000018003160c     ConEmuTh.obj
 0002:0000a628       $unwind$??$swprintf_c@$0IA@@@YAHAEAY0IA@_WPEB_WZZ 0000000180031628     Display.obj
 0002:0000a628       $unwind$??$sprintf_c@$0CI@@@YAHAEAY0CI@DPEBDZZ 0000000180031628     common-kernel64:WThreads.obj
 0002:0000a628       $unwind$??$swprintf_c@$0CAA@@@YAHAEAY0CAA@_WPEB_WZZ 0000000180031628     ConEmuTh.obj
 0002:0000a628       $unwind$??$swprintf_c@$0MI@@@YAHAEAY0MI@_WPEB_WZZ 0000000180031628     ConEmuTh2800.obj
 0002:0000a630       $unwind$?type_case_s@?$output_processor@_WV?$string_output_adapter@_W@__crt_stdio_output@@V?$standard_base@_WV?$string_output_adapter@_W@__crt_stdio_output@@@2@@__crt_stdio_output@@AEAA_NXZ 0000000180031630     libucrt:output.obj
 0002:0000a630       $unwind$__acrt_stdio_flush_nolock 0000000180031630     libucrt:fflush.obj
 0002:0000a630       $unwind$?type_case_n@?$output_processor@_WV?$string_output_adapter@_W@__crt_stdio_output@@V?$standard_base@_WV?$string_output_adapter@_W@__crt_stdio_output@@@2@@__crt_stdio_output@@AEAA_NXZ 0000000180031630     libucrt:output.obj
 0002:0000a630       $unwind$__vcrt_InitializeCriticalSectionEx 0000000180031630     libvcruntime:winapi_downlevel.obj
 0002:0000a630       $unwind$__acrt_execute_uninitializers 0000000180031630     libucrt:shared_initialization.obj
 0002:0000a630       $unwind$__acrt_LocaleNameToLCID 0000000180031630     libucrt:winapi_thunks.obj
 0002:0000a630       $unwind$_initterm_e        0000000180031630     libucrt:initterm.obj
 0002:0000a630       $unwind$__acrt_FlsSetValue 0000000180031630     libucrt:winapi_thunks.obj
 0002:0000a630       $unwind$memcpy_s           0000000180031630     libucrt:cfout.obj
 0002:0000a630       $unwind$?ClearQueue@?$CQueueProcessor@PEAUIMAGE_CACHE_INFO@@@@AEAAXXZ 0000000180031630     ImgCache.obj
 0002:0000a630       $unwind$__vcrt_getptd_noexit 0000000180031630     libvcruntime:per_thread_data.obj
 0002:0000a630       $unwind$_exception_enabled 0000000180031630     libucrt:libm_error.obj
 0002:0000a630       $unwind$?OnSettingsChanged@CeFullPanelInfo@@QEAAHH@Z 0000000180031630     Display.obj
 0002:0000a630       $unwind$?type_case_n@?$output_processor@DV?$string_output_adapter@D@__crt_stdio_output@@V?$standard_base@DV?$string_output_adapter@D@__crt_stdio_output@@@2@@__crt_stdio_output@@AEAA_NXZ 0000000180031630     libucrt:output.obj
 0002:0000a630       $unwind$??R<lambda_ad1ced32f4ac17aa236e5ef05d6b3b7c>@@QEBAXXZ 0000000180031630     libucrt:mbctype.obj
 0002:0000a630       $unwind$?free_crt_array_internal@@YAXQEAPEBX_K@Z 0000000180031630     libucrt:inittime.obj
 0002:0000a630       $unwind$?Init@CImgCache@@QEAAXK@Z 0000000180031630     ImgCache.obj
 0002:0000a630       $unwind$??$common_lseek_nolock@_J@@YA_JH_JH@Z 0000000180031630     libucrt:lseek.obj
 0002:0000a630       $unwind$?ProcessSynchroEventCommon@@YAHHPEAX@Z 0000000180031630     ConEmuTh.obj
 0002:0000a630       $unwind$?type_case_s@?$output_processor@DV?$string_output_adapter@D@__crt_stdio_output@@V?$standard_base@DV?$string_output_adapter@D@__crt_stdio_output@@@2@@__crt_stdio_output@@AEAA_NXZ 0000000180031630     libucrt:output.obj
 0002:0000a630       $unwind$?push_back@?$MArray@UtagPROCESSENTRY32W@@@@QEAA_JAEBUtagPROCESSENTRY32W@@@Z 0000000180031630     common-kernel64:MProcess.obj
 0002:0000a630       $unwind$?type_case_Z@?$output_processor@DV?$string_output_adapter@D@__crt_stdio_output@@V?$standard_base@DV?$string_output_adapter@D@__crt_stdio_output@@@2@@__crt_stdio_output@@AEAA_NXZ 0000000180031630     libucrt:output.obj
 0002:0000a630       $unwind$?addsize@?$MArray@UtagPROCESSENTRY32W@@@@QEAA_N_J@Z 0000000180031630     common-kernel64:MProcess.obj
 0002:0000a630       $unwind$?FinalRelease@CeFullPanelInfo@@QEAAXXZ 0000000180031630     Display.obj
 0002:0000a630       $unwind$__acrt_getptd_noexit 0000000180031630     libucrt:per_thread_data.obj
 0002:0000a630       $unwind$_DllMainCRTStartup 0000000180031630     LIBCMT:dll_dllmain.obj
 0002:0000a630       $unwind$?Unquote@@YAPEB_WPEA_W_N@Z 0000000180031630     common-kernel64:CmdLine.obj
 0002:0000a630       $unwind$?AttachInt@CEStr@@AEAAPEB_WAEAPEA_W@Z 0000000180031630     common-kernel64:CEStr.obj
 0002:0000a630       $unwind$?type_case_Z@?$output_processor@_WV?$string_output_adapter@_W@__crt_stdio_output@@V?$standard_base@_WV?$string_output_adapter@_W@__crt_stdio_output@@@2@@__crt_stdio_output@@AEAA_NXZ 0000000180031630     libucrt:output.obj
 0002:0000a640       $unwind$?SettingsLoadW1900@@YAHPEB_WPEAK@Z 0000000180031640     ConEmuTh1900.obj
 0002:0000a658       $unwind$?SettingsSaveW1900@@YAXPEB_WPEAK@Z 0000000180031658     ConEmuTh1900.obj
 0002:0000a670       $unwind$?SetStartupInfoW2800@@YAXPEAX@Z 0000000180031670     ConEmuTh2800.obj
 0002:0000a670       $unwind$?SetStartupInfoW1900@@YAXPEAX@Z 0000000180031670     ConEmuTh1900.obj
 0002:0000a68c       $unwind$?ShowMessageW1900@@YAHPEB_WH@Z 000000018003168c     ConEmuTh1900.obj
 0002:0000a68c       $unwind$?ShowMessageW2800@@YAHPEB_WH@Z 000000018003168c     ConEmuTh2800.obj
 0002:0000a69c       $unwind$?PostMacroW1900@@YAXPEA_W@Z 000000018003169c     ConEmuTh1900.obj
 0002:0000a69c       $unwind$?PostMacroW2800@@YAXPEA_W@Z 000000018003169c     ConEmuTh2800.obj
 0002:0000a6b0       $unwind$?ShowPluginMenuW1900@@YAHXZ 00000001800316b0     ConEmuTh1900.obj
 0002:0000a6cc       $unwind$?LoadPanelInfoW1900@@YAHH@Z 00000001800316cc     ConEmuTh1900.obj
 0002:0000a6cc       $unwind$?LoadPanelInfoW2800@@YAHH@Z 00000001800316cc     ConEmuTh2800.obj
 0002:0000a6f0       $unwind$?LoadPanelItemInfoW1900@@YAXPEAUCeFullPanelInfo@@_J@Z 00000001800316f0     ConEmuTh1900.obj
 0002:0000a70c       $unwind$?CheckFarPanelsW2800@@YA_NXZ 000000018003170c     ConEmuTh2800.obj
 0002:0000a70c       $unwind$?CheckFarPanelsW1900@@YA_NXZ 000000018003170c     ConEmuTh1900.obj
 0002:0000a71c       $unwind$?CheckPanelSettingsW1900@@YAHH@Z 000000018003171c     ConEmuTh1900.obj
 0002:0000a71c       $unwind$?CheckPanelSettingsW2800@@YAHH@Z 000000018003171c     ConEmuTh2800.obj
 0002:0000a730       $unwind$?SetCurrentPanelItemW1900@@YAXH_J0@Z 0000000180031730     ConEmuTh1900.obj
 0002:0000a750       $unwind$?Color2BgIndex@Far3Color@@SAXKHAEAGPEBK@Z 0000000180031750     ConEmuTh1900.obj
 0002:0000a750       $unwind$?FindFrameBottom_ByRight@CRgnDetect@@IEAA_NPEA_WPEAUtag_CharAttr@@HHAEAH22@Z 0000000180031750     common-user64:RgnDetect.obj
 0002:0000a750       $unwind$?FindFrameRight_ByBottom@CRgnDetect@@IEAA_NPEA_WPEAUtag_CharAttr@@HHAEAH22@Z 0000000180031750     common-user64:RgnDetect.obj
 0002:0000a750       $unwind$?FindFrameBottom_ByLeft@CRgnDetect@@IEAA_NPEA_WPEAUtag_CharAttr@@HHAEAH22@Z 0000000180031750     common-user64:RgnDetect.obj
 0002:0000a75c       $unwind$?parse_int_from_format_string@?$output_processor@_WV?$string_output_adapter@_W@__crt_stdio_output@@V?$standard_base@_WV?$string_output_adapter@_W@__crt_stdio_output@@@2@@__crt_stdio_output@@AEAA_NQEAH@Z 000000018003175c     libucrt:output.obj
 0002:0000a75c       $unwind$?FarColor_3_2@@YAEAEBUFarColor@@_N@Z 000000018003175c     ConEmuTh1900.obj
 0002:0000a770       $unwind$?GetFarSetting@@YAHPEAX_KPEB_W@Z 0000000180031770     ConEmuTh2800.obj
 0002:0000a770       $unwind$?GetFarSetting@@YAHPEAX_KPEB_W@Z 0000000180031770     ConEmuTh1900.obj
 0002:0000a770       $unwind$_call_matherr      0000000180031770     libucrt:libm_error.obj
 0002:0000a778       $unwind$?LoadFarSettingsW1900@@YAXPEAUCEFarInterfaceSettings@@PEAUCEFarPanelSettings@@@Z 0000000180031778     ConEmuTh1900.obj
 0002:0000a778       $unwind$?LoadFarSettingsW2800@@YAXPEAUCEFarInterfaceSettings@@PEAUCEFarPanelSettings@@@Z 0000000180031778     ConEmuTh2800.obj
 0002:0000a790       $unwind$GetGlobalInfoW     0000000180031790     ConEmuTh2800.obj
 0002:0000a798       $unwind$?SettingsLoadW2800@@YAHPEB_WPEAK@Z 0000000180031798     ConEmuTh2800.obj
 0002:0000a7b0       $unwind$?SettingsSaveW2800@@YAXPEB_WPEAK@Z 00000001800317b0     ConEmuTh2800.obj
 0002:0000a7c8       $unwind$?ShowPluginMenuW2800@@YAHXZ 00000001800317c8     ConEmuTh2800.obj
 0002:0000a7e8       $unwind$?LoadPanelItemInfoW2800@@YAXPEAUCeFullPanelInfo@@_J@Z 00000001800317e8     ConEmuTh2800.obj
 0002:0000a80c       $unwind$?SetCurrentPanelItemW2800@@YAXH_J0@Z 000000018003180c     ConEmuTh2800.obj
 0002:0000a824       $unwind$?SetCurrentPanelItemW2800Int@@YAXH_J0@Z 0000000180031824     ConEmuTh2800.obj
 0002:0000a844       $unwind$_log10_special     0000000180031844     libucrt:log_special.obj
 0002:0000a844       $unwind$_invalid_parameter_noinfo 0000000180031844     libucrt:invalid_parameter.obj
 0002:0000a844       $unwind$?ShowMessageW995@@YAHPEB_WH@Z 0000000180031844     ConEmuTh995.obj
 0002:0000a844       $unwind$?FreePanelItemUserData2800@@YAXPEAX_KP6A_JXZ@Z 0000000180031844     ConEmuTh2800.obj
 0002:0000a844       $unwind$?ShowMessageA@@YAHPEBDH@Z 0000000180031844     ConEmuThA.obj
 0002:0000a844       $unwind$wctomb_s           0000000180031844     libucrt:wctomb.obj
 0002:0000a84c       $unwind$?SetStartupInfoW995@@YAXPEAX@Z 000000018003184c     ConEmuTh995.obj
 0002:0000a85c       $unwind$?PostMacroA@@YAXPEAD@Z 000000018003185c     ConEmuThA.obj
 0002:0000a85c       $unwind$?PostMacroW995@@YAXPEA_W@Z 000000018003185c     ConEmuTh995.obj
 0002:0000a85c       $unwind$strpbrk            000000018003185c     libucrt:strpbrk.obj
 0002:0000a86c       $unwind$?ShowPluginMenuW995@@YAHXZ 000000018003186c     ConEmuTh995.obj
 0002:0000a884       $unwind$?LoadPanelItemInfoW995@@YAXPEAUCeFullPanelInfo@@_J@Z 0000000180031884     ConEmuTh995.obj
 0002:0000a89c       $unwind$?CheckFarPanelsW995@@YA_NXZ 000000018003189c     ConEmuTh995.obj
 0002:0000a8ac       $unwind$?CheckPanelSettingsW995@@YAHH@Z 00000001800318ac     ConEmuTh995.obj
 0002:0000a8ac       $unwind$wcstol             00000001800318ac     libucrt:strtox.obj
 0002:0000a8ac       $unwind$?CheckThread@?$CQueueProcessor@PEAUIMAGE_CACHE_INFO@@@@IEAAJXZ 00000001800318ac     ImgCache.obj
 0002:0000a8ac       $unwind$strtol             00000001800318ac     libucrt:strtox.obj
 0002:0000a8ac       $unwind$?CheckPanelSettingsA@@YAHH@Z 00000001800318ac     ConEmuThA.obj
 0002:0000a8b4       $unwind$?SetCurrentPanelItemW995@@YAXH_J0@Z 00000001800318b4     ConEmuTh995.obj
 0002:0000a8d4       $unwind$?LoadPanelInfo995@@YAHH@Z 00000001800318d4     ConEmuTh995.obj
 0002:0000a8f8       $unwind$SetStartupInfo     00000001800318f8     ConEmuThA.obj
 0002:0000a908       $unwind$?_VerifyVersionInfo@@YA_NPEAU_OSVERSIONINFOEXW@@K_K@Z 0000000180031908     common-kernel64:WObjects.obj
 0002:0000a908       $unwind$?GetMsgA@@YAPEB_WHPEA_W@Z 0000000180031908     ConEmuThA.obj
 0002:0000a918       $unwind$?ShowPluginMenuA@@YAHXZ 0000000180031918     ConEmuThA.obj
 0002:0000a938       $unwind$?LoadPanelInfoA@@YAHH@Z 0000000180031938     ConEmuThA.obj
 0002:0000a958       $unwind$?CheckFarPanelsA@@YA_NXZ 0000000180031958     ConEmuThA.obj
 0002:0000a96c       $unwind$?SetCurrentPanelItemA@@YAXH_J0@Z 000000018003196c     ConEmuThA.obj
 0002:0000a98c       $unwind$?ReloadResourcesA@@YAXXZ 000000018003198c     ConEmuThA.obj
 0002:0000a9a0       $unwind$?RegisterPanelView@CeFullPanelInfo@@QEAAHXZ 00000001800319a0     Display.obj
 0002:0000a9bc       $unwind$?UnregisterPanelView@CeFullPanelInfo@@QEAAH_N@Z 00000001800319bc     Display.obj
 0002:0000a9d8       $unwind$?CreateView@CeFullPanelInfo@@QEAAPEAUHWND__@@XZ 00000001800319d8     Display.obj
 0002:0000a9fc       $unwind$?ReallocItems@CeFullPanelInfo@@QEAAH_J@Z 00000001800319fc     Display.obj
 0002:0000aa1c       $stateUnwindMap$?ReallocItems@CeFullPanelInfo@@QEAAH_J@Z 0000000180031a1c     Display.obj
 0002:0000aa28       $ip2state$?ReallocItems@CeFullPanelInfo@@QEAAH_J@Z 0000000180031a28     Display.obj
 0002:0000aa40       $unwind$?RequestSetPos@CeFullPanelInfo@@QEAAX_J0H@Z 0000000180031a40     Display.obj
 0002:0000aa50       $unwind$?PaintItem@CeFullPanelInfo@@QEAAHPEAUHDC__@@_JHHPEAUCePluginPanelItem@@PEAUCePluginPanelItemColor@@HHPEAUHBRUSH__@@4K@Z 0000000180031a50     Display.obj
 0002:0000aa50       $unwind$?DisplayWndProc@CeFullPanelInfo@@SA_JPEAUHWND__@@I_K_J@Z 0000000180031a50     Display.obj
 0002:0000aa70       $unwind$?DisplayThread@CeFullPanelInfo@@SAKPEAX@Z 0000000180031a70     Display.obj
 0002:0000aa80       $unwind$?Paint@CeFullPanelInfo@@QEAAXPEAUHWND__@@AEAUtagPAINTSTRUCT@@AEAUtagRECT@@@Z 0000000180031a80     Display.obj
 0002:0000aaa8       $stateUnwindMap$?Paint@CeFullPanelInfo@@QEAAXPEAUHWND__@@AEAUtagPAINTSTRUCT@@AEAUtagRECT@@@Z 0000000180031aa8     Display.obj
 0002:0000aab0       $ip2state$?Paint@CeFullPanelInfo@@QEAAXPEAUHWND__@@AEAUtagPAINTSTRUCT@@AEAUtagRECT@@@Z 0000000180031ab0     Display.obj
 0002:0000aad0       $unwind$?DrawItemText@CeFullPanelInfo@@QEAAHPEAUHDC__@@PEAUtagRECT@@1PEAUCePluginPanelItem@@PEB_WPEAUHBRUSH__@@H@Z 0000000180031ad0     Display.obj
 0002:0000aaf0       $unwind$?LoadItemColors@CeFullPanelInfo@@QEAAX_JPEAUCePluginPanelItem@@PEAUCePluginPanelItemColor@@HH@Z 0000000180031af0     Display.obj
 0002:0000ab08       $unwind$?FarItem2CeItem@CeFullPanelInfo@@QEAAH_JPEB_W1KU_FILETIME@@_KHPEAX3P6A_JXZ3K@Z 0000000180031b08     Display.obj
 0002:0000ab24       $unwind$?CheckDrawDibCreated@CImgCache@@IEAAHXZ 0000000180031b24     ImgCache.obj
 0002:0000ab24       $unwind$?CheckLoadDibCreated@CImgCache@@IEAAHXZ 0000000180031b24     ImgCache.obj
 0002:0000ab40       $unwind$?FindInCache@CImgCache@@IEAAHPEAUCePluginPanelItem@@PEAHI@Z 0000000180031b40     ImgCache.obj
 0002:0000ab58       $unwind$?LoadModules@CImgCache@@IEAAXXZ 0000000180031b58     ImgCache.obj
 0002:0000ab80       $unwind$?FreeModules@CImgCache@@IEAAXXZ 0000000180031b80     ImgCache.obj
 0002:0000ab8c       $unwind$??1CImgCache@@QEAA@XZ 0000000180031b8c     ImgCache.obj
 0002:0000aba0       $ip2state$??1CImgCache@@QEAA@XZ 0000000180031ba0     ImgCache.obj
 0002:0000aba8       $unwind$?RequestItem@CImgCache@@QEAAHPEAUCePluginPanelItem@@I@Z 0000000180031ba8     ImgCache.obj
 0002:0000abc0       $stateUnwindMap$?RequestItem@CImgCache@@QEAAHPEAUCePluginPanelItem@@I@Z 0000000180031bc0     ImgCache.obj
 0002:0000abc8       $ip2state$?RequestItem@CImgCache@@QEAAHPEAUCePluginPanelItem@@I@Z 0000000180031bc8     ImgCache.obj
 0002:0000abe0       $unwind$?PaintItem@CImgCache@@QEAAHPEAUHDC__@@HHHPEAUCePluginPanelItem@@PEAPEB_WPEAH@Z 0000000180031be0     ImgCache.obj
 0002:0000ac00       $unwind$?LoadThumbnail@CImgCache@@QEAAHPEAUIMAGE_CACHE_INFO@@@Z 0000000180031c00     ImgCache.obj
 0002:0000ac1c       $unwind$?LoadShellIcon@CImgCache@@QEAAHPEAUIMAGE_CACHE_INFO@@H@Z 0000000180031c1c     ImgCache.obj
 0002:0000ac3c       $unwind$?Lock@MSectionLockSimple@@QEAAHPEAUMSectionSimple@@K@Z 0000000180031c3c     common-kernel64:MSectionSimple.obj
 0002:0000ac3c       $unwind$?GetBuffer@CEStr@@QEAAPEA_W_J@Z 0000000180031c3c     common-kernel64:CEStr.obj
 0002:0000ac3c       $unwind$?InitializeQueue@?$CQueueProcessor@PEAUIMAGE_CACHE_INFO@@@@AEAAXH@Z 0000000180031c3c     ImgCache.obj
 0002:0000ac3c       $unwind$__TypeMatch        0000000180031c3c     libvcruntime:frame.obj
 0002:0000ac3c       $unwind$?WaitUnlocked@MSection@@IEAAXKK@Z 0000000180031c3c     common-kernel64:MSection.obj
 0002:0000ac3c       $unwind$_initterm          0000000180031c3c     libucrt:initterm.obj
 0002:0000ac3c       $unwind$?process@?$output_processor@_WV?$string_output_adapter@_W@__crt_stdio_output@@V?$standard_base@_WV?$string_output_adapter@_W@__crt_stdio_output@@@2@@__crt_stdio_output@@QEAAHXZ 0000000180031c3c     libucrt:output.obj
 0002:0000ac3c       $unwind$__acrt_initialize_stdio 0000000180031c3c     libucrt:_file.obj
 0002:0000ac3c       $unwind$__GSHandlerCheck_EH 0000000180031c3c     LIBCMT:gshandlereh.obj
 0002:0000ac54       $unwind$?FindOrCreate@?$CQueueProcessor@PEAUIMAGE_CACHE_INFO@@@@AEAAPEAUProcessingItem@1@AEBQEAUIMAGE_CACHE_INFO@@_J_NW4ProcessingPriority@@@Z 0000000180031c54     ImgCache.obj
 0002:0000ac78       $stateUnwindMap$?FindOrCreate@?$CQueueProcessor@PEAUIMAGE_CACHE_INFO@@@@AEAAPEAUProcessingItem@1@AEBQEAUIMAGE_CACHE_INFO@@_J_NW4ProcessingPriority@@@Z 0000000180031c78     ImgCache.obj
 0002:0000ac80       $ip2state$?FindOrCreate@?$CQueueProcessor@PEAUIMAGE_CACHE_INFO@@@@AEAAPEAUProcessingItem@1@AEBQEAUIMAGE_CACHE_INFO@@_J_NW4ProcessingPriority@@@Z 0000000180031c80     ImgCache.obj
 0002:0000ac98       $unwind$??0?$CQueueProcessor@PEAUIMAGE_CACHE_INFO@@@@QEAA@XZ 0000000180031c98     ImgCache.obj
 0002:0000acac       $stateUnwindMap$??0?$CQueueProcessor@PEAUIMAGE_CACHE_INFO@@@@QEAA@XZ 0000000180031cac     ImgCache.obj
 0002:0000acb8       $ip2state$??0?$CQueueProcessor@PEAUIMAGE_CACHE_INFO@@@@QEAA@XZ 0000000180031cb8     ImgCache.obj
 0002:0000acc8       $unwind$??1?$CQueueProcessor@PEAUIMAGE_CACHE_INFO@@@@UEAA@XZ 0000000180031cc8     ImgCache.obj
 0002:0000acd8       $ip2state$??1?$CQueueProcessor@PEAUIMAGE_CACHE_INFO@@@@UEAA@XZ 0000000180031cd8     ImgCache.obj
 0002:0000ace0       $unwind$?ProcessItem@?$CQueueProcessor@PEAUIMAGE_CACHE_INFO@@@@IEAAJPEAUProcessingItem@1@@Z 0000000180031ce0     ImgCache.obj
 0002:0000ad00       $unwind$?ProcessingStep@?$CQueueProcessor@PEAUIMAGE_CACHE_INFO@@@@IEAA_NXZ 0000000180031d00     ImgCache.obj
 0002:0000ad20       $stateUnwindMap$?ProcessingStep@?$CQueueProcessor@PEAUIMAGE_CACHE_INFO@@@@IEAA_NXZ 0000000180031d20     ImgCache.obj
 0002:0000ad28       $ip2state$?ProcessingStep@?$CQueueProcessor@PEAUIMAGE_CACHE_INFO@@@@IEAA_NXZ 0000000180031d28     ImgCache.obj
 0002:0000ad40       $unwind$?apiCreateThread@@YAPEAXP6AKPEAX@Z0PEAKPEBDH@Z 0000000180031d40     common-kernel64:WThreads.obj
 0002:0000ad40       $unwind$_invalid_parameter 0000000180031d40     libucrt:invalid_parameter.obj
 0002:0000ad40       $unwind$?StringCchVPrintfA@@YAJPEAD_KPEBD0@Z 0000000180031d40     common-kernel64:MStrSafe.obj
 0002:0000ad58       $unwind$?swprintf_c@@YAHPEA_W_JPEB_WZZ 0000000180031d58     common-kernel64:MStrSafe.obj
 0002:0000ad58       $unwind$?sprintf_c@@YAHPEAD_JPEBDZZ 0000000180031d58     common-kernel64:MStrSafe.obj
 0002:0000ad64       $unwind$?msprintf@@YAPEB_WPEA_W_KPEB_WZZ 0000000180031d64     common-kernel64:MStrSafe.obj
 0002:0000ad84       $unwind$?LoadAdvApi@MNullDesc@@IEAAHXZ 0000000180031d84     common-kernel64:MSecurity.obj
 0002:0000ad98       $unwind$?LocalSecurity@MNullDesc@@QEAAPEAU_SECURITY_ATTRIBUTES@@XZ 0000000180031d98     common-kernel64:MSecurity.obj
 0002:0000adb4       $unwind$?ExecuteOpenPipe@@YAPEAXPEB_WAEAY0CAI@_W0KKHPEAXH@Z 0000000180031db4     common-kernel64:ConEmuCheck.obj
 0002:0000adcc       $unwind$??$free_environment@_W@@YAXQEAPEA_W@Z 0000000180031dcc     libucrt:environment_initialization.obj
 0002:0000adcc       $unwind$??$free_environment@D@@YAXQEAPEAD@Z 0000000180031dcc     libucrt:environment_initialization.obj
 0002:0000adcc       $unwind$?ExecutePrepareCmd@@YAXPEAUCESERVER_REQ_HDR@@K_K@Z 0000000180031dcc     common-kernel64:ConEmuCheck.obj
 0002:0000adcc       $unwind$?ExecutePrepareCmd@@YAXPEAUCESERVER_REQ@@K_K@Z 0000000180031dcc     common-kernel64:ConEmuCheck.obj
 0002:0000add8       $unwind$?ExecuteGuiCmd@@YAPEAUCESERVER_REQ@@PEAUHWND__@@PEAU1@0H@Z 0000000180031dd8     common-kernel64:ConEmuCheck.obj
 0002:0000adf8       $unwind$?ExecuteCmd@@YAPEAUCESERVER_REQ@@PEB_WPEAU1@KPEAUHWND__@@HKH@Z 0000000180031df8     common-kernel64:ConEmuCheck.obj
 0002:0000ae1c       $unwind$?ModuleName@@YAPEB_WPEB_W@Z 0000000180031e1c     common-kernel64:ConEmuCheck.obj
 0002:0000ae30       $unwind$?isTerminalMode@@YA_NXZ 0000000180031e30     common-kernel64:MProcess.obj
 0002:0000ae48       $unwind$?Find@?$MToolHelp@UtagPROCESSENTRY32W@@$1?Process32FirstW@@YAHPEAXPEAU1@@Z$1?Process32NextW@@YAH01@Z@@QEAA_NP6A_NPEAUtagPROCESSENTRY32W@@_J@Z10@Z 0000000180031e48     common-kernel64:MProcess.obj
 0002:0000ae64       $unwind$?write_string@?$string_output_adapter@D@__crt_stdio_output@@QEBAXQEBDHQEAH1@Z 0000000180031e64     libucrt:output.obj
 0002:0000ae64       $unwind$??$parse_command_line@D@@YAXPEADPEAPEAD0PEA_K2@Z 0000000180031e64     libucrt:argv_parsing.obj
 0002:0000ae64       $unwind$?MyEnterCriticalSection@MSection@@IEAA_NK@Z 0000000180031e64     common-kernel64:MSection.obj
 0002:0000ae64       $unwind$?_GetRangeOfTrysToCheck@@YAPEBU_s_TryBlockMapEntry@@PEA_KPEBU_s_FuncInfo@@HHPEAI2PEAU_xDISPATCHER_CONTEXT@@@Z 0000000180031e64     libvcruntime:risctrnsctrl.obj
 0002:0000ae80       $unwind$?apiTerminateThreadEx@@YAHPEAXKPEBDH@Z 0000000180031e80     common-kernel64:WThreads.obj
 0002:0000ae9c       $unwind$?SetThreadName@@YAXKPEAD@Z 0000000180031e9c     common-kernel64:WThreads.obj
 0002:0000aebc       $unwind$?apiThreadHelper@@YAKPEAX@Z 0000000180031ebc     common-kernel64:WThreads.obj
 0002:0000aed0       $unwind$?FileExists@@YA_NPEB_WPEAK@Z 0000000180031ed0     common-kernel64:WObjects.obj
 0002:0000aef0       $unwind$?lstrmerge@@YAPEA_WPEB_W00000000@Z 0000000180031ef0     common-kernel64:MStrDup.obj
 0002:0000af10       $unwind$?RecreateAndLock@MSectionSimple@@QEAA_NXZ 0000000180031f10     common-kernel64:MSectionSimple.obj
 0002:0000af18       $unwind$??0CEStr@@QEAA@PEB_W00000000@Z 0000000180031f18     common-kernel64:CEStr.obj
 0002:0000af2c       $unwind$??1CRgnDetect@@QEAA@XZ 0000000180031f2c     common-user64:RgnDetect.obj
 0002:0000af40       $ip2state$??1CRgnDetect@@QEAA@XZ 0000000180031f40     common-user64:RgnDetect.obj
 0002:0000af48       $unwind$?PrepareTransparent@CRgnDetect@@QEAAXPEBUCEFAR_INFO_MAPPING@@PEBKPEBU_CONSOLE_SCREEN_BUFFER_INFO@@PEA_WPEAUtag_CharAttr@@HH@Z 0000000180031f48     common-user64:RgnDetect.obj
 0002:0000af70       $unwind$?x_ismbbtype_l@@YAHPEAU__crt_locale_pointers@@IHH@Z 0000000180031f70     libucrt:ismbbyte.obj
 0002:0000af70       $unwind$?PrepareTransparent@CRgnDetect@@QEAAXPEBUCEFAR_INFO_MAPPING@@PEBK@Z 0000000180031f70     common-user64:RgnDetect.obj
 0002:0000af80       $unwind$?OnWriteConsoleOutput@CRgnDetect@@QEAAXPEBU_CHAR_INFO@@U_COORD@@1PEAU_SMALL_RECT@@PEBK@Z 0000000180031f80     common-user64:RgnDetect.obj
 0002:0000af98       $unwind$?InitializeSBI@CRgnDetect@@QEAAHPEBK@Z 0000000180031f98     common-user64:RgnDetect.obj
 0002:0000afb0       $unwind$?DetectDialog@CRgnDetect@@IEAA_NPEA_WPEAUtag_CharAttr@@HHHHPEAH2@Z 0000000180031fb0     common-user64:RgnDetect.obj
 0002:0000afcc       $unwind$?FindDialog_Right@CRgnDetect@@IEAA_NPEA_WPEAUtag_CharAttr@@HHAEAH222AEA_N@Z 0000000180031fcc     common-user64:RgnDetect.obj
 0002:0000afcc       $unwind$?FindDialog_TopLeft@CRgnDetect@@IEAA_NPEA_WPEAUtag_CharAttr@@HHAEAH222AEA_N@Z 0000000180031fcc     common-user64:RgnDetect.obj
 0002:0000afcc       $unwind$__C_specific_handler 0000000180031fcc     libvcruntime:_riscchandler_.obj
 0002:0000afcc       $unwind$?FindDialog_TopRight@CRgnDetect@@IEAA_NPEA_WPEAUtag_CharAttr@@HHAEAH222AEA_N@Z 0000000180031fcc     common-user64:RgnDetect.obj
 0002:0000afcc       $unwind$?FindFrameLeft_ByTop@CRgnDetect@@IEAA_NPEA_WPEAUtag_CharAttr@@HHAEAH22@Z 0000000180031fcc     common-user64:RgnDetect.obj
 0002:0000afcc       $unwind$?FindFrameRight_ByTop@CRgnDetect@@IEAA_NPEA_WPEAUtag_CharAttr@@HHAEAH22@Z 0000000180031fcc     common-user64:RgnDetect.obj
 0002:0000afe8       $unwind$?FindDialog_Left@CRgnDetect@@IEAA_NPEA_WPEAUtag_CharAttr@@HHAEAH222AEA_N@Z 0000000180031fe8     common-user64:RgnDetect.obj
 0002:0000b000       $unwind$?FindDialog_Any@CRgnDetect@@IEAA_NPEA_WPEAUtag_CharAttr@@HHAEAH222AEA_N@Z 0000000180032000     common-user64:RgnDetect.obj
 0002:0000b018       $unwind$?FindDialog_Inner@CRgnDetect@@IEAA_NPEA_WPEAUtag_CharAttr@@HHAEAH2@Z 0000000180032018     common-user64:RgnDetect.obj
 0002:0000b030       $unwind$?FindFrame_TopLeft@CRgnDetect@@IEAA_NPEA_WPEAUtag_CharAttr@@HHAEAH222@Z 0000000180032030     common-user64:RgnDetect.obj
 0002:0000b04c       $unwind$?FindByBackground@CRgnDetect@@IEAA_NPEA_WPEAUtag_CharAttr@@HHAEAH222AEA_N@Z 000000018003204c     common-user64:RgnDetect.obj
 0002:0000b068       $unwind$?ExpandDialogFrame@CRgnDetect@@IEAA_NPEA_WPEAUtag_CharAttr@@HHAEAH2HH22@Z 0000000180032068     common-user64:RgnDetect.obj
 0002:0000b07c       $unwind$?MarkDialog@CRgnDetect@@IEAAHPEA_WPEAUtag_CharAttr@@HHHHHHI_NK@Z 000000018003207c     common-user64:RgnDetect.obj
 0002:0000b094       $unwind$?SearchAppPaths@@YA_NPEB_WAEAUCEStr@@_NPEAU1@@Z 0000000180032094     common-user64:WFiles.obj
 0002:0000b0bc       $stateUnwindMap$?SearchAppPaths@@YA_NPEB_WAEAUCEStr@@_NPEAU1@@Z 00000001800320bc     common-user64:WFiles.obj
 0002:0000b0c8       $ip2state$?SearchAppPaths@@YA_NPEB_WAEAUCEStr@@_NPEAU1@@Z 00000001800320c8     common-user64:WFiles.obj
 0002:0000b0e0       $unwind$__GSHandlerCheckCommon 00000001800320e0     LIBCMT:_gshandler_.obj
 0002:0000b0e8       $xdatasym                  00000001800320e8     LIBCMT:_amdsecgs_.obj
 0002:0000b0ec       $unwind$?dllmain_crt_process_attach@@YAHQEAUHINSTANCE__@@QEAX@Z 00000001800320ec     LIBCMT:dll_dllmain.obj
 0002:0000b128       $unwind$?dllmain_crt_process_detach@@YAH_N@Z 0000000180032128     LIBCMT:dll_dllmain.obj
 0002:0000b15c       $unwind$?dllmain_dispatch@@YAHQEAUHINSTANCE__@@KQEAX@Z 000000018003215c     LIBCMT:dll_dllmain.obj
 0002:0000b184       $unwind$?filt$0@?0??dllmain_dispatch@@YAHQEAUHINSTANCE__@@KQEAX@Z@4HA 0000000180032184     LIBCMT:dll_dllmain.obj
 0002:0000b18c       $unwind$_putwch_nolock     000000018003218c     libucrt:putwch.obj
 0002:0000b18c       $unwind$__report_gsfailure 000000018003218c     LIBCMT:gs_report.obj
 0002:0000b194       $unwind$capture_current_context 0000000180032194     LIBCMT:gs_report.obj
 0002:0000b1a0       $unwind$capture_previous_context 00000001800321a0     LIBCMT:gs_report.obj
 0002:0000b1ac       $unwind$__security_init_cookie 00000001800321ac     LIBCMT:gs_support.obj
 0002:0000b1b8       $unwind$__scrt_is_nonwritable_in_current_image 00000001800321b8     LIBCMT:utility.obj
 0002:0000b1d8       $unwind$__scrt_is_nonwritable_in_current_image$filt$0 00000001800321d8     LIBCMT:utility.obj
 0002:0000b1e0       $unwind$__scrt_initialize_onexit_tables 00000001800321e0     LIBCMT:utility.obj
 0002:0000b1ec       $unwind$__scrt_fastfail    00000001800321ec     LIBCMT:utility_desktop.obj
 0002:0000b1fc       $unwind$__isa_available_init 00000001800321fc     LIBCMT:_cpu_disp_.obj
 0002:0000b210       $xdatasym                  0000000180032210     LIBCMT:_guard_dispatch_.obj
 0002:0000b214       $unwind$?_GetEstablisherFrame@@YAPEA_KPEA_KPEAU_xDISPATCHER_CONTEXT@@PEBU_s_FuncInfo@@0@Z 0000000180032214     libvcruntime:risctrnsctrl.obj
 0002:0000b22c       $unwind$?__FrameUnwindToEmptyState@@YAXPEA_KPEAU_xDISPATCHER_CONTEXT@@PEBU_s_FuncInfo@@@Z 000000018003222c     libvcruntime:risctrnsctrl.obj
 0002:0000b240       $unwind$_CallSETranslator  0000000180032240     libvcruntime:risctrnsctrl.obj
 0002:0000b260       $unwind$_CallSETranslator$filt$0 0000000180032260     libvcruntime:risctrnsctrl.obj
 0002:0000b26c       $unwind$_UnwindNestedFrames 000000018003226c     libvcruntime:risctrnsctrl.obj
 0002:0000b280       $unwind$__CxxFrameHandler3 0000000180032280     libvcruntime:risctrnsctrl.obj
 0002:0000b290       $xdatasym                  0000000180032290     libvcruntime:memcmp.obj
 0002:0000b298       $xdatasym                  0000000180032298     libvcruntime:memcpy.obj
 0002:0000b2a0       $xdatasym                  00000001800322a0     libvcruntime:memset.obj
 0002:0000b2a4       $unwind$strrchr            00000001800322a4     libvcruntime:strrchr.obj
 0002:0000b2a4       $unwind$wcschr             00000001800322a4     libvcruntime:wcschr.obj
 0002:0000b2a4       $unwind$strchr             00000001800322a4     libvcruntime:strchr.obj
 0002:0000b2b0       $xdatasym                  00000001800322b0     libvcruntime:memchr.obj
 0002:0000b2b4       $unwind$__CxxCallCatchBlock 00000001800322b4     libvcruntime:frame.obj
 0002:0000b2f0       $unwind$__CxxCallCatchBlock$fin$1 00000001800322f0     libvcruntime:frame.obj
 0002:0000b2fc       $unwind$__BuildCatchObject 00000001800322fc     libvcruntime:frame.obj
 0002:0000b328       $unwind$__InternalCxxFrameHandler 0000000180032328     libvcruntime:frame.obj
 0002:0000b328       $unwind$_mbtowc_l          0000000180032328     libucrt:mbtowc.obj
 0002:0000b328       $unwind$__acrt_LCMapStringEx 0000000180032328     libucrt:winapi_thunks.obj
 0002:0000b340       $unwind$__FrameUnwindToState 0000000180032340     libvcruntime:frame.obj
 0002:0000b38c       $unwind$?FindHandler@@YAXPEAUEHExceptionRecord@@PEA_KPEAU_CONTEXT@@PEAU_xDISPATCHER_CONTEXT@@PEBU_s_FuncInfo@@EH1@Z 000000018003238c     libvcruntime:frame.obj
 0002:0000b3ac       $unwind$?CatchIt@@YAXPEAUEHExceptionRecord@@PEA_KPEAU_CONTEXT@@PEAU_xDISPATCHER_CONTEXT@@PEBU_s_FuncInfo@@PEBU_s_HandlerType@@PEBU_s_CatchableType@@PEBU_s_TryBlockMapEntry@@H1EE@Z 00000001800323ac     libvcruntime:frame.obj
 0002:0000b3c4       $unwind$?FindHandlerForForeignException@@YAXPEAUEHExceptionRecord@@PEA_KPEAU_CONTEXT@@PEAU_xDISPATCHER_CONTEXT@@PEBU_s_FuncInfo@@HH1@Z 00000001800323c4     libvcruntime:frame.obj
 0002:0000b3dc       $unwind$?try_get_function@@YAPEAXW4function_id@?A0x63058377@@QEBDQEBW4module_id@2@2@Z 00000001800323dc     libucrt:winapi_thunks.obj
 0002:0000b3dc       $unwind$?try_get_function@@YAPEAXW4function_id@?A0x89697e75@@QEBDQEBW4module_id@2@2@Z 00000001800323dc     libvcruntime:winapi_downlevel.obj
 0002:0000b3dc       $unwind$?write_string@?$string_output_adapter@_W@__crt_stdio_output@@QEBAXQEB_WHQEAH1@Z 00000001800323dc     libucrt:output.obj
 0002:0000b3dc       $unwind$?IsInExceptionSpec@@YAEPEAUEHExceptionRecord@@PEBU_s_ESTypeList@@@Z 00000001800323dc     libvcruntime:frame.obj
 0002:0000b3f8       $unwind$__BuildCatchObjectHelper 00000001800323f8     libvcruntime:frame.obj
 0002:0000b438       $xdatasym                  0000000180032438     libvcruntime:_jmpuwind_.obj
 0002:0000b44c       $unwind$__vcrt_initialize_winapi_thunks 000000018003244c     libvcruntime:winapi_downlevel.obj
 0002:0000b44c       $unwind$__acrt_initialize_winapi_thunks 000000018003244c     libucrt:winapi_thunks.obj
 0002:0000b454       $unwind$__vcrt_uninitialize_winapi_thunks 0000000180032454     libvcruntime:winapi_downlevel.obj
 0002:0000b460       $xdatasym                  0000000180032460     libvcruntime:handlers.obj
 0002:0000b468       $unwind$__DestructExceptionObject 0000000180032468     libvcruntime:ehhelpers.obj
 0002:0000b488       $unwind$?initialize_stdio_handles_nolock@@YAXXZ 0000000180032488     libucrt:ioinit.obj
 0002:0000b488       $unwind$_free_osfhnd       0000000180032488     libucrt:osfinfo.obj
 0002:0000b488       $unwind$__std_exception_copy 0000000180032488     libvcruntime:std_exception.obj
 0002:0000b49c       $unwind$_CxxThrowException 000000018003249c     libvcruntime:throw.obj
 0002:0000b4ac       $unwind$__stdio_common_vsprintf 00000001800324ac     libucrt:output.obj
 0002:0000b4ac       $unwind$__stdio_common_vswprintf 00000001800324ac     libucrt:output.obj
 0002:0000b4d0       $unwind$?process@?$output_processor@DV?$string_output_adapter@D@__crt_stdio_output@@V?$standard_base@DV?$string_output_adapter@D@__crt_stdio_output@@@2@@__crt_stdio_output@@QEAAHXZ 00000001800324d0     libucrt:output.obj
 0002:0000b4e0       $unwind$?parse_int_from_format_string@?$output_processor@DV?$string_output_adapter@D@__crt_stdio_output@@V?$standard_base@DV?$string_output_adapter@D@__crt_stdio_output@@@2@@__crt_stdio_output@@AEAA_NQEAH@Z 00000001800324e0     libucrt:output.obj
 0002:0000b4f4       $unwind$?state_case_type@?$output_processor@DV?$string_output_adapter@D@__crt_stdio_output@@V?$standard_base@DV?$string_output_adapter@D@__crt_stdio_output@@@2@@__crt_stdio_output@@AEAA_NXZ 00000001800324f4     libucrt:output.obj
 0002:0000b50c       $unwind$?type_case_a@?$output_processor@DV?$string_output_adapter@D@__crt_stdio_output@@V?$standard_base@DV?$string_output_adapter@D@__crt_stdio_output@@@2@@__crt_stdio_output@@AEAA_NXZ 000000018003250c     libucrt:output.obj
 0002:0000b518       $unwind$?write_stored_string_tchar@?$output_processor@DV?$string_output_adapter@D@__crt_stdio_output@@V?$standard_base@DV?$string_output_adapter@D@__crt_stdio_output@@@2@@__crt_stdio_output@@AEAA_ND@Z 0000000180032518     libucrt:output.obj
 0002:0000b530       $unwind$?state_case_type@?$output_processor@_WV?$string_output_adapter@_W@__crt_stdio_output@@V?$standard_base@_WV?$string_output_adapter@_W@__crt_stdio_output@@@2@@__crt_stdio_output@@AEAA_NXZ 0000000180032530     libucrt:output.obj
 0002:0000b554       $unwind$?type_case_c_tchar@?$output_processor@_WV?$string_output_adapter@_W@__crt_stdio_output@@V?$standard_base@_WV?$string_output_adapter@_W@__crt_stdio_output@@@2@@__crt_stdio_output@@AEAA_N_W@Z 0000000180032554     libucrt:output.obj
 0002:0000b564       $unwind$?type_case_a@?$output_processor@_WV?$string_output_adapter@_W@__crt_stdio_output@@V?$standard_base@_WV?$string_output_adapter@_W@__crt_stdio_output@@@2@@__crt_stdio_output@@AEAA_NXZ 0000000180032564     libucrt:output.obj
 0002:0000b574       $unwind$?write_stored_string_tchar@?$output_processor@_WV?$string_output_adapter@_W@__crt_stdio_output@@V?$standard_base@_WV?$string_output_adapter@_W@__crt_stdio_output@@@2@@__crt_stdio_output@@AEAA_N_W@Z 0000000180032574     libucrt:output.obj
 0002:0000b588       $unwind$??$write_multiple_characters@V?$string_output_adapter@_W@__crt_stdio_output@@D@__crt_stdio_output@@YAXAEBV?$string_output_adapter@_W@0@DHQEAH@Z 0000000180032588     libucrt:output.obj
 0002:0000b594       $unwind$??$parse_integer@KV?$c_string_character_source@D@__crt_strtox@@@__crt_strtox@@YAKQEAU__crt_locale_pointers@@V?$c_string_character_source@D@0@H_N@Z 0000000180032594     libucrt:strtox.obj
 0002:0000b5b0       $unwind$??$parse_integer@KV?$c_string_character_source@_W@__crt_strtox@@@__crt_strtox@@YAKQEAU__crt_locale_pointers@@V?$c_string_character_source@_W@0@H_N@Z 00000001800325b0     libucrt:strtox.obj
 0002:0000b5cc       $unwind$?common_exit@@YAXHW4_crt_exit_cleanup_mode@@W4_crt_exit_return_mode@@@Z 00000001800325cc     libucrt:exit.obj
 0002:0000b60c       $unwind$_configure_narrow_argv 000000018003260c     libucrt:argv_parsing.obj
 0002:0000b620       $unwind$_execute_onexit_table 0000000180032620     libucrt:onexit.obj
 0002:0000b628       $unwind$??$?RV<lambda_e24bbb7b643b32fcea6fa61b31d4c984>@@AEAV<lambda_275893d493268fdec8709772e3fcec0e>@@V<lambda_9d71df4d7cf3f480f8d633942495c3b0>@@@?$__crt_seh_guarded_call@H@@QEAAH$$QEAV<lambda_e24bbb7b643b32fcea6fa61b31d4c984>@@AEAV<lambda_275893d493268fdec8709772e3fcec0e>@@$$QEAV<lambda_9d71df4d7cf3f480f8d633942495c3b0>@@@Z 0000000180032628     libucrt:onexit.obj
 0002:0000b658       $unwind$terminate          0000000180032658     libucrt:terminate.obj
 0002:0000b678       $xdatasym                  0000000180032678     libucrt:strncmp.obj
 0002:0000b67c       $unwind$__acrt_call_reportfault 000000018003267c     libucrt:invalid_parameter.obj
 0002:0000b69c       $unwind$_isleadbyte_l      000000018003269c     libucrt:_wctype.obj
 0002:0000b69c       $unwind$?getSystemCP@@YAHH@Z 000000018003269c     libucrt:mbctype.obj
 0002:0000b69c       $unwind$isdigit            000000018003269c     libucrt:_ctype.obj
 0002:0000b6a4       $unwind$_tolower_l         00000001800326a4     libucrt:tolower_toupper.obj
 0002:0000b6b4       $unwind$_wctomb_s_l        00000001800326b4     libucrt:wctomb.obj
 0002:0000b6c4       $unwind$strnlen            00000001800326c4     libucrt:strnlen.obj
 0002:0000b6c4       $unwind$wcsnlen            00000001800326c4     libucrt:strnlen.obj
 0002:0000b6cc       $unwind$?construct_ptd_array@@YAXQEAU__acrt_ptd@@@Z 00000001800326cc     libucrt:per_thread_data.obj
 0002:0000b6d4       $unwind$?destroy_ptd_array@@YAXQEAU__acrt_ptd@@@Z 00000001800326d4     libucrt:per_thread_data.obj
 0002:0000b6dc       $unwind$??$?RV<lambda_72d1df2b273a38828b1ce30cbf4cdab5>@@AEAV<lambda_876a65b173b8412d3a47c70a915b0cf4>@@V<lambda_41932305e351933ebe8f8be3ed8bb5dc>@@@?$__crt_seh_guarded_call@X@@QEAAX$$QEAV<lambda_72d1df2b273a38828b1ce30cbf4cdab5>@@AEAV<lambda_876a65b173b8412d3a47c70a915b0cf4>@@$$QEAV<lambda_41932305e351933ebe8f8be3ed8bb5dc>@@@Z 00000001800326dc     libucrt:per_thread_data.obj
 0002:0000b700       $unwind$??$?RV<lambda_5e887d1dcbef67a5eb4283622ba103bf>@@AEAV<lambda_4466841279450cc726390878d4a41900>@@V<lambda_341c25c0346d94847f1f3c463c57e077>@@@?$__crt_seh_guarded_call@X@@QEAAX$$QEAV<lambda_5e887d1dcbef67a5eb4283622ba103bf>@@AEAV<lambda_4466841279450cc726390878d4a41900>@@$$QEAV<lambda_341c25c0346d94847f1f3c463c57e077>@@@Z 0000000180032700     libucrt:per_thread_data.obj
 0002:0000b724       $unwind$??$?RV<lambda_46352004c1216016012b18bd6f87e700>@@AEAV<lambda_3bd07e1a1191394380780325891bf33f>@@V<lambda_334532d3f185bcaa59b5be82d7d22bff>@@@?$__crt_seh_guarded_call@X@@QEAAX$$QEAV<lambda_46352004c1216016012b18bd6f87e700>@@AEAV<lambda_3bd07e1a1191394380780325891bf33f>@@$$QEAV<lambda_334532d3f185bcaa59b5be82d7d22bff>@@@Z 0000000180032724     libucrt:per_thread_data.obj
 0002:0000b748       $unwind$??$?RV<lambda_fb3a7dec4e47f37f22dae91bb15c9095>@@AEAV<lambda_698284760c8add0bfb0756c19673e34b>@@V<lambda_dfb8eca1e75fef3034a8fb18dd509707>@@@?$__crt_seh_guarded_call@X@@QEAAX$$QEAV<lambda_fb3a7dec4e47f37f22dae91bb15c9095>@@AEAV<lambda_698284760c8add0bfb0756c19673e34b>@@$$QEAV<lambda_dfb8eca1e75fef3034a8fb18dd509707>@@@Z 0000000180032748     libucrt:per_thread_data.obj
 0002:0000b76c       $unwind$__acrt_fp_format   000000018003276c     libucrt:cvt.obj
 0002:0000b788       $unwind$?fp_format_nan_or_infinity@@YAHW4__acrt_fp_class@@_NPEAD_K1@Z 0000000180032788     libucrt:cvt.obj
 0002:0000b79c       $unwind$?fp_format_e_internal@@YAHQEAD_KH_NIQEAU_strflt@@2QEAU__crt_locale_pointers@@@Z 000000018003279c     libucrt:cvt.obj
 0002:0000b7b4       $unwind$?fp_format_e@@YAHQEBNQEAD_K12H_NIQEAU__crt_locale_pointers@@@Z 00000001800327b4     libucrt:cvt.obj
 0002:0000b7c8       $unwind$?fp_format_a@@YAHQEBNPEAD_KQEAD2H_NIQEAU__crt_locale_pointers@@@Z 00000001800327c8     libucrt:cvt.obj
 0002:0000b7e4       $unwind$__dcrt_get_narrow_environment_from_os 00000001800327e4     libucrt:get_environment_from_os.obj
 0002:0000b7e4       $unwind$?fp_format_f_internal@@YAHQEAD_KHQEAU_strflt@@_NQEAU__crt_locale_pointers@@@Z 00000001800327e4     libucrt:cvt.obj
 0002:0000b7fc       $unwind$?fp_format_g@@YAHQEBNQEAD_K12H_NIQEAU__crt_locale_pointers@@@Z 00000001800327fc     libucrt:cvt.obj
 0002:0000b810       $unwind$__acrt_uninitialize_locale 0000000180032810     libucrt:wsetlocale.obj
 0002:0000b830       $unwind$__acrt_initialize_lowio 0000000180032830     libucrt:ioinit.obj
 0002:0000b850       $unwind$?initialize_inherited_file_handles_nolock@@YAXXZ 0000000180032850     libucrt:ioinit.obj
 0002:0000b86c       $unwind$iswctype           000000018003286c     libucrt:iswctype.obj
 0002:0000b86c       $unwind$__acrt_is_packaged_app 000000018003286c     libucrt:winapi_thunks.obj
 0002:0000b878       $unwind$_isctype_l         0000000180032878     libucrt:isctype.obj
 0002:0000b894       $unwind$??$common_expand_argv_wildcards@D@@YAHQEAPEADQEAPEAPEAD@Z 0000000180032894     libucrt:argv_wildcards.obj
 0002:0000b8ac       $unwind$??$expand_argument_wildcards@D@@YAHQEAD0AEAV?$argument_list@D@?A0xca0879c4@@@Z 00000001800328ac     libucrt:argv_wildcards.obj
 0002:0000b8cc       $unwind$__acrt_update_thread_multibyte_data 00000001800328cc     libucrt:mbctype.obj
 0002:0000b8f0       $unwind$_setmbcp_nolock    00000001800328f0     libucrt:mbctype.obj
 0002:0000b910       $unwind$?setSBUpLow@@YAXPEAU__crt_multibyte_data@@@Z 0000000180032910     libucrt:mbctype.obj
 0002:0000b92c       $unwind$?setmbcp_internal@@YAHH_N@Z 000000018003292c     libucrt:mbctype.obj
 0002:0000b93c       $unwind$??$?RV<lambda_99476a1ad63dd22509b5d3e65b0ffc95>@@AEAV<lambda_ad1ced32f4ac17aa236e5ef05d6b3b7c>@@V<lambda_f7424dd8d45958661754dc4f2697e9c3>@@@?$__crt_seh_guarded_call@X@@QEAAX$$QEAV<lambda_99476a1ad63dd22509b5d3e65b0ffc95>@@AEAV<lambda_ad1ced32f4ac17aa236e5ef05d6b3b7c>@@$$QEAV<lambda_f7424dd8d45958661754dc4f2697e9c3>@@@Z 000000018003293c     libucrt:mbctype.obj
 0002:0000b960       $unwind$_query_new_handler 0000000180032960     libucrt:new_handler.obj
 0002:0000b980       $unwind$__acrt_get_sigabrt_handler 0000000180032980     libucrt:signal.obj
 0002:0000b988       $unwind$raise              0000000180032988     libucrt:signal.obj
 0002:0000b9b4       $unwind$??$?RV<lambda_c36588078e9f5dfd39652860aa6b3aaf>@@AEAV<lambda_ec61778202f4f5fc7e7711acc23c3bca>@@V<lambda_dc9d2797ccde5d239b4a0efae8ebd7db>@@@?$__crt_seh_guarded_call@P6AXH@Z@@QEAAP6AXH@Z$$QEAV<lambda_c36588078e9f5dfd39652860aa6b3aaf>@@AEAV<lambda_ec61778202f4f5fc7e7711acc23c3bca>@@$$QEAV<lambda_dc9d2797ccde5d239b4a0efae8ebd7db>@@@Z 00000001800329b4     libucrt:signal.obj
 0002:0000b9d8       $unwind$__acrt_LCMapStringA 00000001800329d8     libucrt:lcmapstringa.obj
 0002:0000b9e8       $unwind$?__acrt_LCMapStringA_stat@@YAHPEAU__crt_locale_pointers@@PEB_WKPEBDHPEADHHH@Z 00000001800329e8     libucrt:lcmapstringa.obj
 0002:0000ba10       $unwind$__acrt_update_thread_locale_data 0000000180032a10     libucrt:locale_refcounting.obj
 0002:0000ba34       $unwind$__acrt_fltout      0000000180032a34     libucrt:cfout.obj
 0002:0000ba54       $unwind$?divide@__crt_strtox@@YA_KAEAUbig_integer@1@AEBU21@@Z 0000000180032a54     libucrt:cfout.obj
 0002:0000ba74       $chain$5$?divide@__crt_strtox@@YA_KAEAUbig_integer@1@AEBU21@@Z 0000000180032a74     libucrt:cfout.obj
 0002:0000ba88       $chain$6$?divide@__crt_strtox@@YA_KAEAUbig_integer@1@AEBU21@@Z 0000000180032a88     libucrt:cfout.obj
 0002:0000ba98       $unwind$_fcloseall         0000000180032a98     libucrt:closeall.obj
 0002:0000babc       $unwind$common_flush_all   0000000180032abc     libucrt:fflush.obj
 0002:0000baf8       $unwind$__acrt_locale_free_monetary 0000000180032af8     libucrt:initmon.obj
 0002:0000bb00       $unwind$__acrt_locale_free_time 0000000180032b00     libucrt:inittime.obj
 0002:0000bb10       $unwind$__acrt_GetStringTypeA 0000000180032b10     libucrt:getstringtypea.obj
 0002:0000bb38       $unwind$__acrt_lowio_destroy_handle_array 0000000180032b38     libucrt:osfinfo.obj
 0002:0000bb48       $unwind$__acrt_lowio_ensure_fh_exists 0000000180032b48     libucrt:osfinfo.obj
 0002:0000bb74       $unwind$?GetTableIndexFromLocaleName@@YAHPEB_W@Z 0000000180032b74     libucrt:lcidtoname_downlevel.obj
 0002:0000bb8c       $unwind$qsort              0000000180032b8c     libucrt:qsort.obj
 0002:0000bba4       $chain$4$qsort             0000000180032ba4     libucrt:qsort.obj
 0002:0000bbc8       $chain$5$qsort             0000000180032bc8     libucrt:qsort.obj
 0002:0000bbd8       $unwind$?shortsort@@YAXPEAD0_KP6AHPEBX2@Z@Z 0000000180032bd8     libucrt:qsort.obj
 0002:0000bbe8       $chain$2$?shortsort@@YAXPEAD0_KP6AHPEBX2@Z@Z 0000000180032be8     libucrt:qsort.obj
 0002:0000bc04       $chain$3$?shortsort@@YAXPEAD0_KP6AHPEBX2@Z@Z 0000000180032c04     libucrt:qsort.obj
 0002:0000bc14       $unwind$_mbsdec_l          0000000180032c14     libucrt:mbsdec.obj
 0002:0000bc20       $xdatasym                  0000000180032c20     libucrt:log10.obj
 0002:0000bc2c       $unwind$_write             0000000180032c2c     libucrt:write.obj
 0002:0000bc5c       $unwind$_write_nolock      0000000180032c5c     libucrt:write.obj
 0002:0000bc74       $unwind$?write_double_translated_ansi_nolock@@YA?AUwrite_result@?A0x9c548279@@HQEBDI@Z 0000000180032c74     libucrt:write.obj
 0002:0000bc94       $unwind$?write_text_ansi_nolock@@YA?AUwrite_result@?A0x9c548279@@HQEBDI@Z 0000000180032c94     libucrt:write.obj
 0002:0000bc94       $unwind$?write_text_utf16le_nolock@@YA?AUwrite_result@?A0x9c548279@@HQEBDI@Z 0000000180032c94     libucrt:write.obj
 0002:0000bcb4       $unwind$?write_text_utf8_nolock@@YA?AUwrite_result@?A0x9c548279@@HQEBDI@Z 0000000180032cb4     libucrt:write.obj
 0002:0000bcd8       $unwind$fclose             0000000180032cd8     libucrt:fclose.obj
 0002:0000bcfc       $unwind$_close             0000000180032cfc     libucrt:close.obj
 0002:0000bcfc       $unwind$_commit            0000000180032cfc     libucrt:commit.obj
 0002:0000bd04       $unwind$??$?RV<lambda_b521505b218e5242e90febf6bfebc422>@@AEAV<lambda_6978c1fb23f02e42e1d9e99668cc68aa>@@V<lambda_314360699dd331753a4119843814e9a7>@@@?$__crt_seh_guarded_call@H@@QEAAH$$QEAV<lambda_b521505b218e5242e90febf6bfebc422>@@AEAV<lambda_6978c1fb23f02e42e1d9e99668cc68aa>@@$$QEAV<lambda_314360699dd331753a4119843814e9a7>@@@Z 0000000180032d04     libucrt:commit.obj
 0002:0000bd28       $unwind$common_control87   0000000180032d28     libucrt:ieee.obj
 0002:0000bd58       $unwind$_handle_error      0000000180032d58     libucrt:libm_error.obj
 0002:0000bd78       $unwind$__acrt_initialize_fma3 0000000180032d78     libucrt:fma3_available.obj
 0002:0000bd80       $unwind$_log_special_common 0000000180032d80     libucrt:log_special.obj
 0002:0000bd8c       $unwind$??$?RV<lambda_bfedae4ebbf01fab1bb6dcc6a9e276e0>@@AEAV<lambda_2fe9b910cf3cbf4a0ab98a02ba45b3ec>@@V<lambda_237c231691f317818eb88cc1d5d642d6>@@@?$__crt_seh_guarded_call@H@@QEAAH$$QEAV<lambda_bfedae4ebbf01fab1bb6dcc6a9e276e0>@@AEAV<lambda_2fe9b910cf3cbf4a0ab98a02ba45b3ec>@@$$QEAV<lambda_237c231691f317818eb88cc1d5d642d6>@@@Z 0000000180032d8c     libucrt:close.obj
 0002:0000bdb0       $xdatasym                  0000000180032db0     libucrt:fpsr.obj
 0002:0000bdb8       $unwind$_raise_exc         0000000180032db8     libucrt:fpexcept.obj
 0002:0000bdb8       $unwind$__dcrt_lowio_initialize_console_output 0000000180032db8     libucrt:initcon.obj
 0002:0000bdc0       $unwind$_raise_exc_ex      0000000180032dc0     libucrt:fpexcept.obj
 0002:0000bdd4       $unwind$_ctrlfp            0000000180032dd4     libucrt:fpctrl.obj
 0002:0000bdfc       $unwind$_IsNonwritableInCurrentImage 0000000180032dfc     LIBCMT:pesect.obj
 0002:0000be20       $xdatasym                  0000000180032e20     LIBCMT:_chkstk_.obj
 0002:0000beb0       .edata                     0000000180032eb0     ConEmuTh.x64.exp
 0002:0000bed8       rgpv                       0000000180032ed8     ConEmuTh.x64.exp
 0002:0000bf0c       rgszName                   0000000180032f0c     ConEmuTh.x64.exp
 0002:0000bf40       rgwOrd                     0000000180032f40     ConEmuTh.x64.exp
 0002:0000bf5a       szName                     0000000180032f5a     ConEmuTh.x64.exp
 0002:0000bf6b       $N00001                    0000000180032f6b     ConEmuTh.x64.exp
 0002:0000bf7a       $N00002                    0000000180032f7a     ConEmuTh.x64.exp
 0002:0000bf80       $N00003                    0000000180032f80     ConEmuTh.x64.exp
 0002:0000bf88       $N00004                    0000000180032f88     ConEmuTh.x64.exp
 0002:0000bf91       $N00005                    0000000180032f91     ConEmuTh.x64.exp
 0002:0000bfa0       $N00006                    0000000180032fa0     ConEmuTh.x64.exp
 0002:0000bfb1       $N00007                    0000000180032fb1     ConEmuTh.x64.exp
 0002:0000bfc3       $N00008                    0000000180032fc3     ConEmuTh.x64.exp
 0002:0000bfd1       $N00009                    0000000180032fd1     ConEmuTh.x64.exp
 0002:0000bfdc       $N00010                    0000000180032fdc     ConEmuTh.x64.exp
 0002:0000bfe8       $N00011                    0000000180032fe8     ConEmuTh.x64.exp
 0002:0000bffd       $N00012                    0000000180032ffd     ConEmuTh.x64.exp
 0002:0000c00c       $N00013                    000000018003300c     ConEmuTh.x64.exp
 0002:0000c762       .idata$6                   0000000180033762     version:VERSION.dll
 0002:0000ca94       .idata$6                   0000000180033a94     kernel32:KERNEL32.dll
 0002:0000cd28       .idata$6                   0000000180033d28     user32:USER32.dll
 0002:0000ce7a       .idata$6                   0000000180033e7a     gdi32:GDI32.dll
 0002:0000ceda       .idata$6                   0000000180033eda     advapi32:ADVAPI32.dll
 0002:0000cefa       .idata$6                   0000000180033efa     shell32:SHELL32.dll
 0002:0000cf28       .idata$6                   0000000180033f28     ole32:ole32.dll
 0003:00000100       ?__vcrt_flsindex@@3KA      0000000180035100     libvcruntime:per_thread_data.obj
 0003:00000120       errno_no_memory            0000000180035120     libucrt:errno.obj
 0003:00000124       doserrno_no_memory         0000000180035124     libucrt:errno.obj
 0003:00000128       __acrt_flsindex            0000000180035128     libucrt:per_thread_data.obj
 0003:000005f0       __rgctypeflag              00000001800355f0     libucrt:mbctype.obj
 0003:00000600       __rgcode_page_info         0000000180035600     libucrt:mbctype.obj
 0003:000009b0       ?dazSupported@?1??common_control87@@9@9 00000001800359b0     libucrt:ieee.obj
 0003:000009c0       ?dazSupported@?1??_ctrlfp@@9@9 00000001800359c0     libucrt:fpctrl.obj
 0003:00021a58       ?sbInClearing@?1??ProcessConsoleInput@@YAHHPEAU_INPUT_RECORD@@KPEAK@Z@4_NA 0000000180056a58     ConEmuTh.obj
 0003:00021a80       ?szMenu@?1??GetPluginInfoW1900@@YAXPEAX@Z@4PAPEA_WA 0000000180056a80     ConEmuTh1900.obj
 0003:00021a90       ?szMenu1@?1??GetPluginInfoW1900@@YAXPEAX@Z@4PA_WA 0000000180056a90     ConEmuTh1900.obj
 0003:00021ca0       ?szMenu@?1??GetPluginInfoW2800@@YAXPEAX@Z@4PAPEA_WA 0000000180056ca0     ConEmuTh2800.obj
 0003:00021cb0       ?szMenu1@?1??GetPluginInfoW2800@@YAXPEAX@Z@4PA_WA 0000000180056cb0     ConEmuTh2800.obj
 0003:00021ec0       ?gszRootKeyW995@@3PEA_WEA  0000000180056ec0     ConEmuTh995.obj
 0003:00021ec8       ?szMenu@?1??GetPluginInfoW995@@YAXPEAX@Z@4PAPEA_WA 0000000180056ec8     ConEmuTh995.obj
 0003:00021ed0       ?szMenu1@?1??GetPluginInfoW995@@YAXPEAX@Z@4PA_WA 0000000180056ed0     ConEmuTh995.obj
 0003:000220e0       ?gszRootKeyA@@3PEA_WEA     00000001800570e0     ConEmuThA.obj
 0003:000220e8       ?szMenu@?1??GetPluginInfo@@9@4PAPEADA 00000001800570e8     ConEmuThA.obj
 0003:000220f0       ?szMenu1@?1??GetPluginInfo@@9@4PADA 00000001800570f0     ConEmuThA.obj
 0003:00022210       ?hClass@@3GA               0000000180057210     Display.obj
 0003:00022260       ?szFile@?1??ModuleName@@YAPEB_WPEB_W@Z@4PA_WA 0000000180057260     common-kernel64:ConEmuCheck.obj
 0003:000222a0       ?TerminalMode@?1??isTerminalMode@@YA_NXZ@4_NA 00000001800572a0     common-kernel64:MProcess.obj
 0003:000222a1       ?TerminalChecked@?1??isTerminalMode@@YA_NXZ@4_NA 00000001800572a1     common-kernel64:MProcess.obj
 0003:000222c0       ?g_Threads@@3PAUConEmuThreadInfo@@A 00000001800572c0     common-kernel64:WThreads.obj
 0003:0002aac0       ?gh_UnknownTerminatedThread@@3PEAXEA 000000018005fac0     common-kernel64:WThreads.obj
 0003:0002aad0       ?rtlVerifyVersionInfo@?1??_VerifyVersionInfo@@YA_NPEAU_OSVERSIONINFOEXW@@K_K@Z@4P6AH0K1@ZEA 000000018005fad0     common-kernel64:WObjects.obj
 0003:0002aad8       ?hasRtl@?1??_VerifyVersionInfo@@YA_NPEAU_OSVERSIONINFOEXW@@K_K@Z@4HA 000000018005fad8     common-kernel64:WObjects.obj
 0003:0002aadc       ?is64bitOs@?1??IsWindows64@@YA_NXZ@4_NA 000000018005fadc     common-kernel64:WObjects.obj
 0003:0002aadd       ?isOsChecked@?1??IsWindows64@@YA_NXZ@4_NA 000000018005fadd     common-kernel64:WObjects.obj
 0003:0002aade       ?gbInTransparentAssert@@3_NA 000000018005fade     common-user64:RgnDetect.obj
 0003:0002aae0       ?__proc_attached@@3HA      000000018005fae0     LIBCMT:dll_dllmain.obj
 0003:0002aaf0       GS_ExceptionRecord         000000018005faf0     LIBCMT:gs_report.obj
 0003:0002ab90       GS_ContextRecord           000000018005fb90     LIBCMT:gs_report.obj
 0003:0002b07c       ?module_local_atexit_table_initialized@@3_NA 000000018006007c     LIBCMT:utility.obj
 0003:0002b088       ?module_local_atexit_table@@3U_onexit_table_t@@A 0000000180060088     LIBCMT:utility.obj
 0003:0002b0a0       ?module_local_at_quick_exit_table@@3U_onexit_table_t@@A 00000001800600a0     LIBCMT:utility.obj
 0003:0002b0b8       ?is_initialized_as_dll@@3_NA 00000001800600b8     LIBCMT:utility.obj
 0003:0002b0d0       ?__vcrt_startup_thread_ptd@@3U__vcrt_ptd@@A 00000001800600d0     libvcruntime:per_thread_data.obj
 0003:0002b188       ?heap@@3V_HeapManager@@A   0000000180060188     libvcruntime:undname.obj
 0003:0002b1b0       __vcrt_lock_table          00000001800601b0     libvcruntime:locks.obj
 0003:0002b1d8       __vcrt_locks_initialized   00000001800601d8     libvcruntime:locks.obj
 0003:0002b1e0       ?module_handles@@3PAPEAUHINSTANCE__@@A 00000001800601e0     libvcruntime:winapi_downlevel.obj
 0003:0002b1f8       ?encoded_function_pointers@@3PAPEAXA 00000001800601f8     libvcruntime:winapi_downlevel.obj
 0003:0002b230       c_termination_complete     0000000180060230     libucrt:exit.obj
 0003:0002b238       thread_local_exit_callback_func 0000000180060238     libucrt:exit.obj
 0003:0002b240       ?c_exit_complete@?5??common_exit@@YAXHW4_crt_exit_cleanup_mode@@W4_crt_exit_return_mode@@@Z@4_NA 0000000180060240     libucrt:exit.obj
 0003:0002b250       ?program_name@?5???$common_configure_argv@D@@YAHW4_crt_argv_mode@@@Z@4PADA 0000000180060250     libucrt:argv_parsing.obj
 0003:0002b3a8       __acrt_invalid_parameter_handler 00000001800603a8     libucrt:invalid_parameter.obj
 0003:0002b3c0       enable_percent_n           00000001800603c0     libucrt:printf_count_output.obj
 0003:0002b800       __acrt_lock_table          0000000180060800     libucrt:locks.obj
 0003:0002ba08       __acrt_locks_initialized   0000000180060a08     libucrt:locks.obj
 0003:0002ba10       module_handles             0000000180060a10     libucrt:winapi_thunks.obj
 0003:0002bab0       encoded_function_pointers  0000000180060ab0     libucrt:winapi_thunks.obj
 0003:0002bbb0       ?state_cache@?1??__acrt_is_packaged_app@@9@4JA 0000000180060bb0     libucrt:winapi_thunks.obj
 0003:0002bbcc       fSystemSet                 0000000180060bcc     libucrt:mbctype.obj
 0003:0002bbd8       ?initialized@?1??__acrt_initialize_multibyte@@9@4_NA 0000000180060bd8     libucrt:mbctype.obj
 0003:0002bc10       __acrt_new_handler         0000000180060c10     libucrt:new_handler.obj
 0003:0002bc18       ctrlc_action               0000000180060c18     libucrt:signal.obj
 0003:0002bc20       ctrlbreak_action           0000000180060c20     libucrt:signal.obj
 0003:0002bc28       abort_action               0000000180060c28     libucrt:signal.obj
 0003:0002bc30       term_action                0000000180060c30     libucrt:signal.obj
 0003:0002bc38       user_matherr               0000000180060c38     libucrt:matherr.obj
 0003:0002bc40       __acrt_global_new_mode     0000000180060c40     libucrt:new_mode.obj
 0003:0002bc4c       __acrt_app_type            0000000180060c4c     libucrt:report_runtime_error.obj
 0004:00000000       $pdata$?StringCchCopyW@@YAJPEA_W_KPEB_W@Z 0000000180061000     ConEmuTh.obj
 0004:0000000c       $pdata$?StringCchCatW@@YAJPEA_W_KPEB_W@Z 000000018006100c     ConEmuTh.obj
 0004:00000018       $pdata$?StringCchVPrintfW@@YAJPEA_W_KPEB_WPEAD@Z 0000000180061018     ConEmuTh.obj
 0004:00000024       $pdata$?ExitFARW3@@YAXPEAX@Z 0000000180061024     ConEmuTh.obj
 0004:00000024       $pdata$ExitFARW            0000000180061024     ConEmuTh.obj
 0004:00000030       $pdata$SetStartupInfoW     0000000180061030     ConEmuTh.obj
 0004:0000003c       $pdata$?LoadModuleVersion@@YA_NPEB_WAEAUtagVS_FIXEDFILEINFO@@PEA_W_K@Z 000000018006103c     ConEmuTh.obj
 0004:00000048       $pdata$?LoadFarVersion@@YA_NAEAUFarVersion@@AEAY0CAA@_W@Z 0000000180061048     ConEmuTh.obj
 0004:00000054       $pdata$?FreeItem@CePluginPanelItem@@QEAAXXZ 0000000180061054     ConEmuTh.obj
 0004:00000060       $pdata$?FreeUserData@CePluginPanelItem@@QEAAXXZ 0000000180061060     ConEmuTh.obj
 0004:0000006c       $pdata$?LoadThSet@@YAHK@Z  000000018006106c     ConEmuTh.obj
 0004:00000078       $pdata$?OpenPluginWcmn@@YAPEAXH_J_N@Z 0000000180061078     ConEmuTh.obj
 0004:00000084       $pdata$?SettingsLoadReg@@YAHPEB_W0PEAK@Z 0000000180061084     ConEmuTh.obj
 0004:00000090       $pdata$?SettingsLoadOther@@YAXPEB_W@Z 0000000180061090     ConEmuTh.obj
 0004:0000009c       $pdata$?SettingsSaveReg@@YAXPEB_W0PEAK@Z 000000018006109c     ConEmuTh.obj
 0004:000000a8       $pdata$?SavePanelViewState@@YAXHK@Z 00000001800610a8     ConEmuTh.obj
 0004:000000b4       $pdata$?EntryPoint@@YAXH_J_N@Z 00000001800610b4     ConEmuTh.obj
 0004:000000c0       $pdata$?LoadFarVersion@@YAHXZ 00000001800610c0     ConEmuTh.obj
 0004:000000cc       $pdata$?StartPlugin@@YAXH@Z 00000001800610cc     ConEmuTh.obj
 0004:000000d8       $pdata$?dtor$0@?0??StartPlugin@@YAXH@Z@4HA 00000001800610d8     ConEmuTh.obj
 0004:000000e4       $pdata$?ExitPlugin@@YAXXZ  00000001800610e4     ConEmuTh.obj
 0004:000000f0       $pdata$?PostMacro@@YAXPEA_W@Z 00000001800610f0     ConEmuTh.obj
 0004:000000fc       $pdata$?ReloadPanelsInfo@@YAXXZ 00000001800610fc     ConEmuTh.obj
 0004:00000108       $pdata$?CheckWindows@@YA_NXZ 0000000180061108     ConEmuTh.obj
 0004:00000114       $pdata$?UpdateEnvVar@@YAXH@Z 0000000180061114     ConEmuTh.obj
 0004:00000120       $pdata$?IsThumbnailsActive@@YAPEAUCeFullPanelInfo@@H@Z 0000000180061120     ConEmuTh.obj
 0004:0000012c       $pdata$?GetFarRect@@YAHPEAU_SMALL_RECT@@@Z 000000018006112c     ConEmuTh.obj
 0004:00000138       $pdata$?ExecuteInMainThread@@YAXPEAUConEmuThSynchroArg@@@Z 0000000180061138     ConEmuTh.obj
 0004:00000144       $pdata$?CheckConEmu@@YAHH@Z 0000000180061144     ConEmuTh.obj
 0004:00000150       $pdata$?OnPrePeekConsole@@YAHPEAXPEAU_INPUT_RECORD@@KPEAKPEAH@Z 0000000180061150     ConEmuTh.obj
 0004:0000015c       $pdata$?OnPostPeekConsole@@YAHPEAXPEAU_INPUT_RECORD@@KPEAKPEAH@Z 000000018006115c     ConEmuTh.obj
 0004:00000168       $pdata$?OnPostReadConsole@@YAHPEAXPEAU_INPUT_RECORD@@KPEAKPEAH@Z 0000000180061168     ConEmuTh.obj
 0004:00000174       $pdata$?OnPreWriteConsoleOutput@@YAHPEAXPEBU_CHAR_INFO@@U_COORD@@2PEAU_SMALL_RECT@@@Z 0000000180061174     ConEmuTh.obj
 0004:00000180       $pdata$?ShowLastError@@YAHXZ 0000000180061180     ConEmuTh.obj
 0004:0000018c       $pdata$?CheckVarsInitialized@@YAXXZ 000000018006118c     ConEmuTh.obj
 0004:00000198       $pdata$?dtor$0@?0??CheckVarsInitialized@@YAXXZ@4HA 0000000180061198     ConEmuTh.obj
 0004:000001a4       $pdata$?dtor$1@?0??CheckVarsInitialized@@YAXXZ@4HA 00000001800611a4     ConEmuTh.obj
 0004:000001a4       $pdata$?dtor$2@?0??CheckVarsInitialized@@YAXXZ@4HA 00000001800611a4     ConEmuTh.obj
 0004:000001b0       $pdata$?ProcessConsoleInput@@YAHHPEAU_INPUT_RECORD@@KPEAK@Z 00000001800611b0     ConEmuTh.obj
 0004:000001bc       $pdata$?OnReadyForPanelsReload@@YAXXZ 00000001800611bc     ConEmuTh.obj
 0004:000001c8       $pdata$?ReloadResourcesW@@YAXXZ 00000001800611c8     ConEmuTh.obj
 0004:000001d4       $pdata$?GetMainThreadId@@YAKXZ 00000001800611d4     ConEmuTh.obj
 0004:000001e0       $pdata$?ChangeExports@@YA_NPEBUExportFunc@@PEAUHINSTANCE__@@@Z 00000001800611e0     ConEmuTh.obj
 0004:000001ec       $pdata$DllMain             00000001800611ec     ConEmuTh.obj
 0004:000001f8       $pdata$?OpenW@@YAPEAXPEBUOpenInfo@@@Z 00000001800611f8     ConEmuTh.obj
 0004:00000204       $pdata$?InitName@?$MFileMapping@UPanelViewSetMapping@@@@QEAAPEB_WPEB_WKK@Z 0000000180061204     ConEmuTh.obj
 0004:00000204       $pdata$?InitName@?$MFileMapping@Utag_DetectedDialog@@@@QEAAPEB_WPEB_WKK@Z 0000000180061204     ConEmuTh.obj
 0004:00000210       $pdata$?InternalOpenCreate@?$MFileMapping@Utag_DetectedDialog@@@@IEAAPEAUtag_DetectedDialog@@HHH@Z 0000000180061210     ConEmuTh.obj
 0004:0000021c       $pdata$??_G?$MFileMapping@Utag_DetectedDialog@@@@QEAAPEAXI@Z 000000018006121c     ConEmuTh.obj
 0004:00000228       $pdata$??$swprintf_c@$0CAA@@@YAHAEAY0CAA@_WPEB_WZZ 0000000180061228     ConEmuTh.obj
 0004:00000234       $pdata$?ProcessSynchroEventCommon@@YAHHPEAX@Z 0000000180061234     ConEmuTh.obj
 0004:00000240       $pdata$?InternalOpenCreate@?$MFileMapping@UPanelViewSetMapping@@@@IEAAPEAUPanelViewSetMapping@@HHH@Z 0000000180061240     ConEmuTh.obj
 0004:0000024c       $pdata$??1?$MFileMapping@UPanelViewSetMapping@@@@QEAA@XZ 000000018006124c     ConEmuTh.obj
 0004:00000258       $pdata$?GetPluginInfoW1900@@YAXPEAX@Z 0000000180061258     ConEmuTh1900.obj
 0004:00000264       $pdata$?SettingsLoadW1900@@YAHPEB_WPEAK@Z 0000000180061264     ConEmuTh1900.obj
 0004:00000270       $pdata$?SettingsSaveW1900@@YAXPEB_WPEAK@Z 0000000180061270     ConEmuTh1900.obj
 0004:0000027c       $pdata$?ExitFARW1900@@YAXXZ 000000018006127c     ConEmuTh1900.obj
 0004:00000288       $pdata$?SetStartupInfoW1900@@YAXPEAX@Z 0000000180061288     ConEmuTh1900.obj
 0004:00000294       $pdata$?ShowMessageW1900@@YAHHH@Z 0000000180061294     ConEmuTh1900.obj
 0004:000002a0       $pdata$?ShowMessageW1900@@YAHPEB_WH@Z 00000001800612a0     ConEmuTh1900.obj
 0004:000002ac       $pdata$?PostMacroW1900@@YAXPEA_W@Z 00000001800612ac     ConEmuTh1900.obj
 0004:000002b8       $pdata$?ShowPluginMenuW1900@@YAHXZ 00000001800612b8     ConEmuTh1900.obj
 0004:000002c4       $pdata$?LoadPanelInfoW1900@@YAHH@Z 00000001800612c4     ConEmuTh1900.obj
 0004:000002d0       $pdata$?ReloadPanelsInfoW1900@@YAXXZ 00000001800612d0     ConEmuTh1900.obj
 0004:000002dc       $pdata$?LoadPanelItemInfoW1900@@YAXPEAUCeFullPanelInfo@@_J@Z 00000001800612dc     ConEmuTh1900.obj
 0004:000002e8       $pdata$?CheckFarPanelsW1900@@YA_NXZ 00000001800612e8     ConEmuTh1900.obj
 0004:000002f4       $pdata$?CheckPanelSettingsW1900@@YAHH@Z 00000001800612f4     ConEmuTh1900.obj
 0004:00000300       $pdata$?GetFarRectW1900@@YAXPEAU_SMALL_RECT@@@Z 0000000180061300     ConEmuTh1900.obj
 0004:0000030c       $pdata$?ExecuteInMainThreadW1900@@YAXPEAUConEmuThSynchroArg@@@Z 000000018006130c     ConEmuTh1900.obj
 0004:00000318       $pdata$?SetCurrentPanelItemW1900@@YAXH_J0@Z 0000000180061318     ConEmuTh1900.obj
 0004:00000324       $pdata$?Color2FgIndex@Far3Color@@SAXKAEAGPEBK@Z 0000000180061324     ConEmuTh1900.obj
 0004:00000330       $pdata$?Color2BgIndex@Far3Color@@SAXKHAEAGPEBK@Z 0000000180061330     ConEmuTh1900.obj
 0004:0000033c       $pdata$?FarColor_3_2@@YAEAEBUFarColor@@_N@Z 000000018006133c     ConEmuTh1900.obj
 0004:00000348       $pdata$?GetFarSetting@@YAHPEAX_KPEB_W@Z 0000000180061348     ConEmuTh1900.obj
 0004:00000354       $pdata$?LoadFarSettingsW1900@@YAXPEAUCEFarInterfaceSettings@@PEAUCEFarPanelSettings@@@Z 0000000180061354     ConEmuTh1900.obj
 0004:00000360       $pdata$GetGlobalInfoW      0000000180061360     ConEmuTh2800.obj
 0004:0000036c       $pdata$?GetPluginInfoW2800@@YAXPEAX@Z 000000018006136c     ConEmuTh2800.obj
 0004:00000378       $pdata$?SettingsLoadW2800@@YAHPEB_WPEAK@Z 0000000180061378     ConEmuTh2800.obj
 0004:00000384       $pdata$?SettingsSaveW2800@@YAXPEB_WPEAK@Z 0000000180061384     ConEmuTh2800.obj
 0004:00000390       $pdata$?ExitFARW2800@@YAXXZ 0000000180061390     ConEmuTh2800.obj
 0004:0000039c       $pdata$?SetStartupInfoW2800@@YAXPEAX@Z 000000018006139c     ConEmuTh2800.obj
 0004:000003a8       $pdata$?OpenW2800@@YAPEAXPEBX@Z 00000001800613a8     ConEmuTh2800.obj
 0004:000003b4       $pdata$?ShowMessageW2800@@YAHHH@Z 00000001800613b4     ConEmuTh2800.obj
 0004:000003c0       $pdata$?ShowMessageW2800@@YAHPEB_WH@Z 00000001800613c0     ConEmuTh2800.obj
 0004:000003cc       $pdata$?PostMacroW2800@@YAXPEA_W@Z 00000001800613cc     ConEmuTh2800.obj
 0004:000003d8       $pdata$?ShowPluginMenuW2800@@YAHXZ 00000001800613d8     ConEmuTh2800.obj
 0004:000003e4       $pdata$?LoadPanelInfoW2800@@YAHH@Z 00000001800613e4     ConEmuTh2800.obj
 0004:000003f0       $pdata$?ReloadPanelsInfoW2800@@YAXXZ 00000001800613f0     ConEmuTh2800.obj
 0004:000003fc       $pdata$?LoadPanelItemInfoW2800@@YAXPEAUCeFullPanelInfo@@_J@Z 00000001800613fc     ConEmuTh2800.obj
 0004:00000408       $pdata$?CheckFarPanelsW2800@@YA_NXZ 0000000180061408     ConEmuTh2800.obj
 0004:00000414       $pdata$?CheckPanelSettingsW2800@@YAHH@Z 0000000180061414     ConEmuTh2800.obj
 0004:00000420       $pdata$?GetFarRectW2800@@YAXPEAU_SMALL_RECT@@@Z 0000000180061420     ConEmuTh2800.obj
 0004:0000042c       $pdata$?ExecuteInMainThreadW2800@@YAXPEAUConEmuThSynchroArg@@@Z 000000018006142c     ConEmuTh2800.obj
 0004:00000438       $pdata$?SetCurrentPanelItemW2800@@YAXH_J0@Z 0000000180061438     ConEmuTh2800.obj
 0004:00000444       $pdata$?SetCurrentPanelItemW2800Int@@YAXH_J0@Z 0000000180061444     ConEmuTh2800.obj
 0004:00000450       $pdata$?ProcessSynchroEventW3@@YA_JPEAX@Z 0000000180061450     ConEmuTh2800.obj
 0004:0000045c       $pdata$?FreePanelItemUserData2800@@YAXPEAX_KP6A_JXZ@Z 000000018006145c     ConEmuTh2800.obj
 0004:00000468       $pdata$?GetFarSetting@@YAHPEAX_KPEB_W@Z 0000000180061468     ConEmuTh2800.obj
 0004:00000474       $pdata$?LoadFarSettingsW2800@@YAXPEAUCEFarInterfaceSettings@@PEAUCEFarPanelSettings@@@Z 0000000180061474     ConEmuTh2800.obj
 0004:00000480       $pdata$??$swprintf_c@$0MI@@@YAHAEAY0MI@_WPEB_WZZ 0000000180061480     ConEmuTh2800.obj
 0004:0000048c       $pdata$?GetPluginInfoW995@@YAXPEAX@Z 000000018006148c     ConEmuTh995.obj
 0004:00000498       $pdata$?ExitFARW995@@YAXXZ 0000000180061498     ConEmuTh995.obj
 0004:000004a4       $pdata$?SetStartupInfoW995@@YAXPEAX@Z 00000001800614a4     ConEmuTh995.obj
 0004:000004b0       $pdata$?ShowMessageW995@@YAHHH@Z 00000001800614b0     ConEmuTh995.obj
 0004:000004bc       $pdata$?ShowMessageW995@@YAHPEB_WH@Z 00000001800614bc     ConEmuTh995.obj
 0004:000004c8       $pdata$?PostMacroW995@@YAXPEA_W@Z 00000001800614c8     ConEmuTh995.obj
 0004:000004d4       $pdata$?ShowPluginMenuW995@@YAHXZ 00000001800614d4     ConEmuTh995.obj
 0004:000004e0       $pdata$?ReloadPanelsInfoW995@@YAXXZ 00000001800614e0     ConEmuTh995.obj
 0004:000004ec       $pdata$?LoadPanelItemInfoW995@@YAXPEAUCeFullPanelInfo@@_J@Z 00000001800614ec     ConEmuTh995.obj
 0004:000004f8       $pdata$?CheckFarPanelsW995@@YA_NXZ 00000001800614f8     ConEmuTh995.obj
 0004:00000504       $pdata$?CheckPanelSettingsW995@@YAHH@Z 0000000180061504     ConEmuTh995.obj
 0004:00000510       $pdata$?GetFarRectW995@@YAXPEAU_SMALL_RECT@@@Z 0000000180061510     ConEmuTh995.obj
 0004:0000051c       $pdata$?ExecuteInMainThreadW995@@YAXPEAUConEmuThSynchroArg@@@Z 000000018006151c     ConEmuTh995.obj
 0004:00000528       $pdata$?SetCurrentPanelItemW995@@YAXH_J0@Z 0000000180061528     ConEmuTh995.obj
 0004:00000534       $pdata$?LoadFarSettingsW995@@YAXPEAUCEFarInterfaceSettings@@PEAUCEFarPanelSettings@@@Z 0000000180061534     ConEmuTh995.obj
 0004:00000540       $pdata$?LoadPanelInfo995@@YAHH@Z 0000000180061540     ConEmuTh995.obj
 0004:0000054c       $pdata$ExitFAR             000000018006154c     ConEmuThA.obj
 0004:00000558       $pdata$GetMinFarVersion    0000000180061558     ConEmuThA.obj
 0004:00000564       $pdata$GetPluginInfo       0000000180061564     ConEmuThA.obj
 0004:00000570       $pdata$OpenPlugin          0000000180061570     ConEmuThA.obj
 0004:0000057c       $pdata$SetStartupInfo      000000018006157c     ConEmuThA.obj
 0004:00000588       $pdata$?ShowMessageA@@YAHHH@Z 0000000180061588     ConEmuThA.obj
 0004:00000594       $pdata$?ShowMessageA@@YAHPEBDH@Z 0000000180061594     ConEmuThA.obj
 0004:000005a0       $pdata$?PostMacroA@@YAXPEAD@Z 00000001800615a0     ConEmuThA.obj
 0004:000005ac       $pdata$?GetMsgA@@YAPEB_WHPEA_W@Z 00000001800615ac     ConEmuThA.obj
 0004:000005b8       $pdata$?ShowPluginMenuA@@YAHXZ 00000001800615b8     ConEmuThA.obj
 0004:000005c4       $pdata$?LoadPanelInfoA@@YAHH@Z 00000001800615c4     ConEmuThA.obj
 0004:000005d0       $pdata$?ReloadPanelsInfoA@@YAXXZ 00000001800615d0     ConEmuThA.obj
 0004:000005dc       $pdata$?CheckFarPanelsA@@YA_NXZ 00000001800615dc     ConEmuThA.obj
 0004:000005e8       $pdata$?CheckPanelSettingsA@@YAHH@Z 00000001800615e8     ConEmuThA.obj
 0004:000005f4       $pdata$?SetCurrentPanelItemA@@YAXH_J0@Z 00000001800615f4     ConEmuThA.obj
 0004:00000600       $pdata$?ReloadResourcesA@@YAXXZ 0000000180061600     ConEmuThA.obj
 0004:0000060c       $pdata$?LoadFarSettingsA@@YAXPEAUCEFarInterfaceSettings@@PEAUCEFarPanelSettings@@@Z 000000018006160c     ConEmuThA.obj
 0004:00000618       $pdata$?RegisterPanelView@CeFullPanelInfo@@QEAAHXZ 0000000180061618     Display.obj
 0004:00000624       $pdata$?UnregisterPanelView@CeFullPanelInfo@@QEAAH_N@Z 0000000180061624     Display.obj
 0004:00000630       $pdata$?Close@CeFullPanelInfo@@QEAAXXZ 0000000180061630     Display.obj
 0004:0000063c       $pdata$?CreateView@CeFullPanelInfo@@QEAAPEAUHWND__@@XZ 000000018006163c     Display.obj
 0004:00000648       $pdata$?ReallocItems@CeFullPanelInfo@@QEAAH_J@Z 0000000180061648     Display.obj
 0004:00000654       $pdata$?FinalRelease@CeFullPanelInfo@@QEAAXXZ 0000000180061654     Display.obj
 0004:00000660       $pdata$?DisplayReloadPanel@CeFullPanelInfo@@QEAAXXZ 0000000180061660     Display.obj
 0004:0000066c       $pdata$?RequestSetPos@CeFullPanelInfo@@QEAAX_J0H@Z 000000018006166c     Display.obj
 0004:00000678       $pdata$?DisplayWndProc@CeFullPanelInfo@@SA_JPEAUHWND__@@I_K_J@Z 0000000180061678     Display.obj
 0004:00000684       $pdata$?DisplayThread@CeFullPanelInfo@@SAKPEAX@Z 0000000180061684     Display.obj
 0004:00000690       $pdata$?CalcTopPanelItem@CeFullPanelInfo@@QEAA_J_J0@Z 0000000180061690     Display.obj
 0004:0000069c       $pdata$?Invalidate@CeFullPanelInfo@@QEAAXXZ 000000018006169c     Display.obj
 0004:000006a8       $pdata$?InvalidateAll@CeFullPanelInfo@@SAXXZ 00000001800616a8     Display.obj
 0004:000006b4       $pdata$?Paint@CeFullPanelInfo@@QEAAXPEAUHWND__@@AEAUtagPAINTSTRUCT@@AEAUtagRECT@@@Z 00000001800616b4     Display.obj
 0004:000006c0       $pdata$?PaintItem@CeFullPanelInfo@@QEAAHPEAUHDC__@@_JHHPEAUCePluginPanelItem@@PEAUCePluginPanelItemColor@@HHPEAUHBRUSH__@@4K@Z 00000001800616c0     Display.obj
 0004:000006cc       $pdata$?DrawItemText@CeFullPanelInfo@@QEAAHPEAUHDC__@@PEAUtagRECT@@1PEAUCePluginPanelItem@@PEB_WPEAUHBRUSH__@@H@Z 00000001800616cc     Display.obj
 0004:000006d8       $pdata$?OnSettingsChanged@CeFullPanelInfo@@QEAAHH@Z 00000001800616d8     Display.obj
 0004:000006e4       $pdata$?GetIndexFromWndCoord@CeFullPanelInfo@@QEAAHHHAEA_J@Z 00000001800616e4     Display.obj
 0004:000006f0       $pdata$?GetItemColors@CeFullPanelInfo@@QEAAPEAUHBRUSH__@@_JPEAUCePluginPanelItem@@PEAUCePluginPanelItemColor@@HAEAK3@Z 00000001800616f0     Display.obj
 0004:000006fc       $pdata$?LoadItemColors@CeFullPanelInfo@@QEAAX_JPEAUCePluginPanelItem@@PEAUCePluginPanelItemColor@@HH@Z 00000001800616fc     Display.obj
 0004:00000708       $pdata$?FarItem2CeItem@CeFullPanelInfo@@QEAAH_JPEB_W1KU_FILETIME@@_KHPEAX3P6A_JXZ3K@Z 0000000180061708     Display.obj
 0004:00000714       $pdata$??$swprintf_c@$0IA@@@YAHAEAY0IA@_WPEB_WZZ 0000000180061714     Display.obj
 0004:00000720       $pdata$?CheckLoadDibCreated@CImgCache@@IEAAHXZ 0000000180061720     ImgCache.obj
 0004:0000072c       $pdata$?CheckDrawDibCreated@CImgCache@@IEAAHXZ 000000018006172c     ImgCache.obj
 0004:00000738       $pdata$?FindInCache@CImgCache@@IEAAHPEAUCePluginPanelItem@@PEAHI@Z 0000000180061738     ImgCache.obj
 0004:00000744       $pdata$?CopyBits@CImgCache@@IEAAXU_COORD@@PEAEK01@Z 0000000180061744     ImgCache.obj
 0004:00000750       $pdata$?LoadModules@CImgCache@@IEAAXXZ 0000000180061750     ImgCache.obj
 0004:0000075c       $pdata$?FreeModules@CImgCache@@IEAAXXZ 000000018006175c     ImgCache.obj
 0004:00000768       $pdata$??0CImgCache@@QEAA@PEAUHINSTANCE__@@@Z 0000000180061768     ImgCache.obj
 0004:00000774       $pdata$??1CImgCache@@QEAA@XZ 0000000180061774     ImgCache.obj
 0004:00000780       $pdata$?SetCacheLocation@CImgCache@@QEAAXPEB_W@Z 0000000180061780     ImgCache.obj
 0004:0000078c       $pdata$?Reset@CImgCache@@QEAAXXZ 000000018006178c     ImgCache.obj
 0004:00000798       $pdata$?Init@CImgCache@@QEAAXK@Z 0000000180061798     ImgCache.obj
 0004:000007a4       $pdata$?RequestItem@CImgCache@@QEAAHPEAUCePluginPanelItem@@I@Z 00000001800617a4     ImgCache.obj
 0004:000007b0       $pdata$?dtor$0@?0??RequestItem@CImgCache@@QEAAHPEAUCePluginPanelItem@@I@Z@4HA 00000001800617b0     ImgCache.obj
 0004:000007bc       $pdata$?PaintItem@CImgCache@@QEAAHPEAUHDC__@@HHHPEAUCePluginPanelItem@@PEAPEB_WPEAH@Z 00000001800617bc     ImgCache.obj
 0004:000007c8       $pdata$?LoadThumbnail@CImgCache@@QEAAHPEAUIMAGE_CACHE_INFO@@@Z 00000001800617c8     ImgCache.obj
 0004:000007d4       $pdata$?LoadShellIcon@CImgCache@@QEAAHPEAUIMAGE_CACHE_INFO@@H@Z 00000001800617d4     ImgCache.obj
 0004:000007e0       $pdata$?InitializeQueue@?$CQueueProcessor@PEAUIMAGE_CACHE_INFO@@@@AEAAXH@Z 00000001800617e0     ImgCache.obj
 0004:000007ec       $pdata$?ClearQueue@?$CQueueProcessor@PEAUIMAGE_CACHE_INFO@@@@AEAAXXZ 00000001800617ec     ImgCache.obj
 0004:000007f8       $pdata$?FindOrCreate@?$CQueueProcessor@PEAUIMAGE_CACHE_INFO@@@@AEAAPEAUProcessingItem@1@AEBQEAUIMAGE_CACHE_INFO@@_J_NW4ProcessingPriority@@@Z 00000001800617f8     ImgCache.obj
 0004:00000804       $pdata$??0?$CQueueProcessor@PEAUIMAGE_CACHE_INFO@@@@QEAA@XZ 0000000180061804     ImgCache.obj
 0004:00000810       $pdata$?dtor$0@?0???0?$CQueueProcessor@PEAUIMAGE_CACHE_INFO@@@@QEAA@XZ@4HA 0000000180061810     ImgCache.obj
 0004:0000081c       $pdata$??1?$CQueueProcessor@PEAUIMAGE_CACHE_INFO@@@@UEAA@XZ 000000018006181c     ImgCache.obj
 0004:00000828       $pdata$?CopyItem@?$CQueueProcessor@PEAUIMAGE_CACHE_INFO@@@@MEAAXPEBQEAUIMAGE_CACHE_INFO@@PEAPEAU2@@Z 0000000180061828     ImgCache.obj
 0004:00000834       $pdata$?ProcessItem@?$CQueueProcessor@PEAUIMAGE_CACHE_INFO@@@@IEAAJPEAUProcessingItem@1@@Z 0000000180061834     ImgCache.obj
 0004:00000840       $pdata$?ProcessingStep@?$CQueueProcessor@PEAUIMAGE_CACHE_INFO@@@@IEAA_NXZ 0000000180061840     ImgCache.obj
 0004:0000084c       $pdata$?ProcessingThread@?$CQueueProcessor@PEAUIMAGE_CACHE_INFO@@@@KAKPEAX@Z 000000018006184c     ImgCache.obj
 0004:00000858       $pdata$?CheckThread@?$CQueueProcessor@PEAUIMAGE_CACHE_INFO@@@@IEAAJXZ 0000000180061858     ImgCache.obj
 0004:00000864       $pdata$??_G?$CQueueProcessor@PEAUIMAGE_CACHE_INFO@@@@UEAAPEAXI@Z 0000000180061864     ImgCache.obj
 0004:00000864       $pdata$??_GCImgLoader@@UEAAPEAXI@Z 0000000180061864     ImgCache.obj
 0004:00000870       $pdata$?ProcessItem@CImgLoader@@UEAAJAEAPEAUIMAGE_CACHE_INFO@@_J@Z 0000000180061870     ImgCache.obj
 0004:0000087c       $pdata$?OnThreadStarted@CImgLoader@@UEAAJXZ 000000018006187c     ImgCache.obj
 0004:00000888       $pdata$??$SafeDelete@UMSectionSimple@@@@YAXAEAPEAUMSectionSimple@@@Z 0000000180061888     ImgCache.obj
 0004:00000894       $pdata$??2@YAPEAX_K@Z      0000000180061894     common-kernel64:Memory.obj
 0004:000008a0       $pdata$??_V@YAXPEAX@Z      00000001800618a0     common-kernel64:Memory.obj
 0004:000008a0       $pdata$??3@YAXPEAX@Z       00000001800618a0     common-kernel64:Memory.obj
 0004:000008a0       $pdata$?xf_free@@YAXPEAX@Z 00000001800618a0     common-kernel64:Memory.obj
 0004:000008ac       $pdata$?HeapInitialize@@YA_NXZ 00000001800618ac     common-kernel64:Memory.obj
 0004:000008b8       $pdata$?HeapDeinitialize@@YAXXZ 00000001800618b8     common-kernel64:Memory.obj
 0004:000008c4       $pdata$?StringCchVPrintfA@@YAJPEAD_KPEBD0@Z 00000001800618c4     common-kernel64:MStrSafe.obj
 0004:000008d0       $pdata$?swprintf_c@@YAHPEA_W_JPEB_WZZ 00000001800618d0     common-kernel64:MStrSafe.obj
 0004:000008dc       $pdata$?sprintf_c@@YAHPEAD_JPEBDZZ 00000001800618dc     common-kernel64:MStrSafe.obj
 0004:000008e8       $pdata$?msprintf@@YAPEB_WPEA_W_KPEB_WZZ 00000001800618e8     common-kernel64:MStrSafe.obj
 0004:000008f4       $pdata$?LocalSecurity@@YAPEAU_SECURITY_ATTRIBUTES@@XZ 00000001800618f4     common-kernel64:MSecurity.obj
 0004:00000900       $pdata$?ShutdownSecurity@@YAXXZ 0000000180061900     common-kernel64:MSecurity.obj
 0004:0000090c       $pdata$?LoadAdvApi@MNullDesc@@IEAAHXZ 000000018006190c     common-kernel64:MSecurity.obj
 0004:00000918       $pdata$?LocalSecurity@MNullDesc@@QEAAPEAU_SECURITY_ATTRIBUTES@@XZ 0000000180061918     common-kernel64:MSecurity.obj
 0004:00000924       $pdata$??_GMNullDesc@@QEAAPEAXI@Z 0000000180061924     common-kernel64:MSecurity.obj
 0004:00000930       $pdata$?ExecuteOpenPipe@@YAPEAXPEB_WAEAY0CAI@_W0KKHPEAXH@Z 0000000180061930     common-kernel64:ConEmuCheck.obj
 0004:0000093c       $pdata$?ExecuteNewCmd@@YAPEAUCESERVER_REQ@@K_K@Z 000000018006193c     common-kernel64:ConEmuCheck.obj
 0004:00000948       $pdata$?ExecutePrepareCmd@@YAXPEAUCESERVER_REQ@@K_K@Z 0000000180061948     common-kernel64:ConEmuCheck.obj
 0004:00000954       $pdata$?ExecutePrepareCmd@@YAXPEAUCESERVER_REQ_HDR@@K_K@Z 0000000180061954     common-kernel64:ConEmuCheck.obj
 0004:00000960       $pdata$?ExecuteGuiCmd@@YAPEAUCESERVER_REQ@@PEAUHWND__@@PEAU1@0H@Z 0000000180061960     common-kernel64:ConEmuCheck.obj
 0004:0000096c       $pdata$?ExecuteCmd@@YAPEAUCESERVER_REQ@@PEB_WPEAU1@KPEAUHWND__@@HKH@Z 000000018006196c     common-kernel64:ConEmuCheck.obj
 0004:00000978       $pdata$?ExecuteFreeResult@@YAXAEAPEAUCESERVER_REQ@@@Z 0000000180061978     common-kernel64:ConEmuCheck.obj
 0004:00000984       $pdata$?ModuleName@@YAPEB_WPEB_W@Z 0000000180061984     common-kernel64:ConEmuCheck.obj
 0004:00000990       $pdata$?isTerminalMode@@YA_NXZ 0000000180061990     common-kernel64:MProcess.obj
 0004:0000099c       $pdata$?push_back@?$MArray@UtagPROCESSENTRY32W@@@@QEAA_JAEBUtagPROCESSENTRY32W@@@Z 000000018006199c     common-kernel64:MProcess.obj
 0004:000009a8       $pdata$?addsize@?$MArray@UtagPROCESSENTRY32W@@@@QEAA_N_J@Z 00000001800619a8     common-kernel64:MProcess.obj
 0004:000009b4       $pdata$?getNext@?$MToolHelp@UtagPROCESSENTRY32W@@$1?Process32FirstW@@YAHPEAXPEAU1@@Z$1?Process32NextW@@YAH01@Z@@IEAA_NXZ 00000001800619b4     common-kernel64:MProcess.obj
 0004:000009c0       $pdata$??1?$MToolHelp@UtagPROCESSENTRY32W@@$1?Process32FirstW@@YAHPEAXPEAU1@@Z$1?Process32NextW@@YAH01@Z@@UEAA@XZ 00000001800619c0     common-kernel64:MProcess.obj
 0004:000009cc       $pdata$?Open@?$MToolHelp@UtagPROCESSENTRY32W@@$1?Process32FirstW@@YAHPEAXPEAU1@@Z$1?Process32NextW@@YAH01@Z@@QEAA_NXZ 00000001800619cc     common-kernel64:MProcess.obj
 0004:000009d8       $pdata$?Find@?$MToolHelp@UtagPROCESSENTRY32W@@$1?Process32FirstW@@YAHPEAXPEAU1@@Z$1?Process32NextW@@YAH01@Z@@QEAA_NP6A_NPEAUtagPROCESSENTRY32W@@_J@Z10@Z 00000001800619d8     common-kernel64:MProcess.obj
 0004:000009e4       $pdata$??_GMToolHelpProcess@@UEAAPEAXI@Z 00000001800619e4     common-kernel64:MProcess.obj
 0004:000009e4       $pdata$??_G?$MToolHelp@UtagPROCESSENTRY32W@@$1?Process32FirstW@@YAHPEAXPEAU1@@Z$1?Process32NextW@@YAH01@Z@@UEAAPEAXI@Z 00000001800619e4     common-kernel64:MProcess.obj
 0004:000009f0       $pdata$?Init@HkFunc@@QEAA_NPEB_WPEAUHINSTANCE__@@@Z 00000001800619f0     common-kernel64:HkFunc.obj
 0004:000009fc       $pdata$??0MSection@@QEAA@XZ 00000001800619fc     common-kernel64:MSection.obj
 0004:00000a08       $pdata$??1MSection@@QEAA@XZ 0000000180061a08     common-kernel64:MSection.obj
 0004:00000a14       $pdata$?AddRef@MSection@@IEAAXK@Z 0000000180061a14     common-kernel64:MSection.obj
 0004:00000a20       $pdata$?ReleaseRef@MSection@@IEAAHK@Z 0000000180061a20     common-kernel64:MSection.obj
 0004:00000a2c       $pdata$?WaitUnlocked@MSection@@IEAAXKK@Z 0000000180061a2c     common-kernel64:MSection.obj
 0004:00000a38       $pdata$?MyEnterCriticalSection@MSection@@IEAA_NK@Z 0000000180061a38     common-kernel64:MSection.obj
 0004:00000a44       $pdata$?Lock@MSection@@IEAAHHK@Z 0000000180061a44     common-kernel64:MSection.obj
 0004:00000a50       $pdata$?Unlock@MSection@@IEAAXH@Z 0000000180061a50     common-kernel64:MSection.obj
 0004:00000a5c       $pdata$?Lock@MSectionLock@@QEAAHPEAVMSection@@HK@Z 0000000180061a5c     common-kernel64:MSection.obj
 0004:00000a68       $pdata$?Unlock@MSectionLock@@QEAAXXZ 0000000180061a68     common-kernel64:MSection.obj
 0004:00000a74       $pdata$??1MSectionLock@@QEAA@XZ 0000000180061a74     common-kernel64:MSection.obj
 0004:00000a80       $pdata$?apiCreateThread@@YAPEAXP6AKPEAX@Z0PEAKPEBDH@Z 0000000180061a80     common-kernel64:WThreads.obj
 0004:00000a8c       $pdata$?apiTerminateThreadEx@@YAHPEAXKPEBDH@Z 0000000180061a8c     common-kernel64:WThreads.obj
 0004:00000a98       $pdata$?SetThreadName@@YAXKPEAD@Z 0000000180061a98     common-kernel64:WThreads.obj
 0004:00000aa4       $pdata$?apiThreadHelper@@YAKPEAX@Z 0000000180061aa4     common-kernel64:WThreads.obj
 0004:00000ab0       $pdata$??$sprintf_c@$0CI@@@YAHAEAY0CI@DPEBDZZ 0000000180061ab0     common-kernel64:WThreads.obj
 0004:00000abc       $pdata$?StringCchCopyNW@@YAJPEA_W_KPEB_W1@Z 0000000180061abc     common-kernel64:WObjects.obj
 0004:00000ac8       $pdata$?FileExists@@YA_NPEB_WPEAK@Z 0000000180061ac8     common-kernel64:WObjects.obj
 0004:00000ad4       $pdata$?_VerifyVersionInfo@@YA_NPEAU_OSVERSIONINFOEXW@@K_K@Z 0000000180061ad4     common-kernel64:WObjects.obj
 0004:00000ae0       $pdata$?ExpandEnvStr@@YAPEA_WPEB_W@Z 0000000180061ae0     common-kernel64:WObjects.obj
 0004:00000aec       $pdata$?GetEnvVar@@YAPEA_WPEB_W@Z 0000000180061aec     common-kernel64:WObjects.obj
 0004:00000af8       $pdata$?PointToName@@YAPEB_WPEB_W@Z 0000000180061af8     common-kernel64:CmdLine.obj
 0004:00000b04       $pdata$?PointToExt@@YAPEB_WPEB_W@Z 0000000180061b04     common-kernel64:CmdLine.obj
 0004:00000b10       $pdata$?Unquote@@YAPEB_WPEA_W_N@Z 0000000180061b10     common-kernel64:CmdLine.obj
 0004:00000b1c       $pdata$?lstrdup@@YAPEA_WPEB_W_K@Z 0000000180061b1c     common-kernel64:MStrDup.obj
 0004:00000b28       $pdata$?lstrmerge@@YAPEA_WPEB_W00000000@Z 0000000180061b28     common-kernel64:MStrDup.obj
 0004:00000b34       $pdata$??0MSectionSimple@@QEAA@_N@Z 0000000180061b34     common-kernel64:MSectionSimple.obj
 0004:00000b40       $pdata$??1MSectionSimple@@QEAA@XZ 0000000180061b40     common-kernel64:MSectionSimple.obj
 0004:00000b40       $pdata$?Close@MSectionSimple@@QEAAXXZ 0000000180061b40     common-kernel64:MSectionSimple.obj
 0004:00000b4c       $pdata$?Init@MSectionSimple@@QEAAXXZ 0000000180061b4c     common-kernel64:MSectionSimple.obj
 0004:00000b58       $pdata$?TryEnter@MSectionSimple@@QEAA_NXZ 0000000180061b58     common-kernel64:MSectionSimple.obj
 0004:00000b64       $pdata$?RecreateAndLock@MSectionSimple@@QEAA_NXZ 0000000180061b64     common-kernel64:MSectionSimple.obj
 0004:00000b70       $pdata$?Lock@MSectionLockSimple@@QEAAHPEAUMSectionSimple@@K@Z 0000000180061b70     common-kernel64:MSectionSimple.obj
 0004:00000b7c       $pdata$?Unlock@MSectionLockSimple@@QEAAXXZ 0000000180061b7c     common-kernel64:MSectionSimple.obj
 0004:00000b88       $pdata$??1MSectionLockSimple@@QEAA@XZ 0000000180061b88     common-kernel64:MSectionSimple.obj
 0004:00000b94       $pdata$?AttachInt@CEStr@@AEAAPEB_WAEAPEA_W@Z 0000000180061b94     common-kernel64:CEStr.obj
 0004:00000ba0       $pdata$?GetMaxCount@CEStr@@QEAA_JXZ 0000000180061ba0     common-kernel64:CEStr.obj
 0004:00000bac       $pdata$?GetBuffer@CEStr@@QEAAPEA_W_J@Z 0000000180061bac     common-kernel64:CEStr.obj
 0004:00000bb8       $pdata$?Set@CEStr@@QEAAPEB_WPEB_W_J@Z 0000000180061bb8     common-kernel64:CEStr.obj
 0004:00000bc4       $pdata$?SavePathVar@CEStr@@QEAAXPEB_W@Z 0000000180061bc4     common-kernel64:CEStr.obj
 0004:00000bd0       $pdata$??0CEStr@@QEAA@PEB_W00000000@Z 0000000180061bd0     common-kernel64:CEStr.obj
 0004:00000bdc       $pdata$??1CEStr@@QEAA@XZ   0000000180061bdc     common-kernel64:CEStr.obj
 0004:00000be8       $pdata$?Free@MModule@@QEAAXXZ 0000000180061be8     common-kernel64:MModule.obj
 0004:00000bf4       $pdata$??0CRgnDetect@@QEAA@XZ 0000000180061bf4     common-user64:RgnDetect.obj
 0004:00000c00       $pdata$??1CRgnDetect@@QEAA@XZ 0000000180061c00     common-user64:RgnDetect.obj
 0004:00000c0c       $pdata$?PrepareTransparent@CRgnDetect@@QEAAXPEBUCEFAR_INFO_MAPPING@@PEBKPEBU_CONSOLE_SCREEN_BUFFER_INFO@@PEA_WPEAUtag_CharAttr@@HH@Z 0000000180061c0c     common-user64:RgnDetect.obj
 0004:00000c18       $pdata$?PrepareTransparent@CRgnDetect@@QEAAXPEBUCEFAR_INFO_MAPPING@@PEBK@Z 0000000180061c18     common-user64:RgnDetect.obj
 0004:00000c24       $pdata$?OnWriteConsoleOutput@CRgnDetect@@QEAAXPEBU_CHAR_INFO@@U_COORD@@1PEAU_SMALL_RECT@@PEBK@Z 0000000180061c24     common-user64:RgnDetect.obj
 0004:00000c30       $pdata$?InitializeSBI@CRgnDetect@@QEAAHPEBK@Z 0000000180061c30     common-user64:RgnDetect.obj
 0004:00000c3c       $pdata$?DetectDialog@CRgnDetect@@IEAA_NPEA_WPEAUtag_CharAttr@@HHHHPEAH2@Z 0000000180061c3c     common-user64:RgnDetect.obj
 0004:00000c48       $pdata$?FindDialog_TopLeft@CRgnDetect@@IEAA_NPEA_WPEAUtag_CharAttr@@HHAEAH222AEA_N@Z 0000000180061c48     common-user64:RgnDetect.obj
 0004:00000c54       $pdata$?FindDialog_TopRight@CRgnDetect@@IEAA_NPEA_WPEAUtag_CharAttr@@HHAEAH222AEA_N@Z 0000000180061c54     common-user64:RgnDetect.obj
 0004:00000c60       $pdata$?FindDialog_Left@CRgnDetect@@IEAA_NPEA_WPEAUtag_CharAttr@@HHAEAH222AEA_N@Z 0000000180061c60     common-user64:RgnDetect.obj
 0004:00000c6c       $pdata$?FindDialog_Right@CRgnDetect@@IEAA_NPEA_WPEAUtag_CharAttr@@HHAEAH222AEA_N@Z 0000000180061c6c     common-user64:RgnDetect.obj
 0004:00000c78       $pdata$?FindDialog_Any@CRgnDetect@@IEAA_NPEA_WPEAUtag_CharAttr@@HHAEAH222AEA_N@Z 0000000180061c78     common-user64:RgnDetect.obj
 0004:00000c84       $pdata$?FindDialog_Inner@CRgnDetect@@IEAA_NPEA_WPEAUtag_CharAttr@@HHAEAH2@Z 0000000180061c84     common-user64:RgnDetect.obj
 0004:00000c90       $pdata$?FindFrame_TopLeft@CRgnDetect@@IEAA_NPEA_WPEAUtag_CharAttr@@HHAEAH222@Z 0000000180061c90     common-user64:RgnDetect.obj
 0004:00000c9c       $pdata$?FindFrameTop_ByRight@CRgnDetect@@IEAA_NPEA_WPEAUtag_CharAttr@@HHAEAH22@Z 0000000180061c9c     common-user64:RgnDetect.obj
 0004:00000ca8       $pdata$?FindFrameTop_ByLeft@CRgnDetect@@IEAA_NPEA_WPEAUtag_CharAttr@@HHAEAH22@Z 0000000180061ca8     common-user64:RgnDetect.obj
 0004:00000cb4       $pdata$?FindFrameBottom_ByRight@CRgnDetect@@IEAA_NPEA_WPEAUtag_CharAttr@@HHAEAH22@Z 0000000180061cb4     common-user64:RgnDetect.obj
 0004:00000cc0       $pdata$?FindFrameBottom_ByLeft@CRgnDetect@@IEAA_NPEA_WPEAUtag_CharAttr@@HHAEAH22@Z 0000000180061cc0     common-user64:RgnDetect.obj
 0004:00000ccc       $pdata$?FindFrameRight_ByTop@CRgnDetect@@IEAA_NPEA_WPEAUtag_CharAttr@@HHAEAH22@Z 0000000180061ccc     common-user64:RgnDetect.obj
 0004:00000cd8       $pdata$?FindFrameRight_ByBottom@CRgnDetect@@IEAA_NPEA_WPEAUtag_CharAttr@@HHAEAH22@Z 0000000180061cd8     common-user64:RgnDetect.obj
 0004:00000ce4       $pdata$?FindFrameLeft_ByTop@CRgnDetect@@IEAA_NPEA_WPEAUtag_CharAttr@@HHAEAH22@Z 0000000180061ce4     common-user64:RgnDetect.obj
 0004:00000cf0       $pdata$?FindFrameLeft_ByBottom@CRgnDetect@@IEAA_NPEA_WPEAUtag_CharAttr@@HHAEAH22@Z 0000000180061cf0     common-user64:RgnDetect.obj
 0004:00000cfc       $pdata$?FindByBackground@CRgnDetect@@IEAA_NPEA_WPEAUtag_CharAttr@@HHAEAH222AEA_N@Z 0000000180061cfc     common-user64:RgnDetect.obj
 0004:00000d08       $pdata$?ExpandDialogFrame@CRgnDetect@@IEAA_NPEA_WPEAUtag_CharAttr@@HHAEAH2HH22@Z 0000000180061d08     common-user64:RgnDetect.obj
 0004:00000d14       $pdata$?MarkDialog@CRgnDetect@@IEAAHPEA_WPEAUtag_CharAttr@@HHHHHHI_NK@Z 0000000180061d14     common-user64:RgnDetect.obj
 0004:00000d20       $pdata$?SearchAppPaths@@YA_NPEB_WAEAUCEStr@@_NPEAU1@@Z 0000000180061d20     common-user64:WFiles.obj
 0004:00000d2c       $pdata$?apiShowWindow@@YA_NPEAUHWND__@@H@Z 0000000180061d2c     common-user64:WUser.obj
 0004:00000d38       $pdata$__GSHandlerCheckCommon 0000000180061d38     LIBCMT:_gshandler_.obj
 0004:00000d44       $pdata$__GSHandlerCheck    0000000180061d44     LIBCMT:_gshandler_.obj
 0004:00000d50       $pdata$__GSHandlerCheck_EH 0000000180061d50     LIBCMT:gshandlereh.obj
 0004:00000d68       $pdata$??_Gtype_info@@UEAAPEAXI@Z 0000000180061d68     LIBCMT:std_type_info_static.obj
 0004:00000d74       $pdata$?dllmain_crt_process_attach@@YAHQEAUHINSTANCE__@@QEAX@Z 0000000180061d74     LIBCMT:dll_dllmain.obj
 0004:00000d80       $pdata$?fin$0@?0??dllmain_crt_process_attach@@YAHQEAUHINSTANCE__@@QEAX@Z@4HA 0000000180061d80     LIBCMT:dll_dllmain.obj
 0004:00000d8c       $pdata$?dllmain_crt_process_detach@@YAH_N@Z 0000000180061d8c     LIBCMT:dll_dllmain.obj
 0004:00000d98       $pdata$?fin$0@?0??dllmain_crt_process_detach@@YAH_N@Z@4HA 0000000180061d98     LIBCMT:dll_dllmain.obj
 0004:00000da4       $pdata$?dllmain_crt_dispatch@@YAHQEAUHINSTANCE__@@KQEAX@Z 0000000180061da4     LIBCMT:dll_dllmain.obj
 0004:00000db0       $pdata$?dllmain_dispatch@@YAHQEAUHINSTANCE__@@KQEAX@Z 0000000180061db0     LIBCMT:dll_dllmain.obj
 0004:00000dbc       $pdata$?filt$0@?0??dllmain_dispatch@@YAHQEAUHINSTANCE__@@KQEAX@Z@4HA 0000000180061dbc     LIBCMT:dll_dllmain.obj
 0004:00000dc8       $pdata$_DllMainCRTStartup  0000000180061dc8     LIBCMT:dll_dllmain.obj
 0004:00000dd4       $pdata$__report_securityfailure 0000000180061dd4     LIBCMT:gs_report.obj
 0004:00000de0       $pdata$__report_rangecheckfailure 0000000180061de0     LIBCMT:gs_report.obj
 0004:00000dec       $pdata$__report_gsfailure  0000000180061dec     LIBCMT:gs_report.obj
 0004:00000df8       $pdata$capture_current_context 0000000180061df8     LIBCMT:gs_report.obj
 0004:00000e04       $pdata$capture_previous_context 0000000180061e04     LIBCMT:gs_report.obj
 0004:00000e10       $pdata$__raise_securityfailure 0000000180061e10     LIBCMT:gs_report.obj
 0004:00000e1c       $pdata$__security_init_cookie 0000000180061e1c     LIBCMT:gs_support.obj
 0004:00000e28       $pdata$__scrt_initialize_default_local_stdio_options 0000000180061e28     LIBCMT:default_local_stdio_options.obj
 0004:00000e34       $pdata$__scrt_is_nonwritable_in_current_image 0000000180061e34     LIBCMT:utility.obj
 0004:00000e40       $pdata$__scrt_is_nonwritable_in_current_image$filt$0 0000000180061e40     LIBCMT:utility.obj
 0004:00000e4c       $pdata$__scrt_acquire_startup_lock 0000000180061e4c     LIBCMT:utility.obj
 0004:00000e58       $pdata$__scrt_release_startup_lock 0000000180061e58     LIBCMT:utility.obj
 0004:00000e64       $pdata$__scrt_initialize_crt 0000000180061e64     LIBCMT:utility.obj
 0004:00000e70       $pdata$__scrt_uninitialize_crt 0000000180061e70     LIBCMT:utility.obj
 0004:00000e7c       $pdata$__scrt_initialize_onexit_tables 0000000180061e7c     LIBCMT:utility.obj
 0004:00000e88       $pdata$__scrt_dllmain_exception_filter 0000000180061e88     LIBCMT:utility.obj
 0004:00000e94       $pdata$__scrt_dllmain_before_initialize_c 0000000180061e94     LIBCMT:utility.obj
 0004:00000ea0       $pdata$__scrt_dllmain_after_initialize_c 0000000180061ea0     LIBCMT:utility.obj
 0004:00000eac       $pdata$__scrt_dllmain_uninitialize_c 0000000180061eac     LIBCMT:utility.obj
 0004:00000eb8       $pdata$__scrt_dllmain_uninitialize_critical 0000000180061eb8     LIBCMT:utility.obj
 0004:00000ec4       $pdata$__scrt_dllmain_crt_thread_attach 0000000180061ec4     LIBCMT:utility.obj
 0004:00000ed0       $pdata$__scrt_dllmain_crt_thread_detach 0000000180061ed0     LIBCMT:utility.obj
 0004:00000edc       $pdata$__scrt_fastfail     0000000180061edc     LIBCMT:utility_desktop.obj
 0004:00000ee8       $pdata$_RTC_Initialize     0000000180061ee8     LIBCMT:_initsect_.obj
 0004:00000ef4       $pdata$_RTC_Terminate      0000000180061ef4     LIBCMT:_initsect_.obj
 0004:00000f00       $pdata$__isa_available_init 0000000180061f00     LIBCMT:_cpu_disp_.obj
 0004:00000f18       $pdata$?_GetEstablisherFrame@@YAPEA_KPEA_KPEAU_xDISPATCHER_CONTEXT@@PEBU_s_FuncInfo@@0@Z 0000000180061f18     libvcruntime:risctrnsctrl.obj
 0004:00000f24       $pdata$_GetImageBase       0000000180061f24     libvcruntime:risctrnsctrl.obj
 0004:00000f30       $pdata$_SetImageBase       0000000180061f30     libvcruntime:risctrnsctrl.obj
 0004:00000f3c       $pdata$_GetThrowImageBase  0000000180061f3c     libvcruntime:risctrnsctrl.obj
 0004:00000f48       $pdata$_SetThrowImageBase  0000000180061f48     libvcruntime:risctrnsctrl.obj
 0004:00000f54       $pdata$?__FrameUnwindToEmptyState@@YAXPEA_KPEAU_xDISPATCHER_CONTEXT@@PEBU_s_FuncInfo@@@Z 0000000180061f54     libvcruntime:risctrnsctrl.obj
 0004:00000f60       $pdata$_CallSETranslator   0000000180061f60     libvcruntime:risctrnsctrl.obj
 0004:00000f6c       $pdata$_CallSETranslator$filt$0 0000000180061f6c     libvcruntime:risctrnsctrl.obj
 0004:00000f78       $pdata$?_GetRangeOfTrysToCheck@@YAPEBU_s_TryBlockMapEntry@@PEA_KPEBU_s_FuncInfo@@HHPEAI2PEAU_xDISPATCHER_CONTEXT@@@Z 0000000180061f78     libvcruntime:risctrnsctrl.obj
 0004:00000f84       $pdata$_UnwindNestedFrames 0000000180061f84     libvcruntime:risctrnsctrl.obj
 0004:00000f90       $pdata$?_ExecutionInCatch@@YAHPEAU_xDISPATCHER_CONTEXT@@PEBU_s_FuncInfo@@@Z 0000000180061f90     libvcruntime:risctrnsctrl.obj
 0004:00000f9c       $pdata$_CreateFrameInfo    0000000180061f9c     libvcruntime:risctrnsctrl.obj
 0004:00000fa8       $pdata$_FindAndUnlinkFrame 0000000180061fa8     libvcruntime:risctrnsctrl.obj
 0004:00000fb4       $pdata$__CxxFrameHandler3  0000000180061fb4     libvcruntime:risctrnsctrl.obj
 0004:00000fe4       $pdata$wcschr              0000000180061fe4     libvcruntime:wcschr.obj
 0004:00000ff0       $pdata$__C_specific_handler 0000000180061ff0     libvcruntime:_riscchandler_.obj
 0004:00000ffc       $pdata$strchr              0000000180061ffc     libvcruntime:strchr.obj
 0004:00001008       $pdata$strrchr             0000000180062008     libvcruntime:strrchr.obj
 0004:00001020       $pdata$__std_type_info_destroy_list 0000000180062020     libvcruntime:std_type_info.obj
 0004:0000102c       $pdata$__vcrt_initialize   000000018006202c     libvcruntime:initialization.obj
 0004:00001038       $pdata$__vcrt_uninitialize 0000000180062038     libvcruntime:initialization.obj
 0004:00001044       $pdata$__vcrt_uninitialize_critical 0000000180062044     libvcruntime:initialization.obj
 0004:00001050       $pdata$__vcrt_thread_attach 0000000180062050     libvcruntime:initialization.obj
 0004:0000105c       $pdata$__vcrt_thread_detach 000000018006205c     libvcruntime:initialization.obj
 0004:00001068       $pdata$__vcrt_initialize_ptd 0000000180062068     libvcruntime:per_thread_data.obj
 0004:00001074       $pdata$__vcrt_uninitialize_ptd 0000000180062074     libvcruntime:per_thread_data.obj
 0004:00001080       $pdata$__vcrt_getptd       0000000180062080     libvcruntime:per_thread_data.obj
 0004:0000108c       $pdata$__vcrt_getptd_noexit 000000018006208c     libvcruntime:per_thread_data.obj
 0004:00001098       $pdata$__vcrt_freeptd      0000000180062098     libvcruntime:per_thread_data.obj
 0004:000010a4       $pdata$__vcrt_freefls      00000001800620a4     libvcruntime:per_thread_data.obj
 0004:000010b0       $pdata$?__GetCurrentState@@YAHPEA_KPEAU_xDISPATCHER_CONTEXT@@PEBU_s_FuncInfo@@@Z 00000001800620b0     libvcruntime:riscehstate.obj
 0004:000010bc       $pdata$?__SetUnwindTryBlock@@YAXPEA_KPEAU_xDISPATCHER_CONTEXT@@PEBU_s_FuncInfo@@H@Z 00000001800620bc     libvcruntime:riscehstate.obj
 0004:000010c8       $pdata$?__GetUnwindTryBlock@@YAHPEA_KPEAU_xDISPATCHER_CONTEXT@@PEBU_s_FuncInfo@@@Z 00000001800620c8     libvcruntime:riscehstate.obj
 0004:000010d4       $pdata$?__StateFromIp@@YAHPEBU_s_FuncInfo@@PEAU_xDISPATCHER_CONTEXT@@_K@Z 00000001800620d4     libvcruntime:riscehstate.obj
 0004:000010e0       $pdata$__CxxCallCatchBlock 00000001800620e0     libvcruntime:frame.obj
 0004:000010ec       $pdata$__CxxCallCatchBlock$filt$0 00000001800620ec     libvcruntime:frame.obj
 0004:000010f8       $pdata$__CxxCallCatchBlock$fin$1 00000001800620f8     libvcruntime:frame.obj
 0004:00001104       $pdata$??0exception@std@@QEAA@AEBV01@@Z 0000000180062104     libvcruntime:frame.obj
 0004:00001110       $pdata$??_Gbad_exception@std@@UEAAPEAXI@Z 0000000180062110     libvcruntime:frame.obj
 0004:00001110       $pdata$??_Gexception@std@@UEAAPEAXI@Z 0000000180062110     libvcruntime:frame.obj
 0004:0000111c       $pdata$??0bad_exception@std@@QEAA@AEBV01@@Z 000000018006211c     libvcruntime:frame.obj
 0004:00001128       $pdata$__BuildCatchObject  0000000180062128     libvcruntime:frame.obj
 0004:00001134       $pdata$__TypeMatch         0000000180062134     libvcruntime:frame.obj
 0004:00001140       $pdata$__InternalCxxFrameHandler 0000000180062140     libvcruntime:frame.obj
 0004:0000114c       $pdata$__FrameUnwindToState 000000018006214c     libvcruntime:frame.obj
 0004:00001158       $pdata$__FrameUnwindToState$filt$0 0000000180062158     libvcruntime:frame.obj
 0004:00001164       $pdata$__FrameUnwindToState$fin$1 0000000180062164     libvcruntime:frame.obj
 0004:00001170       $pdata$?FindHandler@@YAXPEAUEHExceptionRecord@@PEA_KPEAU_CONTEXT@@PEAU_xDISPATCHER_CONTEXT@@PEBU_s_FuncInfo@@EH1@Z 0000000180062170     libvcruntime:frame.obj
 0004:0000117c       $pdata$?CatchIt@@YAXPEAUEHExceptionRecord@@PEA_KPEAU_CONTEXT@@PEAU_xDISPATCHER_CONTEXT@@PEBU_s_FuncInfo@@PEBU_s_HandlerType@@PEBU_s_CatchableType@@PEBU_s_TryBlockMapEntry@@H1EE@Z 000000018006217c     libvcruntime:frame.obj
 0004:00001188       $pdata$?FindHandlerForForeignException@@YAXPEAUEHExceptionRecord@@PEA_KPEAU_CONTEXT@@PEAU_xDISPATCHER_CONTEXT@@PEBU_s_FuncInfo@@HH1@Z 0000000180062188     libvcruntime:frame.obj
 0004:00001194       $pdata$?ExFilterRethrow@@YAHPEAU_EXCEPTION_POINTERS@@PEAUEHExceptionRecord@@PEAH@Z 0000000180062194     libvcruntime:frame.obj
 0004:000011a0       $pdata$?IsInExceptionSpec@@YAEPEAUEHExceptionRecord@@PEBU_s_ESTypeList@@@Z 00000001800621a0     libvcruntime:frame.obj
 0004:000011ac       $pdata$__BuildCatchObjectHelper 00000001800621ac     libvcruntime:frame.obj
 0004:000011e8       $pdata$__vcrt_initialize_locks 00000001800621e8     libvcruntime:locks.obj
 0004:000011f4       $pdata$__vcrt_uninitialize_locks 00000001800621f4     libvcruntime:locks.obj
 0004:00001200       $pdata$__vcrt_FlsAlloc     0000000180062200     libvcruntime:winapi_downlevel.obj
 0004:0000120c       $pdata$__vcrt_FlsFree      000000018006220c     libvcruntime:winapi_downlevel.obj
 0004:00001218       $pdata$__vcrt_FlsGetValue  0000000180062218     libvcruntime:winapi_downlevel.obj
 0004:00001224       $pdata$__vcrt_FlsSetValue  0000000180062224     libvcruntime:winapi_downlevel.obj
 0004:00001230       $pdata$__vcrt_InitializeCriticalSectionEx 0000000180062230     libvcruntime:winapi_downlevel.obj
 0004:0000123c       $pdata$__vcrt_initialize_winapi_thunks 000000018006223c     libvcruntime:winapi_downlevel.obj
 0004:00001248       $pdata$__vcrt_uninitialize_winapi_thunks 0000000180062248     libvcruntime:winapi_downlevel.obj
 0004:00001254       $pdata$?try_get_function@@YAPEAXW4function_id@?A0x89697e75@@QEBDQEBW4module_id@2@2@Z 0000000180062254     libvcruntime:winapi_downlevel.obj
 0004:0000126c       $pdata$_IsExceptionObjectToBeDestroyed 000000018006226c     libvcruntime:ehhelpers.obj
 0004:00001278       $pdata$__FrameUnwindFilter 0000000180062278     libvcruntime:ehhelpers.obj
 0004:00001284       $pdata$__DestructExceptionObject 0000000180062284     libvcruntime:ehhelpers.obj
 0004:00001290       $pdata$__DestructExceptionObject$filt$0 0000000180062290     libvcruntime:ehhelpers.obj
 0004:0000129c       $pdata$__std_exception_copy 000000018006229c     libvcruntime:std_exception.obj
 0004:000012a8       $pdata$__std_exception_destroy 00000001800622a8     libvcruntime:std_exception.obj
 0004:000012b4       $pdata$_CxxThrowException  00000001800622b4     libvcruntime:throw.obj
 0004:000012c0       $pdata$??0_LocaleUpdate@@QEAA@QEAU__crt_locale_pointers@@@Z 00000001800622c0     libucrt:output.obj
 0004:000012cc       $pdata$__stdio_common_vswprintf 00000001800622cc     libucrt:output.obj
 0004:000012d8       $pdata$__stdio_common_vsprintf 00000001800622d8     libucrt:output.obj
 0004:000012e4       $pdata$?force_decimal_point@__crt_stdio_output@@YAXPEADQEAU__crt_locale_pointers@@@Z 00000001800622e4     libucrt:output.obj
 0004:000012f0       $pdata$?write_string@?$string_output_adapter@D@__crt_stdio_output@@QEBAXQEBDHQEAH1@Z 00000001800622f0     libucrt:output.obj
 0004:000012fc       $pdata$??0?$output_processor@DV?$string_output_adapter@D@__crt_stdio_output@@V?$standard_base@DV?$string_output_adapter@D@__crt_stdio_output@@@2@@__crt_stdio_output@@QEAA@AEBV?$string_output_adapter@D@1@_KQEBDQEAU__crt_locale_pointers@@QEAD@Z 00000001800622fc     libucrt:output.obj
 0004:00001308       $pdata$?process@?$output_processor@DV?$string_output_adapter@D@__crt_stdio_output@@V?$standard_base@DV?$string_output_adapter@D@__crt_stdio_output@@@2@@__crt_stdio_output@@QEAAHXZ 0000000180062308     libucrt:output.obj
 0004:00001314       $pdata$?state_case_normal@?$output_processor@DV?$string_output_adapter@D@__crt_stdio_output@@V?$standard_base@DV?$string_output_adapter@D@__crt_stdio_output@@@2@@__crt_stdio_output@@AEAA_NXZ 0000000180062314     libucrt:output.obj
 0004:00001320       $pdata$?state_case_normal_tchar@?$output_processor@DV?$string_output_adapter@D@__crt_stdio_output@@V?$standard_base@DV?$string_output_adapter@D@__crt_stdio_output@@@2@@__crt_stdio_output@@AEAA_ND@Z 0000000180062320     libucrt:output.obj
 0004:0000132c       $pdata$?parse_int_from_format_string@?$output_processor@DV?$string_output_adapter@D@__crt_stdio_output@@V?$standard_base@DV?$string_output_adapter@D@__crt_stdio_output@@@2@@__crt_stdio_output@@AEAA_NQEAH@Z 000000018006232c     libucrt:output.obj
 0004:00001338       $pdata$?state_case_size@?$output_processor@DV?$string_output_adapter@D@__crt_stdio_output@@V?$standard_base@DV?$string_output_adapter@D@__crt_stdio_output@@@2@@__crt_stdio_output@@AEAA_NXZ 0000000180062338     libucrt:output.obj
 0004:00001344       $pdata$?state_case_type@?$output_processor@DV?$string_output_adapter@D@__crt_stdio_output@@V?$standard_base@DV?$string_output_adapter@D@__crt_stdio_output@@@2@@__crt_stdio_output@@AEAA_NXZ 0000000180062344     libucrt:output.obj
 0004:00001350       $pdata$?type_case_c_tchar@?$output_processor@DV?$string_output_adapter@D@__crt_stdio_output@@V?$standard_base@DV?$string_output_adapter@D@__crt_stdio_output@@@2@@__crt_stdio_output@@AEAA_ND@Z 0000000180062350     libucrt:output.obj
 0004:0000135c       $pdata$?type_case_Z@?$output_processor@DV?$string_output_adapter@D@__crt_stdio_output@@V?$standard_base@DV?$string_output_adapter@D@__crt_stdio_output@@@2@@__crt_stdio_output@@AEAA_NXZ 000000018006235c     libucrt:output.obj
 0004:00001368       $pdata$?type_case_s@?$output_processor@DV?$string_output_adapter@D@__crt_stdio_output@@V?$standard_base@DV?$string_output_adapter@D@__crt_stdio_output@@@2@@__crt_stdio_output@@AEAA_NXZ 0000000180062368     libucrt:output.obj
 0004:00001374       $pdata$?type_case_a@?$output_processor@DV?$string_output_adapter@D@__crt_stdio_output@@V?$standard_base@DV?$string_output_adapter@D@__crt_stdio_output@@@2@@__crt_stdio_output@@AEAA_NXZ 0000000180062374     libucrt:output.obj
 0004:00001380       $pdata$?type_case_integer@?$output_processor@DV?$string_output_adapter@D@__crt_stdio_output@@V?$standard_base@DV?$string_output_adapter@D@__crt_stdio_output@@@2@@__crt_stdio_output@@AEAA_NI_N@Z 0000000180062380     libucrt:output.obj
 0004:00001380       $pdata$?type_case_integer@?$output_processor@_WV?$string_output_adapter@_W@__crt_stdio_output@@V?$standard_base@_WV?$string_output_adapter@_W@__crt_stdio_output@@@2@@__crt_stdio_output@@AEAA_NI_N@Z 0000000180062380     libucrt:output.obj
 0004:0000138c       $pdata$?type_case_n@?$output_processor@_WV?$string_output_adapter@_W@__crt_stdio_output@@V?$standard_base@_WV?$string_output_adapter@_W@__crt_stdio_output@@@2@@__crt_stdio_output@@AEAA_NXZ 000000018006238c     libucrt:output.obj
 0004:0000138c       $pdata$?type_case_n@?$output_processor@DV?$string_output_adapter@D@__crt_stdio_output@@V?$standard_base@DV?$string_output_adapter@D@__crt_stdio_output@@@2@@__crt_stdio_output@@AEAA_NXZ 000000018006238c     libucrt:output.obj
 0004:00001398       $pdata$?write_stored_string_tchar@?$output_processor@DV?$string_output_adapter@D@__crt_stdio_output@@V?$standard_base@DV?$string_output_adapter@D@__crt_stdio_output@@@2@@__crt_stdio_output@@AEAA_ND@Z 0000000180062398     libucrt:output.obj
 0004:000013a4       $pdata$?write_string@?$string_output_adapter@_W@__crt_stdio_output@@QEBAXQEB_WHQEAH1@Z 00000001800623a4     libucrt:output.obj
 0004:000013b0       $pdata$??0?$output_processor@_WV?$string_output_adapter@_W@__crt_stdio_output@@V?$standard_base@_WV?$string_output_adapter@_W@__crt_stdio_output@@@2@@__crt_stdio_output@@QEAA@AEBV?$string_output_adapter@_W@1@_KQEB_WQEAU__crt_locale_pointers@@QEAD@Z 00000001800623b0     libucrt:output.obj
 0004:000013bc       $pdata$?process@?$output_processor@_WV?$string_output_adapter@_W@__crt_stdio_output@@V?$standard_base@_WV?$string_output_adapter@_W@__crt_stdio_output@@@2@@__crt_stdio_output@@QEAAHXZ 00000001800623bc     libucrt:output.obj
 0004:000013c8       $pdata$?parse_int_from_format_string@?$output_processor@_WV?$string_output_adapter@_W@__crt_stdio_output@@V?$standard_base@_WV?$string_output_adapter@_W@__crt_stdio_output@@@2@@__crt_stdio_output@@AEAA_NQEAH@Z 00000001800623c8     libucrt:output.obj
 0004:000013d4       $pdata$?state_case_size@?$output_processor@_WV?$string_output_adapter@_W@__crt_stdio_output@@V?$standard_base@_WV?$string_output_adapter@_W@__crt_stdio_output@@@2@@__crt_stdio_output@@AEAA_NXZ 00000001800623d4     libucrt:output.obj
 0004:000013e0       $pdata$?state_case_type@?$output_processor@_WV?$string_output_adapter@_W@__crt_stdio_output@@V?$standard_base@_WV?$string_output_adapter@_W@__crt_stdio_output@@@2@@__crt_stdio_output@@AEAA_NXZ 00000001800623e0     libucrt:output.obj
 0004:000013ec       $pdata$?type_case_c_tchar@?$output_processor@_WV?$string_output_adapter@_W@__crt_stdio_output@@V?$standard_base@_WV?$string_output_adapter@_W@__crt_stdio_output@@@2@@__crt_stdio_output@@AEAA_N_W@Z 00000001800623ec     libucrt:output.obj
 0004:000013f8       $pdata$?type_case_Z@?$output_processor@_WV?$string_output_adapter@_W@__crt_stdio_output@@V?$standard_base@_WV?$string_output_adapter@_W@__crt_stdio_output@@@2@@__crt_stdio_output@@AEAA_NXZ 00000001800623f8     libucrt:output.obj
 0004:00001404       $pdata$?type_case_s@?$output_processor@_WV?$string_output_adapter@_W@__crt_stdio_output@@V?$standard_base@_WV?$string_output_adapter@_W@__crt_stdio_output@@@2@@__crt_stdio_output@@AEAA_NXZ 0000000180062404     libucrt:output.obj
 0004:00001410       $pdata$?type_case_a@?$output_processor@_WV?$string_output_adapter@_W@__crt_stdio_output@@V?$standard_base@_WV?$string_output_adapter@_W@__crt_stdio_output@@@2@@__crt_stdio_output@@AEAA_NXZ 0000000180062410     libucrt:output.obj
 0004:0000141c       $pdata$?write_stored_string_tchar@?$output_processor@_WV?$string_output_adapter@_W@__crt_stdio_output@@V?$standard_base@_WV?$string_output_adapter@_W@__crt_stdio_output@@@2@@__crt_stdio_output@@AEAA_N_W@Z 000000018006241c     libucrt:output.obj
 0004:00001428       $pdata$??$write_multiple_characters@V?$string_output_adapter@D@__crt_stdio_output@@D@__crt_stdio_output@@YAXAEBV?$string_output_adapter@D@0@DHQEAH@Z 0000000180062428     libucrt:output.obj
 0004:00001434       $pdata$??$write_multiple_characters@V?$string_output_adapter@_W@__crt_stdio_output@@D@__crt_stdio_output@@YAXAEBV?$string_output_adapter@_W@0@DHQEAH@Z 0000000180062434     libucrt:output.obj
 0004:00001440       $pdata$??$ensure_buffer_is_big_enough@D@formatting_buffer@__crt_stdio_output@@QEAA_N_K@Z 0000000180062440     libucrt:output.obj
 0004:0000144c       $pdata$??$type_case_integer_parse_into_buffer@_K@?$output_processor@_WV?$string_output_adapter@_W@__crt_stdio_output@@V?$standard_base@_WV?$string_output_adapter@_W@__crt_stdio_output@@@2@@__crt_stdio_output@@AEAAX_KI_N@Z 000000018006244c     libucrt:output.obj
 0004:0000144c       $pdata$??$type_case_integer_parse_into_buffer@_K@?$output_processor@DV?$string_output_adapter@D@__crt_stdio_output@@V?$standard_base@DV?$string_output_adapter@D@__crt_stdio_output@@@2@@__crt_stdio_output@@AEAAX_KI_N@Z 000000018006244c     libucrt:output.obj
 0004:00001458       $pdata$??$type_case_integer_parse_into_buffer@I@?$output_processor@_WV?$string_output_adapter@_W@__crt_stdio_output@@V?$standard_base@_WV?$string_output_adapter@_W@__crt_stdio_output@@@2@@__crt_stdio_output@@AEAAXII_N@Z 0000000180062458     libucrt:output.obj
 0004:00001458       $pdata$??$type_case_integer_parse_into_buffer@I@?$output_processor@DV?$string_output_adapter@D@__crt_stdio_output@@V?$standard_base@DV?$string_output_adapter@D@__crt_stdio_output@@@2@@__crt_stdio_output@@AEAAXII_N@Z 0000000180062458     libucrt:output.obj
 0004:00001464       $pdata$wcstol              0000000180062464     libucrt:strtox.obj
 0004:00001470       $pdata$strtol              0000000180062470     libucrt:strtox.obj
 0004:0000147c       $pdata$??$parse_integer@KV?$c_string_character_source@D@__crt_strtox@@@__crt_strtox@@YAKQEAU__crt_locale_pointers@@V?$c_string_character_source@D@0@H_N@Z 000000018006247c     libucrt:strtox.obj
 0004:00001488       $pdata$??$parse_integer@KV?$c_string_character_source@_W@__crt_strtox@@@__crt_strtox@@YAKQEAU__crt_locale_pointers@@V?$c_string_character_source@_W@0@H_N@Z 0000000180062488     libucrt:strtox.obj
 0004:00001494       $pdata$_initterm           0000000180062494     libucrt:initterm.obj
 0004:000014a0       $pdata$_initterm_e         00000001800624a0     libucrt:initterm.obj
 0004:000014ac       $pdata$_seh_filter_exe     00000001800624ac     libucrt:exception_filter.obj
 0004:000014b8       $pdata$?try_cor_exit_process@@YAXI@Z 00000001800624b8     libucrt:exit.obj
 0004:000014c4       $pdata$?exit_or_terminate_process@@YAXI@Z 00000001800624c4     libucrt:exit.obj
 0004:000014d0       $pdata$?common_exit@@YAXHW4_crt_exit_cleanup_mode@@W4_crt_exit_return_mode@@@Z 00000001800624d0     libucrt:exit.obj
 0004:000014dc       $pdata$?filt$0@?0??common_exit@@YAXHW4_crt_exit_cleanup_mode@@W4_crt_exit_return_mode@@@Z@4HA 00000001800624dc     libucrt:exit.obj
 0004:000014e8       $pdata$?fin$1@?0??common_exit@@YAXHW4_crt_exit_cleanup_mode@@W4_crt_exit_return_mode@@@Z@4HA 00000001800624e8     libucrt:exit.obj
 0004:000014f4       $pdata$_configure_narrow_argv 00000001800624f4     libucrt:argv_parsing.obj
 0004:00001500       $pdata$__acrt_allocate_buffer_for_argv 0000000180062500     libucrt:argv_parsing.obj
 0004:0000150c       $pdata$??$parse_command_line@D@@YAXPEADPEAPEAD0PEA_K2@Z 000000018006250c     libucrt:argv_parsing.obj
 0004:00001518       $pdata$__dcrt_uninitialize_environments_nolock 0000000180062518     libucrt:environment_initialization.obj
 0004:00001524       $pdata$??$common_initialize_environment_nolock@D@@YAHXZ 0000000180062524     libucrt:environment_initialization.obj
 0004:00001530       $pdata$??$uninitialize_environment_internal@D@@YAXAEAPEAPEAD@Z 0000000180062530     libucrt:environment_initialization.obj
 0004:0000153c       $pdata$??$uninitialize_environment_internal@_W@@YAXAEAPEAPEA_W@Z 000000018006253c     libucrt:environment_initialization.obj
 0004:00001548       $pdata$??$free_environment@_W@@YAXQEAPEA_W@Z 0000000180062548     libucrt:environment_initialization.obj
 0004:00001548       $pdata$??$free_environment@D@@YAXQEAPEAD@Z 0000000180062548     libucrt:environment_initialization.obj
 0004:00001554       $pdata$??$create_environment@D@@YAQEAPEADQEAD@Z 0000000180062554     libucrt:environment_initialization.obj
 0004:00001560       $pdata$_execute_onexit_table 0000000180062560     libucrt:onexit.obj
 0004:0000156c       $pdata$??$?RV<lambda_e24bbb7b643b32fcea6fa61b31d4c984>@@AEAV<lambda_275893d493268fdec8709772e3fcec0e>@@V<lambda_9d71df4d7cf3f480f8d633942495c3b0>@@@?$__crt_seh_guarded_call@H@@QEAAH$$QEAV<lambda_e24bbb7b643b32fcea6fa61b31d4c984>@@AEAV<lambda_275893d493268fdec8709772e3fcec0e>@@$$QEAV<lambda_9d71df4d7cf3f480f8d633942495c3b0>@@@Z 000000018006256c     libucrt:onexit.obj
 0004:00001578       $pdata$?fin$0@?0???$?RV<lambda_e24bbb7b643b32fcea6fa61b31d4c984>@@AEAV<lambda_275893d493268fdec8709772e3fcec0e>@@V<lambda_9d71df4d7cf3f480f8d633942495c3b0>@@@?$__crt_seh_guarded_call@H@@QEAAH$$QEAV<lambda_e24bbb7b643b32fcea6fa61b31d4c984>@@AEAV<lambda_275893d493268fdec8709772e3fcec0e>@@$$QEAV<lambda_9d71df4d7cf3f480f8d633942495c3b0>@@@Z@4HA 0000000180062578     libucrt:onexit.obj
 0004:00001584       $pdata$__acrt_uninitialize_critical 0000000180062584     libucrt:initialization.obj
 0004:00001590       $pdata$__acrt_thread_attach 0000000180062590     libucrt:initialization.obj
 0004:0000159c       $pdata$__acrt_thread_detach 000000018006259c     libucrt:initialization.obj
 0004:000015a8       $pdata$initialize_c        00000001800625a8     libucrt:initialization.obj
 0004:000015b4       $pdata$uninitialize_environment 00000001800625b4     libucrt:initialization.obj
 0004:000015c0       $pdata$initialize_pointers 00000001800625c0     libucrt:initialization.obj
 0004:000015cc       $pdata$uninitialize_allocated_memory 00000001800625cc     libucrt:initialization.obj
 0004:000015d8       $pdata$terminate           00000001800625d8     libucrt:terminate.obj
 0004:000015e4       $pdata$strcpy_s            00000001800625e4     libucrt:strcpy_s.obj
 0004:000015f0       $pdata$abort               00000001800625f0     libucrt:abort.obj
 0004:00001608       $pdata$_invalid_parameter_noinfo 0000000180062608     libucrt:invalid_parameter.obj
 0004:00001614       $pdata$_invoke_watson      0000000180062614     libucrt:invalid_parameter.obj
 0004:00001620       $pdata$__acrt_call_reportfault 0000000180062620     libucrt:invalid_parameter.obj
 0004:0000162c       $pdata$_invalid_parameter  000000018006262c     libucrt:invalid_parameter.obj
 0004:00001638       $pdata$isdigit             0000000180062638     libucrt:_ctype.obj
 0004:00001644       $pdata$tolower             0000000180062644     libucrt:tolower_toupper.obj
 0004:00001650       $pdata$_tolower_l          0000000180062650     libucrt:tolower_toupper.obj
 0004:0000165c       $pdata$?internal_isupper_l@@YA_NHQEAU__crt_locale_pointers@@@Z 000000018006265c     libucrt:tolower_toupper.obj
 0004:00001668       $pdata$_errno              0000000180062668     libucrt:errno.obj
 0004:00001674       $pdata$__doserrno          0000000180062674     libucrt:errno.obj
 0004:00001680       $pdata$__acrt_errno_map_os_error 0000000180062680     libucrt:errno.obj
 0004:0000168c       $pdata$_free_base          000000018006268c     libucrt:free_base.obj
 0004:00001698       $pdata$_malloc_base        0000000180062698     libucrt:malloc_base.obj
 0004:000016a4       $pdata$_mbtowc_l           00000001800626a4     libucrt:mbtowc.obj
 0004:000016b0       $pdata$wctomb_s            00000001800626b0     libucrt:wctomb.obj
 0004:000016bc       $pdata$_wctomb_s_l         00000001800626bc     libucrt:wctomb.obj
 0004:000016c8       $pdata$wcsnlen             00000001800626c8     libucrt:strnlen.obj
 0004:000016d4       $pdata$strnlen             00000001800626d4     libucrt:strnlen.obj
 0004:000016e0       $pdata$__acrt_initialize_ptd 00000001800626e0     libucrt:per_thread_data.obj
 0004:000016ec       $pdata$__acrt_uninitialize_ptd 00000001800626ec     libucrt:per_thread_data.obj
 0004:000016f8       $pdata$__acrt_getptd       00000001800626f8     libucrt:per_thread_data.obj
 0004:00001704       $pdata$__acrt_getptd_noexit 0000000180062704     libucrt:per_thread_data.obj
 0004:00001710       $pdata$__acrt_freeptd      0000000180062710     libucrt:per_thread_data.obj
 0004:0000171c       $pdata$?destroy_fls@@YAXPEAX@Z 000000018006271c     libucrt:per_thread_data.obj
 0004:00001728       $pdata$?replace_current_thread_locale_nolock@@YAXQEAU__acrt_ptd@@QEAU__crt_locale_data@@@Z 0000000180062728     libucrt:per_thread_data.obj
 0004:00001734       $pdata$?construct_ptd_array@@YAXQEAU__acrt_ptd@@@Z 0000000180062734     libucrt:per_thread_data.obj
 0004:00001740       $pdata$?destroy_ptd_array@@YAXQEAU__acrt_ptd@@@Z 0000000180062740     libucrt:per_thread_data.obj
 0004:0000174c       $pdata$??$?RV<lambda_72d1df2b273a38828b1ce30cbf4cdab5>@@AEAV<lambda_876a65b173b8412d3a47c70a915b0cf4>@@V<lambda_41932305e351933ebe8f8be3ed8bb5dc>@@@?$__crt_seh_guarded_call@X@@QEAAX$$QEAV<lambda_72d1df2b273a38828b1ce30cbf4cdab5>@@AEAV<lambda_876a65b173b8412d3a47c70a915b0cf4>@@$$QEAV<lambda_41932305e351933ebe8f8be3ed8bb5dc>@@@Z 000000018006274c     libucrt:per_thread_data.obj
 0004:00001758       $pdata$?fin$0@?0???$?RV<lambda_fb3a7dec4e47f37f22dae91bb15c9095>@@AEAV<lambda_698284760c8add0bfb0756c19673e34b>@@V<lambda_dfb8eca1e75fef3034a8fb18dd509707>@@@?$__crt_seh_guarded_call@X@@QEAAX$$QEAV<lambda_fb3a7dec4e47f37f22dae91bb15c9095>@@AEAV<lambda_698284760c8add0bfb0756c19673e34b>@@$$QEAV<lambda_dfb8eca1e75fef3034a8fb18dd509707>@@@Z@4HA 0000000180062758     libucrt:per_thread_data.obj
 0004:00001758       $pdata$?fin$0@?0???$?RV<lambda_5e887d1dcbef67a5eb4283622ba103bf>@@AEAV<lambda_4466841279450cc726390878d4a41900>@@V<lambda_341c25c0346d94847f1f3c463c57e077>@@@?$__crt_seh_guarded_call@X@@QEAAX$$QEAV<lambda_5e887d1dcbef67a5eb4283622ba103bf>@@AEAV<lambda_4466841279450cc726390878d4a41900>@@$$QEAV<lambda_341c25c0346d94847f1f3c463c57e077>@@@Z@4HA 0000000180062758     libucrt:per_thread_data.obj
 0004:00001758       $pdata$?fin$0@?0???$?RV<lambda_99476a1ad63dd22509b5d3e65b0ffc95>@@AEAV<lambda_ad1ced32f4ac17aa236e5ef05d6b3b7c>@@V<lambda_f7424dd8d45958661754dc4f2697e9c3>@@@?$__crt_seh_guarded_call@X@@QEAAX$$QEAV<lambda_99476a1ad63dd22509b5d3e65b0ffc95>@@AEAV<lambda_ad1ced32f4ac17aa236e5ef05d6b3b7c>@@$$QEAV<lambda_f7424dd8d45958661754dc4f2697e9c3>@@@Z@4HA 0000000180062758     libucrt:mbctype.obj
 0004:00001758       $pdata$?fin$0@?0???$?RV<lambda_46352004c1216016012b18bd6f87e700>@@AEAV<lambda_3bd07e1a1191394380780325891bf33f>@@V<lambda_334532d3f185bcaa59b5be82d7d22bff>@@@?$__crt_seh_guarded_call@X@@QEAAX$$QEAV<lambda_46352004c1216016012b18bd6f87e700>@@AEAV<lambda_3bd07e1a1191394380780325891bf33f>@@$$QEAV<lambda_334532d3f185bcaa59b5be82d7d22bff>@@@Z@4HA 0000000180062758     libucrt:per_thread_data.obj
 0004:00001758       $pdata$?fin$0@?0???$?RV<lambda_c36588078e9f5dfd39652860aa6b3aaf>@@AEAV<lambda_ec61778202f4f5fc7e7711acc23c3bca>@@V<lambda_dc9d2797ccde5d239b4a0efae8ebd7db>@@@?$__crt_seh_guarded_call@P6AXH@Z@@QEAAP6AXH@Z$$QEAV<lambda_c36588078e9f5dfd39652860aa6b3aaf>@@AEAV<lambda_ec61778202f4f5fc7e7711acc23c3bca>@@$$QEAV<lambda_dc9d2797ccde5d239b4a0efae8ebd7db>@@@Z@4HA 0000000180062758     libucrt:signal.obj
 0004:00001758       $pdata$?fin$0@?0???$?RV<lambda_72d1df2b273a38828b1ce30cbf4cdab5>@@AEAV<lambda_876a65b173b8412d3a47c70a915b0cf4>@@V<lambda_41932305e351933ebe8f8be3ed8bb5dc>@@@?$__crt_seh_guarded_call@X@@QEAAX$$QEAV<lambda_72d1df2b273a38828b1ce30cbf4cdab5>@@AEAV<lambda_876a65b173b8412d3a47c70a915b0cf4>@@$$QEAV<lambda_41932305e351933ebe8f8be3ed8bb5dc>@@@Z@4HA 0000000180062758     libucrt:per_thread_data.obj
 0004:00001764       $pdata$??$?RV<lambda_5e887d1dcbef67a5eb4283622ba103bf>@@AEAV<lambda_4466841279450cc726390878d4a41900>@@V<lambda_341c25c0346d94847f1f3c463c57e077>@@@?$__crt_seh_guarded_call@X@@QEAAX$$QEAV<lambda_5e887d1dcbef67a5eb4283622ba103bf>@@AEAV<lambda_4466841279450cc726390878d4a41900>@@$$QEAV<lambda_341c25c0346d94847f1f3c463c57e077>@@@Z 0000000180062764     libucrt:per_thread_data.obj
 0004:00001770       $pdata$??$?RV<lambda_46352004c1216016012b18bd6f87e700>@@AEAV<lambda_3bd07e1a1191394380780325891bf33f>@@V<lambda_334532d3f185bcaa59b5be82d7d22bff>@@@?$__crt_seh_guarded_call@X@@QEAAX$$QEAV<lambda_46352004c1216016012b18bd6f87e700>@@AEAV<lambda_3bd07e1a1191394380780325891bf33f>@@$$QEAV<lambda_334532d3f185bcaa59b5be82d7d22bff>@@@Z 0000000180062770     libucrt:per_thread_data.obj
 0004:0000177c       $pdata$??$?RV<lambda_fb3a7dec4e47f37f22dae91bb15c9095>@@AEAV<lambda_698284760c8add0bfb0756c19673e34b>@@V<lambda_dfb8eca1e75fef3034a8fb18dd509707>@@@?$__crt_seh_guarded_call@X@@QEAAX$$QEAV<lambda_fb3a7dec4e47f37f22dae91bb15c9095>@@AEAV<lambda_698284760c8add0bfb0756c19673e34b>@@$$QEAV<lambda_dfb8eca1e75fef3034a8fb18dd509707>@@@Z 000000018006277c     libucrt:per_thread_data.obj
 0004:00001788       $pdata$__acrt_update_locale_info 0000000180062788     libucrt:locale_update.obj
 0004:00001794       $pdata$__acrt_update_multibyte_info 0000000180062794     libucrt:locale_update.obj
 0004:000017a0       $pdata$__acrt_fp_format    00000001800627a0     libucrt:cvt.obj
 0004:000017ac       $pdata$?fp_format_nan_or_infinity@@YAHW4__acrt_fp_class@@_NPEAD_K1@Z 00000001800627ac     libucrt:cvt.obj
 0004:000017b8       $pdata$?fp_format_e_internal@@YAHQEAD_KH_NIQEAU_strflt@@2QEAU__crt_locale_pointers@@@Z 00000001800627b8     libucrt:cvt.obj
 0004:000017c4       $pdata$?fp_format_e@@YAHQEBNQEAD_K12H_NIQEAU__crt_locale_pointers@@@Z 00000001800627c4     libucrt:cvt.obj
 0004:000017d0       $pdata$?fp_format_a@@YAHQEBNPEAD_KQEAD2H_NIQEAU__crt_locale_pointers@@@Z 00000001800627d0     libucrt:cvt.obj
 0004:000017dc       $pdata$?fp_format_f_internal@@YAHQEAD_KHQEAU_strflt@@_NQEAU__crt_locale_pointers@@@Z 00000001800627dc     libucrt:cvt.obj
 0004:000017e8       $pdata$?fp_format_g@@YAHQEBNQEAD_K12H_NIQEAU__crt_locale_pointers@@@Z 00000001800627e8     libucrt:cvt.obj
 0004:000017f4       $pdata$_fileno             00000001800627f4     libucrt:fileno.obj
 0004:00001800       $pdata$__acrt_initialize_stdio 0000000180062800     libucrt:_file.obj
 0004:0000180c       $pdata$__acrt_uninitialize_stdio 000000018006280c     libucrt:_file.obj
 0004:00001818       $pdata$__acrt_uninitialize_locale 0000000180062818     libucrt:wsetlocale.obj
 0004:00001824       $pdata$__acrt_uninitialize_locale$fin$0 0000000180062824     libucrt:wsetlocale.obj
 0004:00001824       $pdata$__acrt_update_thread_locale_data$fin$0 0000000180062824     libucrt:locale_refcounting.obj
 0004:00001830       $pdata$__acrt_initialize_lowio 0000000180062830     libucrt:ioinit.obj
 0004:0000183c       $pdata$__acrt_lowio_ensure_fh_exists$fin$0 000000018006283c     libucrt:osfinfo.obj
 0004:0000183c       $pdata$__acrt_initialize_lowio$fin$0 000000018006283c     libucrt:ioinit.obj
 0004:00001848       $pdata$__acrt_uninitialize_lowio 0000000180062848     libucrt:ioinit.obj
 0004:00001854       $pdata$?initialize_inherited_file_handles_nolock@@YAXXZ 0000000180062854     libucrt:ioinit.obj
 0004:00001860       $pdata$?initialize_stdio_handles_nolock@@YAXXZ 0000000180062860     libucrt:ioinit.obj
 0004:0000186c       $pdata$__pctype_func       000000018006286c     libucrt:ctype.obj
 0004:00001878       $pdata$iswctype            0000000180062878     libucrt:iswctype.obj
 0004:00001884       $pdata$_isctype_l          0000000180062884     libucrt:isctype.obj
 0004:00001890       $pdata$__acrt_initialize_locks 0000000180062890     libucrt:locks.obj
 0004:0000189c       $pdata$__acrt_uninitialize_locks 000000018006289c     libucrt:locks.obj
 0004:000018a8       $pdata$__acrt_FlsAlloc     00000001800628a8     libucrt:winapi_thunks.obj
 0004:000018b4       $pdata$__acrt_FlsFree      00000001800628b4     libucrt:winapi_thunks.obj
 0004:000018c0       $pdata$__acrt_FlsGetValue  00000001800628c0     libucrt:winapi_thunks.obj
 0004:000018cc       $pdata$__acrt_FlsSetValue  00000001800628cc     libucrt:winapi_thunks.obj
 0004:000018d8       $pdata$__acrt_initialize_winapi_thunks 00000001800628d8     libucrt:winapi_thunks.obj
 0004:000018e4       $pdata$__acrt_uninitialize_winapi_thunks 00000001800628e4     libucrt:winapi_thunks.obj
 0004:000018f0       $pdata$__acrt_InitializeCriticalSectionEx 00000001800628f0     libucrt:winapi_thunks.obj
 0004:000018fc       $pdata$__acrt_LCMapStringEx 00000001800628fc     libucrt:winapi_thunks.obj
 0004:00001908       $pdata$__acrt_LocaleNameToLCID 0000000180062908     libucrt:winapi_thunks.obj
 0004:00001914       $pdata$__acrt_is_packaged_app 0000000180062914     libucrt:winapi_thunks.obj
 0004:00001920       $pdata$?try_get_function@@YAPEAXW4function_id@?A0x63058377@@QEBDQEBW4module_id@2@2@Z 0000000180062920     libucrt:winapi_thunks.obj
 0004:0000192c       $pdata$_calloc_base        000000018006292c     libucrt:calloc_base.obj
 0004:00001938       $pdata$??$common_expand_argv_wildcards@D@@YAHQEAPEADQEAPEAPEAD@Z 0000000180062938     libucrt:argv_wildcards.obj
 0004:00001944       $pdata$?expand_if_necessary@?$argument_list@D@?A0xca0879c4@@AEAAHXZ 0000000180062944     libucrt:argv_wildcards.obj
 0004:00001950       $pdata$??$copy_and_add_argument_to_buffer@D@@YAHQEBD0_KAEAV?$argument_list@D@?A0xca0879c4@@@Z 0000000180062950     libucrt:argv_wildcards.obj
 0004:0000195c       $pdata$??$expand_argument_wildcards@D@@YAHQEAD0AEAV?$argument_list@D@?A0xca0879c4@@@Z 000000018006295c     libucrt:argv_wildcards.obj
 0004:00001968       $pdata$__acrt_update_thread_multibyte_data 0000000180062968     libucrt:mbctype.obj
 0004:00001974       $pdata$__acrt_update_thread_multibyte_data$fin$0 0000000180062974     libucrt:mbctype.obj
 0004:00001980       $pdata$__acrt_initialize_multibyte 0000000180062980     libucrt:mbctype.obj
 0004:0000198c       $pdata$_setmbcp_nolock     000000018006298c     libucrt:mbctype.obj
 0004:00001998       $pdata$?getSystemCP@@YAHH@Z 0000000180062998     libucrt:mbctype.obj
 0004:000019a4       $pdata$?setSBCS@@YAXPEAU__crt_multibyte_data@@@Z 00000001800629a4     libucrt:mbctype.obj
 0004:000019b0       $pdata$?setSBUpLow@@YAXPEAU__crt_multibyte_data@@@Z 00000001800629b0     libucrt:mbctype.obj
 0004:000019bc       $pdata$?setmbcp_internal@@YAHH_N@Z 00000001800629bc     libucrt:mbctype.obj
 0004:000019c8       $pdata$??R<lambda_ad1ced32f4ac17aa236e5ef05d6b3b7c>@@QEBAXXZ 00000001800629c8     libucrt:mbctype.obj
 0004:000019d4       $pdata$??$?RV<lambda_99476a1ad63dd22509b5d3e65b0ffc95>@@AEAV<lambda_ad1ced32f4ac17aa236e5ef05d6b3b7c>@@V<lambda_f7424dd8d45958661754dc4f2697e9c3>@@@?$__crt_seh_guarded_call@X@@QEAAX$$QEAV<lambda_99476a1ad63dd22509b5d3e65b0ffc95>@@AEAV<lambda_ad1ced32f4ac17aa236e5ef05d6b3b7c>@@$$QEAV<lambda_f7424dd8d45958661754dc4f2697e9c3>@@@Z 00000001800629d4     libucrt:mbctype.obj
 0004:000019e0       $pdata$?x_ismbbtype_l@@YAHPEAU__crt_locale_pointers@@IHH@Z 00000001800629e0     libucrt:ismbbyte.obj
 0004:000019ec       $pdata$__acrt_initialize_command_line 00000001800629ec     libucrt:argv_data.obj
 0004:000019f8       $pdata$__dcrt_get_narrow_environment_from_os 00000001800629f8     libucrt:get_environment_from_os.obj
 0004:00001a04       $pdata$_recalloc_base      0000000180062a04     libucrt:recalloc.obj
 0004:00001a10       $pdata$__acrt_initialize_heap 0000000180062a10     libucrt:heap_handle.obj
 0004:00001a1c       $pdata$__acrt_execute_initializers 0000000180062a1c     libucrt:shared_initialization.obj
 0004:00001a28       $pdata$__acrt_execute_uninitializers 0000000180062a28     libucrt:shared_initialization.obj
 0004:00001a34       $pdata$_callnewh           0000000180062a34     libucrt:new_handler.obj
 0004:00001a40       $pdata$_query_new_handler  0000000180062a40     libucrt:new_handler.obj
 0004:00001a4c       $pdata$_query_new_handler$fin$0 0000000180062a4c     libucrt:new_handler.obj
 0004:00001a58       $pdata$__acrt_get_sigabrt_handler 0000000180062a58     libucrt:signal.obj
 0004:00001a64       $pdata$raise               0000000180062a64     libucrt:signal.obj
 0004:00001a70       $pdata$raise$fin$0         0000000180062a70     libucrt:signal.obj
 0004:00001a7c       $pdata$??$?RV<lambda_c36588078e9f5dfd39652860aa6b3aaf>@@AEAV<lambda_ec61778202f4f5fc7e7711acc23c3bca>@@V<lambda_dc9d2797ccde5d239b4a0efae8ebd7db>@@@?$__crt_seh_guarded_call@P6AXH@Z@@QEAAP6AXH@Z$$QEAV<lambda_c36588078e9f5dfd39652860aa6b3aaf>@@AEAV<lambda_ec61778202f4f5fc7e7711acc23c3bca>@@$$QEAV<lambda_dc9d2797ccde5d239b4a0efae8ebd7db>@@@Z 0000000180062a7c     libucrt:signal.obj
 0004:00001a88       $pdata$__acrt_invoke_user_matherr 0000000180062a88     libucrt:matherr.obj
 0004:00001a94       $pdata$_isleadbyte_l       0000000180062a94     libucrt:_wctype.obj
 0004:00001aa0       $pdata$__acrt_LCMapStringA 0000000180062aa0     libucrt:lcmapstringa.obj
 0004:00001aac       $pdata$?__acrt_LCMapStringA_stat@@YAHPEAU__crt_locale_pointers@@PEB_WKPEBDHPEADHHH@Z 0000000180062aac     libucrt:lcmapstringa.obj
 0004:00001ab8       $pdata$__acrt_release_locale_ref 0000000180062ab8     libucrt:locale_refcounting.obj
 0004:00001ac4       $pdata$__acrt_free_locale  0000000180062ac4     libucrt:locale_refcounting.obj
 0004:00001ad0       $pdata$__acrt_locale_free_lc_time_if_unreferenced 0000000180062ad0     libucrt:locale_refcounting.obj
 0004:00001adc       $pdata$__acrt_update_thread_locale_data 0000000180062adc     libucrt:locale_refcounting.obj
 0004:00001ae8       $pdata$_updatetlocinfoEx_nolock 0000000180062ae8     libucrt:locale_refcounting.obj
 0004:00001af4       $pdata$__acrt_fp_strflt_to_string 0000000180062af4     libucrt:_fptostr.obj
 0004:00001b00       $pdata$memcpy_s            0000000180062b00     libucrt:cfout.obj
 0004:00001b0c       $pdata$__acrt_fltout       0000000180062b0c     libucrt:cfout.obj
 0004:00001b18       $pdata$?divide@__crt_strtox@@YA_KAEAUbig_integer@1@AEBU21@@Z 0000000180062b18     libucrt:cfout.obj
 0004:00001b24       $pdata$5$?divide@__crt_strtox@@YA_KAEAUbig_integer@1@AEBU21@@Z 0000000180062b24     libucrt:cfout.obj
 0004:00001b30       $pdata$6$?divide@__crt_strtox@@YA_KAEAUbig_integer@1@AEBU21@@Z 0000000180062b30     libucrt:cfout.obj
 0004:00001b3c       $pdata$_fcloseall          0000000180062b3c     libucrt:closeall.obj
 0004:00001b48       $pdata$_fcloseall$fin$0    0000000180062b48     libucrt:closeall.obj
 0004:00001b54       $pdata$_fflush_nolock      0000000180062b54     libucrt:fflush.obj
 0004:00001b60       $pdata$__acrt_stdio_flush_nolock 0000000180062b60     libucrt:fflush.obj
 0004:00001b6c       $pdata$common_flush_all    0000000180062b6c     libucrt:fflush.obj
 0004:00001b78       $pdata$common_flush_all$fin$0 0000000180062b78     libucrt:fflush.obj
 0004:00001b84       $pdata$common_flush_all$fin$1 0000000180062b84     libucrt:fflush.obj
 0004:00001b90       $pdata$__acrt_stdio_free_buffer_nolock 0000000180062b90     libucrt:_freebuf.obj
 0004:00001b9c       $pdata$_isatty             0000000180062b9c     libucrt:isatty.obj
 0004:00001ba8       $pdata$__acrt_locale_free_monetary 0000000180062ba8     libucrt:initmon.obj
 0004:00001bb4       $pdata$__acrt_locale_free_numeric 0000000180062bb4     libucrt:initnum.obj
 0004:00001bc0       $pdata$__acrt_locale_free_time 0000000180062bc0     libucrt:inittime.obj
 0004:00001bcc       $pdata$?free_crt_array_internal@@YAXQEAPEBX_K@Z 0000000180062bcc     libucrt:inittime.obj
 0004:00001bd8       $pdata$__acrt_GetStringTypeA 0000000180062bd8     libucrt:getstringtypea.obj
 0004:00001be4       $pdata$_get_osfhandle      0000000180062be4     libucrt:osfinfo.obj
 0004:00001bf0       $pdata$_free_osfhnd        0000000180062bf0     libucrt:osfinfo.obj
 0004:00001bfc       $pdata$__acrt_lowio_create_handle_array 0000000180062bfc     libucrt:osfinfo.obj
 0004:00001c08       $pdata$__acrt_lowio_destroy_handle_array 0000000180062c08     libucrt:osfinfo.obj
 0004:00001c14       $pdata$__acrt_lowio_ensure_fh_exists 0000000180062c14     libucrt:osfinfo.obj
 0004:00001c20       $pdata$__acrt_DownlevelLocaleNameToLCID 0000000180062c20     libucrt:lcidtoname_downlevel.obj
 0004:00001c2c       $pdata$?GetTableIndexFromLocaleName@@YAHPEB_W@Z 0000000180062c2c     libucrt:lcidtoname_downlevel.obj
 0004:00001c38       $pdata$qsort               0000000180062c38     libucrt:qsort.obj
 0004:00001c44       $pdata$4$qsort             0000000180062c44     libucrt:qsort.obj
 0004:00001c50       $pdata$5$qsort             0000000180062c50     libucrt:qsort.obj
 0004:00001c5c       $pdata$?shortsort@@YAXPEAD0_KP6AHPEBX2@Z@Z 0000000180062c5c     libucrt:qsort.obj
 0004:00001c68       $pdata$2$?shortsort@@YAXPEAD0_KP6AHPEBX2@Z@Z 0000000180062c68     libucrt:qsort.obj
 0004:00001c74       $pdata$3$?shortsort@@YAXPEAD0_KP6AHPEBX2@Z@Z 0000000180062c74     libucrt:qsort.obj
 0004:00001c80       $pdata$strncpy_s           0000000180062c80     libucrt:strncpy_s.obj
 0004:00001c8c       $pdata$strpbrk             0000000180062c8c     libucrt:strpbrk.obj
 0004:00001c98       $pdata$_mbsdec_l           0000000180062c98     libucrt:mbsdec.obj
 0004:00001ca4       $pdata$?initialize_multibyte@@YAHXZ 0000000180062ca4     libucrt:multibyte_initializer.obj
 0004:00001cb0       $pdata$_msize              0000000180062cb0     libucrt:msize.obj
 0004:00001cbc       $pdata$_realloc_base       0000000180062cbc     libucrt:realloc_base.obj
 0004:00001cc8       $pdata$fegetenv            0000000180062cc8     libucrt:fegetenv.obj
 0004:00001cd4       $pdata$fesetenv            0000000180062cd4     libucrt:fesetenv.obj
 0004:00001ce0       $pdata$feholdexcept        0000000180062ce0     libucrt:feholdexcept.obj
 0004:00001cf8       $pdata$_write              0000000180062cf8     libucrt:write.obj
 0004:00001d04       $pdata$_write$fin$0        0000000180062d04     libucrt:write.obj
 0004:00001d10       $pdata$_write_nolock       0000000180062d10     libucrt:write.obj
 0004:00001d1c       $pdata$?write_double_translated_ansi_nolock@@YA?AUwrite_result@?A0x9c548279@@HQEBDI@Z 0000000180062d1c     libucrt:write.obj
 0004:00001d28       $pdata$?write_text_ansi_nolock@@YA?AUwrite_result@?A0x9c548279@@HQEBDI@Z 0000000180062d28     libucrt:write.obj
 0004:00001d34       $pdata$?write_text_utf16le_nolock@@YA?AUwrite_result@?A0x9c548279@@HQEBDI@Z 0000000180062d34     libucrt:write.obj
 0004:00001d40       $pdata$?write_text_utf8_nolock@@YA?AUwrite_result@?A0x9c548279@@HQEBDI@Z 0000000180062d40     libucrt:write.obj
 0004:00001d4c       $pdata$??$common_lseek_nolock@_J@@YA_JH_JH@Z 0000000180062d4c     libucrt:lseek.obj
 0004:00001d58       $pdata$fclose              0000000180062d58     libucrt:fclose.obj
 0004:00001d64       $pdata$fclose$fin$0        0000000180062d64     libucrt:fclose.obj
 0004:00001d70       $pdata$_fclose_nolock      0000000180062d70     libucrt:fclose.obj
 0004:00001d7c       $pdata$_commit             0000000180062d7c     libucrt:commit.obj
 0004:00001d88       $pdata$??$?RV<lambda_b521505b218e5242e90febf6bfebc422>@@AEAV<lambda_6978c1fb23f02e42e1d9e99668cc68aa>@@V<lambda_314360699dd331753a4119843814e9a7>@@@?$__crt_seh_guarded_call@H@@QEAAH$$QEAV<lambda_b521505b218e5242e90febf6bfebc422>@@AEAV<lambda_6978c1fb23f02e42e1d9e99668cc68aa>@@$$QEAV<lambda_314360699dd331753a4119843814e9a7>@@@Z 0000000180062d88     libucrt:commit.obj
 0004:00001d94       $pdata$?fin$0@?0???$?RV<lambda_bfedae4ebbf01fab1bb6dcc6a9e276e0>@@AEAV<lambda_2fe9b910cf3cbf4a0ab98a02ba45b3ec>@@V<lambda_237c231691f317818eb88cc1d5d642d6>@@@?$__crt_seh_guarded_call@H@@QEAAH$$QEAV<lambda_bfedae4ebbf01fab1bb6dcc6a9e276e0>@@AEAV<lambda_2fe9b910cf3cbf4a0ab98a02ba45b3ec>@@$$QEAV<lambda_237c231691f317818eb88cc1d5d642d6>@@@Z@4HA 0000000180062d94     libucrt:close.obj
 0004:00001d94       $pdata$?fin$0@?0???$?RV<lambda_b521505b218e5242e90febf6bfebc422>@@AEAV<lambda_6978c1fb23f02e42e1d9e99668cc68aa>@@V<lambda_314360699dd331753a4119843814e9a7>@@@?$__crt_seh_guarded_call@H@@QEAAH$$QEAV<lambda_b521505b218e5242e90febf6bfebc422>@@AEAV<lambda_6978c1fb23f02e42e1d9e99668cc68aa>@@$$QEAV<lambda_314360699dd331753a4119843814e9a7>@@@Z@4HA 0000000180062d94     libucrt:commit.obj
 0004:00001da0       $pdata$_setfpstatusword    0000000180062da0     libucrt:_fenvutils.obj
 0004:00001dac       $pdata$_getfpcontrolword   0000000180062dac     libucrt:_fenvutils.obj
 0004:00001db8       $pdata$_getfpstatusword    0000000180062db8     libucrt:_fenvutils.obj
 0004:00001dc4       $pdata$_clearfp            0000000180062dc4     libucrt:ieee.obj
 0004:00001dd0       $pdata$common_control87    0000000180062dd0     libucrt:ieee.obj
 0004:00001ddc       $pdata$_ctrlfp$filt$0      0000000180062ddc     libucrt:fpctrl.obj
 0004:00001ddc       $pdata$common_control87$filt$0 0000000180062ddc     libucrt:ieee.obj
 0004:00001de8       $pdata$_call_matherr       0000000180062de8     libucrt:libm_error.obj
 0004:00001df4       $pdata$_exception_enabled  0000000180062df4     libucrt:libm_error.obj
 0004:00001e00       $pdata$_handle_error       0000000180062e00     libucrt:libm_error.obj
 0004:00001e0c       $pdata$__acrt_initialize_fma3 0000000180062e0c     libucrt:fma3_available.obj
 0004:00001e18       $pdata$_log_special_common 0000000180062e18     libucrt:log_special.obj
 0004:00001e24       $pdata$_log10_special      0000000180062e24     libucrt:log_special.obj
 0004:00001e30       $pdata$_putwch_nolock      0000000180062e30     libucrt:putwch.obj
 0004:00001e3c       $pdata$_close              0000000180062e3c     libucrt:close.obj
 0004:00001e48       $pdata$_close_nolock       0000000180062e48     libucrt:close.obj
 0004:00001e54       $pdata$??$?RV<lambda_bfedae4ebbf01fab1bb6dcc6a9e276e0>@@AEAV<lambda_2fe9b910cf3cbf4a0ab98a02ba45b3ec>@@V<lambda_237c231691f317818eb88cc1d5d642d6>@@@?$__crt_seh_guarded_call@H@@QEAAH$$QEAV<lambda_bfedae4ebbf01fab1bb6dcc6a9e276e0>@@AEAV<lambda_2fe9b910cf3cbf4a0ab98a02ba45b3ec>@@$$QEAV<lambda_237c231691f317818eb88cc1d5d642d6>@@@Z 0000000180062e54     libucrt:close.obj
 0004:00001e6c       $pdata$_set_errno_from_matherr 0000000180062e6c     libucrt:fpexcept.obj
 0004:00001e78       $pdata$_raise_exc          0000000180062e78     libucrt:fpexcept.obj
 0004:00001e84       $pdata$_raise_exc_ex       0000000180062e84     libucrt:fpexcept.obj
 0004:00001e90       $pdata$_clrfp              0000000180062e90     libucrt:fpctrl.obj
 0004:00001e9c       $pdata$_ctrlfp             0000000180062e9c     libucrt:fpctrl.obj
 0004:00001ea8       $pdata$_statfp             0000000180062ea8     libucrt:fpctrl.obj
 0004:00001eb4       $pdata$_set_statfp         0000000180062eb4     libucrt:fpctrl.obj
 0004:00001ec0       $pdata$__dcrt_lowio_initialize_console_output 0000000180062ec0     libucrt:initcon.obj
 0004:00001ecc       $pdata$__dcrt_terminate_console_output 0000000180062ecc     libucrt:initcon.obj
 0004:00001ed8       $pdata$_IsNonwritableInCurrentImage 0000000180062ed8     LIBCMT:pesect.obj
 0004:00001ee4       $pdata$_IsNonwritableInCurrentImage$filt$0 0000000180062ee4     LIBCMT:pesect.obj
 0005:00000130       $R000000                   0000000180063130     ConEmuTh.res
 0005:00000450       $R000320                   0000000180063450     ConEmuTh.res
 0005:000014f8       $R0013C8                   00000001800644f8     ConEmuTh.res
 0005:00001510       $R0013E0                   0000000180064510     ConEmuTh.res
